 hcd_hsh2

 Timestamp is 4fb05c71 (Mon May 14 13:14:25 2012)

 Preferred load address is 10000000

 Start         Length     Name                   Class
 0001:00000000 00000004H .CRT$XCA                CODE
 0001:00000004 00000004H .CRT$XCZ                CODE
 0001:00000008 00000004H .CRT$XIA                CODE
 0001:0000000c 00000004H .CRT$XIZ                CODE
 0001:00000010 00000004H .CRT$XPA                CODE
 0001:00000014 00000004H .CRT$XPZ                CODE
 0001:00000018 00000004H .CRT$XTA                CODE
 0001:0000001c 00000004H .CRT$XTZ                CODE
 0001:00000020 0000ebc2H .rdata                  CODE
 0001:0000ebe4 00000025H .rdata$debug            CODE
 0001:0000ec0c 00037f4cH .text                   CODE
 0001:00046b58 00000234H .xdata                  CODE
 0001:00046d8c 0000003cH .idata$2                CODE
 0001:00046dc8 00000014H .idata$3                CODE
 0001:00046ddc 00000158H .idata$4                CODE
 0001:00046f34 000000d4H .idata$6                CODE
 0001:00047010 00000100H .edata                  CODE
 0002:00000000 00000158H .idata$5                DATA
 0002:00000158 000007e8H .data                   DATA
 0002:00000940 00000094H .bss                    DATA
 0003:00000000 000013f8H .pdata                  DATA

  Address         Publics by Value              Rva+Base       Lib:Object

 0000:00000000       ___safe_se_handler_count   00000000     <absolute>
 0000:00000000       ___safe_se_handler_table   00000000     <absolute>
 0001:00000000       __xc_a                     10001000     corelib0:crt0init.obj
 0001:00000004       __xc_z                     10001004     corelib0:crt0init.obj
 0001:00000008       __xi_a                     10001008     corelib0:crt0init.obj
 0001:0000000c       __xi_z                     1000100c     corelib0:crt0init.obj
 0001:00000010       __xp_a                     10001010     corelib0:crt0init.obj
 0001:00000014       __xp_z                     10001014     corelib0:crt0init.obj
 0001:00000018       __xt_a                     10001018     corelib0:crt0init.obj
 0001:0000001c       __xt_z                     1000101c     corelib0:crt0init.obj
 0001:0000003c       ??_C@_1BM@DNPIJEGO@?$AAH?$AA2?$AA?5?$AAH?$AAi?$AAg?$AAh?$AA?5?$AAS?$AAp?$AAe?$AAe?$AAd?$AA?$AA@ 1000103c     i_hwinit.obj
 0001:000000e8       ??_C@_1FI@MMEIOCFC@?$AAI?$AAn?$AAi?$AAt?$AAi?$AAa?$AAl?$AAi?$AAz?$AAe?$AAT?$AAr?$AAa?$AAn?$AAs?$AAc?$AAe?$AAi?$AAv?$AAe?$AAr?$AA?3?$AA?5?$AAI?$AAR?$AAQ?$AA?$DN?$AA?$CF?$AAd?$AA?0?$AA?5?$AAs@ 100010e8     i_hwinit.obj
 0001:00000140       ??_C@_1GC@PLPEIKOF@?$AAU?$AAS?$AAB?$AA?5?$AAH?$AAo?$AAs?$AAt?$AA?5?$AAl?$AAo?$AAa?$AAd?$AA?5?$AAf?$AAa?$AAi?$AAl?$AAu?$AAr?$AAe?$AA?5?$AAb?$AAe?$AAc?$AAa?$AAu?$AAs?$AAe?$AA?5?$AAU?$AAs@ 10001140     i_hwinit.obj
 0001:000001a4       ??_C@_1DK@LEKGNGA@?$AAH?$AAi?$AAg?$AAh?$AA?5?$AAS?$AAp?$AAe?$AAe?$AAd?$AA?5?$AAU?$AAS?$AAB?$AA?5?$AAH?$AAo?$AAs?$AAt?$AA?5?$AAP?$AAo?$AAr?$AAt?$AA?5?$AA2?$AA?$AN?$AA?6?$AA?$AA@ 100011a4     i_hwinit.obj
 0001:000001e0       ??_C@_1DM@NCNLGOJP@?$AAH?$AAo?$AAs?$AAt?$AA?5?$AAd?$AAo?$AAe?$AAs?$AA?5?$AAn?$AAo?$AAt?$AA?5?$AAc?$AAo?$AAn?$AAt?$AAr?$AAo?$AAl?$AA?5?$AAp?$AAo?$AAw?$AAe?$AAr?$AA?$AN?$AA?6?$AA?$AA@ 100011e0     i_hwinit.obj
 0001:000002b0       ??_C@_1GM@KKEMFHME@?$AA?9?$AAP?$AAo?$AAr?$AAt?$AA?$CI?$AA?$CF?$AAd?$AA?$CJ?$AA?3?$AAB?$AAS?$AAP?$AAU?$AAS?$AAB?$AAC?$AAl?$AAo?$AAc?$AAk?$AAC?$AAr?$AAe?$AAa?$AAt?$AAe?$AAF?$AAi?$AAl?$AAe?$AAM@ 100012b0     i_usbclock.obj
 0001:00000320       ??_C@_1GO@KPNBKEAO@?$AAP?$AAo?$AAr?$AAt?$AA?$CI?$AA?$CF?$AAd?$AA?$CJ?$AA?3?$AAB?$AAS?$AAP?$AAU?$AAS?$AAB?$AAC?$AAl?$AAo?$AAc?$AAk?$AAC?$AAr?$AAe?$AAa?$AAt?$AAe?$AAF?$AAi?$AAl?$AAe?$AAM?$AAa@ 10001320     i_usbclock.obj
 0001:00000390       ??_C@_1FE@GNDFGBM@?$AAP?$AAo?$AAr?$AAt?$AA?$CI?$AA?$CF?$AAd?$AA?$CJ?$AA?5?$AAO?$AAp?$AAe?$AAn?$AA?5?$AAe?$AAx?$AAi?$AAs?$AAt?$AAi?$AAn?$AAg?$AA?5?$AAU?$AAS?$AAB?$AA_?$AAC?$AAL?$AAO?$AAC?$AAK@ 10001390     i_usbclock.obj
 0001:000003e8       ??_C@_1FI@ECFJDMMH@?$AAP?$AAo?$AAr?$AAt?$AA?$CI?$AA?$CF?$AAd?$AA?$CJ?$AA?3?$AAF?$AAi?$AAr?$AAs?$AAt?$AA?5?$AAt?$AAo?$AA?5?$AAc?$AAr?$AAe?$AAa?$AAt?$AAe?$AA?5?$AAU?$AAS?$AAB?$AA_?$AAC?$AAL?$AAO@ 100013e8     i_usbclock.obj
 0001:00000440       ??_C@_1FC@NEMMIEIK@?$AAF?$AAa?$AAi?$AAl?$AAu?$AAr?$AAe?$AA?5?$AAt?$AAo?$AA?5?$AAC?$AAr?$AAe?$AAa?$AAt?$AAe?$AA?5?$AAF?$AAi?$AAl?$AAe?$AA?5?$AAM?$AAa?$AAp?$AAp?$AAi?$AAn?$AAg?$AA?5?$AAf@ 10001440     i_usbclock.obj
 0001:00000494       ??_C@_1CC@BJPGGDNC@?$AAU?$AAS?$AAB?$AA_?$AAC?$AAL?$AAO?$AAC?$AAK?$AA_?$AAG?$AAA?$AAT?$AAI?$AAN?$AAG?$AA?$AA@ 10001494     i_usbclock.obj
 0001:000004b8       ??_C@_1EG@CGIBPELK@?$AAP?$AAo?$AAr?$AAt?$AA?$CI?$AA?$CF?$AAd?$AA?$CJ?$AA?3?$AAB?$AAS?$AAP?$AAU?$AAS?$AAB?$AAC?$AAr?$AAe?$AAa?$AAt?$AAe?$AAF?$AAi?$AAl?$AAe?$AAM?$AAa?$AAp?$AAp?$AAi?$AAn?$AAg@ 100014b8     i_usbclock.obj
 0001:00000500       ??_C@_1IC@FDNBOOON@?$AAP?$AAo?$AAr?$AAt?$AA?$CI?$AA?$CF?$AAd?$AA?$CJ?$AA?5?$AA?9?$AA?5?$AAU?$AAS?$AAB?$AAC?$AAl?$AAo?$AAc?$AAk?$AAC?$AAa?$AAn?$AAC?$AAl?$AAo?$AAc?$AAk?$AAG?$AAa?$AAt?$AAi?$AAn@ 10001500     i_usbclock.obj
 0001:00000584       ??_C@_1DA@CLIJDNJA@?$AAU?$AAS?$AAB?$AAC?$AAl?$AAo?$AAc?$AAk?$AA?5?$AA?$CF?$AAs?$AA?5?$AAr?$AAe?$AAt?$AAu?$AAr?$AAn?$AA?5?$AA?$CF?$AAd?$AA?$AN?$AA?6?$AA?$AA@ 10001584     i_usbclock.obj
 0001:000005b4       ??_C@_1M@HCOOECOK@?$AAF?$AAA?$AAL?$AAS?$AAE?$AA?$AA@ 100015b4     i_usbclock.obj
 0001:000005c0       ??_C@_19ELAAHEEL@?$AAT?$AAR?$AAU?$AAE?$AA?$AA@ 100015c0     i_usbclock.obj
 0001:000005d0       ??_C@_1FM@HIIFJIHO@?$AAD?$AAi?$AAs?$AAa?$AAb?$AAl?$AAe?$AA?5?$AAF?$AAa?$AAi?$AAl?$AA?0?$AA?5?$AAN?$AAe?$AAe?$AAd?$AA?5?$AAt?$AAo?$AA?5?$AAc?$AAh?$AAe?$AAc?$AAk?$AA?0?$AA?5?$AAc?$AAu?$AAr@ 100015d0     i_usbclock.obj
 0001:00000630       ??_C@_1FK@HJNHKCPL@?$AAE?$AAn?$AAa?$AAb?$AAl?$AAe?$AA?5?$AAF?$AAa?$AAi?$AAl?$AA?0?$AA?5?$AAN?$AAe?$AAe?$AAd?$AA?5?$AAt?$AAo?$AA?5?$AAc?$AAh?$AAe?$AAc?$AAk?$AA?0?$AA?5?$AAc?$AAu?$AAr?$AAr@ 10001630     i_usbclock.obj
 0001:00000690       ??_C@_1FI@MBIBGPGK@?$AAU?$AAS?$AAB?$AAC?$AAl?$AAo?$AAc?$AAk?$AAS?$AAe?$AAt?$AA?3?$AA?5?$AAD?$AAD?$AAK?$AAC?$AAl?$AAo?$AAc?$AAk?$AAS?$AAe?$AAt?$AAG?$AAa?$AAt?$AAi?$AAn?$AAg?$AAM?$AAo@ 10001690     i_usbclock.obj
 0001:000006e8       ??_C@_1FC@PCOPMCOB@?$AAU?$AAS?$AAB?$AAC?$AAl?$AAo?$AAc?$AAk?$AAS?$AAe?$AAt?$AA?3?$AA?5?$AAD?$AAD?$AAK?$AAC?$AAl?$AAo?$AAc?$AAk?$AAC?$AAo?$AAn?$AAf?$AAi?$AAg?$AAB?$AAa?$AAu?$AAd?$AA?5@ 100016e8     i_usbclock.obj
 0001:000007d0       ??_C@_1EK@IBIELIGM@?$AAC?$AAa?$AAn?$AAn?$AAo?$AAt?$AA?5?$AAo?$AAb?$AAt?$AAa?$AAi?$AAn?$AA?5?$AAt?$AAh?$AAe?$AA?5?$AAs?$AAi?$AAl?$AAi?$AAc?$AAo?$AAn?$AA?5?$AAv?$AAe?$AAr?$AAs?$AAi?$AAo@ 100017d0     i_usbutils.obj
 0001:0000081c       ??_C@_1CI@OHCJFJPM@?$AAE?$AAR?$AAR?$AAO?$AAR?$AA?3?$AA?5?$AA?$CF?$AAs?$AA?5?$AAl?$AAi?$AAn?$AAe?$AA?5?$AA?$CF?$AAd?$AA?3?$AA?5?$AA?$AA@ 1000181c     i_usbutils.obj
 0001:00000844       ??_C@_1DK@BFKDMFPD@?$AA?4?$AA?2?$AA?4?$AA?4?$AA?2?$AA?4?$AA?4?$AA?2?$AAU?$AAS?$AAB?$AAC?$AAo?$AAm?$AAm?$AAo?$AAn?$AA?2?$AAU?$AAs?$AAb?$AAU?$AAt?$AAi?$AAl?$AAs?$AA?4?$AAc?$AA?$AA@ 10001844     i_usbutils.obj
 0001:00000880       ??_C@_1DK@JPBDFEOB@?$AAD?$AAE?$AAV?$AAI?$AAC?$AAE?$AA_?$AAC?$AAO?$AAN?$AAF?$AAI?$AAG?$AA_?$AAS?$AAT?$AAA?$AAT?$AAU?$AAS?$AA_?$AAI?$AAN?$AAV?$AAA?$AAL?$AAI?$AAD?$AA?$AA@ 10001880     usbh_usb2com_common_topaz_v1:hcddrv.obj
 0001:000008bc       ??_C@_1DE@IMCKALLA@?$AAD?$AAE?$AAV?$AAI?$AAC?$AAE?$AA_?$AAC?$AAO?$AAN?$AAF?$AAI?$AAG?$AA_?$AAS?$AAT?$AAA?$AAT?$AAU?$AAS?$AA_?$AAD?$AAO?$AAN?$AAE?$AA?$AA@ 100018bc     usbh_usb2com_common_topaz_v1:hcddrv.obj
 0001:000008f0       ??_C@_1DI@CEGNOBAM@?$AAD?$AAE?$AAV?$AAI?$AAC?$AAE?$AA_?$AAC?$AAO?$AAN?$AAF?$AAI?$AAG?$AA_?$AAS?$AAT?$AAA?$AAT?$AAU?$AAS?$AA_?$AAF?$AAA?$AAI?$AAL?$AAE?$AAD?$AA?$AA@ 100018f0     usbh_usb2com_common_topaz_v1:hcddrv.obj
 0001:00000928       ??_C@_1HO@PGHDEMEK@?$AAD?$AAE?$AAV?$AAI?$AAC?$AAE?$AA_?$AAC?$AAO?$AAN?$AAF?$AAI?$AAG?$AA_?$AAS?$AAT?$AAA?$AAT?$AAU?$AAS?$AA_?$AAS?$AAI?$AAG?$AAN?$AAA?$AAL?$AA_?$AAN?$AAE?$AAW?$AA_@ 10001928     usbh_usb2com_common_topaz_v1:hcddrv.obj
 0001:000009a8       ??_C@_1II@FBBOBKGN@?$AAD?$AAE?$AAV?$AAI?$AAC?$AAE?$AA_?$AAC?$AAO?$AAN?$AAF?$AAI?$AAG?$AA_?$AAS?$AAT?$AAA?$AAT?$AAU?$AAS?$AA_?$AAI?$AAN?$AAS?$AAE?$AAR?$AAT?$AA_?$AAN?$AAE?$AAW?$AA_@ 100019a8     usbh_usb2com_common_topaz_v1:hcddrv.obj
 0001:00000a30       ??_C@_1FC@LCLFDJDO@?$AAD?$AAE?$AAV?$AAI?$AAC?$AAE?$AA_?$AAC?$AAO?$AAN?$AAF?$AAI?$AAG?$AA_?$AAS?$AAT?$AAA?$AAT?$AAU?$AAS?$AA_?$AAC?$AAR?$AAE?$AAA?$AAT?$AAE?$AA_?$AAN?$AAE?$AAW?$AA_@ 10001a30     usbh_usb2com_common_topaz_v1:hcddrv.obj
 0001:00000a88       ??_C@_1EI@COKEBMOE@?$AAD?$AAE?$AAV?$AAI?$AAC?$AAE?$AA_?$AAC?$AAO?$AAN?$AAF?$AAI?$AAG?$AA_?$AAS?$AAT?$AAA?$AAT?$AAU?$AAS?$AA_?$AAC?$AAR?$AAE?$AAA?$AAT?$AAE?$AA_?$AAN?$AAE?$AAW?$AA_@ 10001a88     usbh_usb2com_common_topaz_v1:hcddrv.obj
 0001:00000ad0       ??_C@_1GG@HPGGGHKI@?$AAD?$AAE?$AAV?$AAI?$AAC?$AAE?$AA_?$AAC?$AAO?$AAN?$AAF?$AAI?$AAG?$AA_?$AAS?$AAT?$AAA?$AAT?$AAU?$AAS?$AA_?$AAS?$AAC?$AAH?$AAE?$AAD?$AAU?$AAL?$AAI?$AAN?$AAG?$AA_@ 10001ad0     usbh_usb2com_common_topaz_v1:hcddrv.obj
 0001:00000b38       ??_C@_1HG@KPBCOGEF@?$AAD?$AAE?$AAV?$AAI?$AAC?$AAE?$AA_?$AAC?$AAO?$AAN?$AAF?$AAI?$AAG?$AA_?$AAS?$AAT?$AAA?$AAT?$AAU?$AAS?$AA_?$AAS?$AAC?$AAH?$AAE?$AAD?$AAU?$AAL?$AAI?$AAN?$AAG?$AA_@ 10001b38     usbh_usb2com_common_topaz_v1:hcddrv.obj
 0001:00000bb0       ??_C@_1FG@CFFAAPDL@?$AAD?$AAE?$AAV?$AAI?$AAC?$AAE?$AA_?$AAC?$AAO?$AAN?$AAF?$AAI?$AAG?$AA_?$AAS?$AAT?$AAA?$AAT?$AAU?$AAS?$AA_?$AAS?$AAC?$AAH?$AAE?$AAD?$AAU?$AAL?$AAI?$AAN?$AAG?$AA_@ 10001bb0     usbh_usb2com_common_topaz_v1:hcddrv.obj
 0001:00000c08       ??_C@_1GA@NDHJOKMM@?$AAD?$AAE?$AAV?$AAI?$AAC?$AAE?$AA_?$AAC?$AAO?$AAN?$AAF?$AAI?$AAG?$AA_?$AAS?$AAT?$AAA?$AAT?$AAU?$AAS?$AA_?$AAD?$AAE?$AAT?$AAE?$AAR?$AAM?$AAI?$AAN?$AAE?$AA_?$AAC@ 10001c08     usbh_usb2com_common_topaz_v1:hcddrv.obj
 0001:00000c68       ??_C@_1GM@JADKDKDC@?$AAD?$AAE?$AAV?$AAI?$AAC?$AAE?$AA_?$AAC?$AAO?$AAN?$AAF?$AAI?$AAG?$AA_?$AAS?$AAT?$AAA?$AAT?$AAU?$AAS?$AA_?$AAS?$AAC?$AAH?$AAE?$AAD?$AAU?$AAL?$AAI?$AAN?$AAG?$AA_@ 10001c68     usbh_usb2com_common_topaz_v1:hcddrv.obj
 0001:00000cd8       ??_C@_1HM@NPLCKJLH@?$AAD?$AAE?$AAV?$AAI?$AAC?$AAE?$AA_?$AAC?$AAO?$AAN?$AAF?$AAI?$AAG?$AA_?$AAS?$AAT?$AAA?$AAT?$AAU?$AAS?$AA_?$AAS?$AAC?$AAH?$AAE?$AAD?$AAU?$AAL?$AAI?$AAN?$AAG?$AA_@ 10001cd8     usbh_usb2com_common_topaz_v1:hcddrv.obj
 0001:00000d58       ??_C@_1HE@MEMGEMJJ@?$AAD?$AAE?$AAV?$AAI?$AAC?$AAE?$AA_?$AAC?$AAO?$AAN?$AAF?$AAI?$AAG?$AA_?$AAS?$AAT?$AAA?$AAT?$AAU?$AAS?$AA_?$AAS?$AAE?$AAT?$AAU?$AAP?$AA_?$AAC?$AAO?$AAN?$AAF?$AAI@ 10001d58     usbh_usb2com_common_topaz_v1:hcddrv.obj
 0001:00000dd0       ??_C@_1GM@BCHKIAPP@?$AAD?$AAE?$AAV?$AAI?$AAC?$AAE?$AA_?$AAC?$AAO?$AAN?$AAF?$AAI?$AAG?$AA_?$AAS?$AAT?$AAA?$AAT?$AAU?$AAS?$AA_?$AAS?$AAC?$AAH?$AAE?$AAD?$AAU?$AAL?$AAI?$AAN?$AAG?$AA_@ 10001dd0     usbh_usb2com_common_topaz_v1:hcddrv.obj
 0001:00000e40       ??_C@_1HM@FNPCBDHK@?$AAD?$AAE?$AAV?$AAI?$AAC?$AAE?$AA_?$AAC?$AAO?$AAN?$AAF?$AAI?$AAG?$AA_?$AAS?$AAT?$AAA?$AAT?$AAU?$AAS?$AA_?$AAS?$AAC?$AAH?$AAE?$AAD?$AAU?$AAL?$AAI?$AAN?$AAG?$AA_@ 10001e40     usbh_usb2com_common_topaz_v1:hcddrv.obj
 0001:00000ec0       ??_C@_1EI@BBOOKHNN@?$AAD?$AAE?$AAV?$AAI?$AAC?$AAE?$AA_?$AAC?$AAO?$AAN?$AAF?$AAI?$AAG?$AA_?$AAS?$AAT?$AAA?$AAT?$AAU?$AAS?$AA_?$AAL?$AAE?$AAA?$AAV?$AAE?$AA_?$AAA?$AAD?$AAD?$AAR?$AAE@ 10001ec0     usbh_usb2com_common_topaz_v1:hcddrv.obj
 0001:00000f08       ??_C@_1FI@LGLHPFAK@?$AAD?$AAE?$AAV?$AAI?$AAC?$AAE?$AA_?$AAC?$AAO?$AAN?$AAF?$AAI?$AAG?$AA_?$AAS?$AAT?$AAA?$AAT?$AAU?$AAS?$AA_?$AAS?$AAC?$AAH?$AAE?$AAD?$AAU?$AAL?$AAI?$AAN?$AAG?$AA_@ 10001f08     usbh_usb2com_common_topaz_v1:hcddrv.obj
 0001:00000f60       ??_C@_1HG@BLNLBKIO@?$AAD?$AAE?$AAV?$AAI?$AAC?$AAE?$AA_?$AAC?$AAO?$AAN?$AAF?$AAI?$AAG?$AA_?$AAS?$AAT?$AAA?$AAT?$AAU?$AAS?$AA_?$AAS?$AAC?$AAH?$AAE?$AAD?$AAU?$AAL?$AAI?$AAN?$AAG?$AA_@ 10001f60     usbh_usb2com_common_topaz_v1:hcddrv.obj
 0001:00000fd8       ??_C@_1FG@NMCKCJLL@?$AAD?$AAE?$AAV?$AAI?$AAC?$AAE?$AA_?$AAC?$AAO?$AAN?$AAF?$AAI?$AAG?$AA_?$AAS?$AAT?$AAA?$AAT?$AAU?$AAS?$AA_?$AAR?$AAE?$AAS?$AAE?$AAT?$AA_?$AAA?$AAN?$AAD?$AA_?$AAE@ 10001fd8     usbh_usb2com_common_topaz_v1:hcddrv.obj
 0001:00001030       ??_C@_1EI@KNOIBOPH@?$AAD?$AAE?$AAV?$AAI?$AAC?$AAE?$AA_?$AAC?$AAO?$AAN?$AAF?$AAI?$AAG?$AA_?$AAS?$AAT?$AAA?$AAT?$AAU?$AAS?$AA_?$AAU?$AAS?$AAI?$AAN?$AAG?$AA_?$AAA?$AAD?$AAD?$AAR?$AAE@ 10002030     usbh_usb2com_common_topaz_v1:hcddrv.obj
 0001:00001078       ??_C@_1FI@COMJHLEF@?$AAD?$AAE?$AAV?$AAI?$AAC?$AAE?$AA_?$AAC?$AAO?$AAN?$AAF?$AAI?$AAG?$AA_?$AAS?$AAT?$AAA?$AAT?$AAU?$AAS?$AA_?$AAO?$AAP?$AAE?$AAN?$AAI?$AAN?$AAG?$AA_?$AAE?$AAN?$AAD@ 10002078     usbh_usb2com_common_topaz_v1:hcddrv.obj
 0001:000010d0       ??_C@_1DA@JAPEOLC@?$AAH?$AAC?$AAD?$AA?5?$AAd?$AAr?$AAi?$AAv?$AAe?$AAr?$AA?5?$AAD?$AAL?$AAL?$AA?5?$AAa?$AAt?$AAt?$AAa?$AAc?$AAh?$AA?$AN?$AA?6?$AA?$AA@ 100020d0     usbh_usb2com_common_topaz_v1:hcddrv.obj
 0001:00001100       ??_C@_1FK@FNONLNGN@?$AA?$CF?$AAs?$AA?3?$AA?5?$AAD?$AAE?$AAB?$AAU?$AAG?$AAC?$AAH?$AAK?$AA?5?$AAf?$AAa?$AAi?$AAl?$AAe?$AAd?$AA?5?$AAi?$AAn?$AA?5?$AAf?$AAi?$AAl?$AAe?$AA?5?$AA?$CF?$AAs?$AA?5?$AAa@ 10002100     usbh_usb2com_common_topaz_v1:hcddrv.obj
 0001:0000115c       ??_C@_1BA@LEPJIIOK@?$AAU?$AAn?$AAk?$AAn?$AAo?$AAw?$AAn?$AA?$AA@ 1000215c     usbh_usb2com_common_topaz_v1:hcddrv.obj
 0001:00001170       ??_C@_1ME@NILHHCOC@?$AAC?$AA?3?$AA?2?$AAW?$AAI?$AAN?$AAC?$AAE?$AAR?$AAO?$AAO?$AAT?$AAS?$AA?2?$AAT?$AAo?$AAp?$AAa?$AAz?$AA?2?$AAW?$AAI?$AAN?$AAC?$AAE?$AA6?$AA0?$AA0?$AA?2?$AAp?$AAl?$AAa@ 10002170     usbh_usb2com_common_topaz_v1:hcddrv.obj
 0001:00001238       ??_C@_1EA@EHNJJFN@?$AAU?$AAS?$AAB?$AA2?$AAC?$AAO?$AAM?$AA?3?$AAH?$AAc?$AAd?$AAM?$AAd?$AAd?$AA_?$AAP?$AAo?$AAw?$AAe?$AAr?$AAU?$AAp?$AA?5?$AAc?$AAa?$AAl?$AAl?$AAe?$AAd?$AA?$AN?$AA?6?$AA?$AA@ 10002238     usbh_usb2com_common_topaz_v1:hcddrv.obj
 0001:00001278       ??_C@_1DG@INPFIHHA@?$AAH?$AAc?$AAd?$AAM?$AAd?$AAd?$AA_?$AAS?$AAe?$AAt?$AAS?$AAu?$AAb?$AAH?$AAu?$AAb?$AAT?$AAe?$AAs?$AAt?$AAM?$AAo?$AAd?$AAe?$AA?$AN?$AA?6?$AA?$AA@ 10002278     usbh_usb2com_common_topaz_v1:hcddrv.obj
 0001:000012b0       ??_C@_1GG@BEPGMBBL@?$AAE?$AAH?$AAC?$AAD?$AA?$CB?$AAH?$AAC?$AAD?$AA_?$AAI?$AAn?$AAi?$AAt?$AA?5?$AAR?$AAe?$AAg?$AAQ?$AAu?$AAe?$AAr?$AAy?$AAV?$AAa?$AAl?$AAu?$AAe?$AAE?$AAx?$AA?$CI?$AA?$CF?$AAs@ 100022b0     usbh_usb2com_common_topaz_v1:hcddrv.obj
 0001:00001318       ??_C@_17KACEIPNC@?$AAK?$AAe?$AAy?$AA?$AA@ 10002318     usbh_usb2com_common_topaz_v1:hcddrv.obj
 0001:00001320       ??_C@_1FM@DDECOKKC@?$AAE?$AAH?$AAC?$AAD?$AA?$CB?$AAH?$AAC?$AAD?$AA_?$AAI?$AAn?$AAi?$AAt?$AA?5?$AAR?$AAe?$AAg?$AAO?$AAp?$AAe?$AAn?$AAK?$AAe?$AAy?$AAE?$AAx?$AA?$CI?$AA?$CF?$AAs?$AA?$CJ?$AA?5?$AAr@ 10002320     usbh_usb2com_common_topaz_v1:hcddrv.obj
 0001:0000137c       ??_C@_1CA@CLOGNIBH@?$AAE?$AAH?$AAC?$AAD?$AA?$CB?$AAH?$AAC?$AAD?$AA_?$AAI?$AAn?$AAi?$AAt?$AA?$AN?$AA?6?$AA?$AA@ 1000237c     usbh_usb2com_common_topaz_v1:hcddrv.obj
 0001:0000139c       ??_C@_1BI@BHLBGEOK@?$AAP?$AAr?$AAi?$AAo?$AAr?$AAi?$AAt?$AAy?$AA2?$AA5?$AA6?$AA?$AA@ 1000239c     usbh_usb2com_common_topaz_v1:hcddrv.obj
 0001:000013b4       ??_C@_1CG@PDHPMGPJ@?$AAU?$AAH?$AAC?$AAD?$AA?3?$AA?5?$AAH?$AAC?$AAD?$AA_?$AAD?$AAe?$AAi?$AAn?$AAi?$AAt?$AA?$AN?$AA?6?$AA?$AA@ 100023b4     usbh_usb2com_common_topaz_v1:hcddrv.obj
 0001:000013e0       ??_7CHcd@@6B@              100023e0     usbh_usb2com_common_topaz_v1:hcd.obj
 0001:00001450       ??_C@_1GG@IMKOLEF@?$AA?9?$AAC?$AAH?$AAc?$AAd?$AA?3?$AA?3?$AAO?$AAp?$AAe?$AAn?$AAP?$AAi?$AAp?$AAe?$AA?5?$AAf?$AAo?$AAr?$AA?5?$AAa?$AAd?$AAd?$AAr?$AAe?$AAs?$AAs?$AA?5?$AA?$CF?$AAd?$AA?0?$AA?5@ 10002450     usbh_usb2com_common_topaz_v1:hcd.obj
 0001:000014b8       ??_C@_1EO@POAKMOKK@?$AA?$CL?$AAC?$AAH?$AAc?$AAd?$AA?3?$AA?3?$AAO?$AAp?$AAe?$AAn?$AAP?$AAi?$AAp?$AAe?$AA?5?$AAf?$AAo?$AAr?$AA?5?$AAd?$AAe?$AAv?$AAi?$AAc?$AAe?$AA?5?$AAo?$AAn?$AA?5?$AAa?$AAd@ 100024b8     usbh_usb2com_common_topaz_v1:hcd.obj
 0001:00001508       ??_C@_1II@BLHGDNFM@?$AA?9?$AAC?$AAH?$AAc?$AAd?$AA?3?$AA?3?$AAC?$AAl?$AAo?$AAs?$AAe?$AAP?$AAi?$AAp?$AAe?$AA?5?$AA?9?$AA?5?$AAa?$AAd?$AAd?$AAr?$AAe?$AAs?$AAs?$AA?5?$AA?$DN?$AA?5?$AA?$CF?$AAd?$AA?0@ 10002508     usbh_usb2com_common_topaz_v1:hcd.obj
 0001:00001590       ??_C@_1GC@NJMEDGCO@?$AA?$CL?$AAC?$AAH?$AAc?$AAd?$AA?3?$AA?3?$AAC?$AAl?$AAo?$AAs?$AAe?$AAP?$AAi?$AAp?$AAe?$AA?5?$AA?9?$AA?5?$AAa?$AAd?$AAd?$AAr?$AAe?$AAs?$AAs?$AA?5?$AA?$DN?$AA?5?$AA?$CF?$AAd?$AA?0@ 10002590     usbh_usb2com_common_topaz_v1:hcd.obj
 0001:000015f8       ??_C@_1FC@IHEAIAGM@?$AA?9?$AAC?$AAH?$AAc?$AAd?$AA?3?$AA?3?$AAI?$AAs?$AAs?$AAu?$AAe?$AAT?$AAr?$AAa?$AAn?$AAs?$AAf?$AAe?$AAr?$AA?5?$AA?9?$AA?5?$AAr?$AAe?$AAt?$AAu?$AAr?$AAi?$AAn?$AAg?$AA?5@ 100025f8     usbh_usb2com_common_topaz_v1:hcd.obj
 0001:00001650       ??_C@_1PM@ELCLLPLD@?$AA?$CL?$AAC?$AAH?$AAc?$AAd?$AA?3?$AA?3?$AAI?$AAs?$AAs?$AAu?$AAe?$AAT?$AAr?$AAa?$AAn?$AAs?$AAf?$AAe?$AAr?$AA?5?$AA?9?$AA?5?$AAa?$AAd?$AAd?$AAr?$AAe?$AAs?$AAs?$AA?5?$AA?$DN@ 10002650     usbh_usb2com_common_topaz_v1:hcd.obj
 0001:00001750       ??_C@_1JA@FCGAMPLO@?$AA?9?$AAC?$AAH?$AAc?$AAd?$AA?3?$AA?3?$AAA?$AAb?$AAo?$AAr?$AAt?$AAT?$AAr?$AAa?$AAn?$AAs?$AAf?$AAe?$AAr?$AA?5?$AA?9?$AA?5?$AAa?$AAd?$AAd?$AAr?$AAe?$AAs?$AAs?$AA?5?$AA?$DN@ 10002750     usbh_usb2com_common_topaz_v1:hcd.obj
 0001:000017e0       ??_C@_1JC@PLEKCCMG@?$AA?$CL?$AAC?$AAH?$AAc?$AAd?$AA?3?$AA?3?$AAA?$AAb?$AAo?$AAr?$AAt?$AAT?$AAr?$AAa?$AAn?$AAs?$AAf?$AAe?$AAr?$AA?5?$AA?9?$AA?5?$AAa?$AAd?$AAd?$AAr?$AAe?$AAs?$AAs?$AA?5?$AA?$DN@ 100027e0     usbh_usb2com_common_topaz_v1:hcd.obj
 0001:00001878       ??_C@_1KE@LBCAOHB@?$AA?9?$AAC?$AAH?$AAc?$AAd?$AA?3?$AA?3?$AAI?$AAs?$AAP?$AAi?$AAp?$AAe?$AAH?$AAa?$AAl?$AAt?$AAe?$AAd?$AA?5?$AA?9?$AA?5?$AAa?$AAd?$AAd?$AAr?$AAe?$AAs?$AAs?$AA?5?$AA?$DN?$AA?5@ 10002878     usbh_usb2com_common_topaz_v1:hcd.obj
 0001:00001920       ??_C@_1GI@FPOGNJBG@?$AA?$CL?$AAC?$AAH?$AAc?$AAd?$AA?3?$AA?3?$AAI?$AAs?$AAP?$AAi?$AAp?$AAe?$AAH?$AAa?$AAl?$AAt?$AAe?$AAd?$AA?5?$AA?9?$AA?5?$AAa?$AAd?$AAd?$AAr?$AAe?$AAs?$AAs?$AA?5?$AA?$DN?$AA?5@ 10002920     usbh_usb2com_common_topaz_v1:hcd.obj
 0001:00001988       ??_C@_1II@FAPMMDIC@?$AA?9?$AAC?$AAH?$AAc?$AAd?$AA?3?$AA?3?$AAR?$AAe?$AAs?$AAe?$AAt?$AAP?$AAi?$AAp?$AAe?$AA?5?$AA?9?$AA?5?$AAa?$AAd?$AAd?$AAr?$AAe?$AAs?$AAs?$AA?5?$AA?$DN?$AA?5?$AA?$CF?$AAd?$AA?0@ 10002988     usbh_usb2com_common_topaz_v1:hcd.obj
 0001:00001a10       ??_C@_1GC@CCBOPNIE@?$AA?$CL?$AAC?$AAH?$AAc?$AAd?$AA?3?$AA?3?$AAR?$AAe?$AAs?$AAe?$AAt?$AAP?$AAi?$AAp?$AAe?$AA?5?$AA?9?$AA?5?$AAa?$AAd?$AAd?$AAr?$AAe?$AAs?$AAs?$AA?5?$AA?$DN?$AA?5?$AA?$CF?$AAd?$AA?0@ 10002a10     usbh_usb2com_common_topaz_v1:hcd.obj
 0001:00001a78       ??_C@_1HA@DBAOPMNC@?$AA?9?$AAC?$AAH?$AAc?$AAd?$AA?3?$AA?3?$AAD?$AAi?$AAs?$AAa?$AAb?$AAl?$AAe?$AAD?$AAe?$AAv?$AAi?$AAc?$AAe?$AA?5?$AA?9?$AA?5?$AAa?$AAd?$AAd?$AAr?$AAe?$AAs?$AAs?$AA?5?$AA?$DN@ 10002a78     usbh_usb2com_common_topaz_v1:hcd.obj
 0001:00001ae8       ??_C@_1GC@CKNGPFE@?$AA?$CL?$AAC?$AAH?$AAc?$AAd?$AA?3?$AA?3?$AAD?$AAi?$AAs?$AAa?$AAb?$AAl?$AAe?$AAD?$AAe?$AAv?$AAi?$AAc?$AAe?$AA?5?$AA?9?$AA?5?$AAa?$AAd?$AAd?$AAr?$AAe?$AAs?$AAs?$AA?5?$AA?$DN@ 10002ae8     usbh_usb2com_common_topaz_v1:hcd.obj
 0001:00001b50       ??_C@_1IM@FNOGFBBE@?$AA?9?$AAC?$AAH?$AAc?$AAd?$AA?3?$AA?3?$AAS?$AAu?$AAs?$AAp?$AAe?$AAn?$AAd?$AAR?$AAe?$AAs?$AAu?$AAm?$AAe?$AA?5?$AA?9?$AA?5?$AAa?$AAd?$AAd?$AAr?$AAe?$AAs?$AAs?$AA?5?$AA?$DN@ 10002b50     usbh_usb2com_common_topaz_v1:hcd.obj
 0001:00001be0       ??_C@_1GK@JHFDANOI@?$AA?$CL?$AAC?$AAH?$AAc?$AAd?$AA?3?$AA?3?$AAS?$AAu?$AAs?$AAp?$AAe?$AAn?$AAd?$AAR?$AAe?$AAs?$AAu?$AAm?$AAe?$AA?5?$AA?9?$AA?5?$AAa?$AAd?$AAd?$AAr?$AAe?$AAs?$AAs?$AA?5?$AA?$DN@ 10002be0     usbh_usb2com_common_topaz_v1:hcd.obj
 0001:00001c50       ??_C@_1KA@FJCCGHGB@?$AAC?$AAP?$AAh?$AAy?$AAs?$AAM?$AAe?$AAm?$AA?5?$AA?5?$AAN?$AAo?$AAr?$AAm?$AAa?$AAl?$AA?5?$AAA?$AAl?$AAl?$AAo?$AAc?$AA?5?$AAR?$AAe?$AAg?$AAi?$AAo?$AAn?$AA?5?$AAP?$AAh@ 10002c50     usbh_usb2com_common_topaz_v1:cphysmem.obj
 0001:00001cf0       ??_C@_1KA@PJOEMMCM@?$AAC?$AAP?$AAh?$AAy?$AAs?$AAM?$AAe?$AAm?$AA?5?$AAH?$AAi?$AAg?$AAh?$AAP?$AAr?$AAi?$AA?5?$AAA?$AAl?$AAl?$AAo?$AAc?$AA?5?$AAR?$AAe?$AAg?$AAi?$AAo?$AAn?$AA?5?$AAP?$AAh@ 10002cf0     usbh_usb2com_common_topaz_v1:cphysmem.obj
 0001:00001d90       ??_C@_1KA@JBKPJKEP@?$AAC?$AAP?$AAh?$AAy?$AAs?$AAM?$AAe?$AAm?$AA?5?$AAS?$AAp?$AAe?$AAc?$AAi?$AAa?$AAl?$AA?5?$AAA?$AAl?$AAl?$AAo?$AAc?$AA?5?$AAR?$AAe?$AAg?$AAi?$AAo?$AAn?$AA?5?$AAP?$AAh@ 10002d90     usbh_usb2com_common_topaz_v1:cphysmem.obj
 0001:00001e30       ??_C@_1KA@PIBOCLFE@?$AAC?$AAP?$AAh?$AAy?$AAs?$AAM?$AAe?$AAm?$AA?5?$AA?5?$AA?5?$AAT?$AAo?$AAt?$AAa?$AAl?$AA?5?$AAA?$AAl?$AAl?$AAo?$AAc?$AA?5?$AAR?$AAe?$AAg?$AAi?$AAo?$AAn?$AA?5?$AAP?$AAh@ 10002e30     usbh_usb2com_common_topaz_v1:cphysmem.obj
 0001:00001ed0       ??_C@_1FA@ICCPJKCO@?$AAA?$AAl?$AAl?$AAo?$AAc?$AAa?$AAt?$AAi?$AAn?$AAg?$AA?5?$AAD?$AAM?$AAA?$AA?5?$AAb?$AAu?$AAf?$AAf?$AAe?$AAr?$AA?5?$AAf?$AAr?$AAo?$AAm?$AA?5?$AAs?$AAy?$AAs?$AAt?$AAe@ 10002ed0     usbh_usb2com_common_topaz_v1:cphysmem.obj
 0001:00001f20       ??_C@_1EA@LENIGCOC@?$AAD?$AAM?$AAA?$AA?5?$AAb?$AAu?$AAf?$AAf?$AAe?$AAr?$AA?5?$AAp?$AAa?$AAs?$AAs?$AAe?$AAd?$AA?5?$AAi?$AAn?$AA?5?$AAf?$AAr?$AAo?$AAm?$AA?5?$AAP?$AAD?$AAD?$AA?$AN?$AA?6?$AA?$AA@ 10002f20     usbh_usb2com_common_topaz_v1:cphysmem.obj
 0001:00001f60       ??_C@_1MI@LKBLMIGD@?$AAC?$AA?3?$AA?2?$AAW?$AAI?$AAN?$AAC?$AAE?$AAR?$AAO?$AAO?$AAT?$AAS?$AA?2?$AAT?$AAo?$AAp?$AAa?$AAz?$AA?2?$AAW?$AAI?$AAN?$AAC?$AAE?$AA6?$AA0?$AA0?$AA?2?$AAp?$AAl?$AAa@ 10002f60     usbh_usb2com_common_topaz_v1:cphysmem.obj
 0001:00002028       ??_C@_1GE@MMCCLEGJ@?$AAC?$AAP?$AAh?$AAy?$AAs?$AAM?$AAe?$AAm?$AA?5?$AAI?$AAn?$AAi?$AAt?$AA?5?$AA?3?$AA?5?$AAH?$AAi?$AAg?$AAh?$AAP?$AAr?$AAi?$AA?5?$AAF?$AAr?$AAe?$AAe?$AA?5?$AAH?$AAe?$AAa@ 10003028     usbh_usb2com_common_topaz_v1:cphysmem.obj
 0001:00002090       ??_C@_1FO@GMLOFHA@?$AAC?$AAP?$AAh?$AAy?$AAs?$AAM?$AAe?$AAm?$AA?5?$AAI?$AAn?$AAi?$AAt?$AA?5?$AA?3?$AA?5?$AAM?$AAa?$AAi?$AAn?$AA?5?$AAF?$AAr?$AAe?$AAe?$AA?5?$AAH?$AAe?$AAa?$AAp?$AA?5?$AAN@ 10003090     usbh_usb2com_common_topaz_v1:cphysmem.obj
 0001:000020f0       ??_C@_1CC@BENCJCHP@?$AAF?$AAr?$AAe?$AAe?$AA?5?$AAL?$AAo?$AAw?$AA?5?$AAP?$AAr?$AAi?$AA?5?$AAM?$AAe?$AAm?$AA?$AA@ 100030f0     usbh_usb2com_common_topaz_v1:cphysmem.obj
 0001:00002118       ??_C@_1JM@GLIPFLD@?$AAC?$AAP?$AAh?$AAy?$AAs?$AAM?$AAe?$AAm?$AA?5?$AAI?$AAn?$AAi?$AAt?$AA?5?$AA?3?$AA?5?$AAH?$AAi?$AAg?$AAh?$AAP?$AAr?$AAi?$AAF?$AAr?$AAe?$AAe?$AAL?$AAi?$AAs?$AAt?$AAH@ 10003118     usbh_usb2com_common_topaz_v1:cphysmem.obj
 0001:000021b8       ??_C@_1IA@BJAEEMDH@?$AAC?$AAP?$AAh?$AAy?$AAs?$AAM?$AAe?$AAm?$AA?5?$AAI?$AAn?$AAi?$AAt?$AA?5?$AA?3?$AA?5?$AAF?$AAr?$AAe?$AAe?$AAL?$AAi?$AAs?$AAt?$AAH?$AAe?$AAa?$AAd?$AA?5?$AA?$DN?$AA?5?$AA0@ 100031b8     usbh_usb2com_common_topaz_v1:cphysmem.obj
 0001:00002238       ??_C@_1FI@PMOPNGBB@?$AAC?$AAP?$AAh?$AAy?$AAs?$AAM?$AAe?$AAm?$AA?5?$AAI?$AAn?$AAi?$AAt?$AA?5?$AA?3?$AA?5?$AAN?$AAo?$AAd?$AAe?$AAF?$AAr?$AAe?$AAe?$AAL?$AAi?$AAs?$AAt?$AAH?$AAe?$AAa?$AAd@ 10003238     usbh_usb2com_common_topaz_v1:cphysmem.obj
 0001:00002290       ??_C@_1FG@KBIHBEP@?$AAC?$AAP?$AAh?$AAy?$AAs?$AAM?$AAe?$AAm?$AA?5?$AAV?$AAa?$AAl?$AAi?$AAd?$AAa?$AAt?$AAe?$AAH?$AAe?$AAa?$AAp?$AAs?$AA?5?$AA?3?$AA?5?$AAN?$AAo?$AAd?$AAe?$AAs?$AA?5?$AAF@ 10003290     usbh_usb2com_common_topaz_v1:cphysmem.obj
 0001:000022e8       ??_C@_1HE@BKCBJCLG@?$AAC?$AAP?$AAh?$AAy?$AAs?$AAM?$AAe?$AAm?$AA?5?$AAV?$AAa?$AAl?$AAi?$AAd?$AAa?$AAt?$AAe?$AAH?$AAe?$AAa?$AAp?$AAs?$AA?5?$AA?3?$AA?5?$AAI?$AAn?$AAv?$AAa?$AAl?$AAi?$AAd@ 100032e8     usbh_usb2com_common_topaz_v1:cphysmem.obj
 0001:00002360       ??_C@_1HI@EIJALODG@?$AAC?$AAP?$AAh?$AAy?$AAs?$AAM?$AAe?$AAm?$AA?5?$AAV?$AAa?$AAl?$AAi?$AAd?$AAa?$AAt?$AAe?$AAH?$AAe?$AAa?$AAp?$AAs?$AA?5?$AA?3?$AA?5?$AAW?$AAe?$AA?8?$AAv?$AAe?$AA?5?$AAl@ 10003360     usbh_usb2com_common_topaz_v1:cphysmem.obj
 0001:000023d8       ??_C@_1IK@IOHNCDME@?$AAC?$AAP?$AAh?$AAy?$AAs?$AAM?$AAe?$AAm?$AA?5?$AAV?$AAa?$AAl?$AAi?$AAd?$AAa?$AAt?$AAe?$AAH?$AAe?$AAa?$AAp?$AAs?$AA?5?$AA?3?$AA?5?$AAF?$AAr?$AAe?$AAe?$AAS?$AAi?$AAz@ 100033d8     usbh_usb2com_common_topaz_v1:cphysmem.obj
 0001:00002468       ??_C@_1GO@BBFMJBGE@?$AAC?$AAP?$AAh?$AAy?$AAs?$AAM?$AAe?$AAm?$AA?5?$AAV?$AAa?$AAl?$AAi?$AAd?$AAa?$AAt?$AAe?$AAH?$AAe?$AAa?$AAp?$AAs?$AA?5?$AA?3?$AA?5?$AAI?$AAn?$AAv?$AAa?$AAl?$AAi?$AAd@ 10003468     usbh_usb2com_common_topaz_v1:cphysmem.obj
 0001:000024d8       ??_C@_1JM@FJJCMIHE@?$AAI?$AAn?$AAU?$AAs?$AAe?$AAL?$AAi?$AAs?$AAt?$AA?$CI?$AAp?$AAr?$AAi?$AA?5?$AA?$DN?$AA?5?$AA?$CF?$AAd?$AA?$CJ?$AA?5?$AA?3?$AA?5?$AAp?$AAN?$AAo?$AAd?$AAe?$AA?5?$AAs?$AAi?$AAz?$AAe@ 100034d8     usbh_usb2com_common_topaz_v1:cphysmem.obj
 0001:00002578       ??_C@_1GM@JDBBEPGD@?$AAC?$AAP?$AAh?$AAy?$AAs?$AAM?$AAe?$AAm?$AA?5?$AAV?$AAa?$AAl?$AAi?$AAd?$AAa?$AAt?$AAe?$AAH?$AAe?$AAa?$AAp?$AAs?$AA?5?$AA?3?$AA?5?$AAI?$AAn?$AAv?$AAa?$AAl?$AAi?$AAd@ 10003578     usbh_usb2com_common_topaz_v1:cphysmem.obj
 0001:000025e8       ??_C@_1HE@LFOBKGBN@?$AAC?$AAP?$AAh?$AAy?$AAs?$AAM?$AAe?$AAm?$AA?5?$AAV?$AAa?$AAl?$AAi?$AAd?$AAa?$AAt?$AAe?$AAH?$AAe?$AAa?$AAp?$AAs?$AA?5?$AA?3?$AA?5?$AAF?$AAr?$AAe?$AAe?$AA?5?$AAL?$AAi@ 100035e8     usbh_usb2com_common_topaz_v1:cphysmem.obj
 0001:00002660       ??_C@_1JK@ENFIOHDK@?$AAF?$AAr?$AAe?$AAe?$AAL?$AAi?$AAs?$AAt?$AA?$CI?$AAp?$AAr?$AAi?$AA?5?$AA?$DN?$AA?5?$AA?$CF?$AAd?$AA?$CJ?$AA?5?$AA?3?$AA?5?$AAp?$AAN?$AAo?$AAd?$AAe?$AA?5?$AAs?$AAi?$AAz?$AAe?$AA?5@ 10003660     usbh_usb2com_common_topaz_v1:cphysmem.obj
 0001:00002700       ??_C@_1ME@KNFABPNB@?$AAc?$AA?3?$AA?2?$AAw?$AAi?$AAn?$AAc?$AAe?$AAr?$AAo?$AAo?$AAt?$AAs?$AA?2?$AAt?$AAo?$AAp?$AAa?$AAz?$AA?2?$AAw?$AAi?$AAn?$AAc?$AAe?$AA6?$AA0?$AA0?$AA?2?$AAp?$AAl?$AAa@ 10003700     usbh_usb2com_common_topaz_v1:cphysmem.obj
 0001:000027c4       ??_C@_1BK@HELANJJ@?$AAD?$AAe?$AAf?$AAa?$AAu?$AAl?$AAt?$AA?5?$AAD?$AAe?$AAs?$AAc?$AA?$AA@ 100037c4     usbh_usb2com_common_topaz_v1:cphysmem.obj
 0001:000027e0       ??_C@_1BK@DHHEGMON@?$AAD?$AAe?$AAl?$AAe?$AAt?$AAe?$AAd?$AA?5?$AAN?$AAo?$AAd?$AAe?$AA?$AA@ 100037e0     usbh_usb2com_common_topaz_v1:cphysmem.obj
 0001:00002800       ??_C@_1FO@DKILOPHK@?$AAC?$AAP?$AAh?$AAy?$AAs?$AAM?$AAe?$AAm?$AA?5?$AAA?$AAl?$AAl?$AAo?$AAc?$AAa?$AAt?$AAe?$AAM?$AAe?$AAm?$AAo?$AAr?$AAy?$AA?5?$AA?3?$AA?5?$AAb?$AAS?$AAp?$AAe?$AAc?$AAi@ 10003800     usbh_usb2com_common_topaz_v1:cphysmem.obj
 0001:00002860       ??_C@_1JG@MNOBEEOD@?$AAC?$AAP?$AAh?$AAy?$AAs?$AAM?$AAe?$AAm?$AA?5?$AAA?$AAl?$AAl?$AAo?$AAc?$AAa?$AAt?$AAe?$AAM?$AAe?$AAm?$AAo?$AAr?$AAy?$AA?5?$AA?3?$AA?5?$AAP?$AAA?$AA?5?$AA?$DN?$AA?5?$AA0@ 10003860     usbh_usb2com_common_topaz_v1:cphysmem.obj
 0001:000028f8       ??_C@_1FM@OOLOAMIO@?$AAC?$AAP?$AAh?$AAy?$AAs?$AAM?$AAe?$AAm?$AA?5?$AAA?$AAl?$AAl?$AAo?$AAc?$AAa?$AAt?$AAe?$AAM?$AAe?$AAm?$AAo?$AAr?$AAy?$AA?5?$AA?3?$AA?5?$AAN?$AAo?$AA?5?$AAm?$AAe?$AAm@ 100038f8     usbh_usb2com_common_topaz_v1:cphysmem.obj
 0001:00002958       ??_C@_1HA@LDBHCAGE@?$AAC?$AAP?$AAh?$AAy?$AAs?$AAM?$AAe?$AAm?$AA?3?$AA?5?$AAH?$AAe?$AAa?$AAp?$AA?5?$AAp?$AAr?$AAi?$AA?5?$AA?$DN?$AA?5?$AA?$CF?$AAd?$AA?5?$AAb?$AAe?$AAf?$AAo?$AAr?$AAe?$AA?5?$AAa@ 10003958     usbh_usb2com_common_topaz_v1:cphysmem.obj
 0001:000029c8       ??_C@_1FK@GOKAFDHN@?$AAA?$AAl?$AAl?$AAo?$AAc?$AAa?$AAt?$AAe?$AAM?$AAe?$AAm?$AAo?$AAr?$AAy?$AA?5?$AAD?$AAe?$AAs?$AAc?$AA?5?$AA?$DN?$AA?5?$AA?$CF?$AAs?$AA?3?$AA?5?$AA?$CI?$AAr?$AAo?$AAu?$AAn?$AAd@ 100039c8     usbh_usb2com_common_topaz_v1:cphysmem.obj
 0001:00002a28       ??_C@_1GC@CLHBJKAN@?$AAC?$AAP?$AAh?$AAy?$AAs?$AAM?$AAe?$AAm?$AA?3?$AA?5?$AAH?$AAe?$AAa?$AAp?$AA?5?$AAp?$AAr?$AAi?$AA?5?$AA?$DN?$AA?5?$AA?$CF?$AAd?$AA?5?$AAa?$AAf?$AAt?$AAe?$AAr?$AA?5?$AAf?$AAr@ 10003a28     usbh_usb2com_common_topaz_v1:cphysmem.obj
 0001:00002a8c       ??_C@_1BK@BIHKKMPG@?$AAF?$AAr?$AAe?$AAe?$AAd?$AA?5?$AAM?$AAe?$AAm?$AAo?$AAr?$AAy?$AA?$AA@ 10003a8c     usbh_usb2com_common_topaz_v1:cphysmem.obj
 0001:00002aa8       ??_C@_1IO@GHNBCJEB@?$AAC?$AAP?$AAh?$AAy?$AAs?$AAM?$AAe?$AAm?$AA?5?$AAF?$AAr?$AAe?$AAe?$AAM?$AAe?$AAm?$AAo?$AAr?$AAy?$AA?5?$AA?3?$AA?5?$AAP?$AAA?$AA?5?$AA?$DN?$AA?5?$AA0?$AAx?$AA?$CF?$AA0?$AA8@ 10003aa8     usbh_usb2com_common_topaz_v1:cphysmem.obj
 0001:00002b38       ??_C@_1GE@CAKPDPGE@?$AAC?$AAP?$AAh?$AAy?$AAs?$AAM?$AAe?$AAm?$AA?3?$AA?5?$AAH?$AAe?$AAa?$AAp?$AA?5?$AAp?$AAr?$AAi?$AA?5?$AA?$DN?$AA?5?$AA?$CF?$AAd?$AA?5?$AAb?$AAe?$AAf?$AAo?$AAr?$AAe?$AA?5?$AAf@ 10003b38     usbh_usb2com_common_topaz_v1:cphysmem.obj
 0001:00002b9c       ??_7CDeviceGlobal@@6B@     10003b9c     usbh_usb2com_common_topaz_v1:cdevice.obj
 0001:00002bb0       ??_C@_1EA@JHPLNJAE@?$AA?9?$AAC?$AAD?$AAe?$AAv?$AAi?$AAc?$AAe?$AA?3?$AA?3?$AAI?$AAn?$AAi?$AAt?$AAi?$AAa?$AAl?$AAi?$AAz?$AAe?$AA?0?$AA?5?$AAs?$AAu?$AAc?$AAc?$AAe?$AAs?$AAs?$AA?$CB?$AA?6?$AA?$AA@ 10003bb0     usbh_usb2com_common_topaz_v1:cdevice.obj
 0001:00002bf0       ??_C@_1GO@JGJHIIIJ@?$AA?9?$AAC?$AAD?$AAe?$AAv?$AAi?$AAc?$AAe?$AA?3?$AA?3?$AAI?$AAn?$AAi?$AAt?$AAi?$AAa?$AAl?$AAi?$AAz?$AAe?$AA?5?$AA?9?$AA?5?$AAC?$AAo?$AAu?$AAl?$AAd?$AA?5?$AAn?$AAo?$AAt@ 10003bf0     usbh_usb2com_common_topaz_v1:cdevice.obj
 0001:00002c60       ??_C@_1CO@MCCAIHAO@?$AAH?$AAc?$AAd?$AAS?$AAe?$AAl?$AAe?$AAc?$AAt?$AAC?$AAo?$AAn?$AAf?$AAi?$AAg?$AAu?$AAr?$AAa?$AAt?$AAi?$AAo?$AAn?$AA?$AA@ 10003c60     usbh_usb2com_common_topaz_v1:cdevice.obj
 0001:00002c90       ??_C@_1CE@KAKNBFJP@?$AAH?$AAc?$AAd?$AAD?$AAe?$AAv?$AAi?$AAc?$AAe?$AAD?$AAe?$AAt?$AAa?$AAc?$AAh?$AAe?$AAd?$AA?$AA@ 10003c90     usbh_usb2com_common_topaz_v1:cdevice.obj
 0001:00002cb4       ??_C@_1CE@MBINLHH@?$AAH?$AAc?$AAd?$AAD?$AAe?$AAv?$AAi?$AAc?$AAe?$AAA?$AAt?$AAt?$AAa?$AAc?$AAh?$AAe?$AAd?$AA?$AA@ 10003cb4     usbh_usb2com_common_topaz_v1:cdevice.obj
 0001:00002cd8       ??_C@_1BE@NANPENDH@?$AAH?$AAc?$AAd?$AAA?$AAt?$AAt?$AAa?$AAc?$AAh?$AA?$AA@ 10003cd8     usbh_usb2com_common_topaz_v1:cdevice.obj
 0001:00002cf0       ??_C@_1GC@NHBDHMML@?$AA?9?$AAC?$AAD?$AAe?$AAv?$AAi?$AAc?$AAe?$AA?3?$AA?3?$AAI?$AAn?$AAi?$AAt?$AAi?$AAa?$AAl?$AAi?$AAz?$AAe?$AA?5?$AA?9?$AA?5?$AAC?$AAo?$AAu?$AAl?$AAd?$AA?5?$AAn?$AAo?$AAt@ 10003cf0     usbh_usb2com_common_topaz_v1:cdevice.obj
 0001:00002d54       ??_C@_1BC@MPAIGMIO@?$AAU?$AAS?$AAB?$AAD?$AA?4?$AAD?$AAL?$AAL?$AA?$AA@ 10003d54     usbh_usb2com_common_topaz_v1:cdevice.obj
 0001:00002d68       ??_C@_1MG@JOMKLAFK@?$AAC?$AA?3?$AA?2?$AAW?$AAI?$AAN?$AAC?$AAE?$AAR?$AAO?$AAO?$AAT?$AAS?$AA?2?$AAT?$AAo?$AAp?$AAa?$AAz?$AA?2?$AAW?$AAI?$AAN?$AAC?$AAE?$AA6?$AA0?$AA0?$AA?2?$AAp?$AAl?$AAa@ 10003d68     usbh_usb2com_common_topaz_v1:cdevice.obj
 0001:00002e30       ??_C@_1DI@FHCICPGN@?$AA?$CL?$AAC?$AAD?$AAe?$AAv?$AAi?$AAc?$AAe?$AAG?$AAl?$AAo?$AAb?$AAa?$AAl?$AA?3?$AA?3?$AAI?$AAn?$AAi?$AAt?$AAi?$AAa?$AAl?$AAi?$AAz?$AAe?$AA?6?$AA?$AA@ 10003e30     usbh_usb2com_common_topaz_v1:cdevice.obj
 0001:00002e68       ??_C@_1DA@LHFPLNDP@?$AA?9?$AAC?$AAD?$AAe?$AAv?$AAi?$AAc?$AAe?$AA?3?$AA?3?$AAD?$AAe?$AAI?$AAn?$AAi?$AAt?$AAi?$AAa?$AAl?$AAi?$AAz?$AAe?$AA?6?$AA?$AA@ 10003e68     usbh_usb2com_common_topaz_v1:cdevice.obj
 0001:00002e98       ??_C@_1BE@MDMBICMJ@?$AAH?$AAc?$AAd?$AAD?$AAe?$AAt?$AAa?$AAc?$AAh?$AA?$AA@ 10003e98     usbh_usb2com_common_topaz_v1:cdevice.obj
 0001:00002eac       ??_C@_1DA@DKPLNHPH@?$AA?$CL?$AAC?$AAD?$AAe?$AAv?$AAi?$AAc?$AAe?$AA?3?$AA?3?$AAD?$AAe?$AAI?$AAn?$AAi?$AAt?$AAi?$AAa?$AAl?$AAi?$AAz?$AAe?$AA?6?$AA?$AA@ 10003eac     usbh_usb2com_common_topaz_v1:cdevice.obj
 0001:00002ee0       ??_C@_1HO@NEAGMBBN@?$AA?9?$AAC?$AAD?$AAe?$AAv?$AAi?$AAc?$AAe?$AA?3?$AA?3?$AAR?$AAe?$AAs?$AAe?$AAr?$AAv?$AAe?$AAA?$AAd?$AAd?$AAr?$AAe?$AAs?$AAs?$AA?0?$AA?5?$AAr?$AAe?$AAt?$AAu?$AAr?$AAn@ 10003ee0     usbh_usb2com_common_topaz_v1:cdevice.obj
 0001:00002f60       ??_C@_1EA@FINECAO@?$AA?$CL?$AAC?$AAD?$AAe?$AAv?$AAi?$AAc?$AAe?$AAG?$AAl?$AAo?$AAb?$AAa?$AAl?$AA?3?$AA?3?$AAR?$AAe?$AAs?$AAe?$AAr?$AAv?$AAe?$AAA?$AAd?$AAd?$AAr?$AAe?$AAs?$AAs?$AA?6?$AA?$AA@ 10003f60     usbh_usb2com_common_topaz_v1:cdevice.obj
 0001:00002fa0       ??_C@_1EM@JAIJPGKI@?$AA?9?$AAC?$AAD?$AAe?$AAv?$AAi?$AAc?$AAe?$AA?3?$AA?3?$AAF?$AAr?$AAe?$AAe?$AAA?$AAd?$AAd?$AAr?$AAe?$AAs?$AAs?$AA?5?$AA?9?$AA?5?$AAa?$AAd?$AAd?$AAr?$AAe?$AAs?$AAs?$AA?5@ 10003fa0     usbh_usb2com_common_topaz_v1:cdevice.obj
 0001:00002ff0       ??_C@_1FI@GOMGBLHC@?$AA?$CL?$AAC?$AAD?$AAe?$AAv?$AAi?$AAc?$AAe?$AAG?$AAl?$AAo?$AAb?$AAa?$AAl?$AA?3?$AA?3?$AAF?$AAr?$AAe?$AAe?$AAA?$AAd?$AAd?$AAr?$AAe?$AAs?$AAs?$AA?5?$AA?9?$AA?5?$AAa?$AAd@ 10003ff0     usbh_usb2com_common_topaz_v1:cdevice.obj
 0001:00003048       ??_C@_1CG@MCANFPKD@?$AA?9?$AAC?$AAD?$AAe?$AAv?$AAi?$AAc?$AAe?$AA?3?$AA?3?$AAC?$AAD?$AAe?$AAv?$AAi?$AAc?$AAe?$AA?6?$AA?$AA@ 10004048     usbh_usb2com_common_topaz_v1:cdevice.obj
 0001:00003070       ??_C@_1CG@FJNNFPGN@?$AA?$CL?$AAC?$AAD?$AAe?$AAv?$AAi?$AAc?$AAe?$AA?3?$AA?3?$AAC?$AAD?$AAe?$AAv?$AAi?$AAc?$AAe?$AA?6?$AA?$AA@ 10004070     usbh_usb2com_common_topaz_v1:cdevice.obj
 0001:00003098       ??_7CDevice@@6B@           10004098     usbh_usb2com_common_topaz_v1:cdevice.obj
 0001:000030d4       ??_C@_1CI@EJOBNDNG@?$AA?9?$AAC?$AAD?$AAe?$AAv?$AAi?$AAc?$AAe?$AA?3?$AA?3?$AA?$HO?$AAC?$AAD?$AAe?$AAv?$AAi?$AAc?$AAe?$AA?6?$AA?$AA@ 100040d4     usbh_usb2com_common_topaz_v1:cdevice.obj
 0001:000030fc       ??_C@_1CI@BMJILCMG@?$AA?$CL?$AAC?$AAD?$AAe?$AAv?$AAi?$AAc?$AAe?$AA?3?$AA?3?$AA?$HO?$AAC?$AAD?$AAe?$AAv?$AAi?$AAc?$AAe?$AA?6?$AA?$AA@ 100040fc     usbh_usb2com_common_topaz_v1:cdevice.obj
 0001:00003128       ??_C@_1IK@BBOLADBJ@?$AA?9?$AAC?$AAD?$AAe?$AAv?$AAi?$AAc?$AAe?$AA?3?$AA?3?$AAC?$AAr?$AAe?$AAa?$AAt?$AAe?$AAU?$AAs?$AAb?$AAC?$AAo?$AAn?$AAf?$AAi?$AAg?$AAu?$AAr?$AAa?$AAt?$AAi?$AAo?$AAn@ 10004128     usbh_usb2com_common_topaz_v1:cdevice.obj
 0001:000031b8       ??_C@_1HE@OBCNJEAP@?$AA?9?$AAC?$AAD?$AAe?$AAv?$AAi?$AAc?$AAe?$AA?3?$AA?3?$AAC?$AAr?$AAe?$AAa?$AAt?$AAe?$AAU?$AAs?$AAb?$AAC?$AAo?$AAn?$AAf?$AAi?$AAg?$AAu?$AAr?$AAa?$AAt?$AAi?$AAo?$AAn@ 100041b8     usbh_usb2com_common_topaz_v1:cdevice.obj
 0001:00003230       ??_C@_1FG@PLHAINKD@?$AA?$CL?$AAC?$AAD?$AAe?$AAv?$AAi?$AAc?$AAe?$AA?3?$AA?3?$AAC?$AAr?$AAe?$AAa?$AAt?$AAe?$AAU?$AAs?$AAb?$AAC?$AAo?$AAn?$AAf?$AAi?$AAg?$AAu?$AAr?$AAa?$AAt?$AAi?$AAo?$AAn@ 10004230     usbh_usb2com_common_topaz_v1:cdevice.obj
 0001:00003288       ??_C@_1FG@CKPOJHLM@?$AA?9?$AAC?$AAD?$AAe?$AAv?$AAi?$AAc?$AAe?$AA?3?$AA?3?$AAD?$AAe?$AAl?$AAe?$AAt?$AAe?$AAU?$AAs?$AAb?$AAC?$AAo?$AAn?$AAf?$AAi?$AAg?$AAu?$AAr?$AAa?$AAt?$AAi?$AAo?$AAn@ 10004288     usbh_usb2com_common_topaz_v1:cdevice.obj
 0001:000032e0       ??_C@_1FG@MDKEDGEC@?$AA?$CL?$AAC?$AAD?$AAe?$AAv?$AAi?$AAc?$AAe?$AA?3?$AA?3?$AAD?$AAe?$AAl?$AAe?$AAt?$AAe?$AAU?$AAs?$AAb?$AAC?$AAo?$AAn?$AAf?$AAi?$AAg?$AAu?$AAr?$AAa?$AAt?$AAi?$AAo?$AAn@ 100042e0     usbh_usb2com_common_topaz_v1:cdevice.obj
 0001:00003338       ??_C@_1HI@HLMBKNMH@?$AA?9?$AAC?$AAD?$AAe?$AAv?$AAi?$AAc?$AAe?$AA?$CI?$AA?$CF?$AAs?$AA?5?$AAt?$AAi?$AAe?$AAr?$AA?5?$AA?$CF?$AAd?$AA?$CJ?$AA?3?$AA?3?$AAA?$AAl?$AAl?$AAo?$AAc?$AAa?$AAt?$AAe?$AAP?$AAi@ 10004338     usbh_usb2com_common_topaz_v1:cdevice.obj
 0001:000033b0       ??_C@_1GK@EPJKGPON@?$AAC?$AAD?$AAe?$AAv?$AAi?$AAc?$AAe?$AA?$CI?$AA?$CF?$AAs?$AA?5?$AAt?$AAi?$AAe?$AAr?$AA?5?$AA?$CF?$AAd?$AA?$CJ?$AA?3?$AA?3?$AAA?$AAl?$AAl?$AAo?$AAc?$AAa?$AAt?$AAe?$AAP?$AAi?$AAp@ 100043b0     usbh_usb2com_common_topaz_v1:cdevice.obj
 0001:00003420       ??_C@_1JE@NPCBHKBA@?$AAC?$AAD?$AAe?$AAv?$AAi?$AAc?$AAe?$AA?$CI?$AA?$CF?$AAs?$AA?5?$AAt?$AAi?$AAe?$AAr?$AA?5?$AA?$CF?$AAd?$AA?$CJ?$AA?3?$AA?3?$AAA?$AAl?$AAl?$AAo?$AAc?$AAa?$AAt?$AAe?$AAP?$AAi?$AAp@ 10004420     usbh_usb2com_common_topaz_v1:cdevice.obj
 0001:000034b8       ??_C@_1FC@EIACOBNP@?$AA?$CL?$AAC?$AAD?$AAe?$AAv?$AAi?$AAc?$AAe?$AA?$CI?$AA?$CF?$AAs?$AA?5?$AAt?$AAi?$AAe?$AAr?$AA?5?$AA?$CF?$AAd?$AA?$CJ?$AA?3?$AA?3?$AAA?$AAl?$AAl?$AAo?$AAc?$AAa?$AAt?$AAe?$AAP?$AAi@ 100044b8     usbh_usb2com_common_topaz_v1:cdevice.obj
 0001:0000350c       ??_C@_1DK@MGILKFGP@?$AA?9?$AAD?$AAu?$AAm?$AAp?$AA?5?$AAU?$AAS?$AAB?$AA_?$AAD?$AAE?$AAV?$AAI?$AAC?$AAE?$AA_?$AAD?$AAE?$AAS?$AAC?$AAR?$AAI?$AAP?$AAT?$AAO?$AAR?$AA?6?$AA?$AA@ 1000450c     usbh_usb2com_common_topaz_v1:cdevice.obj
 0001:00003548       ??_C@_1DM@HKEDEOHI@?$AA?7?$AAb?$AAN?$AAu?$AAm?$AAC?$AAo?$AAn?$AAf?$AAi?$AAg?$AAu?$AAr?$AAa?$AAt?$AAi?$AAo?$AAn?$AAs?$AA?5?$AA?$DN?$AA?5?$AA0?$AAx?$AA?$CF?$AA0?$AA2?$AAx?$AA?6?$AA?$AA@ 10004548     usbh_usb2com_common_topaz_v1:cdevice.obj
 0001:00003584       ??_C@_1DC@KFEMFLN@?$AA?7?$AAi?$AAS?$AAe?$AAr?$AAi?$AAa?$AAl?$AAN?$AAu?$AAm?$AAb?$AAe?$AAr?$AA?5?$AA?$DN?$AA?5?$AA0?$AAx?$AA?$CF?$AA0?$AA2?$AAx?$AA?6?$AA?$AA@ 10004584     usbh_usb2com_common_topaz_v1:cdevice.obj
 0001:000035b8       ??_C@_1CI@KLPGHDHJ@?$AA?7?$AAi?$AAP?$AAr?$AAo?$AAd?$AAu?$AAc?$AAt?$AA?5?$AA?$DN?$AA?5?$AA0?$AAx?$AA?$CF?$AA0?$AA2?$AAx?$AA?6?$AA?$AA@ 100045b8     usbh_usb2com_common_topaz_v1:cdevice.obj
 0001:000035e0       ??_C@_1DC@GGENBBGM@?$AA?7?$AAi?$AAM?$AAa?$AAn?$AAu?$AAf?$AAa?$AAc?$AAt?$AAu?$AAr?$AAe?$AAr?$AA?5?$AA?$DN?$AA?5?$AA0?$AAx?$AA?$CF?$AA0?$AA2?$AAx?$AA?6?$AA?$AA@ 100045e0     usbh_usb2com_common_topaz_v1:cdevice.obj
 0001:00003614       ??_C@_1CK@PABHMLCI@?$AA?7?$AAb?$AAc?$AAd?$AAD?$AAe?$AAv?$AAi?$AAc?$AAe?$AA?5?$AA?$DN?$AA?5?$AA0?$AAx?$AA?$CF?$AA0?$AA4?$AAx?$AA?6?$AA?$AA@ 10004614     usbh_usb2com_common_topaz_v1:cdevice.obj
 0001:00003640       ??_C@_1CK@POCACHBF@?$AA?7?$AAi?$AAd?$AAP?$AAr?$AAo?$AAd?$AAu?$AAc?$AAt?$AA?5?$AA?$DN?$AA?5?$AA0?$AAx?$AA?$CF?$AA0?$AA4?$AAx?$AA?6?$AA?$AA@ 10004640     usbh_usb2com_common_topaz_v1:cdevice.obj
 0001:0000366c       ??_C@_1CI@DKBCNBPN@?$AA?7?$AAi?$AAd?$AAV?$AAe?$AAn?$AAd?$AAo?$AAr?$AA?5?$AA?$DN?$AA?5?$AA0?$AAx?$AA?$CF?$AA0?$AA4?$AAx?$AA?6?$AA?$AA@ 1000466c     usbh_usb2com_common_topaz_v1:cdevice.obj
 0001:00003694       ??_C@_1DG@DNBBNAFE@?$AA?7?$AAb?$AAM?$AAa?$AAx?$AAP?$AAa?$AAc?$AAk?$AAe?$AAt?$AAS?$AAi?$AAz?$AAe?$AA0?$AA?5?$AA?$DN?$AA?5?$AA0?$AAx?$AA?$CF?$AA0?$AA2?$AAx?$AA?6?$AA?$AA@ 10004694     usbh_usb2com_common_topaz_v1:cdevice.obj
 0001:000036cc       ??_C@_1DG@ILHCOCOC@?$AA?7?$AAb?$AAD?$AAe?$AAv?$AAi?$AAc?$AAe?$AAP?$AAr?$AAo?$AAt?$AAo?$AAc?$AAo?$AAl?$AA?5?$AA?$DN?$AA?5?$AA0?$AAx?$AA?$CF?$AA0?$AA2?$AAx?$AA?6?$AA?$AA@ 100046cc     usbh_usb2com_common_topaz_v1:cdevice.obj
 0001:00003704       ??_C@_1DG@ECOHLBJB@?$AA?7?$AAb?$AAD?$AAe?$AAv?$AAi?$AAc?$AAe?$AAS?$AAu?$AAb?$AAC?$AAl?$AAa?$AAs?$AAs?$AA?5?$AA?$DN?$AA?5?$AA0?$AAx?$AA?$CF?$AA0?$AA2?$AAx?$AA?6?$AA?$AA@ 10004704     usbh_usb2com_common_topaz_v1:cdevice.obj
 0001:0000373c       ??_C@_1DA@OGADBMKG@?$AA?7?$AAb?$AAD?$AAe?$AAv?$AAi?$AAc?$AAe?$AAC?$AAl?$AAa?$AAs?$AAs?$AA?5?$AA?$DN?$AA?5?$AA0?$AAx?$AA?$CF?$AA0?$AA2?$AAx?$AA?6?$AA?$AA@ 1000473c     usbh_usb2com_common_topaz_v1:cdevice.obj
 0001:0000376c       ??_C@_1CE@KILHOIAM@?$AA?7?$AAb?$AAc?$AAd?$AAU?$AAS?$AAB?$AA?5?$AA?$DN?$AA?5?$AA0?$AAx?$AA?$CF?$AA0?$AA4?$AAx?$AA?6?$AA?$AA@ 1000476c     usbh_usb2com_common_topaz_v1:cdevice.obj
 0001:00003790       ??_C@_1DG@KKACGDHH@?$AA?7?$AAb?$AAD?$AAe?$AAs?$AAc?$AAr?$AAi?$AAp?$AAt?$AAo?$AAr?$AAT?$AAy?$AAp?$AAe?$AA?5?$AA?$DN?$AA?5?$AA0?$AAx?$AA?$CF?$AA0?$AA2?$AAx?$AA?6?$AA?$AA@ 10004790     usbh_usb2com_common_topaz_v1:cdevice.obj
 0001:000037c8       ??_C@_1CG@HCKNJKHJ@?$AA?7?$AAb?$AAL?$AAe?$AAn?$AAg?$AAt?$AAh?$AA?5?$AA?$DN?$AA?5?$AA0?$AAx?$AA?$CF?$AA0?$AA2?$AAx?$AA?6?$AA?$AA@ 100047c8     usbh_usb2com_common_topaz_v1:cdevice.obj
 0001:000037f0       ??_C@_1DK@KDGIICEE@?$AA?$CL?$AAD?$AAu?$AAm?$AAp?$AA?5?$AAU?$AAS?$AAB?$AA_?$AAD?$AAE?$AAV?$AAI?$AAC?$AAE?$AA_?$AAD?$AAE?$AAS?$AAC?$AAR?$AAI?$AAP?$AAT?$AAO?$AAR?$AA?6?$AA?$AA@ 100047f0     usbh_usb2com_common_topaz_v1:cdevice.obj
 0001:00003830       ??_C@_1EI@GPGKHEHH@?$AA?9?$AAD?$AAu?$AAm?$AAp?$AA?5?$AAU?$AAS?$AAB?$AA_?$AAC?$AAO?$AAN?$AAF?$AAI?$AAG?$AAU?$AAR?$AAA?$AAT?$AAI?$AAO?$AAN?$AA_?$AAD?$AAE?$AAS?$AAC?$AAR?$AAI?$AAP?$AAT@ 10004830     usbh_usb2com_common_topaz_v1:cdevice.obj
 0001:00003878       ??_C@_1CI@BHMCOMDM@?$AA?7?$AAM?$AAa?$AAx?$AAP?$AAo?$AAw?$AAe?$AAr?$AA?5?$AA?$DN?$AA?5?$AA0?$AAx?$AA?$CF?$AA0?$AA2?$AAx?$AA?6?$AA?$AA@ 10004878     usbh_usb2com_common_topaz_v1:cdevice.obj
 0001:000038a0       ??_C@_1EI@OGFINNGI@?$AA?7?$AA?7?$AAb?$AAm?$AAA?$AAt?$AAt?$AAr?$AAi?$AAb?$AAu?$AAt?$AAe?$AAs?$AA?0?$AA?5?$AAR?$AAe?$AAm?$AAo?$AAt?$AAe?$AA?5?$AAW?$AAa?$AAk?$AAe?$AAu?$AAp?$AA?5?$AA?$DN?$AA?5@ 100048a0     usbh_usb2com_common_topaz_v1:cdevice.obj
 0001:000038e8       ??_C@_1EG@JGMNAAKF@?$AA?7?$AA?7?$AAb?$AAm?$AAA?$AAt?$AAt?$AAr?$AAi?$AAb?$AAu?$AAt?$AAe?$AAs?$AA?0?$AA?5?$AAS?$AAe?$AAl?$AAf?$AA?5?$AAP?$AAo?$AAw?$AAe?$AAr?$AAe?$AAd?$AA?5?$AA?$DN?$AA?5?$AA?$CF@ 100048e8     usbh_usb2com_common_topaz_v1:cdevice.obj
 0001:00003930       ??_C@_1EE@FIOJAKAP@?$AA?7?$AA?7?$AAb?$AAm?$AAA?$AAt?$AAt?$AAr?$AAi?$AAb?$AAu?$AAt?$AAe?$AAs?$AA?0?$AA?5?$AAB?$AAu?$AAs?$AA?5?$AAP?$AAo?$AAw?$AAe?$AAr?$AAe?$AAd?$AA?5?$AA?$DN?$AA?5?$AA?$CF?$AAd@ 10004930     usbh_usb2com_common_topaz_v1:cdevice.obj
 0001:00003974       ??_C@_1DA@LCDJCEML@?$AA?7?$AAb?$AAm?$AAA?$AAt?$AAt?$AAr?$AAi?$AAb?$AAu?$AAt?$AAe?$AAs?$AA?5?$AA?$DN?$AA?5?$AA0?$AAx?$AA?$CF?$AA0?$AA2?$AAx?$AA?6?$AA?$AA@ 10004974     usbh_usb2com_common_topaz_v1:cdevice.obj
 0001:000039a4       ??_C@_1DE@DPPBJEKC@?$AA?7?$AAi?$AAC?$AAo?$AAn?$AAf?$AAi?$AAg?$AAu?$AAr?$AAa?$AAt?$AAi?$AAo?$AAn?$AA?5?$AA?$DN?$AA?5?$AA0?$AAx?$AA?$CF?$AA0?$AA2?$AAx?$AA?6?$AA?$AA@ 100049a4     usbh_usb2com_common_topaz_v1:cdevice.obj
 0001:000039d8       ??_C@_1DO@IEJMMIGI@?$AA?7?$AAb?$AAC?$AAo?$AAn?$AAf?$AAi?$AAg?$AAu?$AAr?$AAa?$AAt?$AAi?$AAo?$AAn?$AAV?$AAa?$AAl?$AAu?$AAe?$AA?5?$AA?$DN?$AA?5?$AA0?$AAx?$AA?$CF?$AA0?$AA2?$AAx?$AA?6?$AA?$AA@ 100049d8     usbh_usb2com_common_topaz_v1:cdevice.obj
 0001:00003a18       ??_C@_1DE@CEAKMJHK@?$AA?7?$AAb?$AAN?$AAu?$AAm?$AAI?$AAn?$AAt?$AAe?$AAr?$AAf?$AAa?$AAc?$AAe?$AAs?$AA?5?$AA?$DN?$AA?5?$AA0?$AAx?$AA?$CF?$AA0?$AA2?$AAx?$AA?6?$AA?$AA@ 10004a18     usbh_usb2com_common_topaz_v1:cdevice.obj
 0001:00003a4c       ??_C@_1DA@BIBJMFOD@?$AA?7?$AAw?$AAT?$AAo?$AAt?$AAa?$AAl?$AAL?$AAe?$AAn?$AAg?$AAt?$AAh?$AA?5?$AA?$DN?$AA?5?$AA0?$AAx?$AA?$CF?$AA0?$AA4?$AAx?$AA?6?$AA?$AA@ 10004a4c     usbh_usb2com_common_topaz_v1:cdevice.obj
 0001:00003a80       ??_C@_1EI@DNLDJBIN@?$AA?$CL?$AAD?$AAu?$AAm?$AAp?$AA?5?$AAU?$AAS?$AAB?$AA_?$AAC?$AAO?$AAN?$AAF?$AAI?$AAG?$AAU?$AAR?$AAA?$AAT?$AAI?$AAO?$AAN?$AA_?$AAD?$AAE?$AAS?$AAC?$AAR?$AAI?$AAP?$AAT@ 10004a80     usbh_usb2com_common_topaz_v1:cdevice.obj
 0001:00003ac8       ??_C@_1EA@GKDHLAHP@?$AA?9?$AAD?$AAu?$AAm?$AAp?$AA?5?$AAU?$AAS?$AAB?$AA_?$AAI?$AAN?$AAT?$AAE?$AAR?$AAF?$AAA?$AAC?$AAE?$AA_?$AAD?$AAE?$AAS?$AAC?$AAR?$AAI?$AAP?$AAT?$AAO?$AAR?$AA?6?$AA?$AA@ 10004ac8     usbh_usb2com_common_topaz_v1:cdevice.obj
 0001:00003b08       ??_C@_1CM@MOJHGEFA@?$AA?7?$AAi?$AAI?$AAn?$AAt?$AAe?$AAr?$AAf?$AAa?$AAc?$AAe?$AA?5?$AA?$DN?$AA?5?$AA0?$AAx?$AA?$CF?$AA0?$AA2?$AAx?$AA?6?$AA?$AA@ 10004b08     usbh_usb2com_common_topaz_v1:cdevice.obj
 0001:00003b34       ??_C@_1DM@NGGHHJBN@?$AA?7?$AAb?$AAI?$AAn?$AAt?$AAe?$AAr?$AAf?$AAa?$AAc?$AAe?$AAP?$AAr?$AAo?$AAt?$AAo?$AAc?$AAo?$AAl?$AA?5?$AA?$DN?$AA?5?$AA0?$AAx?$AA?$CF?$AA0?$AA2?$AAx?$AA?6?$AA?$AA@ 10004b34     usbh_usb2com_common_topaz_v1:cdevice.obj
 0001:00003b70       ??_C@_1DM@BPPCCKGO@?$AA?7?$AAb?$AAI?$AAn?$AAt?$AAe?$AAr?$AAf?$AAa?$AAc?$AAe?$AAS?$AAu?$AAb?$AAC?$AAl?$AAa?$AAs?$AAs?$AA?5?$AA?$DN?$AA?5?$AA0?$AAx?$AA?$CF?$AA0?$AA2?$AAx?$AA?6?$AA?$AA@ 10004b70     usbh_usb2com_common_topaz_v1:cdevice.obj
 0001:00003bac       ??_C@_1DG@GGHLMIAK@?$AA?7?$AAb?$AAI?$AAn?$AAt?$AAe?$AAr?$AAf?$AAa?$AAc?$AAe?$AAC?$AAl?$AAa?$AAs?$AAs?$AA?5?$AA?$DN?$AA?5?$AA0?$AAx?$AA?$CF?$AA0?$AA2?$AAx?$AA?6?$AA?$AA@ 10004bac     usbh_usb2com_common_topaz_v1:cdevice.obj
 0001:00003be4       ??_C@_1DC@PJPDJIP@?$AA?7?$AAb?$AAN?$AAu?$AAm?$AAE?$AAn?$AAd?$AAp?$AAo?$AAi?$AAn?$AAt?$AAs?$AA?5?$AA?$DN?$AA?5?$AA0?$AAx?$AA?$CF?$AA0?$AA2?$AAx?$AA?6?$AA?$AA@ 10004be4     usbh_usb2com_common_topaz_v1:cdevice.obj
 0001:00003c18       ??_C@_1DK@MJEAGMPA@?$AA?7?$AAb?$AAA?$AAl?$AAt?$AAe?$AAr?$AAn?$AAa?$AAt?$AAe?$AAS?$AAe?$AAt?$AAt?$AAi?$AAn?$AAg?$AA?5?$AA?$DN?$AA?5?$AA0?$AAx?$AA?$CF?$AA0?$AA2?$AAx?$AA?6?$AA?$AA@ 10004c18     usbh_usb2com_common_topaz_v1:cdevice.obj
 0001:00003c54       ??_C@_1DI@OBBAOB@?$AA?7?$AAb?$AAI?$AAn?$AAt?$AAe?$AAr?$AAf?$AAa?$AAc?$AAe?$AAN?$AAu?$AAm?$AAb?$AAe?$AAr?$AA?5?$AA?$DN?$AA?5?$AA0?$AAx?$AA?$CF?$AA0?$AA2?$AAx?$AA?6?$AA?$AA@ 10004c54     usbh_usb2com_common_topaz_v1:cdevice.obj
 0001:00003c90       ??_C@_1EA@POGLFBID@?$AA?$CL?$AAD?$AAu?$AAm?$AAp?$AA?5?$AAU?$AAS?$AAB?$AA_?$AAI?$AAN?$AAT?$AAE?$AAR?$AAF?$AAA?$AAC?$AAE?$AA_?$AAD?$AAE?$AAS?$AAC?$AAR?$AAI?$AAP?$AAT?$AAO?$AAR?$AA?6?$AA?$AA@ 10004c90     usbh_usb2com_common_topaz_v1:cdevice.obj
 0001:00003cd0       ??_C@_1DO@PFLJDGOH@?$AA?9?$AAD?$AAu?$AAm?$AAp?$AA?5?$AAU?$AAS?$AAB?$AA_?$AAE?$AAN?$AAD?$AAP?$AAO?$AAI?$AAN?$AAT?$AA_?$AAD?$AAE?$AAS?$AAC?$AAR?$AAI?$AAP?$AAT?$AAO?$AAR?$AA?6?$AA?$AA@ 10004cd0     usbh_usb2com_common_topaz_v1:cdevice.obj
 0001:00003d10       ??_C@_1CK@LLJPEFDK@?$AA?7?$AAb?$AAI?$AAn?$AAt?$AAe?$AAr?$AAv?$AAa?$AAl?$AA?5?$AA?$DN?$AA?5?$AA0?$AAx?$AA?$CF?$AA0?$AA2?$AAx?$AA?6?$AA?$AA@ 10004d10     usbh_usb2com_common_topaz_v1:cdevice.obj
 0001:00003d3c       ??_C@_1DE@FKEFDAJI@?$AA?7?$AAw?$AAM?$AAa?$AAx?$AAP?$AAa?$AAc?$AAk?$AAe?$AAt?$AAS?$AAi?$AAz?$AAe?$AA?5?$AA?$DN?$AA?5?$AA0?$AAx?$AA?$CF?$AA0?$AA4?$AAx?$AA?6?$AA?$AA@ 10004d3c     usbh_usb2com_common_topaz_v1:cdevice.obj
 0001:00003d70       ??_C@_1EI@IBEEEFHL@?$AA?7?$AA?7?$AAb?$AAm?$AAA?$AAt?$AAt?$AAr?$AAi?$AAb?$AAu?$AAt?$AAe?$AAs?$AA?0?$AA?5?$AAe?$AAn?$AAd?$AAp?$AAo?$AAi?$AAn?$AAt?$AA?5?$AAt?$AAy?$AAp?$AAe?$AA?5?$AA?$DN?$AA?5@ 10004d70     usbh_usb2com_common_topaz_v1:cdevice.obj
 0001:00003db8       ??_C@_1EI@JPGNKMBJ@?$AA?7?$AA?7?$AAb?$AAE?$AAn?$AAd?$AAp?$AAo?$AAi?$AAn?$AAt?$AAA?$AAd?$AAd?$AAr?$AAe?$AAs?$AAs?$AA?0?$AA?5?$AAd?$AAi?$AAr?$AAe?$AAc?$AAt?$AAi?$AAo?$AAn?$AA?5?$AA?$DN?$AA?5@ 10004db8     usbh_usb2com_common_topaz_v1:cdevice.obj
 0001:00003e00       ??_C@_17HCEMPBGG@?$AAO?$AAU?$AAT?$AA?$AA@ 10004e00     usbh_usb2com_common_topaz_v1:cdevice.obj
 0001:00003e08       ??_C@_15BNKBCKPG@?$AAI?$AAN?$AA?$AA@ 10004e08     usbh_usb2com_common_topaz_v1:cdevice.obj
 0001:00003e10       ??_C@_1EK@FBMFPAGP@?$AA?7?$AA?7?$AAb?$AAE?$AAn?$AAd?$AAp?$AAo?$AAi?$AAn?$AAt?$AAA?$AAd?$AAd?$AAr?$AAe?$AAs?$AAs?$AA?0?$AA?5?$AAe?$AAn?$AAd?$AAp?$AAo?$AAi?$AAn?$AAt?$AA?5?$AA?$CD?$AA?5?$AA?$DN@ 10004e10     usbh_usb2com_common_topaz_v1:cdevice.obj
 0001:00003e5c       ??_C@_1DI@MCPDKGOI@?$AA?7?$AAb?$AAE?$AAn?$AAd?$AAp?$AAo?$AAi?$AAn?$AAt?$AAA?$AAd?$AAd?$AAr?$AAe?$AAs?$AAs?$AA?5?$AA?$DN?$AA?5?$AA0?$AAx?$AA?$CF?$AA0?$AA2?$AAx?$AA?6?$AA?$AA@ 10004e5c     usbh_usb2com_common_topaz_v1:cdevice.obj
 0001:00003e94       ??_C@_1DO@PHADHLEF@?$AA?$CL?$AAD?$AAu?$AAm?$AAp?$AA?5?$AAU?$AAS?$AAB?$AA_?$AAE?$AAN?$AAD?$AAP?$AAO?$AAI?$AAN?$AAT?$AA_?$AAD?$AAE?$AAS?$AAC?$AAR?$AAI?$AAP?$AAT?$AAO?$AAR?$AA?6?$AA?$AA@ 10004e94     usbh_usb2com_common_topaz_v1:cdevice.obj
 0001:00003ed4       ??_C@_1BA@FCLNFMPO@?$AAC?$AAO?$AAN?$AAT?$AAR?$AAO?$AAL?$AA?$AA@ 10004ed4     usbh_usb2com_common_topaz_v1:cdevice.obj
 0001:00003ee4       ??_C@_1BI@EGKNLPFO@?$AAI?$AAS?$AAO?$AAC?$AAH?$AAR?$AAO?$AAN?$AAO?$AAU?$AAS?$AA?$AA@ 10004ee4     usbh_usb2com_common_topaz_v1:cdevice.obj
 0001:00003efc       ??_C@_19KPHDKIJN@?$AAB?$AAU?$AAL?$AAK?$AA?$AA@ 10004efc     usbh_usb2com_common_topaz_v1:cdevice.obj
 0001:00003f08       ??_C@_1BE@HPDKKJEA@?$AAI?$AAN?$AAT?$AAE?$AAR?$AAR?$AAU?$AAP?$AAT?$AA?$AA@ 10004f08     usbh_usb2com_common_topaz_v1:cdevice.obj
 0001:00003f20       ??_C@_1EC@KLPCLDKE@?$AA?9?$AAD?$AAu?$AAm?$AAp?$AA?5?$AAe?$AAx?$AAt?$AAe?$AAn?$AAd?$AAe?$AAd?$AA?5?$AAb?$AAy?$AAt?$AAe?$AAs?$AA?0?$AA?5?$AAs?$AAi?$AAz?$AAe?$AA?5?$AA?$DN?$AA?5?$AA?$CF?$AAd?$AA?6@ 10004f20     usbh_usb2com_common_topaz_v1:cdevice.obj
 0001:00003f64       ??_C@_1DE@GIBFNBPI@?$AA?7?$AAB?$AAy?$AAt?$AAe?$AAs?$AA?5?$AA?$CF?$AAd?$AA?5?$AAt?$AAo?$AA?5?$AA?$CF?$AAd?$AA?5?$AA?$DN?$AA?5?$AA0?$AAx?$AA?$CF?$AA0?$AA8?$AAx?$AA?6?$AA?$AA@ 10004f64     usbh_usb2com_common_topaz_v1:cdevice.obj
 0001:00003f98       ??_C@_1EC@MEPGFLKH@?$AA?$CL?$AAD?$AAu?$AAm?$AAp?$AA?5?$AAe?$AAx?$AAt?$AAe?$AAn?$AAd?$AAe?$AAd?$AA?5?$AAb?$AAy?$AAt?$AAe?$AAs?$AA?0?$AA?5?$AAs?$AAi?$AAz?$AAe?$AA?5?$AA?$DN?$AA?5?$AA?$CF?$AAd?$AA?6@ 10004f98     usbh_usb2com_common_topaz_v1:cdevice.obj
 0001:00003fe0       ??_C@_1FC@MKNFGBBO@?$AAC?$AAd?$AAe?$AAv?$AAi?$AAc?$AAe?$AA?3?$AA?5?$AAC?$AAr?$AAe?$AAa?$AAt?$AAe?$AA?5?$AAE?$AAv?$AAe?$AAn?$AAt?$AA?5?$AAF?$AAa?$AAi?$AAl?$AAe?$AAd?$AA?5?$AAf?$AAo?$AAr@ 10004fe0     usbh_usb2com_common_topaz_v1:cdevice.obj
 0001:00004038       ??_C@_1EI@DLCCEPPA@?$AAC?$AAD?$AAe?$AAv?$AAi?$AAc?$AAe?$AA?3?$AA?5?$AAC?$AAr?$AAe?$AAa?$AAt?$AAe?$AAd?$AA?5?$AAa?$AA?5?$AAn?$AAe?$AAw?$AA?5?$AAF?$AAu?$AAn?$AAc?$AA?5?$AAE?$AAv?$AAe?$AAn@ 10005038     usbh_usb2com_common_topaz_v1:cdevice.obj
 0001:00004080       ??_C@_1FC@IHBOEJHC@?$AAC?$AAd?$AAe?$AAv?$AAi?$AAc?$AAe?$AA?3?$AA?5?$AAO?$AAp?$AAe?$AAn?$AAe?$AAd?$AA?5?$AAa?$AAn?$AA?5?$AAe?$AAx?$AAi?$AAs?$AAt?$AAi?$AAn?$AAg?$AA?5?$AAF?$AAu?$AAn?$AAc@ 10005080     usbh_usb2com_common_topaz_v1:cdevice.obj
 0001:000040d4       ??_C@_1BE@KCBNNJPA@?$AAU?$AAS?$AAB?$AAD?$AAe?$AAt?$AAa?$AAc?$AAh?$AA?$AA@ 100050d4     usbh_usb2com_common_topaz_v1:cdevice.obj
 0001:000040e8       ??_C@_1BK@DEBFAAFC@?$AA?9?$AAC?$AAH?$AAu?$AAb?$AA?3?$AA?3?$AAC?$AAH?$AAu?$AAb?$AA?6?$AA?$AA@ 100050e8     usbh_usb2com_common_topaz_v1:cdevice.obj
 0001:00004104       ??_C@_1BK@LMLNNOD@?$AA?$CL?$AAC?$AAH?$AAu?$AAb?$AA?3?$AA?3?$AAC?$AAH?$AAu?$AAb?$AA?6?$AA?$AA@ 10005104     usbh_usb2com_common_topaz_v1:cdevice.obj
 0001:00004120       ??_7CHub@@6B@              10005120     usbh_usb2com_common_topaz_v1:cdevice.obj
 0001:00004188       ??_C@_1FK@LOPDGCEF@?$AAC?$AAH?$AAu?$AAb?$AA?$CI?$AA?$CF?$AAs?$AA?5?$AAt?$AAi?$AAe?$AAr?$AA?5?$AA?$CF?$AAd?$AA?$CJ?$AA?3?$AA?3?$AA?5?$AAR?$AAe?$AAs?$AAu?$AAm?$AAe?$AAN?$AAo?$AAt?$AAi?$AAf?$AAi?$AAc@ 10005188     usbh_usb2com_common_topaz_v1:cdevice.obj
 0001:000041e4       ??_C@_1BM@IFFKMHML@?$AA?9?$AAC?$AAH?$AAu?$AAb?$AA?3?$AA?3?$AA?$HO?$AAC?$AAH?$AAu?$AAb?$AA?6?$AA?$AA@ 100051e4     usbh_usb2com_common_topaz_v1:cdevice.obj
 0001:00004200       ??_C@_1BM@IAOGMJIF@?$AA?$CL?$AAC?$AAH?$AAu?$AAb?$AA?3?$AA?3?$AA?$HO?$AAC?$AAH?$AAu?$AAb?$AA?6?$AA?$AA@ 10005200     usbh_usb2com_common_topaz_v1:cdevice.obj
 0001:00004220       ??_C@_1IO@PBDBAMLH@?$AA?9?$AAC?$AAH?$AAu?$AAb?$AA?$CI?$AA?$CF?$AAs?$AA?5?$AAt?$AAi?$AAe?$AAr?$AA?5?$AA?$CF?$AAd?$AA?$CJ?$AA?3?$AA?3?$AAH?$AAu?$AAb?$AAS?$AAt?$AAa?$AAt?$AAu?$AAs?$AAC?$AAh?$AAa?$AAn@ 10005220     usbh_usb2com_common_topaz_v1:cdevice.obj
 0001:000042b0       ??_C@_1IM@FADCMJIB@?$AAC?$AAH?$AAu?$AAb?$AA?$CI?$AA?$CF?$AAs?$AA?5?$AAt?$AAi?$AAe?$AAr?$AA?5?$AA?$CF?$AAd?$AA?$CJ?$AA?3?$AA?3?$AAH?$AAu?$AAb?$AAS?$AAt?$AAa?$AAt?$AAu?$AAs?$AAC?$AAh?$AAa?$AAn?$AAg@ 100052b0     usbh_usb2com_common_topaz_v1:cdevice.obj
 0001:00004340       ??_C@_1KC@HAEJMCEO@?$AAC?$AAH?$AAu?$AAb?$AA?$CI?$AA?$CF?$AAs?$AA?5?$AAt?$AAi?$AAe?$AAr?$AA?5?$AA?$CF?$AAd?$AA?$CJ?$AA?3?$AA?3?$AAH?$AAu?$AAb?$AAS?$AAt?$AAa?$AAt?$AAu?$AAs?$AAC?$AAh?$AAa?$AAn?$AAg@ 10005340     usbh_usb2com_common_topaz_v1:cdevice.obj
 0001:000043e8       ??_C@_1IM@EDNNMFKN@?$AAC?$AAH?$AAu?$AAb?$AA?$CI?$AA?$CF?$AAs?$AA?5?$AAt?$AAi?$AAe?$AAr?$AA?5?$AA?$CF?$AAd?$AA?$CJ?$AA?3?$AA?3?$AAH?$AAu?$AAb?$AAS?$AAt?$AAa?$AAt?$AAu?$AAs?$AAC?$AAh?$AAa?$AAn?$AAg@ 100053e8     usbh_usb2com_common_topaz_v1:cdevice.obj
 0001:00004478       ??_C@_1PM@EEDHHKA@?$AAC?$AAH?$AAu?$AAb?$AA?$CI?$AA?$CF?$AAs?$AA?5?$AAt?$AAi?$AAe?$AAr?$AA?5?$AA?$CF?$AAd?$AA?$CJ?$AA?3?$AA?3?$AAH?$AAu?$AAb?$AAS?$AAt?$AAa?$AAt?$AAu?$AAs?$AAC?$AAh?$AAa?$AAn?$AAg@ 10005478     usbh_usb2com_common_topaz_v1:cdevice.obj
 0001:00004578       ??_C@_1GC@EOPJDNON@?$AAh?$AAu?$AAb?$AAS?$AAt?$AAa?$AAt?$AAu?$AAs?$AA?4?$AAc?$AAh?$AAa?$AAn?$AAg?$AAe?$AA?4?$AAp?$AAo?$AAr?$AAt?$AA?4?$AAC?$AAo?$AAn?$AAn?$AAe?$AAc?$AAt?$AAS?$AAt?$AAa@ 10005578     usbh_usb2com_common_topaz_v1:cdevice.obj
 0001:000045dc       ??_C@_1DK@FOIHOBDN@?$AAh?$AAu?$AAb?$AAS?$AAt?$AAa?$AAt?$AAu?$AAs?$AA?5?$AAF?$AAo?$AAr?$AAc?$AAe?$AAD?$AAe?$AAt?$AAa?$AAc?$AAh?$AA?5?$AA?$DN?$AA?5?$AA?$CF?$AAd?$AA?$AN?$AA?6?$AA?$AA@ 100055dc     usbh_usb2com_common_topaz_v1:cdevice.obj
 0001:00004618       ??_C@_1DO@FNMMJLDI@?$AAh?$AAu?$AAb?$AAS?$AAt?$AAa?$AAt?$AAu?$AAs?$AA?5?$AAP?$AAo?$AAr?$AAt?$AAC?$AAo?$AAn?$AAn?$AAe?$AAc?$AAt?$AAe?$AAd?$AA?5?$AA?$DN?$AA?5?$AA?$CF?$AAd?$AA?$AN?$AA?6?$AA?$AA@ 10005618     usbh_usb2com_common_topaz_v1:cdevice.obj
 0001:00004658       ??_C@_1DK@IDFICJDI@?$AAh?$AAu?$AAb?$AAS?$AAt?$AAa?$AAt?$AAu?$AAs?$AA?5?$AAP?$AAo?$AAr?$AAt?$AAE?$AAn?$AAa?$AAb?$AAl?$AAe?$AAd?$AA?5?$AA?$DN?$AA?5?$AA?$CF?$AAd?$AA?$AN?$AA?6?$AA?$AA@ 10005658     usbh_usb2com_common_topaz_v1:cdevice.obj
 0001:00004698       ??_C@_1EE@NMIDHFNG@?$AAh?$AAu?$AAb?$AAS?$AAt?$AAa?$AAt?$AAu?$AAs?$AA?5?$AAP?$AAo?$AAr?$AAt?$AAE?$AAn?$AAa?$AAb?$AAl?$AAe?$AAC?$AAh?$AAa?$AAn?$AAg?$AAe?$AA?5?$AA?$DN?$AA?5?$AA?$CF?$AAd?$AA?$AN@ 10005698     usbh_usb2com_common_topaz_v1:cdevice.obj
 0001:000046e0       ??_C@_1KK@GDICOEKP@?$AAC?$AAH?$AAu?$AAb?$AA?$CI?$AA?$CF?$AAs?$AA?5?$AAt?$AAi?$AAe?$AAr?$AA?5?$AA?$CF?$AAd?$AA?$CJ?$AA?3?$AA?3?$AAH?$AAu?$AAb?$AAS?$AAt?$AAa?$AAt?$AAu?$AAs?$AAC?$AAh?$AAa?$AAn?$AAg@ 100056e0     usbh_usb2com_common_topaz_v1:cdevice.obj
 0001:00004790       ??_C@_1JI@MHBMAJKN@?$AAC?$AAH?$AAu?$AAb?$AA?$CI?$AA?$CF?$AAs?$AA?5?$AAt?$AAi?$AAe?$AAr?$AA?5?$AA?$CF?$AAd?$AA?$CJ?$AA?3?$AA?3?$AAH?$AAu?$AAb?$AAS?$AAt?$AAa?$AAt?$AAu?$AAs?$AAC?$AAh?$AAa?$AAn?$AAg@ 10005790     usbh_usb2com_common_topaz_v1:cdevice.obj
 0001:00004828       ??_C@_1GG@KLDEFPJM@?$AAC?$AAH?$AAu?$AAb?$AA?$CI?$AA?$CF?$AAs?$AA?5?$AAt?$AAi?$AAe?$AAr?$AA?5?$AA?$CF?$AAd?$AA?$CJ?$AA?3?$AA?3?$AA?5?$AAS?$AAu?$AAs?$AAp?$AAe?$AAn?$AAd?$AA?5?$AAD?$AAe?$AAv?$AAi?$AAc@ 10005828     usbh_usb2com_common_topaz_v1:cdevice.obj
 0001:00004890       ??_C@_19JDHDJODM@?$AAF?$AAA?$AAI?$AAL?$AA?$AA@ 10005890     usbh_usb2com_common_topaz_v1:cdevice.obj
 0001:0000489c       ??_C@_1BA@JFDCMKFN@?$AAS?$AAu?$AAc?$AAc?$AAe?$AAs?$AAs?$AA?$AA@ 1000589c     usbh_usb2com_common_topaz_v1:cdevice.obj
 0001:000048ac       ??_C@_1DE@GJLHELMP@?$AAG?$AAe?$AAt?$AAF?$AAo?$AAr?$AAc?$AAe?$AAR?$AAe?$AAA?$AAt?$AAt?$AAa?$AAc?$AAh?$AA?5?$AA?$DN?$AA?5?$AA0?$AAx?$AA?$CF?$AAx?$AA?$AN?$AA?6?$AA?$AA@ 100058ac     usbh_usb2com_common_topaz_v1:cdevice.obj
 0001:000048e0       ??_C@_1FM@BCEGBMEC@?$AAH?$AAu?$AAb?$AAP?$AAo?$AAr?$AAt?$AAS?$AAt?$AAa?$AAt?$AAu?$AAs?$AAC?$AAh?$AAa?$AAn?$AAg?$AAe?$AA?5?$AAr?$AAe?$AAq?$AAu?$AAe?$AAs?$AAt?$AA?5?$AAb?$AAa?$AAc?$AAk@ 100058e0     usbh_usb2com_common_topaz_v1:cdevice.obj
 0001:00004940       ??_C@_1FE@KFAAOPKI@?$AA?$CL?$AAC?$AAH?$AAu?$AAb?$AA?$CI?$AA?$CF?$AAs?$AA?5?$AAt?$AAi?$AAe?$AAr?$AA?5?$AA?$CF?$AAd?$AA?$CJ?$AA?3?$AA?3?$AAH?$AAu?$AAb?$AAS?$AAt?$AAa?$AAt?$AAu?$AAs?$AAC?$AAh?$AAa?$AAn@ 10005940     usbh_usb2com_common_topaz_v1:cdevice.obj
 0001:00004994       ??_C@_1DK@CEOCGHBG@?$AAC?$AAH?$AAu?$AAb?$AA?3?$AA?3?$AAS?$AAu?$AAb?$AAH?$AAu?$AAb?$AAT?$AAe?$AAs?$AAt?$AAM?$AAo?$AAd?$AAe?$AAE?$AAn?$AAa?$AAb?$AAl?$AAe?$AA?$AN?$AA?6?$AA?$AA@ 10005994     usbh_usb2com_common_topaz_v1:cdevice.obj
 0001:000049d0       ??_C@_1IA@LJFJLBFJ@?$AAC?$AAH?$AAu?$AAb?$AA?$CI?$AA?$CF?$AAs?$AA?5?$AAt?$AAi?$AAe?$AAr?$AA?5?$AA?$CF?$AAd?$AA?$CJ?$AA?3?$AA?3?$AAD?$AAi?$AAs?$AAa?$AAb?$AAl?$AAe?$AAD?$AAe?$AAv?$AAi?$AAc?$AAe?$AA?5@ 100059d0     usbh_usb2com_common_topaz_v1:cdevice.obj
 0001:00004a50       ??_C@_1KC@CMBFBEHD@?$AA?9?$AAC?$AAH?$AAu?$AAb?$AA?$CI?$AA?$CF?$AAs?$AA?5?$AAt?$AAi?$AAe?$AAr?$AA?5?$AA?$CF?$AAd?$AA?$CJ?$AA?3?$AA?3?$AAS?$AAu?$AAs?$AAp?$AAe?$AAn?$AAd?$AAR?$AAe?$AAs?$AAu?$AAm?$AAe@ 10005a50     usbh_usb2com_common_topaz_v1:cdevice.obj
 0001:00004af8       ??_C@_1IA@DMLFEMLF@?$AA?$CL?$AAC?$AAH?$AAu?$AAb?$AA?$CI?$AA?$CF?$AAs?$AA?5?$AAt?$AAi?$AAe?$AAr?$AA?5?$AA?$CF?$AAd?$AA?$CJ?$AA?3?$AA?3?$AAS?$AAu?$AAs?$AAp?$AAe?$AAn?$AAd?$AAR?$AAe?$AAs?$AAu?$AAm?$AAe@ 10005af8     usbh_usb2com_common_topaz_v1:cdevice.obj
 0001:00004b78       ??_C@_1DE@MOJKKNGE@?$AA?9?$AAD?$AAu?$AAm?$AAp?$AA?5?$AAU?$AAS?$AAB?$AA_?$AAH?$AAU?$AAB?$AA_?$AAD?$AAE?$AAS?$AAC?$AAR?$AAI?$AAP?$AAT?$AAO?$AAR?$AA?6?$AA?$AA@ 10005b78     usbh_usb2com_common_topaz_v1:cdevice.obj
 0001:00004bb0       ??_C@_1FI@FKNCEHEA@?$AA?7?$AAP?$AAo?$AAr?$AAt?$AAP?$AAw?$AAr?$AAC?$AAt?$AAr?$AAl?$AAM?$AAa?$AAs?$AAk?$AA?5?$AAb?$AAi?$AAt?$AAm?$AAa?$AAs?$AAk?$AA?5?$AAb?$AAy?$AAt?$AAe?$AA?5?$AA?$CD?$AA?$CF@ 10005bb0     usbh_usb2com_common_topaz_v1:cdevice.obj
 0001:00004c08       ??_C@_1FI@MBOKINON@?$AA?7?$AAD?$AAe?$AAv?$AAi?$AAc?$AAe?$AAR?$AAe?$AAm?$AAo?$AAv?$AAa?$AAb?$AAl?$AAe?$AA?5?$AAb?$AAi?$AAt?$AAm?$AAa?$AAs?$AAk?$AA?5?$AAb?$AAy?$AAt?$AAe?$AA?5?$AA?$CD?$AA?$CF@ 10005c08     usbh_usb2com_common_topaz_v1:cdevice.obj
 0001:00004c60       ??_C@_1DM@OFIEHLKD@?$AA?7?$AAb?$AAH?$AAu?$AAb?$AAC?$AAo?$AAn?$AAt?$AAr?$AAo?$AAl?$AAC?$AAu?$AAr?$AAr?$AAe?$AAn?$AAt?$AA?5?$AA?$DN?$AA?5?$AA0?$AAx?$AA?$CF?$AA0?$AA2?$AAx?$AA?6?$AA?$AA@ 10005c60     usbh_usb2com_common_topaz_v1:cdevice.obj
 0001:00004c9c       ??_C@_1DO@EHMENOCN@?$AA?7?$AAb?$AAP?$AAo?$AAw?$AAe?$AAr?$AAO?$AAn?$AAT?$AAo?$AAP?$AAo?$AAw?$AAe?$AAr?$AAG?$AAo?$AAo?$AAd?$AA?5?$AA?$DN?$AA?5?$AA0?$AAx?$AA?$CF?$AA0?$AA2?$AAx?$AA?6?$AA?$AA@ 10005c9c     usbh_usb2com_common_topaz_v1:cdevice.obj
 0001:00004ce0       ??_C@_1GO@KACOCAAE@?$AA?7?$AA?7?$AAw?$AAH?$AAu?$AAb?$AAC?$AAh?$AAa?$AAr?$AAa?$AAc?$AAt?$AAe?$AAr?$AAi?$AAs?$AAt?$AAi?$AAc?$AAs?$AA?0?$AA?5?$AAG?$AAl?$AAo?$AAb?$AAa?$AAl?$AA?5?$AAO?$AAv@ 10005ce0     usbh_usb2com_common_topaz_v1:cdevice.obj
 0001:00004d50       ??_C@_1HG@HEBEECEK@?$AA?7?$AA?7?$AAw?$AAH?$AAu?$AAb?$AAC?$AAh?$AAa?$AAr?$AAa?$AAc?$AAt?$AAe?$AAr?$AAi?$AAs?$AAt?$AAi?$AAc?$AAs?$AA?0?$AA?5?$AAI?$AAn?$AAd?$AAi?$AAv?$AAi?$AAd?$AAu?$AAa@ 10005d50     usbh_usb2com_common_topaz_v1:cdevice.obj
 0001:00004dc8       ??_C@_1GG@PLOBHGPD@?$AA?7?$AA?7?$AAw?$AAH?$AAu?$AAb?$AAC?$AAh?$AAa?$AAr?$AAa?$AAc?$AAt?$AAe?$AAr?$AAi?$AAs?$AAt?$AAi?$AAc?$AAs?$AA?0?$AA?5?$AAN?$AAo?$AA?5?$AAO?$AAv?$AAe?$AAr?$AA?5?$AAC@ 10005dc8     usbh_usb2com_common_topaz_v1:cdevice.obj
 0001:00004e30       ??_C@_1GO@LIJLDPEK@?$AA?7?$AA?7?$AAw?$AAH?$AAu?$AAb?$AAC?$AAh?$AAa?$AAr?$AAa?$AAc?$AAt?$AAe?$AAr?$AAi?$AAs?$AAt?$AAi?$AAc?$AAs?$AA?0?$AA?5?$AAH?$AAu?$AAb?$AA?5?$AA?$CF?$AAs?$AA?5?$AAp?$AAa@ 10005e30     usbh_usb2com_common_topaz_v1:cdevice.obj
 0001:00004ea0       ??_C@_1O@EDGFPFDG@?$AAI?$AAS?$AA?5?$AAN?$AAO?$AAT?$AA?$AA@ 10005ea0     usbh_usb2com_common_topaz_v1:cdevice.obj
 0001:00004eb0       ??_C@_15LPNCKFLE@?$AAI?$AAS?$AA?$AA@ 10005eb0     usbh_usb2com_common_topaz_v1:cdevice.obj
 0001:00004eb8       ??_C@_1GI@CCLJDJKA@?$AA?7?$AA?7?$AAw?$AAH?$AAu?$AAb?$AAC?$AAh?$AAa?$AAr?$AAa?$AAc?$AAt?$AAe?$AAr?$AAi?$AAs?$AAt?$AAi?$AAc?$AAs?$AA?0?$AA?5?$AAG?$AAa?$AAn?$AAg?$AAe?$AAd?$AA?5?$AAP?$AAo@ 10005eb8     usbh_usb2com_common_topaz_v1:cdevice.obj
 0001:00004f20       ??_C@_1HA@PJFBNNAO@?$AA?7?$AA?7?$AAw?$AAH?$AAu?$AAb?$AAC?$AAh?$AAa?$AAr?$AAa?$AAc?$AAt?$AAe?$AAr?$AAi?$AAs?$AAt?$AAi?$AAc?$AAs?$AA?0?$AA?5?$AAI?$AAn?$AAd?$AAi?$AAv?$AAi?$AAd?$AAu?$AAa@ 10005f20     usbh_usb2com_common_topaz_v1:cdevice.obj
 0001:00004f90       ??_C@_1GA@PJHGAPML@?$AA?7?$AA?7?$AAw?$AAH?$AAu?$AAb?$AAC?$AAh?$AAa?$AAr?$AAa?$AAc?$AAt?$AAe?$AAr?$AAi?$AAs?$AAt?$AAi?$AAc?$AAs?$AA?0?$AA?5?$AAN?$AAo?$AA?5?$AAP?$AAo?$AAr?$AAt?$AA?5?$AAP@ 10005f90     usbh_usb2com_common_topaz_v1:cdevice.obj
 0001:00004ff0       ??_C@_1DO@IFBHLDNF@?$AA?7?$AAw?$AAH?$AAu?$AAb?$AAC?$AAh?$AAa?$AAr?$AAa?$AAc?$AAt?$AAe?$AAr?$AAi?$AAs?$AAt?$AAi?$AAc?$AAs?$AA?5?$AA?$DN?$AA?5?$AA0?$AAx?$AA?$CF?$AA0?$AA4?$AAx?$AA?6?$AA?$AA@ 10005ff0     usbh_usb2com_common_topaz_v1:cdevice.obj
 0001:00005030       ??_C@_1DE@FPJADFAL@?$AA?7?$AAb?$AAN?$AAu?$AAm?$AAb?$AAe?$AAr?$AAO?$AAf?$AAP?$AAo?$AAr?$AAt?$AAs?$AA?5?$AA?$DN?$AA?5?$AA0?$AAx?$AA?$CF?$AA0?$AA2?$AAx?$AA?6?$AA?$AA@ 10006030     usbh_usb2com_common_topaz_v1:cdevice.obj
 0001:00005064       ??_C@_1DK@CKNMLPCA@?$AA?7?$AAb?$AAD?$AAe?$AAs?$AAc?$AAr?$AAi?$AAp?$AAt?$AAo?$AAr?$AAL?$AAe?$AAn?$AAg?$AAt?$AAh?$AA?5?$AA?$DN?$AA?5?$AA0?$AAx?$AA?$CF?$AA0?$AA2?$AAx?$AA?6?$AA?$AA@ 10006064     usbh_usb2com_common_topaz_v1:cdevice.obj
 0001:000050a0       ??_C@_1DE@GBEBKDAL@?$AA?$CL?$AAD?$AAu?$AAm?$AAp?$AA?5?$AAU?$AAS?$AAB?$AA_?$AAH?$AAU?$AAB?$AA_?$AAD?$AAE?$AAS?$AAC?$AAR?$AAI?$AAP?$AAT?$AAO?$AAR?$AA?6?$AA?$AA@ 100060a0     usbh_usb2com_common_topaz_v1:cdevice.obj
 0001:000050d4       ??_C@_1BK@GALBKKNF@?$AAN?$AAe?$AAt?$AAM?$AAs?$AAg?$AAB?$AAo?$AAx?$AAE?$AAx?$AAt?$AA?$AA@ 100060d4     usbh_usb2com_common_topaz_v1:cdevice.obj
 0001:000050f0       ??_C@_1BE@BOHEBICI@?$AAn?$AAe?$AAt?$AAu?$AAi?$AA?4?$AAd?$AAl?$AAl?$AA?$AA@ 100060f0     usbh_usb2com_common_topaz_v1:cdevice.obj
 0001:00005104       ??_C@_1CA@GOGEMIHH@?$AAW?$AAa?$AAi?$AAt?$AAF?$AAo?$AAr?$AAA?$AAP?$AAI?$AAR?$AAe?$AAa?$AAd?$AAy?$AA?$AA@ 10006104     usbh_usb2com_common_topaz_v1:cdevice.obj
 0001:00005124       ??_C@_1BM@LLINKHBA@?$AAk?$AA?4?$AAc?$AAo?$AAr?$AAe?$AAd?$AAl?$AAl?$AA?4?$AAd?$AAl?$AAl?$AA?$AA@ 10006124     usbh_usb2com_common_topaz_v1:cdevice.obj
 0001:00005140       ??_C@_1BO@KLPJMMP@?$AAC?$AAe?$AAC?$AAa?$AAl?$AAl?$AAU?$AAs?$AAe?$AAr?$AAP?$AAr?$AAo?$AAc?$AA?$AA@ 10006140     usbh_usb2com_common_topaz_v1:cdevice.obj
 0001:00005160       ??_C@_1JK@CIKNMDOB@?$AA?9?$AAC?$AAH?$AAu?$AAb?$AA?$CI?$AA?$CF?$AAs?$AA?5?$AAt?$AAi?$AAe?$AAr?$AA?5?$AA?$CF?$AAd?$AA?$CJ?$AA?3?$AA?3?$AAA?$AAt?$AAt?$AAa?$AAc?$AAh?$AAD?$AAe?$AAv?$AAi?$AAc?$AAe?$AA?5@ 10006160     usbh_usb2com_common_topaz_v1:cdevice.obj
 0001:00005200       ??_C@_1JM@PDNHGEJD@?$AAC?$AAH?$AAu?$AAb?$AA?$CI?$AA?$CF?$AAs?$AA?5?$AAt?$AAi?$AAe?$AAr?$AA?5?$AA?$CF?$AAd?$AA?$CJ?$AA?3?$AA?3?$AAA?$AAt?$AAt?$AAa?$AAc?$AAh?$AAD?$AAe?$AAv?$AAi?$AAc?$AAe?$AA?5?$AA?9@ 10006200     usbh_usb2com_common_topaz_v1:cdevice.obj
 0001:0000529c       ??_C@_1DI@OCCBGHGB@?$AA?7?$AA?$CB?$AA?$CB?$AA?$CB?$AA?$CB?$AAE?$AAn?$AAu?$AAm?$AAe?$AAr?$AAa?$AAt?$AAi?$AAo?$AAn?$AA?5?$AAD?$AAo?$AAn?$AAe?$AA?$CB?$AA?$CB?$AA?$CB?$AA?$CB?$AA?$AN?$AA?6?$AA?$AA@ 1000629c     usbh_usb2com_common_topaz_v1:cdevice.obj
 0001:000052d8       ??_C@_1HE@EAEFIBJD@?$AAE?$AAx?$AAc?$AAe?$AAe?$AAd?$AA?5?$AAp?$AAo?$AAw?$AAe?$AAr?$AA?5?$AAl?$AAi?$AAm?$AAi?$AAt?$AAa?$AAt?$AAi?$AAo?$AAn?$AA?0?$AA?5?$AAU?$AAS?$AAB?$AA?5?$AAd?$AAe?$AAv@ 100062d8     usbh_usb2com_common_topaz_v1:cdevice.obj
 0001:0000534c       ??_C@_1CO@BBAJLCLO@?$AAC?$AAo?$AAn?$AAf?$AAi?$AAg?$AA?5?$AAP?$AAo?$AAw?$AAe?$AAr?$AA?5?$AA?$DN?$AA?5?$AA?$CF?$AAd?$AA?5?$AAm?$AAA?$AA?$AN?$AA?6?$AA?$AA@ 1000634c     usbh_usb2com_common_topaz_v1:cdevice.obj
 0001:00005380       ??_C@_1IK@GIJBMIGK@?$AAC?$AAH?$AAu?$AAb?$AA?$CI?$AA?$CF?$AAs?$AA?5?$AAt?$AAi?$AAe?$AAr?$AA?5?$AA?$CF?$AAd?$AA?$CJ?$AA?3?$AA?3?$AAA?$AAt?$AAt?$AAa?$AAc?$AAh?$AAD?$AAe?$AAv?$AAi?$AAc?$AAe?$AA?5?$AA?9@ 10006380     usbh_usb2com_common_topaz_v1:cdevice.obj
 0001:00005410       ??_C@_1IA@JDFOHPNL@?$AAC?$AAH?$AAu?$AAb?$AA?$CI?$AA?$CF?$AAs?$AA?5?$AAt?$AAi?$AAe?$AAr?$AA?5?$AA?$CF?$AAd?$AA?$CJ?$AA?3?$AA?3?$AAA?$AAt?$AAt?$AAa?$AAc?$AAh?$AAD?$AAe?$AAv?$AAi?$AAc?$AAe?$AA?5?$AA?9@ 10006410     usbh_usb2com_common_topaz_v1:cdevice.obj
 0001:00005490       ??_C@_1GK@IHAKGPKC@?$AAT?$AAo?$AAo?$AA?5?$AAm?$AAa?$AAn?$AAy?$AA?5?$AAh?$AAu?$AAb?$AA?5?$AAt?$AAi?$AAe?$AAr?$AAs?$AA?0?$AA?5?$AAU?$AAS?$AAB?$AA?5?$AAd?$AAe?$AAv?$AAi?$AAc?$AAe?$AA?5?$AAc@ 10006490     usbh_usb2com_common_topaz_v1:cdevice.obj
 0001:00005500       ??_C@_1OG@CLMEBJJO@?$AAC?$AAH?$AAu?$AAb?$AA?$CI?$AA?$CF?$AAs?$AA?5?$AAt?$AAi?$AAe?$AAr?$AA?5?$AA?$CF?$AAd?$AA?$CJ?$AA?3?$AA?3?$AAA?$AAt?$AAt?$AAa?$AAc?$AAh?$AAD?$AAe?$AAv?$AAi?$AAc?$AAe?$AA?5?$AA?9@ 10006500     usbh_usb2com_common_topaz_v1:cdevice.obj
 0001:000055e8       ??_C@_1GK@PECGIBIC@?$AAC?$AAH?$AAu?$AAb?$AA?$CI?$AA?$CF?$AAs?$AA?5?$AAt?$AAi?$AAe?$AAr?$AA?5?$AA?$CF?$AAd?$AA?$CJ?$AA?3?$AA?3?$AAA?$AAt?$AAt?$AAa?$AAc?$AAh?$AAD?$AAe?$AAv?$AAi?$AAc?$AAe?$AA?5?$AA?9@ 100065e8     usbh_usb2com_common_topaz_v1:cdevice.obj
 0001:00005658       ??_C@_1KE@DPIGKHEM@?$AAC?$AAH?$AAu?$AAb?$AA?$CI?$AA?$CF?$AAs?$AA?5?$AAt?$AAi?$AAe?$AAr?$AA?5?$AA?$CF?$AAd?$AA?$CJ?$AA?3?$AA?3?$AAA?$AAt?$AAt?$AAa?$AAc?$AAh?$AAD?$AAe?$AAv?$AAi?$AAc?$AAe?$AA?5?$AA?9@ 10006658     usbh_usb2com_common_topaz_v1:cdevice.obj
 0001:00005700       ??_C@_1JA@MNHJHALK@?$AAC?$AAH?$AAu?$AAb?$AA?$CI?$AA?$CF?$AAs?$AA?5?$AAt?$AAi?$AAe?$AAr?$AA?5?$AA?$CF?$AAd?$AA?$CJ?$AA?3?$AA?3?$AAA?$AAt?$AAt?$AAa?$AAc?$AAh?$AAD?$AAe?$AAv?$AAi?$AAc?$AAe?$AA?5?$AA?9@ 10006700     usbh_usb2com_common_topaz_v1:cdevice.obj
 0001:00005790       ??_C@_1KE@HOICJLME@?$AAC?$AAH?$AAu?$AAb?$AA?$CI?$AA?$CF?$AAs?$AA?5?$AAt?$AAi?$AAe?$AAr?$AA?5?$AA?$CF?$AAd?$AA?$CJ?$AA?3?$AA?3?$AAA?$AAt?$AAt?$AAa?$AAc?$AAh?$AAD?$AAe?$AAv?$AAi?$AAc?$AAe?$AA?5?$AA?9@ 10006790     usbh_usb2com_common_topaz_v1:cdevice.obj
 0001:00005838       ??_C@_1HK@JHNJCLMB@?$AAC?$AAH?$AAu?$AAb?$AA?$CI?$AA?$CF?$AAs?$AA?5?$AAt?$AAi?$AAe?$AAr?$AA?5?$AA?$CF?$AAd?$AA?$CJ?$AA?3?$AA?3?$AAA?$AAt?$AAt?$AAa?$AAc?$AAh?$AAD?$AAe?$AAv?$AAi?$AAc?$AAe?$AA?5?$AA?9@ 10006838     usbh_usb2com_common_topaz_v1:cdevice.obj
 0001:000058b4       ??_C@_1BA@EOKOFGEP@?$AAI?$AAn?$AAv?$AAa?$AAl?$AAi?$AAd?$AA?$AA@ 100068b4     usbh_usb2com_common_topaz_v1:cdevice.obj
 0001:000058c8       ??_C@_1IA@KFCHKPBM@?$AAC?$AAH?$AAu?$AAb?$AA?$CI?$AA?$CF?$AAs?$AA?5?$AAt?$AAi?$AAe?$AAr?$AA?5?$AA?$CF?$AAd?$AA?$CJ?$AA?3?$AA?3?$AAA?$AAt?$AAt?$AAa?$AAc?$AAh?$AAD?$AAe?$AAv?$AAi?$AAc?$AAe?$AA?5?$AA?9@ 100068c8     usbh_usb2com_common_topaz_v1:cdevice.obj
 0001:00005948       ??_C@_1FG@EBOJJKPN@?$AAA?$AAt?$AAt?$AAa?$AAc?$AAh?$AAD?$AAe?$AAv?$AAi?$AAc?$AAe?$AA?3?$AA?5?$AAw?$AAi?$AAt?$AAh?$AA?5?$AAC?$AAH?$AAu?$AAb?$AA?$CI?$AA0?$AAx?$AA?$CF?$AAx?$AA?$CJ?$AA?5?$AAR?$AAe@ 10006948     usbh_usb2com_common_topaz_v1:cdevice.obj
 0001:000059a0       ??_C@_1HO@NDPINIP@?$AA?$CL?$AAC?$AAH?$AAu?$AAb?$AA?$CI?$AA?$CF?$AAs?$AA?5?$AAt?$AAi?$AAe?$AAr?$AA?5?$AA?$CF?$AAd?$AA?$CJ?$AA?3?$AA?3?$AAA?$AAt?$AAt?$AAa?$AAc?$AAh?$AAD?$AAe?$AAv?$AAi?$AAc?$AAe?$AA?5@ 100069a0     usbh_usb2com_common_topaz_v1:cdevice.obj
 0001:00005a20       ??_C@_1MC@LPCKHMID@?$AA?9?$AAC?$AAH?$AAu?$AAb?$AA?$CI?$AA?$CF?$AAs?$AA?5?$AAt?$AAi?$AAe?$AAr?$AA?5?$AA?$CF?$AAd?$AA?$CJ?$AA?3?$AA?3?$AAG?$AAe?$AAt?$AAD?$AAe?$AAs?$AAc?$AAr?$AAi?$AAp?$AAt?$AAo?$AAr@ 10006a20     usbh_usb2com_common_topaz_v1:cdevice.obj
 0001:00005ae8       ??_C@_1GO@EDOMJKIM@?$AAC?$AAH?$AAu?$AAb?$AA?3?$AA?3?$AAG?$AAe?$AAt?$AAD?$AAe?$AAs?$AAc?$AAr?$AAi?$AAp?$AAt?$AAo?$AAr?$AA?5?$AA?9?$AA?5?$AAf?$AAo?$AAr?$AAc?$AAi?$AAn?$AAg?$AA?5?$AAd?$AAe@ 10006ae8     usbh_usb2com_common_topaz_v1:cdevice.obj
 0001:00005b58       ??_C@_1KG@BKBBKGNO@?$AA?$CL?$AAC?$AAH?$AAu?$AAb?$AA?$CI?$AA?$CF?$AAs?$AA?5?$AAt?$AAi?$AAe?$AAr?$AA?5?$AA?$CF?$AAd?$AA?$CJ?$AA?3?$AA?3?$AAG?$AAe?$AAt?$AAD?$AAe?$AAs?$AAc?$AAr?$AAi?$AAp?$AAt?$AAo?$AAr@ 10006b58     usbh_usb2com_common_topaz_v1:cdevice.obj
 0001:00005c00       ??_C@_1EK@MGLFNGOH@?$AA?9?$AAC?$AAH?$AAu?$AAb?$AA?3?$AA?3?$AAD?$AAe?$AAt?$AAa?$AAc?$AAh?$AAD?$AAo?$AAw?$AAn?$AAs?$AAt?$AAr?$AAe?$AAa?$AAm?$AAD?$AAe?$AAv?$AAi?$AAc?$AAe?$AAT?$AAh?$AAr@ 10006c00     usbh_usb2com_common_topaz_v1:cdevice.obj
 0001:00005c50       ??_C@_1EK@PIIGJLPO@?$AA?$CL?$AAC?$AAH?$AAu?$AAb?$AA?3?$AA?3?$AAD?$AAe?$AAt?$AAa?$AAc?$AAh?$AAD?$AAo?$AAw?$AAn?$AAs?$AAt?$AAr?$AAe?$AAa?$AAm?$AAD?$AAe?$AAv?$AAi?$AAc?$AAe?$AAT?$AAh?$AAr@ 10006c50     usbh_usb2com_common_topaz_v1:cdevice.obj
 0001:00005ca0       ??_C@_1FK@JCHPMIB@?$AA?9?$AAC?$AAH?$AAu?$AAb?$AA?$CI?$AA?$CF?$AAs?$AA?5?$AAt?$AAi?$AAe?$AAr?$AA?5?$AA?$CF?$AAd?$AA?$CJ?$AA?3?$AA?3?$AAD?$AAe?$AAt?$AAa?$AAc?$AAh?$AAD?$AAe?$AAv?$AAi?$AAc?$AAe?$AA?5@ 10006ca0     usbh_usb2com_common_topaz_v1:cdevice.obj
 0001:00005d00       ??_C@_1JO@KEOKNAIJ@?$AAC?$AAH?$AAu?$AAb?$AA?$CI?$AA?$CF?$AAs?$AA?5?$AAt?$AAi?$AAe?$AAr?$AA?5?$AA?$CF?$AAd?$AA?$CJ?$AA?3?$AA?3?$AAD?$AAe?$AAt?$AAa?$AAc?$AAh?$AAD?$AAe?$AAv?$AAi?$AAc?$AAe?$AA?5?$AA?9@ 10006d00     usbh_usb2com_common_topaz_v1:cdevice.obj
 0001:00005da0       ??_C@_1KA@GJGBLDNJ@?$AAC?$AAH?$AAu?$AAb?$AA?$CI?$AA?$CF?$AAs?$AA?5?$AAt?$AAi?$AAe?$AAr?$AA?5?$AA?$CF?$AAd?$AA?$CJ?$AA?3?$AA?3?$AAD?$AAe?$AAt?$AAa?$AAc?$AAh?$AAD?$AAe?$AAv?$AAi?$AAc?$AAe?$AA?5?$AA?9@ 10006da0     usbh_usb2com_common_topaz_v1:cdevice.obj
 0001:00005e40       ??_C@_1LE@IKHCBIJE@?$AAC?$AAH?$AAu?$AAb?$AA?$CI?$AA?$CF?$AAs?$AA?5?$AAt?$AAi?$AAe?$AAr?$AA?5?$AA?$CF?$AAd?$AA?$CJ?$AA?3?$AA?3?$AAD?$AAe?$AAt?$AAa?$AAc?$AAh?$AAD?$AAe?$AAv?$AAi?$AAc?$AAe?$AA?5?$AA?9@ 10006e40     usbh_usb2com_common_topaz_v1:cdevice.obj
 0001:00005ef8       ??_C@_1FK@COKGEFEA@?$AA?$CL?$AAC?$AAH?$AAu?$AAb?$AA?$CI?$AA?$CF?$AAs?$AA?5?$AAt?$AAi?$AAe?$AAr?$AA?5?$AA?$CF?$AAd?$AA?$CJ?$AA?3?$AA?3?$AAD?$AAe?$AAt?$AAa?$AAc?$AAh?$AAD?$AAe?$AAv?$AAi?$AAc?$AAe?$AA?5@ 10006ef8     usbh_usb2com_common_topaz_v1:cdevice.obj
 0001:00005f58       ??_C@_1HG@LCNIGFBM@?$AA?9?$AAC?$AAH?$AAu?$AAb?$AA?$CI?$AA?$CF?$AAs?$AA?5?$AAt?$AAi?$AAe?$AAr?$AA?5?$AA?$CF?$AAd?$AA?$CJ?$AA?3?$AA?3?$AAA?$AAl?$AAl?$AAo?$AAc?$AAa?$AAt?$AAe?$AAD?$AAe?$AAv?$AAi?$AAc@ 10006f58     usbh_usb2com_common_topaz_v1:cdevice.obj
 0001:00005fd0       ??_C@_1GI@EFDHBKMO@?$AAC?$AAH?$AAu?$AAb?$AA?$CI?$AA?$CF?$AAs?$AA?5?$AAt?$AAi?$AAe?$AAr?$AA?5?$AA?$CF?$AAd?$AA?$CJ?$AA?3?$AA?3?$AAA?$AAl?$AAl?$AAo?$AAc?$AAa?$AAt?$AAe?$AAD?$AAe?$AAv?$AAi?$AAc?$AAe@ 10006fd0     usbh_usb2com_common_topaz_v1:cdevice.obj
 0001:00006038       ??_C@_1EE@FLPILJJJ@?$AAC?$AAH?$AAu?$AAb?$AA?3?$AAC?$AAH?$AAu?$AAb?$AA?5?$AAw?$AAi?$AAt?$AAh?$AA?5?$AAn?$AAo?$AA?5?$AAo?$AAf?$AA?5?$AAp?$AAo?$AAr?$AAt?$AAs?$AA?5?$AA?$CI?$AA?$CF?$AAd?$AA?$CJ?$AA?$AN@ 10007038     usbh_usb2com_common_topaz_v1:cdevice.obj
 0001:00006080       ??_C@_1JG@OMFLLIOP@?$AAC?$AAH?$AAu?$AAb?$AA?$CI?$AA?$CF?$AAs?$AA?5?$AAt?$AAi?$AAe?$AAr?$AA?5?$AA?$CF?$AAd?$AA?$CJ?$AA?3?$AA?3?$AAA?$AAl?$AAl?$AAo?$AAc?$AAa?$AAt?$AAe?$AAD?$AAe?$AAv?$AAi?$AAc?$AAe@ 10007080     usbh_usb2com_common_topaz_v1:cdevice.obj
 0001:00006118       ??_C@_1FA@JGCFOODP@?$AA?$CL?$AAC?$AAH?$AAu?$AAb?$AA?$CI?$AA?$CF?$AAs?$AA?5?$AAt?$AAi?$AAe?$AAr?$AA?5?$AA?$CF?$AAd?$AA?$CJ?$AA?3?$AA?3?$AAA?$AAl?$AAl?$AAo?$AAc?$AAa?$AAt?$AAe?$AAD?$AAe?$AAv?$AAi?$AAc@ 10007118     usbh_usb2com_common_topaz_v1:cdevice.obj
 0001:00006168       ??_C@_1EC@CBKBJNBG@?$AA?9?$AAC?$AAH?$AAu?$AAb?$AA?$CI?$AA?$CF?$AAs?$AA?5?$AAt?$AAi?$AAe?$AAr?$AA?5?$AA?$CF?$AAd?$AA?$CJ?$AA?3?$AA?3?$AAH?$AAa?$AAn?$AAd?$AAl?$AAe?$AAD?$AAe?$AAt?$AAa?$AAc?$AAh?$AA?6@ 10007168     usbh_usb2com_common_topaz_v1:cdevice.obj
 0001:000061b0       ??_C@_1IO@KODAFMJG@?$AAC?$AAH?$AAu?$AAb?$AA?$CI?$AA?$CF?$AAs?$AA?5?$AAt?$AAi?$AAe?$AAr?$AA?5?$AA?$CF?$AAd?$AA?$CJ?$AA?3?$AA?3?$AAH?$AAa?$AAn?$AAd?$AAl?$AAe?$AAD?$AAe?$AAt?$AAa?$AAc?$AAh?$AA?5?$AA?9@ 100071b0     usbh_usb2com_common_topaz_v1:cdevice.obj
 0001:00006240       ??_C@_1KO@JIKLHMFD@?$AAC?$AAH?$AAu?$AAb?$AA?$CI?$AA?$CF?$AAs?$AA?5?$AAt?$AAi?$AAe?$AAr?$AA?5?$AA?$CF?$AAd?$AA?$CJ?$AA?3?$AA?3?$AAH?$AAa?$AAn?$AAd?$AAl?$AAe?$AAD?$AAe?$AAt?$AAa?$AAc?$AAh?$AA?5?$AA?9@ 10007240     usbh_usb2com_common_topaz_v1:cdevice.obj
 0001:000062f0       ??_C@_1EC@EOKFHFBF@?$AA?$CL?$AAC?$AAH?$AAu?$AAb?$AA?$CI?$AA?$CF?$AAs?$AA?5?$AAt?$AAi?$AAe?$AAr?$AA?5?$AA?$CF?$AAd?$AA?$CJ?$AA?3?$AA?3?$AAH?$AAa?$AAn?$AAd?$AAl?$AAe?$AAD?$AAe?$AAt?$AAa?$AAc?$AAh?$AA?6@ 100072f0     usbh_usb2com_common_topaz_v1:cdevice.obj
 0001:00006338       ??_C@_1JI@CNCNJHBH@?$AA?9?$AAC?$AAH?$AAu?$AAb?$AA?$CI?$AA?$CF?$AAs?$AA?5?$AAt?$AAi?$AAe?$AAr?$AA?5?$AA?$CF?$AAd?$AA?$CJ?$AA?3?$AA?3?$AAO?$AAp?$AAe?$AAn?$AAP?$AAi?$AAp?$AAe?$AA?5?$AA?9?$AA?5?$AAa?$AAd@ 10007338     usbh_usb2com_common_topaz_v1:cdevice.obj
 0001:000063d0       ??_C@_1FI@NOMFGBIN@?$AA?$CL?$AAC?$AAH?$AAu?$AAb?$AA?$CI?$AA?$CF?$AAs?$AA?5?$AAt?$AAi?$AAe?$AAr?$AA?5?$AA?$CF?$AAd?$AA?$CJ?$AA?3?$AA?3?$AAO?$AAp?$AAe?$AAn?$AAP?$AAi?$AAp?$AAe?$AA?5?$AA?9?$AA?5?$AAa?$AAd@ 100073d0     usbh_usb2com_common_topaz_v1:cdevice.obj
 0001:00006428       ??_C@_1LK@NCLHEMJN@?$AA?9?$AAC?$AAH?$AAu?$AAb?$AA?$CI?$AA?$CF?$AAs?$AA?5?$AAt?$AAi?$AAe?$AAr?$AA?5?$AA?$CF?$AAd?$AA?$CJ?$AA?3?$AA?3?$AAC?$AAl?$AAo?$AAs?$AAe?$AAP?$AAi?$AAp?$AAe?$AA?5?$AA?9?$AA?5?$AAa@ 10007428     usbh_usb2com_common_topaz_v1:cdevice.obj
 0001:000064e8       ??_C@_1HK@EABKNNKI@?$AA?$CL?$AAC?$AAH?$AAu?$AAb?$AA?$CI?$AA?$CF?$AAs?$AA?5?$AAt?$AAi?$AAe?$AAr?$AA?5?$AA?$CF?$AAd?$AA?$CJ?$AA?3?$AA?3?$AAC?$AAl?$AAo?$AAs?$AAe?$AAP?$AAi?$AAp?$AAe?$AA?5?$AA?9?$AA?5?$AAa@ 100074e8     usbh_usb2com_common_topaz_v1:cdevice.obj
 0001:00006568       ??_C@_1LE@GMNJJOHD@?$AA?9?$AAC?$AAH?$AAu?$AAb?$AA?$CI?$AA?$CF?$AAs?$AA?5?$AAt?$AAi?$AAe?$AAr?$AA?5?$AA?$CF?$AAd?$AA?$CJ?$AA?3?$AA?3?$AAI?$AAs?$AAs?$AAu?$AAe?$AAT?$AAr?$AAa?$AAn?$AAs?$AAf?$AAe?$AAr@ 10007568     usbh_usb2com_common_topaz_v1:cdevice.obj
 0001:00006620       ??_C@_1HG@PCAFGNMO@?$AA?$CL?$AAC?$AAH?$AAu?$AAb?$AA?$CI?$AA?$CF?$AAs?$AA?5?$AAt?$AAi?$AAe?$AAr?$AA?5?$AA?$CF?$AAd?$AA?$CJ?$AA?3?$AA?3?$AAI?$AAs?$AAs?$AAu?$AAe?$AAT?$AAr?$AAa?$AAn?$AAs?$AAf?$AAe?$AAr@ 10007620     usbh_usb2com_common_topaz_v1:cdevice.obj
 0001:00006698       ??_C@_1MC@IKDLAGGE@?$AA?9?$AAC?$AAH?$AAu?$AAb?$AA?$CI?$AA?$CF?$AAs?$AA?5?$AAt?$AAi?$AAe?$AAr?$AA?5?$AA?$CF?$AAd?$AA?$CJ?$AA?3?$AA?3?$AAA?$AAb?$AAo?$AAr?$AAt?$AAT?$AAr?$AAa?$AAn?$AAs?$AAf?$AAe?$AAr@ 10007698     usbh_usb2com_common_topaz_v1:cdevice.obj
 0001:00006760       ??_C@_1IC@DBAPCDPC@?$AA?$CL?$AAC?$AAH?$AAu?$AAb?$AA?$CI?$AA?$CF?$AAs?$AA?5?$AAt?$AAi?$AAe?$AAr?$AA?5?$AA?$CF?$AAd?$AA?$CJ?$AA?3?$AA?3?$AAA?$AAb?$AAo?$AAr?$AAt?$AAT?$AAr?$AAa?$AAn?$AAs?$AAf?$AAe?$AAr@ 10007760     usbh_usb2com_common_topaz_v1:cdevice.obj
 0001:000067e8       ??_C@_1LG@INJELGGL@?$AA?9?$AAC?$AAH?$AAu?$AAb?$AA?$CI?$AA?$CF?$AAs?$AA?5?$AAt?$AAi?$AAe?$AAr?$AA?5?$AA?$CF?$AAd?$AA?$CJ?$AA?3?$AA?3?$AAI?$AAs?$AAP?$AAi?$AAp?$AAe?$AAH?$AAa?$AAl?$AAt?$AAe?$AAd?$AA?5@ 100077e8     usbh_usb2com_common_topaz_v1:cdevice.obj
 0001:000068a0       ??_C@_1IA@PMECJFMI@?$AA?$CL?$AAC?$AAH?$AAu?$AAb?$AA?$CI?$AA?$CF?$AAs?$AA?5?$AAt?$AAi?$AAe?$AAr?$AA?5?$AA?$CF?$AAd?$AA?$CJ?$AA?3?$AA?3?$AAI?$AAs?$AAP?$AAi?$AAp?$AAe?$AAH?$AAa?$AAl?$AAt?$AAe?$AAd?$AA?5@ 100078a0     usbh_usb2com_common_topaz_v1:cdevice.obj
 0001:00006920       ??_C@_1LK@IPKBCNF@?$AA?9?$AAC?$AAH?$AAu?$AAb?$AA?$CI?$AA?$CF?$AAs?$AA?5?$AAt?$AAi?$AAe?$AAr?$AA?5?$AA?$CF?$AAd?$AA?$CJ?$AA?3?$AA?3?$AAR?$AAe?$AAs?$AAe?$AAt?$AAP?$AAi?$AAp?$AAe?$AA?5?$AA?9?$AA?5?$AAa@ 10007920     usbh_usb2com_common_topaz_v1:cdevice.obj
 0001:000069e0       ??_C@_1HK@LLMABGAC@?$AA?$CL?$AAC?$AAH?$AAu?$AAb?$AA?$CI?$AA?$CF?$AAs?$AA?5?$AAt?$AAi?$AAe?$AAr?$AA?5?$AA?$CF?$AAd?$AA?$CJ?$AA?3?$AA?3?$AAR?$AAe?$AAs?$AAe?$AAt?$AAP?$AAi?$AAp?$AAe?$AA?5?$AA?9?$AA?5?$AAa@ 100079e0     usbh_usb2com_common_topaz_v1:cdevice.obj
 0001:00006a60       ??_C@_1KC@LNNECAFE@?$AA?9?$AAC?$AAH?$AAu?$AAb?$AA?$CI?$AA?$CF?$AAs?$AA?5?$AAt?$AAi?$AAe?$AAr?$AA?5?$AA?$CF?$AAd?$AA?$CJ?$AA?3?$AA?3?$AAD?$AAi?$AAs?$AAa?$AAb?$AAl?$AAe?$AAD?$AAe?$AAv?$AAi?$AAc?$AAe@ 10007a60     usbh_usb2com_common_topaz_v1:cdevice.obj
 0001:00006b08       ??_C@_1IC@KFLGBCAH@?$AA?$CL?$AAC?$AAH?$AAu?$AAb?$AA?$CI?$AA?$CF?$AAs?$AA?5?$AAt?$AAi?$AAe?$AAr?$AA?5?$AA?$CF?$AAd?$AA?$CJ?$AA?3?$AA?3?$AAD?$AAi?$AAs?$AAa?$AAb?$AAl?$AAe?$AAD?$AAe?$AAv?$AAi?$AAc?$AAe@ 10007b08     usbh_usb2com_common_topaz_v1:cdevice.obj
 0001:00006b90       ??_C@_1LE@MMIJLBC@?$AA?9?$AAC?$AAH?$AAu?$AAb?$AA?$CI?$AA?$CF?$AAs?$AA?5?$AAt?$AAi?$AAe?$AAr?$AA?5?$AA?$CF?$AAd?$AA?$CJ?$AA?3?$AA?3?$AAD?$AAi?$AAs?$AAa?$AAb?$AAl?$AAe?$AAO?$AAf?$AAf?$AAS?$AAt?$AAr@ 10007b90     usbh_usb2com_common_topaz_v1:cdevice.obj
 0001:00006c48       ??_C@_1JE@OBFLIFJ@?$AA?$CL?$AAC?$AAH?$AAu?$AAb?$AA?$CI?$AA?$CF?$AAs?$AA?5?$AAt?$AAi?$AAe?$AAr?$AA?5?$AA?$CF?$AAd?$AA?$CJ?$AA?3?$AA?3?$AAD?$AAi?$AAs?$AAa?$AAb?$AAl?$AAe?$AAO?$AAf?$AAf?$AAS?$AAt?$AAr@ 10007c48     usbh_usb2com_common_topaz_v1:cdevice.obj
 0001:00006cdc       ??_C@_1CK@CJNCFJE@?$AA?9?$AAC?$AAR?$AAo?$AAo?$AAt?$AAH?$AAu?$AAb?$AA?3?$AA?3?$AAC?$AAR?$AAo?$AAo?$AAt?$AAH?$AAu?$AAb?$AA?6?$AA?$AA@ 10007cdc     usbh_usb2com_common_topaz_v1:cdevice.obj
 0001:00006d08       ??_C@_1CK@HCOKDDHC@?$AA?$CL?$AAC?$AAR?$AAo?$AAo?$AAt?$AAH?$AAu?$AAb?$AA?3?$AA?3?$AAC?$AAR?$AAo?$AAo?$AAt?$AAH?$AAu?$AAb?$AA?6?$AA?$AA@ 10007d08     usbh_usb2com_common_topaz_v1:cdevice.obj
 0001:00006d38       ??_7CRootHub@@6B@          10007d38     usbh_usb2com_common_topaz_v1:cdevice.obj
 0001:00006d9c       ??_C@_19LFKAPJKP@?$AAR?$AAo?$AAo?$AAt?$AA?$AA@ 10007d9c     usbh_usb2com_common_topaz_v1:cdevice.obj
 0001:00006da8       ??_C@_1CM@NAKEALML@?$AA?9?$AAC?$AAR?$AAo?$AAo?$AAt?$AAH?$AAu?$AAb?$AA?3?$AA?3?$AA?$HO?$AAC?$AAR?$AAo?$AAo?$AAt?$AAH?$AAu?$AAb?$AA?6?$AA?$AA@ 10007da8     usbh_usb2com_common_topaz_v1:cdevice.obj
 0001:00006dd4       ??_C@_1CM@CMFEJKIH@?$AA?$CL?$AAC?$AAR?$AAo?$AAo?$AAt?$AAH?$AAu?$AAb?$AA?3?$AA?3?$AA?$HO?$AAC?$AAR?$AAo?$AAo?$AAt?$AAH?$AAu?$AAb?$AA?6?$AA?$AA@ 10007dd4     usbh_usb2com_common_topaz_v1:cdevice.obj
 0001:00006e00       ??_C@_1GK@HHCFCMBC@?$AA?9?$AAC?$AAR?$AAo?$AAo?$AAt?$AAH?$AAu?$AAb?$AA?3?$AA?3?$AAE?$AAn?$AAt?$AAe?$AAr?$AAO?$AAp?$AAe?$AAr?$AAa?$AAt?$AAi?$AAo?$AAn?$AAa?$AAl?$AAS?$AAt?$AAa?$AAt?$AAe@ 10007e00     usbh_usb2com_common_topaz_v1:cdevice.obj
 0001:00006e70       ??_C@_1EE@PDDHPKNI@?$AA?$CL?$AAC?$AAR?$AAo?$AAo?$AAt?$AAH?$AAu?$AAb?$AA?3?$AA?3?$AAE?$AAn?$AAt?$AAe?$AAr?$AAO?$AAp?$AAe?$AAr?$AAa?$AAt?$AAi?$AAo?$AAn?$AAa?$AAl?$AAS?$AAt?$AAa?$AAt?$AAe@ 10007e70     usbh_usb2com_common_topaz_v1:cdevice.obj
 0001:00006eb4       ??_C@_1DK@ICPLBLCC@?$AA?9?$AAC?$AAR?$AAo?$AAo?$AAt?$AAH?$AAu?$AAb?$AA?3?$AA?3?$AAP?$AAo?$AAw?$AAe?$AAr?$AAA?$AAl?$AAl?$AAH?$AAu?$AAb?$AAP?$AAo?$AAr?$AAt?$AAs?$AA?6?$AA?$AA@ 10007eb4     usbh_usb2com_common_topaz_v1:cdevice.obj
 0001:00006ef0       ??_C@_1DK@OHBIDMAJ@?$AA?$CL?$AAC?$AAR?$AAo?$AAo?$AAt?$AAH?$AAu?$AAb?$AA?3?$AA?3?$AAP?$AAo?$AAw?$AAe?$AAr?$AAA?$AAl?$AAl?$AAH?$AAu?$AAb?$AAP?$AAo?$AAr?$AAt?$AAs?$AA?6?$AA?$AA@ 10007ef0     usbh_usb2com_common_topaz_v1:cdevice.obj
 0001:00006f30       ??_C@_1HO@ELFNBANG@?$AA?9?$AAC?$AAR?$AAo?$AAo?$AAt?$AAH?$AAu?$AAb?$AA?3?$AA?3?$AAW?$AAa?$AAi?$AAt?$AAF?$AAo?$AAr?$AAP?$AAo?$AAr?$AAt?$AAS?$AAt?$AAa?$AAt?$AAu?$AAs?$AAC?$AAh?$AAa?$AAn@ 10007f30     usbh_usb2com_common_topaz_v1:cdevice.obj
 0001:00006fb0       ??_C@_1EI@OICCPODJ@?$AA?$CL?$AAC?$AAR?$AAo?$AAo?$AAt?$AAH?$AAu?$AAb?$AA?3?$AA?3?$AAW?$AAa?$AAi?$AAt?$AAF?$AAo?$AAr?$AAP?$AAo?$AAr?$AAt?$AAS?$AAt?$AAa?$AAt?$AAu?$AAs?$AAC?$AAh?$AAa?$AAn@ 10007fb0     usbh_usb2com_common_topaz_v1:cdevice.obj
 0001:00006ff8       ??_C@_1GI@PFLBEDL@?$AA?9?$AAC?$AAR?$AAo?$AAo?$AAt?$AAH?$AAu?$AAb?$AA?3?$AA?3?$AAG?$AAe?$AAt?$AAS?$AAt?$AAa?$AAt?$AAu?$AAs?$AA?5?$AA?9?$AA?5?$AAp?$AAo?$AAr?$AAt?$AA?5?$AA?$DN?$AA?5?$AA?$CF?$AAd@ 10007ff8     usbh_usb2com_common_topaz_v1:cdevice.obj
 0001:00007060       ??_C@_1EE@HPELNOPH@?$AA?$CL?$AAC?$AAR?$AAo?$AAo?$AAt?$AAH?$AAu?$AAb?$AA?3?$AA?3?$AAG?$AAe?$AAt?$AAS?$AAt?$AAa?$AAt?$AAu?$AAs?$AA?5?$AA?9?$AA?5?$AAp?$AAo?$AAr?$AAt?$AA?5?$AA?$DN?$AA?5?$AA?$CF?$AAd@ 10008060     usbh_usb2com_common_topaz_v1:cdevice.obj
 0001:000070a8       ??_C@_1HC@FCGCEEHM@?$AA?9?$AAC?$AAR?$AAo?$AAo?$AAt?$AAH?$AAu?$AAb?$AA?3?$AA?3?$AAR?$AAe?$AAs?$AAe?$AAt?$AAA?$AAn?$AAd?$AAE?$AAn?$AAa?$AAb?$AAl?$AAe?$AAP?$AAo?$AAr?$AAt?$AA?5?$AA?9?$AA?5@ 100080a8     usbh_usb2com_common_topaz_v1:cdevice.obj
 0001:00007120       ??_C@_1FG@FLAJCBDG@?$AA?$CL?$AAC?$AAR?$AAo?$AAo?$AAt?$AAH?$AAu?$AAb?$AA?3?$AA?3?$AAR?$AAe?$AAs?$AAe?$AAt?$AAA?$AAn?$AAd?$AAE?$AAn?$AAa?$AAb?$AAl?$AAe?$AAP?$AAo?$AAr?$AAt?$AA?5?$AA?9?$AA?5@ 10008120     usbh_usb2com_common_topaz_v1:cdevice.obj
 0001:00007178       ??_C@_1EI@ICHPNEPH@?$AA?9?$AAC?$AAR?$AAo?$AAo?$AAt?$AAH?$AAu?$AAb?$AA?3?$AA?3?$AAD?$AAi?$AAs?$AAa?$AAb?$AAl?$AAe?$AAP?$AAo?$AAr?$AAt?$AA?5?$AA?9?$AA?5?$AAp?$AAo?$AAr?$AAt?$AA?5?$AA?$DN?$AA?5@ 10008178     usbh_usb2com_common_topaz_v1:cdevice.obj
 0001:000071c0       ??_C@_1EI@NAKGDBAN@?$AA?$CL?$AAC?$AAR?$AAo?$AAo?$AAt?$AAH?$AAu?$AAb?$AA?3?$AA?3?$AAD?$AAi?$AAs?$AAa?$AAb?$AAl?$AAe?$AAP?$AAo?$AAr?$AAt?$AA?5?$AA?9?$AA?5?$AAp?$AAo?$AAr?$AAt?$AA?5?$AA?$DN?$AA?5@ 100081c0     usbh_usb2com_common_topaz_v1:cdevice.obj
 0001:00007208       ??_C@_1LM@CFDGEKIP@?$AA?9?$AAC?$AAR?$AAo?$AAo?$AAt?$AAH?$AAu?$AAb?$AA?3?$AA?3?$AAS?$AAe?$AAt?$AAO?$AAr?$AAC?$AAl?$AAe?$AAa?$AAr?$AAF?$AAe?$AAa?$AAt?$AAu?$AAr?$AAe?$AA?5?$AA?9?$AA?5?$AAp@ 10008208     usbh_usb2com_common_topaz_v1:cdevice.obj
 0001:000072c8       ??_C@_1KG@NIOCCNL@?$AAC?$AAR?$AAo?$AAo?$AAt?$AAH?$AAu?$AAb?$AA?3?$AA?3?$AAS?$AAe?$AAt?$AAO?$AAr?$AAC?$AAl?$AAe?$AAa?$AAr?$AAF?$AAe?$AAa?$AAt?$AAu?$AAr?$AAe?$AA?5?$AA?9?$AA?5?$AAp?$AAo@ 100082c8     usbh_usb2com_common_topaz_v1:cdevice.obj
 0001:00007370       ??_C@_1JI@LGGIGNLA@?$AA?$CL?$AAC?$AAR?$AAo?$AAo?$AAt?$AAH?$AAu?$AAb?$AA?3?$AA?3?$AAS?$AAe?$AAt?$AAO?$AAr?$AAC?$AAl?$AAe?$AAa?$AAr?$AAF?$AAe?$AAa?$AAt?$AAu?$AAr?$AAe?$AA?5?$AA?9?$AA?5?$AAp@ 10008370     usbh_usb2com_common_topaz_v1:cdevice.obj
 0001:00007408       ??_C@_1DK@BLICMNOB@?$AA?9?$AAC?$AAE?$AAx?$AAt?$AAe?$AAr?$AAn?$AAa?$AAl?$AAH?$AAu?$AAb?$AA?3?$AA?3?$AAC?$AAE?$AAx?$AAt?$AAe?$AAr?$AAn?$AAa?$AAl?$AAH?$AAu?$AAb?$AA?6?$AA?$AA@ 10008408     usbh_usb2com_common_topaz_v1:cdevice.obj
 0001:00007444       ??_C@_1DK@HOGBOKMK@?$AA?$CL?$AAC?$AAE?$AAx?$AAt?$AAe?$AAr?$AAn?$AAa?$AAl?$AAH?$AAu?$AAb?$AA?3?$AA?3?$AAC?$AAE?$AAx?$AAt?$AAe?$AAr?$AAn?$AAa?$AAl?$AAH?$AAu?$AAb?$AA?6?$AA?$AA@ 10008444     usbh_usb2com_common_topaz_v1:cdevice.obj
 0001:00007480       ??_7CExternalHub@@6B@      10008480     usbh_usb2com_common_topaz_v1:cdevice.obj
 0001:000074e4       ??_C@_1BC@KMFBFJEN@?$AAE?$AAx?$AAt?$AAe?$AAr?$AAn?$AAa?$AAl?$AA?$AA@ 100084e4     usbh_usb2com_common_topaz_v1:cdevice.obj
 0001:000074f8       ??_C@_1DM@KMIKFLE@?$AA?9?$AAC?$AAE?$AAx?$AAt?$AAe?$AAr?$AAn?$AAa?$AAl?$AAH?$AAu?$AAb?$AA?3?$AA?3?$AA?$HO?$AAC?$AAE?$AAx?$AAt?$AAe?$AAr?$AAn?$AAa?$AAl?$AAH?$AAu?$AAb?$AA?6?$AA?$AA@ 100084f8     usbh_usb2com_common_topaz_v1:cdevice.obj
 0001:00007534       ??_C@_1DM@NJLCIIFF@?$AA?$CL?$AAC?$AAE?$AAx?$AAt?$AAe?$AAr?$AAn?$AAa?$AAl?$AAH?$AAu?$AAb?$AA?3?$AA?3?$AA?$HO?$AAC?$AAE?$AAx?$AAt?$AAe?$AAr?$AAn?$AAa?$AAl?$AAH?$AAu?$AAb?$AA?6?$AA?$AA@ 10008534     usbh_usb2com_common_topaz_v1:cdevice.obj
 0001:00007570       ??_C@_1HC@GNNHIEFI@?$AA?9?$AAC?$AAE?$AAx?$AAt?$AAe?$AAr?$AAn?$AAa?$AAl?$AAH?$AAu?$AAb?$AA?3?$AA?3?$AAE?$AAn?$AAt?$AAe?$AAr?$AAO?$AAp?$AAe?$AAr?$AAa?$AAt?$AAi?$AAo?$AAn?$AAa?$AAl?$AAS@ 10008570     usbh_usb2com_common_topaz_v1:cdevice.obj
 0001:000075e8       ??_C@_1EM@MEILKMHH@?$AA?$CL?$AAC?$AAE?$AAx?$AAt?$AAe?$AAr?$AAn?$AAa?$AAl?$AAH?$AAu?$AAb?$AA?3?$AA?3?$AAE?$AAn?$AAt?$AAe?$AAr?$AAO?$AAp?$AAe?$AAr?$AAa?$AAt?$AAi?$AAo?$AAn?$AAa?$AAl?$AAS@ 100085e8     usbh_usb2com_common_topaz_v1:cdevice.obj
 0001:00007638       ??_C@_1ME@IBBEICDF@?$AA?9?$AAC?$AAE?$AAx?$AAt?$AAe?$AAr?$AAn?$AAa?$AAl?$AAH?$AAu?$AAb?$AA?3?$AA?3?$AAS?$AAe?$AAt?$AAO?$AAr?$AAC?$AAl?$AAe?$AAa?$AAr?$AAF?$AAe?$AAa?$AAt?$AAu?$AAr?$AAe@ 10008638     usbh_usb2com_common_topaz_v1:cdevice.obj
 0001:00007700       ??_C@_1KO@NCFBBEAA@?$AAC?$AAE?$AAx?$AAt?$AAe?$AAr?$AAn?$AAa?$AAl?$AAH?$AAu?$AAb?$AA?3?$AA?3?$AAS?$AAe?$AAt?$AAO?$AAr?$AAC?$AAl?$AAe?$AAa?$AAr?$AAF?$AAe?$AAa?$AAt?$AAu?$AAr?$AAe?$AA?5@ 10008700     usbh_usb2com_common_topaz_v1:cdevice.obj
 0001:000077b0       ??_C@_1GO@MODMIGEA@?$AAC?$AAE?$AAx?$AAt?$AAe?$AAr?$AAn?$AAa?$AAl?$AAH?$AAu?$AAb?$AA?3?$AA?3?$AAS?$AAe?$AAt?$AAO?$AAr?$AAC?$AAl?$AAe?$AAa?$AAr?$AAF?$AAe?$AAa?$AAt?$AAu?$AAr?$AAe?$AA?5@ 100087b0     usbh_usb2com_common_topaz_v1:cdevice.obj
 0001:00007820       ??_C@_1FM@NDFPLGFL@?$AA?9?$AAC?$AAE?$AAx?$AAt?$AAe?$AAr?$AAn?$AAa?$AAl?$AAH?$AAu?$AAb?$AA?3?$AA?3?$AAP?$AAo?$AAw?$AAe?$AAr?$AAA?$AAl?$AAl?$AAH?$AAu?$AAb?$AAP?$AAo?$AAr?$AAt?$AAs?$AA?0@ 10008820     usbh_usb2com_common_topaz_v1:cdevice.obj
 0001:00007880       ??_C@_1FE@CAIBHEOA@?$AAC?$AAE?$AAx?$AAt?$AAe?$AAr?$AAn?$AAa?$AAl?$AAH?$AAu?$AAb?$AA?3?$AA?3?$AAP?$AAo?$AAw?$AAe?$AAr?$AAA?$AAl?$AAl?$AAH?$AAu?$AAb?$AAP?$AAo?$AAr?$AAt?$AAs?$AA?5?$AA?9@ 10008880     usbh_usb2com_common_topaz_v1:cdevice.obj
 0001:000078d8       ??_C@_1EC@EIEJHPIH@?$AA?$CL?$AAC?$AAE?$AAx?$AAt?$AAe?$AAr?$AAn?$AAa?$AAl?$AAH?$AAu?$AAb?$AA?3?$AA?3?$AAP?$AAo?$AAw?$AAe?$AAr?$AAA?$AAl?$AAl?$AAH?$AAu?$AAb?$AAP?$AAo?$AAr?$AAt?$AAs?$AA?6@ 100088d8     usbh_usb2com_common_topaz_v1:cdevice.obj
 0001:00007920       ??_C@_1JI@EPAIPDFE@?$AA?9?$AAC?$AAE?$AAx?$AAt?$AAe?$AAr?$AAn?$AAa?$AAl?$AA?3?$AA?3?$AAG?$AAe?$AAt?$AAS?$AAt?$AAa?$AAt?$AAu?$AAs?$AAC?$AAh?$AAa?$AAn?$AAg?$AAe?$AAB?$AAi?$AAt?$AAm?$AAa@ 10008920     usbh_usb2com_common_topaz_v1:cdevice.obj
 0001:000079b8       ??_C@_1HO@KALJIFCJ@?$AAC?$AAE?$AAx?$AAt?$AAe?$AAr?$AAn?$AAa?$AAl?$AAH?$AAu?$AAb?$AA?3?$AA?3?$AAG?$AAe?$AAt?$AAS?$AAt?$AAa?$AAt?$AAu?$AAs?$AAC?$AAh?$AAa?$AAn?$AAg?$AAe?$AAB?$AAi?$AAt@ 100089b8     usbh_usb2com_common_topaz_v1:cdevice.obj
 0001:00007a38       ??_C@_1EM@DBCILMDF@?$AA?$CL?$AAC?$AAE?$AAx?$AAt?$AAe?$AAr?$AAn?$AAa?$AAl?$AAH?$AAu?$AAb?$AA?3?$AA?3?$AAG?$AAe?$AAt?$AAS?$AAt?$AAa?$AAt?$AAu?$AAs?$AAC?$AAh?$AAa?$AAn?$AAg?$AAe?$AAB?$AAi@ 10008a38     usbh_usb2com_common_topaz_v1:cdevice.obj
 0001:00007a88       ??_C@_1JC@JNLMDHLK@?$AA?9?$AAC?$AAE?$AAx?$AAt?$AAe?$AAr?$AAn?$AAa?$AAl?$AA?3?$AA?3?$AAW?$AAa?$AAi?$AAt?$AAF?$AAo?$AAr?$AAP?$AAo?$AAr?$AAt?$AAS?$AAt?$AAa?$AAt?$AAu?$AAs?$AAC?$AAh?$AAa@ 10008a88     usbh_usb2com_common_topaz_v1:cdevice.obj
 0001:00007b20       ??_C@_1FA@GFNGOBND@?$AA?$CL?$AAC?$AAE?$AAx?$AAt?$AAe?$AAr?$AAn?$AAa?$AAl?$AAH?$AAu?$AAb?$AA?3?$AA?3?$AAW?$AAa?$AAi?$AAt?$AAF?$AAo?$AAr?$AAP?$AAo?$AAr?$AAt?$AAS?$AAt?$AAa?$AAt?$AAu?$AAs@ 10008b20     usbh_usb2com_common_topaz_v1:cdevice.obj
 0001:00007b70       ??_C@_1HA@HBNEJOAD@?$AA?9?$AAC?$AAE?$AAx?$AAt?$AAe?$AAr?$AAn?$AAa?$AAl?$AAH?$AAu?$AAb?$AA?3?$AA?3?$AAG?$AAe?$AAt?$AAS?$AAt?$AAa?$AAt?$AAu?$AAs?$AA?5?$AA?9?$AA?5?$AAp?$AAo?$AAr?$AAt?$AA?5@ 10008b70     usbh_usb2com_common_topaz_v1:cdevice.obj
 0001:00007be0       ??_C@_1EM@EIPHIIFI@?$AA?$CL?$AAC?$AAE?$AAx?$AAt?$AAe?$AAr?$AAn?$AAa?$AAl?$AAH?$AAu?$AAb?$AA?3?$AA?3?$AAG?$AAe?$AAt?$AAS?$AAt?$AAa?$AAt?$AAu?$AAs?$AA?5?$AA?9?$AA?5?$AAp?$AAo?$AAr?$AAt?$AA?5@ 10008be0     usbh_usb2com_common_topaz_v1:cdevice.obj
 0001:00007c30       ??_C@_1HK@OMHBDAGB@?$AA?9?$AAC?$AAE?$AAx?$AAt?$AAe?$AAr?$AAn?$AAa?$AAl?$AAH?$AAu?$AAb?$AA?3?$AA?3?$AAR?$AAe?$AAs?$AAe?$AAt?$AAA?$AAn?$AAd?$AAE?$AAn?$AAa?$AAb?$AAl?$AAe?$AAP?$AAo?$AAr@ 10008c30     usbh_usb2com_common_topaz_v1:cdevice.obj
 0001:00007cb0       ??_C@_1JC@GLHNDCHK@?$AA?9?$AAC?$AAE?$AAx?$AAt?$AAe?$AAr?$AAn?$AAa?$AAl?$AAH?$AAu?$AAb?$AA?3?$AA?3?$AAR?$AAe?$AAs?$AAe?$AAt?$AAA?$AAn?$AAd?$AAE?$AAn?$AAa?$AAb?$AAl?$AAe?$AAP?$AAo?$AAr@ 10008cb0     usbh_usb2com_common_topaz_v1:cdevice.obj
 0001:00007d48       ??_C@_1FO@OOBJEFHK@?$AA?$CL?$AAC?$AAE?$AAx?$AAt?$AAe?$AAr?$AAn?$AAa?$AAl?$AAH?$AAu?$AAb?$AA?3?$AA?3?$AAR?$AAe?$AAs?$AAe?$AAt?$AAA?$AAn?$AAd?$AAE?$AAn?$AAa?$AAb?$AAl?$AAe?$AAP?$AAo?$AAr@ 10008d48     usbh_usb2com_common_topaz_v1:cdevice.obj
 0001:00007da8       ??_C@_1FA@BFIDHOJJ@?$AA?9?$AAC?$AAE?$AAx?$AAt?$AAe?$AAr?$AAn?$AAa?$AAl?$AAH?$AAu?$AAb?$AA?3?$AA?3?$AAD?$AAi?$AAs?$AAa?$AAb?$AAl?$AAe?$AAP?$AAo?$AAr?$AAt?$AA?5?$AA?9?$AA?5?$AAp?$AAo?$AAr@ 10008da8     usbh_usb2com_common_topaz_v1:cdevice.obj
 0001:00007df8       ??_C@_1FA@FNFCCOOH@?$AA?$CL?$AAC?$AAE?$AAx?$AAt?$AAe?$AAr?$AAn?$AAa?$AAl?$AAH?$AAu?$AAb?$AA?3?$AA?3?$AAD?$AAi?$AAs?$AAa?$AAb?$AAl?$AAe?$AAP?$AAo?$AAr?$AAt?$AA?5?$AA?9?$AA?5?$AAp?$AAo?$AAr@ 10008df8     usbh_usb2com_common_topaz_v1:cdevice.obj
 0001:00007e48       ??_C@_1KA@EIDHOGBK@?$AA?$CL?$AAC?$AAE?$AAx?$AAt?$AAe?$AAr?$AAn?$AAa?$AAl?$AAH?$AAu?$AAb?$AA?3?$AA?3?$AAS?$AAe?$AAt?$AAO?$AAr?$AAC?$AAl?$AAe?$AAa?$AAr?$AAF?$AAe?$AAa?$AAt?$AAu?$AAr?$AAe@ 10008e48     usbh_usb2com_common_topaz_v1:cdevice.obj
 0001:00007ee8       ??_C@_1HE@OGFLIABG@?$AA?9?$AAC?$AAE?$AAx?$AAt?$AAe?$AAr?$AAn?$AAa?$AAl?$AAH?$AAu?$AAb?$AA?3?$AA?3?$AAS?$AAe?$AAt?$AAO?$AAr?$AAC?$AAl?$AAe?$AAa?$AAr?$AAR?$AAe?$AAm?$AAo?$AAt?$AAe?$AAW@ 10008ee8     usbh_usb2com_common_topaz_v1:cdevice.obj
 0001:00007f60       ??_C@_1GG@EJGBKNJ@?$AA?$CL?$AAC?$AAE?$AAx?$AAt?$AAe?$AAr?$AAn?$AAa?$AAl?$AAH?$AAu?$AAb?$AA?3?$AA?3?$AAS?$AAe?$AAt?$AAO?$AAr?$AAC?$AAl?$AAe?$AAa?$AAr?$AAR?$AAe?$AAm?$AAo?$AAt?$AAe?$AAW@ 10008f60     usbh_usb2com_common_topaz_v1:cdevice.obj
 0001:00007fc8       ??_C@_1EA@HAHMHPPG@?$AA?9?$AAC?$AAF?$AAu?$AAn?$AAc?$AAt?$AAi?$AAo?$AAn?$AA?$CI?$AAt?$AAi?$AAe?$AAr?$AA?5?$AA?$CF?$AAd?$AA?$CJ?$AA?3?$AA?3?$AAC?$AAF?$AAu?$AAn?$AAc?$AAt?$AAi?$AAo?$AAn?$AA?6?$AA?$AA@ 10008fc8     usbh_usb2com_common_topaz_v1:cdevice.obj
 0001:00008008       ??_C@_1EA@OECAJOAK@?$AA?$CL?$AAC?$AAF?$AAu?$AAn?$AAc?$AAt?$AAi?$AAo?$AAn?$AA?$CI?$AAt?$AAi?$AAe?$AAr?$AA?5?$AA?$CF?$AAd?$AA?$CJ?$AA?3?$AA?3?$AAC?$AAF?$AAu?$AAn?$AAc?$AAt?$AAi?$AAo?$AAn?$AA?6?$AA?$AA@ 10009008     usbh_usb2com_common_topaz_v1:cdevice.obj
 0001:00008048       ??_7CFunction@@6B@         10009048     usbh_usb2com_common_topaz_v1:cdevice.obj
 0001:00008084       ??_C@_1BC@IDPNFFME@?$AAF?$AAu?$AAn?$AAc?$AAt?$AAi?$AAo?$AAn?$AA?$AA@ 10009084     usbh_usb2com_common_topaz_v1:cdevice.obj
 0001:00008098       ??_C@_1EC@FBEPJHCP@?$AA?9?$AAC?$AAF?$AAu?$AAn?$AAc?$AAt?$AAi?$AAo?$AAn?$AA?$CI?$AAt?$AAi?$AAe?$AAr?$AA?5?$AA?$CF?$AAd?$AA?$CJ?$AA?3?$AA?3?$AA?$HO?$AAC?$AAF?$AAu?$AAn?$AAc?$AAt?$AAi?$AAo?$AAn?$AA?6@ 10009098     usbh_usb2com_common_topaz_v1:cdevice.obj
 0001:000080e0       ??_C@_1EC@DOELHPCM@?$AA?$CL?$AAC?$AAF?$AAu?$AAn?$AAc?$AAt?$AAi?$AAo?$AAn?$AA?$CI?$AAt?$AAi?$AAe?$AAr?$AA?5?$AA?$CF?$AAd?$AA?$CJ?$AA?3?$AA?3?$AA?$HO?$AAC?$AAF?$AAu?$AAn?$AAc?$AAt?$AAi?$AAo?$AAn?$AA?6@ 100090e0     usbh_usb2com_common_topaz_v1:cdevice.obj
 0001:00008128       ??_C@_1HO@CKKHIFHP@?$AA?9?$AAC?$AAF?$AAu?$AAn?$AAc?$AAt?$AAi?$AAo?$AAn?$AA?$CI?$AAt?$AAi?$AAe?$AAr?$AA?5?$AA?$CF?$AAd?$AA?$CJ?$AA?3?$AA?3?$AAE?$AAn?$AAt?$AAe?$AAr?$AAO?$AAp?$AAe?$AAr?$AAa?$AAt@ 10009128     usbh_usb2com_common_topaz_v1:cdevice.obj
 0001:000081a8       ??_C@_1GI@DBLMBFBL@?$AAC?$AAF?$AAu?$AAn?$AAc?$AAt?$AAi?$AAo?$AAn?$AA?$CI?$AAt?$AAi?$AAe?$AAr?$AA?5?$AA?$CF?$AAd?$AA?$CJ?$AA?3?$AA?3?$AAE?$AAn?$AAt?$AAe?$AAr?$AAO?$AAp?$AAe?$AAr?$AAa?$AAt?$AAi@ 100091a8     usbh_usb2com_common_topaz_v1:cdevice.obj
 0001:00008210       ??_C@_1DO@NNHBJHPD@?$AAF?$AAa?$AAi?$AAl?$AAu?$AAr?$AAe?$AA?5?$AAt?$AAo?$AA?5?$AAA?$AAl?$AAl?$AAo?$AAc?$AAa?$AAt?$AAe?$AAP?$AAi?$AAp?$AAe?$AAA?$AAr?$AAr?$AAa?$AAy?$AA?$AN?$AA?6?$AA?$AA@ 10009210     usbh_usb2com_common_topaz_v1:cdevice.obj
 0001:00008250       ??_C@_1FI@PNNALGEC@?$AA?$CL?$AAC?$AAF?$AAu?$AAn?$AAc?$AAt?$AAi?$AAo?$AAn?$AA?$CI?$AAt?$AAi?$AAe?$AAr?$AA?5?$AA?$CF?$AAd?$AA?$CJ?$AA?3?$AA?3?$AAE?$AAn?$AAt?$AAe?$AAr?$AAO?$AAp?$AAe?$AAr?$AAa?$AAt@ 10009250     usbh_usb2com_common_topaz_v1:cdevice.obj
 0001:000082a8       ??_C@_1JM@IKMNJOMD@?$AA?9?$AAC?$AAF?$AAu?$AAn?$AAc?$AAt?$AAi?$AAo?$AAn?$AA?$CI?$AAt?$AAi?$AAe?$AAr?$AA?5?$AA?$CF?$AAd?$AA?$CJ?$AA?3?$AA?3?$AAO?$AAp?$AAe?$AAn?$AAP?$AAi?$AAp?$AAe?$AA?5?$AA?9?$AA?5@ 100092a8     usbh_usb2com_common_topaz_v1:cdevice.obj
 0001:00008348       ??_C@_1IK@MOOEIMIB@?$AAC?$AAF?$AAu?$AAn?$AAc?$AAt?$AAi?$AAo?$AAn?$AA?$CI?$AAt?$AAi?$AAe?$AAr?$AA?5?$AA?$CF?$AAd?$AA?$CJ?$AA?3?$AA?3?$AAO?$AAp?$AAe?$AAn?$AAP?$AAi?$AAp?$AAe?$AA?5?$AA?9?$AA?5?$AAo@ 10009348     usbh_usb2com_common_topaz_v1:cdevice.obj
 0001:000083d8       ??_C@_1KM@JACIJAAL@?$AAC?$AAF?$AAu?$AAn?$AAc?$AAt?$AAi?$AAo?$AAn?$AA?$CI?$AAt?$AAi?$AAe?$AAr?$AA?5?$AA?$CF?$AAd?$AA?$CJ?$AA?3?$AA?3?$AAO?$AAp?$AAe?$AAn?$AAP?$AAi?$AAp?$AAe?$AA?5?$AA?9?$AA?5?$AAa@ 100093d8     usbh_usb2com_common_topaz_v1:cdevice.obj
 0001:00008488       ??_C@_1ME@KAFNGAIE@?$AAC?$AAF?$AAu?$AAn?$AAc?$AAt?$AAi?$AAo?$AAn?$AA?$CI?$AAt?$AAi?$AAe?$AAr?$AA?5?$AA?$CF?$AAd?$AA?$CJ?$AA?3?$AA?3?$AAO?$AAp?$AAe?$AAn?$AAP?$AAi?$AAp?$AAe?$AA?5?$AA?9?$AA?5?$AAe@ 10009488     usbh_usb2com_common_topaz_v1:cdevice.obj
 0001:00008550       ??_C@_1FM@LHKAGABP@?$AA?$CL?$AAC?$AAF?$AAu?$AAn?$AAc?$AAt?$AAi?$AAo?$AAn?$AA?$CI?$AAt?$AAi?$AAe?$AAr?$AA?5?$AA?$CF?$AAd?$AA?$CJ?$AA?3?$AA?3?$AAO?$AAp?$AAe?$AAn?$AAP?$AAi?$AAp?$AAe?$AA?5?$AA?9?$AA?5@ 10009550     usbh_usb2com_common_topaz_v1:cdevice.obj
 0001:000085b0       ??_C@_1LE@CFCEGCI@?$AA?9?$AAC?$AAF?$AAu?$AAn?$AAc?$AAt?$AAi?$AAo?$AAn?$AA?$CI?$AAt?$AAi?$AAe?$AAr?$AA?5?$AA?$CF?$AAd?$AA?$CJ?$AA?3?$AA?3?$AAC?$AAl?$AAo?$AAs?$AAe?$AAP?$AAi?$AAp?$AAe?$AA?5?$AA?9@ 100095b0     usbh_usb2com_common_topaz_v1:cdevice.obj
 0001:00008668       ??_C@_1KG@MIBBGHMA@?$AAC?$AAF?$AAu?$AAn?$AAc?$AAt?$AAi?$AAo?$AAn?$AA?$CI?$AAt?$AAi?$AAe?$AAr?$AA?5?$AA?$CF?$AAd?$AA?$CJ?$AA?3?$AA?3?$AAC?$AAl?$AAo?$AAs?$AAe?$AAP?$AAi?$AAp?$AAe?$AA?5?$AA?9?$AA?5@ 10009668     usbh_usb2com_common_topaz_v1:cdevice.obj
 0001:00008710       ??_C@_1IA@LNBOPBH@?$AAC?$AAF?$AAu?$AAn?$AAc?$AAt?$AAi?$AAo?$AAn?$AA?$CI?$AAt?$AAi?$AAe?$AAr?$AA?5?$AA?$CF?$AAd?$AA?$CJ?$AA?3?$AA?3?$AAC?$AAl?$AAo?$AAs?$AAe?$AAP?$AAi?$AAp?$AAe?$AA?5?$AA?9?$AA?5@ 10009710     usbh_usb2com_common_topaz_v1:cdevice.obj
 0001:00008790       ??_C@_1HE@FILFIPFM@?$AA?$CL?$AAC?$AAF?$AAu?$AAn?$AAc?$AAt?$AAi?$AAo?$AAn?$AA?$CI?$AAt?$AAi?$AAe?$AAr?$AA?5?$AA?$CF?$AAd?$AA?$CJ?$AA?3?$AA?3?$AAC?$AAl?$AAo?$AAs?$AAe?$AAP?$AAi?$AAp?$AAe?$AA?5?$AA?9@ 10009790     usbh_usb2com_common_topaz_v1:cdevice.obj
 0001:00008808       ??_C@_1IK@JNPJLHDE@?$AA?9?$AAC?$AAF?$AAu?$AAn?$AAc?$AAt?$AAi?$AAo?$AAn?$AA?$CI?$AAt?$AAi?$AAe?$AAr?$AA?5?$AA?$CF?$AAd?$AA?$CJ?$AA?3?$AA?3?$AAI?$AAs?$AAs?$AAu?$AAe?$AAT?$AAr?$AAa?$AAn?$AAs?$AAf@ 10009808     usbh_usb2com_common_topaz_v1:cdevice.obj
 0001:00008898       ??_C@_1EI@BLOBBPOH@?$AA?$CL?$AAC?$AAF?$AAu?$AAn?$AAc?$AAt?$AAi?$AAo?$AAn?$AA?$CI?$AAt?$AAi?$AAe?$AAr?$AA?5?$AA?$CF?$AAd?$AA?$CJ?$AA?3?$AA?3?$AAI?$AAs?$AAs?$AAu?$AAe?$AAT?$AAr?$AAa?$AAn?$AAs?$AAf@ 10009898     usbh_usb2com_common_topaz_v1:cdevice.obj
 0001:000088e0       ??_C@_1LM@GKIPBFAK@?$AA?9?$AAC?$AAF?$AAu?$AAn?$AAc?$AAt?$AAi?$AAo?$AAn?$AA?$CI?$AAt?$AAi?$AAe?$AAr?$AA?5?$AA?$CF?$AAd?$AA?$CJ?$AA?3?$AA?3?$AAA?$AAb?$AAo?$AAr?$AAt?$AAT?$AAr?$AAa?$AAn?$AAs?$AAf@ 100098e0     usbh_usb2com_common_topaz_v1:cdevice.obj
 0001:000089a0       ??_C@_1HM@LNHMIHEJ@?$AA?$CL?$AAC?$AAF?$AAu?$AAn?$AAc?$AAt?$AAi?$AAo?$AAn?$AA?$CI?$AAt?$AAi?$AAe?$AAr?$AA?5?$AA?$CF?$AAd?$AA?$CJ?$AA?3?$AA?3?$AAA?$AAb?$AAo?$AAr?$AAt?$AAT?$AAr?$AAa?$AAn?$AAs?$AAf@ 100099a0     usbh_usb2com_common_topaz_v1:cdevice.obj
 0001:00008a20       ??_C@_1LK@JJFGCKDD@?$AA?9?$AAC?$AAF?$AAu?$AAn?$AAc?$AAt?$AAi?$AAo?$AAn?$AA?$CI?$AAt?$AAi?$AAe?$AAr?$AA?5?$AA?$CF?$AAd?$AA?$CJ?$AA?3?$AA?3?$AAI?$AAs?$AAP?$AAi?$AAp?$AAe?$AAH?$AAa?$AAl?$AAt?$AAe@ 10009a20     usbh_usb2com_common_topaz_v1:cdevice.obj
 0001:00008ae0       ??_C@_1HK@JILDILFA@?$AA?$CL?$AAC?$AAF?$AAu?$AAn?$AAc?$AAt?$AAi?$AAo?$AAn?$AA?$CI?$AAt?$AAi?$AAe?$AAr?$AA?5?$AA?$CF?$AAd?$AA?$CJ?$AA?3?$AA?3?$AAI?$AAs?$AAP?$AAi?$AAp?$AAe?$AAH?$AAa?$AAl?$AAt?$AAe@ 10009ae0     usbh_usb2com_common_topaz_v1:cdevice.obj
 0001:00008b60       ??_C@_1LE@BINMLMAA@?$AA?9?$AAC?$AAF?$AAu?$AAn?$AAc?$AAt?$AAi?$AAo?$AAn?$AA?$CI?$AAt?$AAi?$AAe?$AAr?$AA?5?$AA?$CF?$AAd?$AA?$CJ?$AA?3?$AA?3?$AAR?$AAe?$AAs?$AAe?$AAt?$AAP?$AAi?$AAp?$AAe?$AA?5?$AA?9@ 10009b60     usbh_usb2com_common_topaz_v1:cdevice.obj
 0001:00008c18       ??_C@_1HE@CMDAIMMM@?$AA?$CL?$AAC?$AAF?$AAu?$AAn?$AAc?$AAt?$AAi?$AAo?$AAn?$AA?$CI?$AAt?$AAi?$AAe?$AAr?$AA?5?$AA?$CF?$AAd?$AA?$CJ?$AA?3?$AA?3?$AAR?$AAe?$AAs?$AAe?$AAt?$AAP?$AAi?$AAp?$AAe?$AA?5?$AA?9@ 10009c18     usbh_usb2com_common_topaz_v1:cdevice.obj
 0001:00008c90       ??_C@_1EG@JMCHJCGL@?$AA?9?$AAC?$AAF?$AAu?$AAn?$AAc?$AAt?$AAi?$AAo?$AAn?$AA?$CI?$AAt?$AAi?$AAe?$AAr?$AA?5?$AA?$CF?$AAd?$AA?$CJ?$AA?3?$AA?3?$AAH?$AAa?$AAn?$AAd?$AAl?$AAe?$AAD?$AAe?$AAt?$AAa?$AAc@ 10009c90     usbh_usb2com_common_topaz_v1:cdevice.obj
 0001:00008cd8       ??_C@_1EG@JAACAFFA@?$AA?$CL?$AAC?$AAF?$AAu?$AAn?$AAc?$AAt?$AAi?$AAo?$AAn?$AA?$CI?$AAt?$AAi?$AAe?$AAr?$AA?5?$AA?$CF?$AAd?$AA?$CJ?$AA?3?$AA?3?$AAH?$AAa?$AAn?$AAd?$AAl?$AAe?$AAD?$AAe?$AAt?$AAa?$AAc@ 10009cd8     usbh_usb2com_common_topaz_v1:cdevice.obj
 0001:00008d20       ??_C@_1OC@CDIKDMDG@?$AA?9?$AAC?$AAF?$AAu?$AAn?$AAc?$AAt?$AAi?$AAo?$AAn?$AA?3?$AA?3?$AAS?$AAe?$AAt?$AAO?$AAr?$AAC?$AAl?$AAe?$AAa?$AAr?$AAF?$AAe?$AAa?$AAt?$AAu?$AAr?$AAe?$AA?5?$AA?9?$AA?5@ 10009d20     usbh_usb2com_common_topaz_v1:cdevice.obj
 0001:00008e08       ??_C@_1MM@KEJIBKLK@?$AAC?$AAF?$AAu?$AAn?$AAc?$AAt?$AAi?$AAo?$AAn?$AA?3?$AA?3?$AAS?$AAe?$AAt?$AAO?$AAr?$AAC?$AAl?$AAe?$AAa?$AAr?$AAF?$AAe?$AAa?$AAt?$AAu?$AAr?$AAe?$AA?5?$AA?9?$AA?5?$AAr@ 10009e08     usbh_usb2com_common_topaz_v1:cdevice.obj
 0001:00008ed8       ??_C@_1KI@NHPPIIBA@?$AA?$CB?$AA?$CB?$AA?$CB?$AAC?$AAF?$AAu?$AAn?$AAc?$AAt?$AAi?$AAo?$AAn?$AA?$CI?$AA?5?$AAt?$AAi?$AAe?$AAr?$AA?5?$AA?$CF?$AAd?$AA?$CJ?$AA?3?$AA?3?$AAS?$AAe?$AAt?$AAO?$AAr?$AAC?$AAl?$AAe@ 10009ed8     usbh_usb2com_common_topaz_v1:cdevice.obj
 0001:00008f80       ??_C@_1LO@LLOAFJJK@?$AA?$CL?$AAC?$AAF?$AAu?$AAn?$AAc?$AAt?$AAi?$AAo?$AAn?$AA?3?$AA?3?$AAS?$AAe?$AAt?$AAO?$AAr?$AAC?$AAl?$AAe?$AAa?$AAr?$AAF?$AAe?$AAa?$AAt?$AAu?$AAr?$AAe?$AA?5?$AA?9?$AA?5@ 10009f80     usbh_usb2com_common_topaz_v1:cdevice.obj
 0001:00009040       ??_C@_1MA@CAEDHJEG@?$AAC?$AA?3?$AA?2?$AAW?$AAI?$AAN?$AAC?$AAE?$AAR?$AAO?$AAO?$AAT?$AAS?$AA?2?$AAT?$AAo?$AAp?$AAa?$AAz?$AA?2?$AAW?$AAI?$AAN?$AAC?$AAE?$AA6?$AA0?$AA0?$AA?2?$AAp?$AAl?$AAa@ 1000a040     usbh_usb2com_common_topaz_v1:sync.obj
 0001:00009100       ??_C@_1BO@MFMGCEN@?$AA?9?$AAC?$AAE?$AAh?$AAc?$AAd?$AA?3?$AA?3?$AAC?$AAE?$AAh?$AAc?$AAd?$AA?6?$AA?$AA@ 1000a100     usbh_ehcdmdd_common_topaz_v1:cehcd.obj
 0001:00009120       ??_C@_1BO@IFBOCIHN@?$AA?$CL?$AAC?$AAE?$AAh?$AAc?$AAd?$AA?3?$AA?3?$AAC?$AAE?$AAh?$AAc?$AAd?$AA?6?$AA?$AA@ 1000a120     usbh_ehcdmdd_common_topaz_v1:cehcd.obj
 0001:00009140       ??_7CEhcd@@6B@             1000a140     usbh_ehcdmdd_common_topaz_v1:cehcd.obj
 0001:000091b8       ??_C@_1CA@MPADNHNK@?$AA?9?$AAC?$AAE?$AAh?$AAc?$AAd?$AA?3?$AA?3?$AA?$HO?$AAC?$AAE?$AAh?$AAc?$AAd?$AA?6?$AA?$AA@ 1000a1b8     usbh_ehcdmdd_common_topaz_v1:cehcd.obj
 0001:000091d8       ??_C@_1CA@IGEMMAOF@?$AA?$CL?$AAC?$AAE?$AAh?$AAc?$AAd?$AA?3?$AA?3?$AA?$HO?$AAC?$AAE?$AAh?$AAc?$AAd?$AA?6?$AA?$AA@ 1000a1d8     usbh_ehcdmdd_common_topaz_v1:cehcd.obj
 0001:000091f8       ??_C@_1CM@DECAPEAG@?$AA?9?$AAC?$AAE?$AAh?$AAc?$AAd?$AA?3?$AA?3?$AAD?$AAe?$AAI?$AAn?$AAi?$AAt?$AAi?$AAa?$AAl?$AAi?$AAz?$AAe?$AA?6?$AA?$AA@ 1000a1f8     usbh_ehcdmdd_common_topaz_v1:cehcd.obj
 0001:00009224       ??_C@_1CM@MINAGFEK@?$AA?$CL?$AAC?$AAE?$AAh?$AAc?$AAd?$AA?3?$AA?3?$AAD?$AAe?$AAI?$AAn?$AAi?$AAt?$AAi?$AAa?$AAl?$AAi?$AAz?$AAe?$AA?6?$AA?$AA@ 1000a224     usbh_ehcdmdd_common_topaz_v1:cehcd.obj
 0001:00009250       ??_C@_1EA@FJFHOJOA@?$AA?9?$AAC?$AAE?$AAh?$AAc?$AAd?$AA?3?$AA?3?$AAI?$AAn?$AAi?$AAt?$AAi?$AAa?$AAl?$AAi?$AAz?$AAe?$AA?4?$AA?5?$AAS?$AAu?$AAc?$AAc?$AAe?$AAs?$AAs?$AA?$CB?$AA?$CB?$AA?$AN?$AA?6?$AA?$AA@ 1000a250     usbh_ehcdmdd_common_topaz_v1:cehcd.obj
 0001:00009290       ??_C@_1GC@CLFDOADC@?$AA?9?$AAC?$AAE?$AAh?$AAc?$AAd?$AA?3?$AA?3?$AAI?$AAn?$AAi?$AAt?$AAi?$AAa?$AAl?$AAi?$AAz?$AAe?$AA?4?$AA?5?$AAE?$AAr?$AAr?$AAo?$AAr?$AA?5?$AAi?$AAn?$AAi?$AAt?$AAi?$AAa@ 1000a290     usbh_ehcdmdd_common_topaz_v1:cehcd.obj
 0001:000092f8       ??_C@_1GO@FCBMJNBH@?$AA?9?$AAC?$AAE?$AAh?$AAc?$AAd?$AA?3?$AA?3?$AAI?$AAn?$AAi?$AAt?$AAi?$AAa?$AAl?$AAi?$AAz?$AAe?$AA?5?$AA?9?$AA?5?$AAu?$AAn?$AAa?$AAb?$AAl?$AAe?$AA?5?$AAt?$AAo?$AA?5?$AAc@ 1000a2f8     usbh_ehcdmdd_common_topaz_v1:cehcd.obj
 0001:00009368       ??_C@_1LM@EKBLHICJ@?$AAC?$AA?3?$AA?2?$AAW?$AAI?$AAN?$AAC?$AAE?$AAR?$AAO?$AAO?$AAT?$AAS?$AA?2?$AAT?$AAo?$AAp?$AAa?$AAz?$AA?2?$AAW?$AAI?$AAN?$AAC?$AAE?$AA6?$AA0?$AA0?$AA?2?$AAP?$AAL?$AAA@ 1000a368     usbh_ehcdmdd_common_topaz_v1:cehcd.obj
 0001:00009428       ??_C@_1JC@CPGBLJL@?$AA?9?$AAC?$AAE?$AAh?$AAc?$AAd?$AA?3?$AA?3?$AAI?$AAn?$AAi?$AAt?$AAi?$AAa?$AAl?$AAi?$AAz?$AAe?$AA?4?$AA?5?$AAE?$AAr?$AAr?$AAo?$AAr?$AA?5?$AA?9?$AA?5?$AAc?$AAo?$AAu?$AAl@ 1000a428     usbh_ehcdmdd_common_topaz_v1:cehcd.obj
 0001:000094bc       ??_C@_1DI@IAIONEJK@?$AA?$CL?$AAC?$AAE?$AAh?$AAc?$AAd?$AA?3?$AA?3?$AAI?$AAn?$AAi?$AAt?$AAi?$AAa?$AAl?$AAi?$AAz?$AAe?$AA?4?$AA?5?$AAE?$AAn?$AAt?$AAr?$AAy?$AA?$AN?$AA?6?$AA?$AA@ 1000a4bc     usbh_ehcdmdd_common_topaz_v1:cehcd.obj
 0001:000094f4       ??_C@_1BO@FNFLKEKD@?$AA?9?$AAC?$AAP?$AAi?$AAp?$AAe?$AA?3?$AA?3?$AAC?$AAP?$AAi?$AAp?$AAe?$AA?6?$AA?$AA@ 1000a4f4     usbh_ehcdmdd_common_topaz_v1:cpipe.obj
 0001:00009514       ??_C@_1BO@NEBJOOJD@?$AA?$CL?$AAC?$AAP?$AAi?$AAp?$AAe?$AA?3?$AA?3?$AAC?$AAP?$AAi?$AAp?$AAe?$AA?6?$AA?$AA@ 1000a514     usbh_ehcdmdd_common_topaz_v1:cpipe.obj
 0001:00009534       ??_7CPipe@@6B@             1000a534     usbh_ehcdmdd_common_topaz_v1:cpipe.obj
 0001:0000956c       ??_7CPipeAbs@@6B@          1000a56c     usbh_ehcdmdd_common_topaz_v1:cpipe.obj
 0001:00009590       ??_C@_1MC@FNHLHGBI@?$AAC?$AA?3?$AA?2?$AAW?$AAI?$AAN?$AAC?$AAE?$AAR?$AAO?$AAO?$AAT?$AAS?$AA?2?$AAT?$AAo?$AAp?$AAa?$AAz?$AA?2?$AAW?$AAI?$AAN?$AAC?$AAE?$AA6?$AA0?$AA0?$AA?2?$AAp?$AAl?$AAa@ 1000a590     usbh_ehcdmdd_common_topaz_v1:cpipe.obj
 0001:00009654       ??_C@_1CA@EGGPAPJO@?$AA?9?$AAC?$AAP?$AAi?$AAp?$AAe?$AA?3?$AA?3?$AA?$HO?$AAC?$AAP?$AAi?$AAp?$AAe?$AA?6?$AA?$AA@ 1000a654     usbh_ehcdmdd_common_topaz_v1:cpipe.obj
 0001:00009674       ??_C@_1CA@PCABIKB@?$AA?$CL?$AAC?$AAP?$AAi?$AAp?$AAe?$AA?3?$AA?3?$AA?$HO?$AAC?$AAP?$AAi?$AAp?$AAe?$AA?6?$AA?$AA@ 1000a674     usbh_ehcdmdd_common_topaz_v1:cpipe.obj
 0001:00009698       ??_C@_1JI@LFEJLGMB@?$AA?9?$AAC?$AAP?$AAi?$AAp?$AAe?$AA?$CI?$AA?$CF?$AAs?$AA?$CJ?$AA?3?$AA?3?$AAI?$AAs?$AAP?$AAi?$AAp?$AAe?$AAH?$AAa?$AAl?$AAt?$AAe?$AAd?$AA?0?$AA?5?$AA?$CK?$AAl?$AAp?$AAb?$AAH?$AAa@ 1000a698     usbh_ehcdmdd_common_topaz_v1:cpipe.obj
 0001:00009730       ??_C@_1LM@KPFMIBJP@?$AAC?$AA?3?$AA?2?$AAW?$AAI?$AAN?$AAC?$AAE?$AAR?$AAO?$AAO?$AAT?$AAS?$AA?2?$AAT?$AAo?$AAp?$AAa?$AAz?$AA?2?$AAW?$AAI?$AAN?$AAC?$AAE?$AA6?$AA0?$AA0?$AA?2?$AAP?$AAL?$AAA@ 1000a730     usbh_ehcdmdd_common_topaz_v1:cpipe.obj
 0001:000097ec       ??_C@_1DE@MCCIDDLK@?$AA?$CL?$AAC?$AAP?$AAi?$AAp?$AAe?$AA?$CI?$AA?$CF?$AAs?$AA?$CJ?$AA?3?$AA?3?$AAI?$AAs?$AAP?$AAi?$AAp?$AAe?$AAH?$AAa?$AAl?$AAt?$AAe?$AAd?$AA?6?$AA?$AA@ 1000a7ec     usbh_ehcdmdd_common_topaz_v1:cpipe.obj
 0001:00009820       ??_C@_1DK@INACOAAB@?$AA?9?$AAC?$AAP?$AAi?$AAp?$AAe?$AA?$CI?$AA?$CF?$AAs?$AA?$CJ?$AA?3?$AA?3?$AAC?$AAl?$AAe?$AAa?$AAr?$AAH?$AAa?$AAl?$AAt?$AAe?$AAd?$AAF?$AAl?$AAa?$AAg?$AA?6?$AA?$AA@ 1000a820     usbh_ehcdmdd_common_topaz_v1:cpipe.obj
 0001:00009860       ??_C@_1IE@IBNINFFO@?$AAC?$AAP?$AAi?$AAp?$AAe?$AA?$CI?$AA?$CF?$AAs?$AA?$CJ?$AA?3?$AA?3?$AAC?$AAl?$AAe?$AAa?$AAr?$AAH?$AAa?$AAl?$AAt?$AAe?$AAd?$AAF?$AAl?$AAa?$AAg?$AA?5?$AA?9?$AA?5?$AAw?$AAa?$AAr@ 1000a860     usbh_ehcdmdd_common_topaz_v1:cpipe.obj
 0001:000098e4       ??_C@_1DK@OIOBMHCK@?$AA?$CL?$AAC?$AAP?$AAi?$AAp?$AAe?$AA?$CI?$AA?$CF?$AAs?$AA?$CJ?$AA?3?$AA?3?$AAC?$AAl?$AAe?$AAa?$AAr?$AAH?$AAa?$AAl?$AAt?$AAe?$AAd?$AAF?$AAl?$AAa?$AAg?$AA?6?$AA?$AA@ 1000a8e4     usbh_ehcdmdd_common_topaz_v1:cpipe.obj
 0001:00009920       ??_C@_1DG@HGODKGLN@?$AA?9?$AAC?$AAQ?$AAu?$AAe?$AAu?$AAe?$AAd?$AAP?$AAi?$AAp?$AAe?$AA?3?$AA?3?$AAC?$AAQ?$AAu?$AAe?$AAu?$AAe?$AAd?$AAP?$AAi?$AAp?$AAe?$AA?6?$AA?$AA@ 1000a920     usbh_ehcdmdd_common_topaz_v1:cpipe.obj
 0001:00009958       ??_C@_1DG@HDDOFDAJ@?$AA?$CL?$AAC?$AAQ?$AAu?$AAe?$AAu?$AAe?$AAd?$AAP?$AAi?$AAp?$AAe?$AA?3?$AA?3?$AAC?$AAQ?$AAu?$AAe?$AAu?$AAe?$AAd?$AAP?$AAi?$AAp?$AAe?$AA?6?$AA?$AA@ 1000a958     usbh_ehcdmdd_common_topaz_v1:cpipe.obj
 0001:00009990       ??_7CQueuedPipe@@6B@       1000a990     usbh_ehcdmdd_common_topaz_v1:cpipe.obj
 0001:000099d0       ??_C@_1DI@OKMEGAFJ@?$AA?9?$AAC?$AAQ?$AAu?$AAe?$AAu?$AAe?$AAd?$AAP?$AAi?$AAp?$AAe?$AA?3?$AA?3?$AA?$HO?$AAC?$AAQ?$AAu?$AAe?$AAu?$AAe?$AAd?$AAP?$AAi?$AAp?$AAe?$AA?6?$AA?$AA@ 1000a9d0     usbh_ehcdmdd_common_topaz_v1:cpipe.obj
 0001:00009a08       ??_C@_1DI@KHLKAIKL@?$AA?$CL?$AAC?$AAQ?$AAu?$AAe?$AAu?$AAe?$AAd?$AAP?$AAi?$AAp?$AAe?$AA?3?$AA?3?$AA?$HO?$AAC?$AAQ?$AAu?$AAe?$AAu?$AAe?$AAd?$AAP?$AAi?$AAp?$AAe?$AA?6?$AA?$AA@ 1000aa08     usbh_ehcdmdd_common_topaz_v1:cpipe.obj
 0001:00009a40       ??_C@_1KO@FHDEKCOL@?$AA?9?$AAC?$AAQ?$AAu?$AAe?$AAu?$AAe?$AAd?$AAP?$AAi?$AAp?$AAe?$AA?$CI?$AA?$CF?$AAs?$AA?$CJ?$AA?3?$AA?3?$AAA?$AAb?$AAo?$AAr?$AAt?$AAT?$AAr?$AAa?$AAn?$AAs?$AAf?$AAe?$AAr?$AA?5@ 1000aa40     usbh_ehcdmdd_common_topaz_v1:cpipe.obj
 0001:00009af0       ??_C@_1KC@DEIOLPMB@?$AAC?$AAQ?$AAu?$AAe?$AAu?$AAe?$AAd?$AAP?$AAi?$AAp?$AAe?$AA?3?$AA?3?$AAA?$AAb?$AAo?$AAr?$AAt?$AAT?$AAr?$AAa?$AAn?$AAs?$AAf?$AAe?$AAr?$AA?5?$AA?9?$AA?5?$AAe?$AAx?$AAc@ 1000aaf0     usbh_ehcdmdd_common_topaz_v1:cpipe.obj
 0001:00009b98       ??_C@_1GM@NGEPGNBL@?$AA?$CL?$AAC?$AAQ?$AAu?$AAe?$AAu?$AAe?$AAd?$AAP?$AAi?$AAp?$AAe?$AA?$CI?$AA?$CF?$AAs?$AA?$CJ?$AA?3?$AA?3?$AAA?$AAb?$AAo?$AAr?$AAt?$AAT?$AAr?$AAa?$AAn?$AAs?$AAf?$AAe?$AAr?$AA?5@ 1000ab98     usbh_ehcdmdd_common_topaz_v1:cpipe.obj
 0001:00009c04       ??_C@_1BA@BOPMONDN@?$AA?4?$AA?2?$AAc?$AAt?$AAd?$AA?4?$AAh?$AA?$AA@ 1000ac04     usbh_ehcdmdd_common_topaz_v1:cpipe.obj
 0001:00009c18       ??_C@_1EG@KEDADMGJ@?$AA?9?$AAC?$AAQ?$AAu?$AAe?$AAu?$AAe?$AAd?$AAP?$AAi?$AAp?$AAe?$AA?$CI?$AA?$CF?$AAs?$AA?$CJ?$AA?3?$AA?3?$AAC?$AAl?$AAe?$AAa?$AAr?$AAH?$AAa?$AAl?$AAt?$AAe?$AAd?$AAF?$AAl?$AAa@ 1000ac18     usbh_ehcdmdd_common_topaz_v1:cpipe.obj
 0001:00009c60       ??_C@_1JA@OOFNJMIL@?$AAC?$AAQ?$AAu?$AAe?$AAu?$AAe?$AAd?$AAP?$AAi?$AAp?$AAe?$AA?$CI?$AA?$CF?$AAs?$AA?$CJ?$AA?3?$AA?3?$AAC?$AAl?$AAe?$AAa?$AAr?$AAH?$AAa?$AAl?$AAt?$AAe?$AAd?$AAF?$AAl?$AAa?$AAg@ 1000ac60     usbh_ehcdmdd_common_topaz_v1:cpipe.obj
 0001:00009cf0       ??_C@_1EG@KIBFKLFC@?$AA?$CL?$AAC?$AAQ?$AAu?$AAe?$AAu?$AAe?$AAd?$AAP?$AAi?$AAp?$AAe?$AA?$CI?$AA?$CF?$AAs?$AA?$CJ?$AA?3?$AA?3?$AAC?$AAl?$AAe?$AAa?$AAr?$AAH?$AAa?$AAl?$AAt?$AAe?$AAd?$AAF?$AAl?$AAa@ 1000acf0     usbh_ehcdmdd_common_topaz_v1:cpipe.obj
 0001:00009d38       ??_C@_1EG@EBGMCDLC@?$AA?9?$AAC?$AAQ?$AAu?$AAe?$AAu?$AAe?$AAd?$AAP?$AAi?$AAp?$AAe?$AA?$CI?$AA?$CF?$AAs?$AA?$CJ?$AA?3?$AA?3?$AAA?$AAb?$AAo?$AAr?$AAt?$AAQ?$AAu?$AAe?$AAu?$AAe?$AA?5?$AA?9?$AA?5?$AA?$CF@ 1000ad38     usbh_ehcdmdd_common_topaz_v1:cpipe.obj
 0001:00009d80       ??_C@_1DO@NGPDGELJ@?$AA?$CL?$AAC?$AAQ?$AAu?$AAe?$AAu?$AAe?$AAd?$AAP?$AAi?$AAp?$AAe?$AA?$CI?$AA?$CF?$AAs?$AA?$CJ?$AA?3?$AA?3?$AAA?$AAb?$AAo?$AAr?$AAt?$AAQ?$AAu?$AAe?$AAu?$AAe?$AA?5?$AA?6?$AA?$AA@ 1000ad80     usbh_ehcdmdd_common_topaz_v1:cpipe.obj
 0001:00009dc0       ??_C@_1JE@GOMEIDDI@?$AA?9?$AAC?$AAP?$AAi?$AAp?$AAe?$AA?$CI?$AA?$CF?$AAs?$AA?$CJ?$AA?3?$AA?3?$AAI?$AAs?$AAs?$AAu?$AAe?$AAT?$AAr?$AAa?$AAn?$AAs?$AAf?$AAe?$AAr?$AA?5?$AA?9?$AA?5?$AAa?$AAd?$AAd?$AAr@ 1000adc0     usbh_ehcdmdd_common_topaz_v1:cpipe.obj
 0001:00009e58       ??_C@_1FC@PKJGBOEE@?$AA?$CL?$AAC?$AAP?$AAi?$AAp?$AAe?$AA?$CI?$AA?$CF?$AAs?$AA?$CJ?$AA?3?$AA?3?$AAI?$AAs?$AAs?$AAu?$AAe?$AAT?$AAr?$AAa?$AAn?$AAs?$AAf?$AAe?$AAr?$AA?0?$AA?5?$AAa?$AAd?$AAd?$AAr?$AAe@ 1000ae58     usbh_ehcdmdd_common_topaz_v1:cpipe.obj
 0001:00009eac       ??_7CQTransfer@@6B@        1000aeac     usbh_ehcdmdd_common_topaz_v1:cpipe.obj
 0001:00009eb8       ??_C@_1DI@HGFMJLPJ@?$AAC?$AAQ?$AAu?$AAe?$AAu?$AAe?$AAP?$AAi?$AAp?$AAe?$AA?3?$AA?3?$AAS?$AAt?$AAo?$AAp?$AAT?$AAr?$AAa?$AAn?$AAs?$AAf?$AAe?$AAr?$AAs?$AA?$AN?$AA?6?$AA?$AA@ 1000aeb8     usbh_ehcdmdd_common_topaz_v1:cpipe.obj
 0001:00009ef0       ??_C@_1LG@LENACAKG@?$AA?9?$AAC?$AAP?$AAi?$AAp?$AAe?$AA?$CI?$AA?$CF?$AAs?$AA?$CJ?$AA?3?$AA?3?$AAS?$AAc?$AAh?$AAe?$AAd?$AAu?$AAl?$AAe?$AAT?$AAr?$AAa?$AAn?$AAs?$AAf?$AAe?$AAr?$AA?5?$AA?9?$AA?5?$AAS@ 1000aef0     usbh_ehcdmdd_common_topaz_v1:cpipe.obj
 0001:00009fa8       ??_C@_1CO@BAFFGEGA@?$AA?9?$AAC?$AAB?$AAu?$AAl?$AAk?$AAP?$AAi?$AAp?$AAe?$AA?3?$AA?3?$AAC?$AAB?$AAu?$AAl?$AAk?$AAP?$AAi?$AAp?$AAe?$AA?6?$AA?$AA@ 1000afa8     usbh_ehcdmdd_common_topaz_v1:cpipe.obj
 0001:00009fd8       ??_C@_1CO@MLJBDLEL@?$AA?$CL?$AAC?$AAB?$AAu?$AAl?$AAk?$AAP?$AAi?$AAp?$AAe?$AA?3?$AA?3?$AAC?$AAB?$AAu?$AAl?$AAk?$AAP?$AAi?$AAp?$AAe?$AA?6?$AA?$AA@ 1000afd8     usbh_ehcdmdd_common_topaz_v1:cpipe.obj
 0001:0000a008       ??_7CBulkPipe@@6B@         1000b008     usbh_ehcdmdd_common_topaz_v1:cpipe.obj
 0001:0000a048       ??_C@_19PBJLGAMD@?$AAB?$AAu?$AAl?$AAk?$AA?$AA@ 1000b048     usbh_ehcdmdd_common_topaz_v1:cpipe.obj
 0001:0000a054       ??_C@_1DA@KHCPKGIF@?$AA?9?$AAC?$AAB?$AAu?$AAl?$AAk?$AAP?$AAi?$AAp?$AAe?$AA?3?$AA?3?$AA?$HO?$AAC?$AAB?$AAu?$AAl?$AAk?$AAP?$AAi?$AAp?$AAe?$AA?6?$AA?$AA@ 1000b054     usbh_ehcdmdd_common_topaz_v1:cpipe.obj
 0001:0000a084       ??_C@_1DA@CKILMMEN@?$AA?$CL?$AAC?$AAB?$AAu?$AAl?$AAk?$AAP?$AAi?$AAp?$AAe?$AA?3?$AA?3?$AA?$HO?$AAC?$AAB?$AAu?$AAl?$AAk?$AAP?$AAi?$AAp?$AAe?$AA?6?$AA?$AA@ 1000b084     usbh_ehcdmdd_common_topaz_v1:cpipe.obj
 0001:0000a0b8       ??_C@_1GO@DDNGLOEL@?$AA?9?$AAC?$AAB?$AAu?$AAl?$AAk?$AAP?$AAi?$AAp?$AAe?$AA?3?$AA?3?$AAO?$AAp?$AAe?$AAn?$AAP?$AAi?$AAp?$AAe?$AA?0?$AA?5?$AAr?$AAe?$AAt?$AAu?$AAr?$AAn?$AAi?$AAn?$AAg?$AA?5@ 1000b0b8     usbh_ehcdmdd_common_topaz_v1:cpipe.obj
 0001:0000a128       ??_C@_1CM@HNACDBOM@?$AA?$CL?$AAC?$AAB?$AAu?$AAl?$AAk?$AAP?$AAi?$AAp?$AAe?$AA?3?$AA?3?$AAO?$AAp?$AAe?$AAn?$AAP?$AAi?$AAp?$AAe?$AA?6?$AA?$AA@ 1000b128     usbh_ehcdmdd_common_topaz_v1:cpipe.obj
 0001:0000a154       ??_C@_1DG@IGDHGBCL@?$AA?$CL?$AAC?$AAB?$AAu?$AAl?$AAk?$AAP?$AAi?$AAp?$AAe?$AA?$CI?$AA?$CF?$AAs?$AA?$CJ?$AA?3?$AA?3?$AAC?$AAl?$AAo?$AAs?$AAe?$AAP?$AAi?$AAp?$AAe?$AA?6?$AA?$AA@ 1000b154     usbh_ehcdmdd_common_topaz_v1:cpipe.obj
 0001:0000a190       ??_C@_1HG@DDFHCFDD@?$AA?$CB?$AAC?$AAB?$AAu?$AAl?$AAk?$AAP?$AAi?$AAp?$AAe?$AA?3?$AA?3?$AAA?$AAr?$AAe?$AAT?$AAr?$AAa?$AAn?$AAs?$AAf?$AAe?$AAr?$AAP?$AAa?$AAr?$AAa?$AAm?$AAe?$AAt?$AAe?$AAr@ 1000b190     usbh_ehcdmdd_common_topaz_v1:cpipe.obj
 0001:0000a208       ??_C@_1DK@PKKLHODC@?$AA?9?$AAC?$AAC?$AAo?$AAn?$AAt?$AAr?$AAo?$AAl?$AAP?$AAi?$AAp?$AAe?$AA?3?$AA?3?$AAC?$AAC?$AAo?$AAn?$AAt?$AAr?$AAo?$AAl?$AAP?$AAi?$AAp?$AAe?$AA?6?$AA?$AA@ 1000b208     usbh_ehcdmdd_common_topaz_v1:cpipe.obj
 0001:0000a244       ??_C@_1DK@JPEIFJBJ@?$AA?$CL?$AAC?$AAC?$AAo?$AAn?$AAt?$AAr?$AAo?$AAl?$AAP?$AAi?$AAp?$AAe?$AA?3?$AA?3?$AAC?$AAC?$AAo?$AAn?$AAt?$AAr?$AAo?$AAl?$AAP?$AAi?$AAp?$AAe?$AA?6?$AA?$AA@ 1000b244     usbh_ehcdmdd_common_topaz_v1:cpipe.obj
 0001:0000a280       ??_7CControlPipe@@6B@      1000b280     usbh_ehcdmdd_common_topaz_v1:cpipe.obj
 0001:0000a2c0       ??_C@_1BA@JGFNDEFA@?$AAC?$AAo?$AAn?$AAt?$AAr?$AAo?$AAl?$AA?$AA@ 1000b2c0     usbh_ehcdmdd_common_topaz_v1:cpipe.obj
 0001:0000a2d0       ??_C@_1DM@HAHKKHKF@?$AA?9?$AAC?$AAC?$AAo?$AAn?$AAt?$AAr?$AAo?$AAl?$AAP?$AAi?$AAp?$AAe?$AA?3?$AA?3?$AA?$HO?$AAC?$AAC?$AAo?$AAn?$AAt?$AAr?$AAo?$AAl?$AAP?$AAi?$AAp?$AAe?$AA?6?$AA?$AA@ 1000b2d0     usbh_ehcdmdd_common_topaz_v1:cpipe.obj
 0001:0000a30c       ??_C@_1DM@KDAAIKEE@?$AA?$CL?$AAC?$AAC?$AAo?$AAn?$AAt?$AAr?$AAo?$AAl?$AAP?$AAi?$AAp?$AAe?$AA?3?$AA?3?$AA?$HO?$AAC?$AAC?$AAo?$AAn?$AAt?$AAr?$AAo?$AAl?$AAP?$AAi?$AAp?$AAe?$AA?6?$AA?$AA@ 1000b30c     usbh_ehcdmdd_common_topaz_v1:cpipe.obj
 0001:0000a348       ??_C@_1DC@GHHCAGFM@?$AA?9?$AAC?$AAC?$AAo?$AAn?$AAt?$AAr?$AAo?$AAl?$AAP?$AAi?$AAp?$AAe?$AA?3?$AA?3?$AAO?$AAp?$AAe?$AAn?$AAP?$AAi?$AAp?$AAe?$AA?6?$AA?$AA@ 1000b348     usbh_ehcdmdd_common_topaz_v1:cpipe.obj
 0001:0000a37c       ??_C@_1DC@MJDGFOPI@?$AA?$CL?$AAC?$AAC?$AAo?$AAn?$AAt?$AAr?$AAo?$AAl?$AAP?$AAi?$AAp?$AAe?$AA?3?$AA?3?$AAO?$AAp?$AAe?$AAn?$AAP?$AAi?$AAp?$AAe?$AA?6?$AA?$AA@ 1000b37c     usbh_ehcdmdd_common_topaz_v1:cpipe.obj
 0001:0000a3b0       ??_C@_1JO@NJHKCDBF@?$AA?9?$AAC?$AAC?$AAo?$AAn?$AAt?$AAr?$AAo?$AAl?$AAP?$AAi?$AAp?$AAe?$AA?3?$AA?3?$AA?3?$AA?3?$AAI?$AAs?$AAs?$AAu?$AAe?$AAT?$AAr?$AAa?$AAn?$AAs?$AAf?$AAe?$AAr?$AA?5?$AA?9@ 1000b3b0     usbh_ehcdmdd_common_topaz_v1:cpipe.obj
 0001:0000a450       ??_C@_1FI@KCIAIEAB@?$AA?$CL?$AAC?$AAC?$AAo?$AAn?$AAt?$AAr?$AAo?$AAl?$AAP?$AAi?$AAp?$AAe?$AA?3?$AA?3?$AAI?$AAs?$AAs?$AAu?$AAe?$AAT?$AAr?$AAa?$AAn?$AAs?$AAf?$AAe?$AAr?$AA?0?$AA?5?$AAa?$AAd@ 1000b450     usbh_ehcdmdd_common_topaz_v1:cpipe.obj
 0001:0000a4a8       ??_C@_1HM@OIBOFPNI@?$AA?9?$AAC?$AAC?$AAo?$AAn?$AAt?$AAr?$AAo?$AAl?$AAP?$AAi?$AAp?$AAe?$AA?3?$AA?3?$AAC?$AAh?$AAa?$AAn?$AAg?$AAe?$AAM?$AAa?$AAx?$AAP?$AAa?$AAc?$AAk?$AAe?$AAt?$AAS?$AAi@ 1000b4a8     usbh_ehcdmdd_common_topaz_v1:cpipe.obj
 0001:0000a528       ??_C@_1HM@LHJEGOH@?$AA?$CL?$AAC?$AAC?$AAo?$AAn?$AAt?$AAr?$AAo?$AAl?$AAP?$AAi?$AAp?$AAe?$AA?3?$AA?3?$AAC?$AAh?$AAa?$AAn?$AAg?$AAe?$AAM?$AAa?$AAx?$AAP?$AAa?$AAc?$AAk?$AAe?$AAt?$AAS?$AAi@ 1000b528     usbh_ehcdmdd_common_topaz_v1:cpipe.obj
 0001:0000a5a8       ??_C@_1HM@GLJMKJHD@?$AA?9?$AAC?$AAC?$AAo?$AAn?$AAt?$AAr?$AAo?$AAl?$AAP?$AAi?$AAp?$AAe?$AA?3?$AA?3?$AAA?$AAr?$AAe?$AAT?$AAr?$AAa?$AAn?$AAs?$AAf?$AAe?$AAr?$AAP?$AAa?$AAr?$AAa?$AAm?$AAe@ 1000b5a8     usbh_ehcdmdd_common_topaz_v1:cpipe.obj
 0001:0000a628       ??_C@_1FG@LOHNLBGH@?$AA?$CL?$AAC?$AAC?$AAo?$AAn?$AAt?$AAr?$AAo?$AAl?$AAP?$AAi?$AAp?$AAe?$AA?3?$AA?3?$AAA?$AAr?$AAe?$AAT?$AAr?$AAa?$AAn?$AAs?$AAf?$AAe?$AAr?$AAP?$AAa?$AAr?$AAa?$AAm?$AAe@ 1000b628     usbh_ehcdmdd_common_topaz_v1:cpipe.obj
 0001:0000a680       ??_C@_1EC@JEMMMPIH@?$AA?9?$AAC?$AAI?$AAn?$AAt?$AAe?$AAr?$AAr?$AAu?$AAp?$AAt?$AAP?$AAi?$AAp?$AAe?$AA?3?$AA?3?$AAC?$AAI?$AAn?$AAt?$AAe?$AAr?$AAr?$AAu?$AAp?$AAt?$AAP?$AAi?$AAp?$AAe?$AA?6@ 1000b680     usbh_ehcdmdd_common_topaz_v1:cpipe.obj
 0001:0000a6c8       ??_C@_1EC@PLMICHIE@?$AA?$CL?$AAC?$AAI?$AAn?$AAt?$AAe?$AAr?$AAr?$AAu?$AAp?$AAt?$AAP?$AAi?$AAp?$AAe?$AA?3?$AA?3?$AAC?$AAI?$AAn?$AAt?$AAe?$AAr?$AAr?$AAu?$AAp?$AAt?$AAP?$AAi?$AAp?$AAe?$AA?6@ 1000b6c8     usbh_ehcdmdd_common_topaz_v1:cpipe.obj
 0001:0000a710       ??_7CInterruptPipe@@6B@    1000b710     usbh_ehcdmdd_common_topaz_v1:cpipe.obj
 0001:0000a750       ??_C@_1BE@PBKDACKD@?$AAI?$AAn?$AAt?$AAe?$AAr?$AAr?$AAu?$AAp?$AAt?$AA?$AA@ 1000b750     usbh_ehcdmdd_common_topaz_v1:cpipe.obj
 0001:0000a768       ??_C@_1EE@DEJPNDGC@?$AA?9?$AAC?$AAI?$AAn?$AAt?$AAe?$AAr?$AAr?$AAu?$AAp?$AAt?$AAP?$AAi?$AAp?$AAe?$AA?3?$AA?3?$AA?$HO?$AAC?$AAI?$AAn?$AAt?$AAe?$AAr?$AAr?$AAu?$AAp?$AAt?$AAP?$AAi?$AAp?$AAe@ 1000b768     usbh_ehcdmdd_common_topaz_v1:cpipe.obj
 0001:0000a7b0       ??_C@_1EE@LBGDIFOP@?$AA?$CL?$AAC?$AAI?$AAn?$AAt?$AAe?$AAr?$AAr?$AAu?$AAp?$AAt?$AAP?$AAi?$AAp?$AAe?$AA?3?$AA?3?$AA?$HO?$AAC?$AAI?$AAn?$AAt?$AAe?$AAr?$AAr?$AAu?$AAp?$AAt?$AAP?$AAi?$AAp?$AAe@ 1000b7b0     usbh_ehcdmdd_common_topaz_v1:cpipe.obj
 0001:0000a7f8       ??_C@_1HI@FOEBHECD@?$AA?9?$AAC?$AAI?$AAn?$AAt?$AAe?$AAr?$AAr?$AAu?$AAp?$AAt?$AAP?$AAi?$AAp?$AAe?$AA?3?$AA?3?$AAO?$AAp?$AAe?$AAn?$AAP?$AAi?$AAp?$AAe?$AA?0?$AA?5?$AAr?$AAe?$AAt?$AAu?$AAr@ 1000b7f8     usbh_ehcdmdd_common_topaz_v1:cpipe.obj
 0001:0000a870       ??_C@_1DG@GPNELIPB@?$AA?$CL?$AAC?$AAI?$AAn?$AAt?$AAe?$AAr?$AAr?$AAu?$AAp?$AAt?$AAP?$AAi?$AAp?$AAe?$AA?3?$AA?3?$AAO?$AAp?$AAe?$AAn?$AAP?$AAi?$AAp?$AAe?$AA?6?$AA?$AA@ 1000b870     usbh_ehcdmdd_common_topaz_v1:cpipe.obj
 0001:0000a8a8       ??_C@_1IA@LIOLNNHC@?$AA?9?$AAC?$AAI?$AAn?$AAt?$AAe?$AAr?$AAr?$AAu?$AAp?$AAt?$AAP?$AAi?$AAp?$AAe?$AA?3?$AA?3?$AAA?$AAr?$AAe?$AAT?$AAr?$AAa?$AAn?$AAs?$AAf?$AAe?$AAr?$AAP?$AAa?$AAr?$AAa@ 1000b8a8     usbh_ehcdmdd_common_topaz_v1:cpipe.obj
 0001:0000a928       ??_C@_1FK@DKADEEOK@?$AA?$CL?$AAC?$AAI?$AAn?$AAt?$AAe?$AAr?$AAr?$AAu?$AAp?$AAt?$AAP?$AAi?$AAp?$AAe?$AA?3?$AA?3?$AAA?$AAr?$AAe?$AAT?$AAr?$AAa?$AAn?$AAs?$AAf?$AAe?$AAr?$AAP?$AAa?$AAr?$AAa@ 1000b928     usbh_ehcdmdd_common_topaz_v1:cpipe.obj
 0001:0000a988       ??_C@_1EK@KOEDIKFD@?$AA?9?$AAC?$AAI?$AAs?$AAo?$AAc?$AAh?$AAr?$AAo?$AAn?$AAo?$AAu?$AAs?$AAP?$AAi?$AAp?$AAe?$AA?3?$AA?3?$AAC?$AAI?$AAs?$AAo?$AAc?$AAh?$AAr?$AAo?$AAn?$AAo?$AAu?$AAs?$AAP@ 1000b988     usbh_ehcdmdd_common_topaz_v1:cpipe.obj
 0001:0000a9d8       ??_C@_1HO@LMFMLCBE@?$AAC?$AAI?$AAs?$AAo?$AAc?$AAh?$AAr?$AAo?$AAn?$AAo?$AAu?$AAs?$AAP?$AAi?$AAp?$AAe?$AA?3?$AA?3?$AAC?$AAI?$AAs?$AAo?$AAc?$AAh?$AAr?$AAo?$AAn?$AAo?$AAu?$AAs?$AAP?$AAi@ 1000b9d8     usbh_ehcdmdd_common_topaz_v1:cpipe.obj
 0001:0000aa58       ??_C@_1EK@JAHAMHEK@?$AA?$CL?$AAC?$AAI?$AAs?$AAo?$AAc?$AAh?$AAr?$AAo?$AAn?$AAo?$AAu?$AAs?$AAP?$AAi?$AAp?$AAe?$AA?3?$AA?3?$AAC?$AAI?$AAs?$AAo?$AAc?$AAh?$AAr?$AAo?$AAn?$AAo?$AAu?$AAs?$AAP@ 1000ba58     usbh_ehcdmdd_common_topaz_v1:cpipe.obj
 0001:0000aaa4       ??_7CIsochronousPipe@@6B@  1000baa4     usbh_ehcdmdd_common_topaz_v1:cpipe.obj
 0001:0000aadc       ??_C@_1BI@FKFHNGHF@?$AAI?$AAs?$AAo?$AAc?$AAh?$AAr?$AAo?$AAn?$AAo?$AAu?$AAs?$AA?$AA@ 1000badc     usbh_ehcdmdd_common_topaz_v1:cpipe.obj
 0001:0000aaf8       ??_C@_1EM@BLDMLENC@?$AA?9?$AAC?$AAI?$AAs?$AAo?$AAc?$AAh?$AAr?$AAo?$AAn?$AAo?$AAu?$AAs?$AAP?$AAi?$AAp?$AAe?$AA?3?$AA?3?$AA?$HO?$AAC?$AAI?$AAs?$AAo?$AAc?$AAh?$AAr?$AAo?$AAn?$AAo?$AAu?$AAs@ 1000baf8     usbh_ehcdmdd_common_topaz_v1:cpipe.obj
 0001:0000ab48       ??_C@_1EM@IIFBBONE@?$AA?$CL?$AAC?$AAI?$AAs?$AAo?$AAc?$AAh?$AAr?$AAo?$AAn?$AAo?$AAu?$AAs?$AAP?$AAi?$AAp?$AAe?$AA?3?$AA?3?$AA?$HO?$AAC?$AAI?$AAs?$AAo?$AAc?$AAh?$AAr?$AAo?$AAn?$AAo?$AAu?$AAs@ 1000bb48     usbh_ehcdmdd_common_topaz_v1:cpipe.obj
 0001:0000ab98       ??_C@_1ME@MIHPHEKP@?$AAC?$AA?3?$AA?2?$AAW?$AAI?$AAN?$AAC?$AAE?$AAR?$AAO?$AAO?$AAT?$AAS?$AA?2?$AAT?$AAo?$AAp?$AAa?$AAz?$AA?2?$AAW?$AAI?$AAN?$AAC?$AAE?$AA6?$AA0?$AA0?$AA?2?$AAp?$AAl?$AAa@ 1000bb98     usbh_ehcdmdd_common_topaz_v1:cpipe.obj
 0001:0000ac60       ??_C@_1JI@ENJAEICO@?$AAC?$AAI?$AAs?$AAo?$AAc?$AAh?$AAr?$AAo?$AAn?$AAo?$AAu?$AAs?$AAP?$AAi?$AAp?$AAe?$AA?3?$AA?3?$AAA?$AAl?$AAl?$AAo?$AAc?$AAa?$AAt?$AAe?$AAC?$AAI?$AAT?$AAD?$AA?3?$AA?5@ 1000bc60     usbh_ehcdmdd_common_topaz_v1:cpipe.obj
 0001:0000acf8       ??_C@_1JM@KEKOKCFN@?$AAC?$AAI?$AAs?$AAo?$AAc?$AAh?$AAr?$AAo?$AAn?$AAo?$AAu?$AAs?$AAP?$AAi?$AAp?$AAe?$AA?3?$AA?3?$AAA?$AAl?$AAl?$AAo?$AAc?$AAa?$AAt?$AAe?$AAC?$AAS?$AAI?$AAT?$AAD?$AA?3@ 1000bcf8     usbh_ehcdmdd_common_topaz_v1:cpipe.obj
 0001:0000ad98       ??_C@_1HM@GAFPALLL@?$AA?9?$AAC?$AAI?$AAs?$AAo?$AAc?$AAh?$AAr?$AAo?$AAn?$AAo?$AAu?$AAs?$AAP?$AAi?$AAp?$AAe?$AA?3?$AA?3?$AAO?$AAp?$AAe?$AAn?$AAP?$AAi?$AAp?$AAe?$AA?0?$AA?5?$AAr?$AAe?$AAt@ 1000bd98     usbh_ehcdmdd_common_topaz_v1:cpipe.obj
 0001:0000ae14       ??_C@_1DK@OPNDEICN@?$AA?$CL?$AAC?$AAI?$AAs?$AAo?$AAc?$AAh?$AAr?$AAo?$AAn?$AAo?$AAu?$AAs?$AAP?$AAi?$AAp?$AAe?$AA?3?$AA?3?$AAO?$AAp?$AAe?$AAn?$AAP?$AAi?$AAp?$AAe?$AA?6?$AA?$AA@ 1000be14     usbh_ehcdmdd_common_topaz_v1:cpipe.obj
 0001:0000ae50       ??_C@_1DM@HPKHCFDD@?$AA?9?$AAC?$AAI?$AAs?$AAo?$AAc?$AAh?$AAr?$AAo?$AAn?$AAo?$AAu?$AAs?$AAP?$AAi?$AAp?$AAe?$AA?3?$AA?3?$AAC?$AAl?$AAo?$AAs?$AAe?$AAP?$AAi?$AAp?$AAe?$AA?6?$AA?$AA@ 1000be50     usbh_ehcdmdd_common_topaz_v1:cpipe.obj
 0001:0000ae8c       ??_C@_1DM@KMNNAINC@?$AA?$CL?$AAC?$AAI?$AAs?$AAo?$AAc?$AAh?$AAr?$AAo?$AAn?$AAo?$AAu?$AAs?$AAP?$AAi?$AAp?$AAe?$AA?3?$AA?3?$AAC?$AAl?$AAo?$AAs?$AAe?$AAP?$AAi?$AAp?$AAe?$AA?6?$AA?$AA@ 1000be8c     usbh_ehcdmdd_common_topaz_v1:cpipe.obj
 0001:0000aec8       ??_C@_1KM@KKLHDMPD@?$AAC?$AAI?$AAs?$AAo?$AAc?$AAh?$AAr?$AAo?$AAn?$AAo?$AAu?$AAs?$AAP?$AAi?$AAp?$AAe?$AA?3?$AA?3?$AAA?$AAb?$AAo?$AAr?$AAt?$AAT?$AAr?$AAa?$AAn?$AAs?$AAf?$AAe?$AAr?$AA?5@ 1000bec8     usbh_ehcdmdd_common_topaz_v1:cpipe.obj
 0001:0000af78       ??_C@_1EE@GNCAFEJO@?$AA?$CL?$AAC?$AAI?$AAs?$AAo?$AAc?$AAh?$AAr?$AAo?$AAn?$AAo?$AAu?$AAs?$AAP?$AAi?$AAp?$AAe?$AA?3?$AA?3?$AAA?$AAb?$AAo?$AAr?$AAt?$AAT?$AAr?$AAa?$AAn?$AAs?$AAf?$AAe?$AAr@ 1000bf78     usbh_ehcdmdd_common_topaz_v1:cpipe.obj
 0001:0000afc0       ??_C@_1LG@FKIKFAPC@?$AA?$CB?$AAC?$AAI?$AAs?$AAo?$AAc?$AAh?$AAr?$AAo?$AAn?$AAo?$AAu?$AAs?$AAP?$AAi?$AAp?$AAe?$AA?3?$AA?3?$AAI?$AAs?$AAs?$AAu?$AAe?$AAT?$AAr?$AAa?$AAn?$AAs?$AAf?$AAe?$AAr@ 1000bfc0     usbh_ehcdmdd_common_topaz_v1:cpipe.obj
 0001:0000b078       ??_C@_1EK@GADJNDHH@?$AA?$CL?$AAC?$AAI?$AAs?$AAo?$AAc?$AAh?$AAr?$AAo?$AAn?$AAo?$AAu?$AAs?$AAP?$AAi?$AAp?$AAe?$AA?3?$AA?3?$AAS?$AAc?$AAh?$AAe?$AAd?$AAu?$AAl?$AAe?$AAT?$AAr?$AAa?$AAn?$AAs@ 1000c078     usbh_ehcdmdd_common_topaz_v1:cpipe.obj
 0001:0000b0c8       ??_C@_1HK@FGMLGCL@?$AA?9?$AAC?$AAI?$AAs?$AAo?$AAc?$AAh?$AAr?$AAo?$AAn?$AAo?$AAu?$AAs?$AAP?$AAi?$AAp?$AAe?$AA?3?$AA?3?$AAC?$AAh?$AAe?$AAc?$AAk?$AAF?$AAo?$AAr?$AAD?$AAo?$AAn?$AAe?$AAT@ 1000c0c8     usbh_ehcdmdd_common_topaz_v1:cpipe.obj
 0001:0000b148       ??_C@_1FE@HLBAALFH@?$AA?$CL?$AAC?$AAI?$AAs?$AAo?$AAc?$AAh?$AAr?$AAo?$AAn?$AAo?$AAu?$AAs?$AAP?$AAi?$AAp?$AAe?$AA?3?$AA?3?$AAC?$AAh?$AAe?$AAc?$AAk?$AAF?$AAo?$AAr?$AAD?$AAo?$AAn?$AAe?$AAT@ 1000c148     usbh_ehcdmdd_common_topaz_v1:cpipe.obj
 0001:0000b1a0       ??_C@_1IE@HJGDLHPI@?$AA?9?$AAC?$AAI?$AAs?$AAo?$AAc?$AAh?$AAr?$AAo?$AAn?$AAo?$AAu?$AAs?$AAP?$AAi?$AAp?$AAe?$AA?3?$AA?3?$AAA?$AAr?$AAe?$AAT?$AAr?$AAa?$AAn?$AAs?$AAf?$AAe?$AAr?$AAP?$AAa@ 1000c1a0     usbh_ehcdmdd_common_topaz_v1:cpipe.obj
 0001:0000b228       ??_C@_1FO@GGCPAHGF@?$AA?$CL?$AAC?$AAI?$AAs?$AAo?$AAc?$AAh?$AAr?$AAo?$AAn?$AAo?$AAu?$AAs?$AAP?$AAi?$AAp?$AAe?$AA?3?$AA?3?$AAA?$AAr?$AAe?$AAT?$AAr?$AAa?$AAn?$AAs?$AAf?$AAe?$AAr?$AAP?$AAa@ 1000c228     usbh_ehcdmdd_common_topaz_v1:cpipe.obj
 0001:0000b288       ??_C@_1MA@HJOIBODM@?$AAC?$AA?3?$AA?2?$AAW?$AAI?$AAN?$AAC?$AAE?$AAR?$AAO?$AAO?$AAT?$AAS?$AA?2?$AAT?$AAo?$AAp?$AAa?$AAz?$AA?2?$AAW?$AAI?$AAN?$AAC?$AAE?$AA6?$AA0?$AA0?$AA?2?$AAP?$AAL?$AAA@ 1000c288     usbh_ehcdmdd_common_topaz_v1:usb2lib.obj
 0001:0000b348       ??_C@_1DK@LALOJPCH@?$AAe?$AAn?$AAd?$AAp?$AAo?$AAi?$AAn?$AAt?$AA?5?$AAa?$AAl?$AAr?$AAe?$AAa?$AAd?$AAy?$AA?5?$AAa?$AAl?$AAl?$AAo?$AAc?$AAa?$AAt?$AAe?$AAd?$AA?$AN?$AA?6?$AA?$AA@ 1000c348     usbh_ehcdmdd_common_topaz_v1:usb2lib.obj
 0001:0000b390       ??_C@_1LI@KICOKNMD@?$AAC?$AA?3?$AA?2?$AAW?$AAI?$AAN?$AAC?$AAE?$AAR?$AAO?$AAO?$AAT?$AAS?$AA?2?$AAT?$AAo?$AAp?$AAa?$AAz?$AA?2?$AAW?$AAI?$AAN?$AAC?$AAE?$AA6?$AA0?$AA0?$AA?2?$AAP?$AAL?$AAA@ 1000c390     usbh_ehcdmdd_common_topaz_v1:chw.obj
 0001:0000b448       ??_7CDummyPipe@@6B@        1000c448     usbh_ehcdmdd_common_topaz_v1:chw.obj
 0001:0000b480       ??_C@_1BA@NBFKLKJD@?$AA?4?$AA?2?$AAc?$AAh?$AAw?$AA?4?$AAh?$AA?$AA@ 1000c480     usbh_ehcdmdd_common_topaz_v1:chw.obj
 0001:0000b490       ??_C@_1M@EOJMLNDL@?$AAD?$AAu?$AAm?$AAm?$AAy?$AA?$AA@ 1000c490     usbh_ehcdmdd_common_topaz_v1:chw.obj
 0001:0000b4a0       ??_C@_1ME@EHKKMEBO@?$AAC?$AA?3?$AA?2?$AAW?$AAI?$AAN?$AAC?$AAE?$AAR?$AAO?$AAO?$AAT?$AAS?$AA?2?$AAT?$AAo?$AAp?$AAa?$AAz?$AA?2?$AAW?$AAI?$AAN?$AAC?$AAE?$AA6?$AA0?$AA0?$AA?2?$AAp?$AAl?$AAa@ 1000c4a0     usbh_ehcdmdd_common_topaz_v1:chw.obj
 0001:0000b568       ??_C@_1IE@FLPBCPAJ@?$AA?9?$AAC?$AAP?$AAi?$AAp?$AAe?$AA?3?$AA?3?$AAI?$AAn?$AAi?$AAt?$AAi?$AAa?$AAl?$AAi?$AAz?$AAe?$AA?4?$AA?5?$AAE?$AAr?$AAr?$AAo?$AAr?$AA?5?$AAc?$AAr?$AAe?$AAa?$AAt?$AAi@ 1000c568     usbh_ehcdmdd_common_topaz_v1:chw.obj
 0001:0000b5f0       ??_C@_1IC@BKOJKGJB@?$AA?9?$AAC?$AAP?$AAi?$AAp?$AAe?$AA?3?$AA?3?$AAI?$AAn?$AAi?$AAt?$AAi?$AAa?$AAl?$AAi?$AAz?$AAe?$AA?4?$AA?5?$AAE?$AAr?$AAr?$AAo?$AAr?$AA?5?$AAc?$AAr?$AAe?$AAa?$AAt?$AAi@ 1000c5f0     usbh_ehcdmdd_common_topaz_v1:chw.obj
 0001:0000b678       ??_C@_1EK@LNDAMOBI@?$AA?9?$AAC?$AAP?$AAi?$AAp?$AAe?$AA?3?$AA?3?$AAC?$AAh?$AAe?$AAc?$AAk?$AAF?$AAo?$AAr?$AAD?$AAo?$AAn?$AAe?$AAT?$AAr?$AAa?$AAn?$AAs?$AAf?$AAe?$AAr?$AAs?$AAT?$AAh?$AAr@ 1000c678     usbh_ehcdmdd_common_topaz_v1:chw.obj
 0001:0000b6c8       ??_C@_1JM@HGCADDMJ@?$AAC?$AAP?$AAi?$AAp?$AAe?$AA?3?$AA?3?$AAC?$AAh?$AAe?$AAc?$AAk?$AAF?$AAo?$AAr?$AAD?$AAo?$AAn?$AAe?$AAT?$AAr?$AAa?$AAn?$AAs?$AAf?$AAe?$AAr?$AAs?$AAT?$AAh?$AAr?$AAe@ 1000c6c8     usbh_ehcdmdd_common_topaz_v1:chw.obj
 0001:0000b768       ??_C@_1HG@FJHGEDDA@?$AAC?$AAP?$AAi?$AAp?$AAe?$AA?3?$AA?3?$AAC?$AAh?$AAe?$AAc?$AAk?$AAF?$AAo?$AAr?$AAD?$AAo?$AAn?$AAe?$AAT?$AAr?$AAa?$AAn?$AAs?$AAf?$AAe?$AAr?$AAs?$AAT?$AAh?$AAr?$AAe@ 1000c768     usbh_ehcdmdd_common_topaz_v1:chw.obj
 0001:0000b7e0       ??_C@_1EK@IDADIDAB@?$AA?$CL?$AAC?$AAP?$AAi?$AAp?$AAe?$AA?3?$AA?3?$AAC?$AAh?$AAe?$AAc?$AAk?$AAF?$AAo?$AAr?$AAD?$AAo?$AAn?$AAe?$AAT?$AAr?$AAa?$AAn?$AAs?$AAf?$AAe?$AAr?$AAs?$AAT?$AAh?$AAr@ 1000c7e0     usbh_ehcdmdd_common_topaz_v1:chw.obj
 0001:0000b82c       ??_C@_1CG@INGKPFMN@?$AAO?$AAT?$AAG?$AA?5?$AAS?$AAu?$AAp?$AAp?$AAo?$AAr?$AAt?$AA?5?$AA?$DN?$AA?5?$AA?$CF?$AAd?$AA?$AN?$AA?6?$AA?$AA@ 1000c82c     usbh_ehcdmdd_common_topaz_v1:chw.obj
 0001:0000b858       ??_C@_1EA@DPCFGDAC@?$AA?$CL?$AAC?$AAH?$AAW?$AA?3?$AA?3?$AAC?$AAH?$AAW?$AA?5?$AAb?$AAa?$AAs?$AAe?$AA?$DN?$AA0?$AAx?$AA?$CF?$AAx?$AA?0?$AA?5?$AAi?$AAn?$AAt?$AAr?$AA?$DN?$AA0?$AAx?$AA?$CF?$AAx?$AA?6?$AA?$AA@ 1000c858     usbh_ehcdmdd_common_topaz_v1:chw.obj
 0001:0000b898       ??_7CHW@@6B@               1000c898     usbh_ehcdmdd_common_topaz_v1:chw.obj
 0001:0000b910       ??_C@_1HG@MBKCEMPB@?$AA?$CB?$AA?$CB?$AA?$CB?$AAW?$AAa?$AAr?$AAn?$AAi?$AAn?$AAg?$AA?$CB?$AA?$CB?$AA?$CB?$AA?5?$AAS?$AAe?$AAt?$AAt?$AAi?$AAn?$AAg?$AA?5?$AAr?$AAe?$AAs?$AAu?$AAm?$AAe?$AA?1?$AAs?$AAu?$AAs@ 1000c910     usbh_ehcdmdd_common_topaz_v1:chw.obj
 0001:0000b988       ??_C@_1GO@MAFPNDIJ@?$AA?$CB?$AA?$CB?$AA?$CB?$AAW?$AAa?$AAr?$AAn?$AAi?$AAn?$AAg?$AA?$CB?$AA?$CB?$AA?$CB?$AA?5?$AAs?$AAt?$AAa?$AAt?$AAu?$AAs?$AA?5?$AAs?$AAh?$AAo?$AAw?$AA?5?$AAe?$AAr?$AAr?$AAo?$AAr?$AA?1@ 1000c988     usbh_ehcdmdd_common_topaz_v1:chw.obj
 0001:0000b9f8       ??_C@_1EO@HMIBCHLC@?$AAC?$AAH?$AAW?$AA?3?$AA?3?$AAI?$AAn?$AAi?$AAt?$AAi?$AAa?$AAl?$AAi?$AAz?$AAe?$AA?5?$AA?9?$AA?5?$AAE?$AAn?$AAa?$AAb?$AAl?$AAe?$AA?5?$AAA?$AAs?$AAy?$AAn?$AAc?$AA?5?$AAS@ 1000c9f8     usbh_ehcdmdd_common_topaz_v1:chw.obj
 0001:0000ba48       ??_C@_1FI@DCMECGHC@?$AAC?$AAH?$AAW?$AA?3?$AA?3?$AAI?$AAn?$AAi?$AAt?$AAi?$AAa?$AAl?$AAi?$AAz?$AAe?$AA?5?$AA?9?$AA?5?$AAs?$AAe?$AAt?$AAt?$AAi?$AAn?$AAg?$AA?5?$AAF?$AAL?$AAB?$AAA?$AAS?$AAE@ 1000ca48     usbh_ehcdmdd_common_topaz_v1:chw.obj
 0001:0000baa0       ??_C@_1EK@HPKPHAGK@?$AAC?$AAH?$AAW?$AA?3?$AA?3?$AAI?$AAn?$AAi?$AAt?$AAi?$AAa?$AAl?$AAi?$AAz?$AAe?$AA?5?$AA?9?$AA?5?$AAs?$AAe?$AAt?$AAt?$AAi?$AAn?$AAg?$AA?5?$AAF?$AAR?$AAN?$AAU?$AAM?$AA?5@ 1000caa0     usbh_ehcdmdd_common_topaz_v1:chw.obj
 0001:0000baf0       ??_C@_1HA@MEOMJIGE@?$AAC?$AAH?$AAW?$AA?3?$AA?3?$AAI?$AAn?$AAi?$AAt?$AAi?$AAa?$AAl?$AAi?$AAz?$AAe?$AA?5?$AA?9?$AA?5?$AAs?$AAe?$AAt?$AAt?$AAi?$AAn?$AAg?$AA?5?$AAU?$AAS?$AAB?$AAI?$AAN?$AAT@ 1000caf0     usbh_ehcdmdd_common_topaz_v1:chw.obj
 0001:0000bb60       ??_C@_1FO@CCFPNPAL@?$AAC?$AAH?$AAW?$AA?3?$AA?3?$AAI?$AAn?$AAi?$AAt?$AAi?$AAa?$AAl?$AAi?$AAz?$AAe?$AA?5?$AA?9?$AA?5?$AAe?$AAn?$AAd?$AA?5?$AAs?$AAi?$AAg?$AAn?$AAa?$AAl?$AAl?$AAi?$AAn?$AAg@ 1000cb60     usbh_ehcdmdd_common_topaz_v1:chw.obj
 0001:0000bbc0       ??_C@_1DI@MBIOGDIA@?$AA?9?$AAC?$AAH?$AAW?$AA?3?$AA?3?$AAI?$AAn?$AAi?$AAt?$AAi?$AAa?$AAl?$AAi?$AAz?$AAe?$AA?0?$AA?5?$AAs?$AAu?$AAc?$AAc?$AAe?$AAs?$AAs?$AA?$CB?$AA?6?$AA?$AA@ 1000cbc0     usbh_ehcdmdd_common_topaz_v1:chw.obj
 0001:0000bbf8       ??_C@_1FG@CKLMEGIM@?$AAC?$AAH?$AAW?$AA?3?$AA?3?$AAI?$AAn?$AAi?$AAt?$AAi?$AAa?$AAl?$AAi?$AAz?$AAe?$AA?5?$AA?9?$AA?5?$AAI?$AAn?$AAi?$AAt?$AAi?$AAa?$AAl?$AA?5?$AAA?$AAl?$AAl?$AA?5?$AAp?$AAo@ 1000cbf8     usbh_ehcdmdd_common_topaz_v1:chw.obj
 0001:0000bc50       ??_C@_1EM@OLPEIAAA@?$AA?9?$AAC?$AAH?$AAW?$AA?3?$AA?3?$AAI?$AAn?$AAi?$AAt?$AAi?$AAa?$AAl?$AAi?$AAz?$AAe?$AA?4?$AA?5?$AAE?$AAr?$AAr?$AAo?$AAr?$AA?5?$AAc?$AAr?$AAe?$AAa?$AAt?$AAi?$AAn?$AAg@ 1000cc50     usbh_ehcdmdd_common_topaz_v1:chw.obj
 0001:0000bca0       ??_C@_1GC@NNLMHGPK@?$AA?9?$AAC?$AAH?$AAW?$AA?3?$AA?3?$AAI?$AAn?$AAi?$AAt?$AAi?$AAa?$AAl?$AAi?$AAz?$AAe?$AA?4?$AA?5?$AAE?$AAr?$AAr?$AAo?$AAr?$AA?5?$AAo?$AAn?$AA?5?$AAI?$AAn?$AAt?$AAe?$AAr@ 1000cca0     usbh_ehcdmdd_common_topaz_v1:chw.obj
 0001:0000bd08       ??_C@_1JA@MHLILIKF@?$AA?9?$AAC?$AAH?$AAW?$AA?3?$AA?3?$AAI?$AAn?$AAi?$AAt?$AAi?$AAa?$AAl?$AAi?$AAz?$AAe?$AA?4?$AA?5?$AAE?$AAr?$AAr?$AAo?$AAr?$AA?5?$AAc?$AAr?$AAe?$AAa?$AAt?$AAi?$AAn?$AAg@ 1000cd08     usbh_ehcdmdd_common_topaz_v1:chw.obj
 0001:0000bd98       ??_C@_1FG@LGOCOJPG@?$AAC?$AAH?$AAW?$AA?3?$AA?3?$AAI?$AAn?$AAi?$AAt?$AAi?$AAa?$AAl?$AAi?$AAz?$AAe?$AA?5?$AA?9?$AA?5?$AAs?$AAi?$AAg?$AAn?$AAa?$AAl?$AAl?$AAi?$AAn?$AAg?$AA?5?$AAg?$AAl?$AAo@ 1000cd98     usbh_ehcdmdd_common_topaz_v1:chw.obj
 0001:0000bdf0       ??_C@_1JC@OFBFENBJ@?$AA?9?$AAC?$AAH?$AAW?$AA?3?$AA?3?$AAI?$AAn?$AAi?$AAt?$AAi?$AAa?$AAl?$AAi?$AAz?$AAe?$AA?5?$AA?9?$AA?5?$AAz?$AAe?$AAr?$AAo?$AA?5?$AAR?$AAe?$AAg?$AAi?$AAs?$AAt?$AAe?$AAr@ 1000cdf0     usbh_ehcdmdd_common_topaz_v1:chw.obj
 0001:0000be84       ??_C@_1CE@HIKDPBAB@?$AA?$CL?$AAC?$AAH?$AAW?$AA?3?$AA?3?$AAI?$AAn?$AAi?$AAt?$AAi?$AAa?$AAl?$AAi?$AAz?$AAe?$AA?6?$AA?$AA@ 1000ce84     usbh_ehcdmdd_common_topaz_v1:chw.obj
 0001:0000bea8       ??_C@_1DK@FFAMHNIM@?$AA?9?$AAC?$AAH?$AAW?$AA?3?$AA?3?$AAE?$AAn?$AAt?$AAe?$AAr?$AAO?$AAp?$AAe?$AAr?$AAa?$AAt?$AAi?$AAo?$AAn?$AAa?$AAl?$AAS?$AAt?$AAa?$AAt?$AAe?$AA?6?$AA?$AA@ 1000cea8     usbh_ehcdmdd_common_topaz_v1:chw.obj
 0001:0000bee8       ??_C@_1GK@MLODPEHP@?$AAC?$AAH?$AAW?$AA?3?$AA?3?$AAE?$AAn?$AAt?$AAe?$AAr?$AAO?$AAp?$AAe?$AAr?$AAa?$AAt?$AAi?$AAo?$AAn?$AAa?$AAl?$AAS?$AAt?$AAa?$AAt?$AAe?$AA?5?$AA?9?$AA?5?$AAs?$AAe?$AAt@ 1000cee8     usbh_ehcdmdd_common_topaz_v1:chw.obj
 0001:0000bf58       ??_C@_1GE@MLJIHIHN@?$AAC?$AAH?$AAW?$AA?3?$AA?3?$AAE?$AAn?$AAt?$AAe?$AAr?$AAO?$AAp?$AAe?$AAr?$AAa?$AAt?$AAi?$AAo?$AAn?$AAa?$AAl?$AAS?$AAt?$AAa?$AAt?$AAe?$AA?5?$AA?9?$AA?5?$AAc?$AAl?$AAe@ 1000cf58     usbh_ehcdmdd_common_topaz_v1:chw.obj
 0001:0000bfbc       ??_C@_1BM@CBMLCADC@?$AAI?$AAn?$AAt?$AAT?$AAh?$AAr?$AAe?$AAs?$AAh?$AAC?$AAt?$AAr?$AAl?$AA?$AA@ 1000cfbc     usbh_ehcdmdd_common_topaz_v1:chw.obj
 0001:0000bfd8       ??_C@_1DK@DAOPFKKH@?$AA?$CL?$AAC?$AAH?$AAW?$AA?3?$AA?3?$AAE?$AAn?$AAt?$AAe?$AAr?$AAO?$AAp?$AAe?$AAr?$AAa?$AAt?$AAi?$AAo?$AAn?$AAa?$AAl?$AAS?$AAt?$AAa?$AAt?$AAe?$AA?6?$AA?$AA@ 1000cfd8     usbh_ehcdmdd_common_topaz_v1:chw.obj
 0001:0000c018       ??_C@_1EA@GDEIKMNI@?$AAS?$AAt?$AAa?$AAr?$AAt?$AAH?$AAo?$AAs?$AAt?$AAC?$AAo?$AAn?$AAt?$AAr?$AAo?$AAl?$AAl?$AAe?$AAr?$AA?5?$AAc?$AAo?$AAm?$AAp?$AAl?$AAe?$AAt?$AAe?$AAd?$AA?$AN?$AA?6?$AA?$AA@ 1000d018     usbh_ehcdmdd_common_topaz_v1:chw.obj
 0001:0000c058       ??_C@_1HA@KLKPLPGO@?$AAF?$AAo?$AAr?$AAc?$AAe?$AA?5?$AAW?$AAa?$AAk?$AAe?$AAU?$AAp?$AA?5?$AAo?$AAn?$AA?5?$AAH?$AAo?$AAs?$AAt?$AA?5?$AAS?$AAu?$AAs?$AAp?$AAe?$AAn?$AAd?$AA?$CI?$AA?$CF?$AAd?$AA?$CJ@ 1000d058     usbh_ehcdmdd_common_topaz_v1:chw.obj
 0001:0000c0c8       ??_C@_1GK@GGOFBDKF@?$AAU?$AAS?$AAB?$AA?5?$AAc?$AAa?$AAn?$AAn?$AAo?$AAt?$AA?5?$AAr?$AAe?$AAi?$AAn?$AAi?$AAt?$AA?5?$AAt?$AAh?$AAe?$AA?5?$AAH?$AAC?$AAD?$AA?5?$AAa?$AAt?$AA?5?$AAC?$AAE?$AA?5@ 1000d0c8     usbh_ehcdmdd_common_topaz_v1:chw.obj
 0001:0000c138       ??_C@_1EE@FFCLNAAM@?$AA?9?$AAC?$AAH?$AAW?$AA?3?$AA?3?$AAL?$AAe?$AAa?$AAv?$AAi?$AAn?$AAg?$AA?5?$AAU?$AAS?$AAB?$AAI?$AAn?$AAt?$AAe?$AAr?$AAr?$AAu?$AAp?$AAt?$AAT?$AAh?$AAr?$AAe?$AAa?$AAd@ 1000d138     usbh_ehcdmdd_common_topaz_v1:chw.obj
 0001:0000c180       ??_C@_1EG@NAIMFBLA@?$AAS?$AAw?$AAi?$AAt?$AAc?$AAh?$AA?5?$AAb?$AAa?$AAc?$AAk?$AA?5?$AAt?$AAo?$AA?5?$AAI?$AAD?$AAL?$AAE?$AA?5?$AAt?$AAi?$AAm?$AAe?$AAo?$AAu?$AAt?$AA?5?$AAm?$AAo?$AAd?$AAe@ 1000d180     usbh_ehcdmdd_common_topaz_v1:chw.obj
 0001:0000c1c8       ??_C@_1FI@CODCNCKO@?$AAE?$AAx?$AAi?$AAt?$AA?5?$AAt?$AAh?$AAe?$AA?5?$AAh?$AAo?$AAs?$AAt?$AA?5?$AAd?$AAr?$AAi?$AAv?$AAe?$AAr?$AA?5?$AAg?$AAo?$AAi?$AAn?$AAg?$AA?5?$AAb?$AAa?$AAc?$AAk?$AA?5@ 1000d1c8     usbh_ehcdmdd_common_topaz_v1:chw.obj
 0001:0000c220       ??_C@_1CE@DJAJDMLE@?$AAW?$AAa?$AAi?$AAt?$AA?5?$AAf?$AAo?$AAr?$AA?5?$AAD?$AAe?$AAt?$AAa?$AAc?$AAh?$AA?$AN?$AA?6?$AA?$AA@ 1000d220     usbh_ehcdmdd_common_topaz_v1:chw.obj
 0001:0000c244       ??_C@_1DE@NCMBIKIN@?$AAH?$AAC?$AAD?$AA?5?$AAR?$AAe?$AAs?$AAu?$AAm?$AAe?$AA?5?$AAf?$AAr?$AAo?$AAm?$AA?5?$AAw?$AAo?$AAr?$AAk?$AAi?$AAn?$AAg?$AA?$AN?$AA?6?$AA?$AA@ 1000d244     usbh_ehcdmdd_common_topaz_v1:chw.obj
 0001:0000c278       ??_C@_1LC@EPNFIBFE@?$AAH?$AAC?$AAD?$AA?5?$AAI?$AAS?$AAT?$AA?3?$AA?5?$AAc?$AAa?$AAn?$AAn?$AAo?$AAt?$AA?5?$AAs?$AAp?$AAi?$AAn?$AA?5?$AAa?$AA?5?$AAn?$AAe?$AAw?$AA?5?$AAt?$AAh?$AAr?$AAe?$AAa@ 1000d278     usbh_ehcdmdd_common_topaz_v1:chw.obj
 0001:0000c330       ??_C@_1EA@GKNBLIK@?$AAP?$AAo?$AAr?$AAt?$AA?5?$AA?$CF?$AAd?$AA?5?$AAn?$AAe?$AAe?$AAd?$AA?5?$AAt?$AAo?$AA?5?$AAw?$AAa?$AAk?$AAe?$AAu?$AAp?$AA?5?$AA?$CI?$AA0?$AAx?$AA?$CF?$AAx?$AA?$CJ?$AA?$AN?$AA?6?$AA?$AA@ 1000d330     usbh_ehcdmdd_common_topaz_v1:chw.obj
 0001:0000c370       ??_C@_1CG@GGAABBIA@?$AAP?$AAo?$AAr?$AAt?$AAS?$AAC?$AA?$FL?$AA0?$AA?$FN?$AA?5?$AA?$DN?$AA?5?$AA0?$AAx?$AA?$CF?$AAx?$AA?$AN?$AA?6?$AA?$AA@ 1000d370     usbh_ehcdmdd_common_topaz_v1:chw.obj
 0001:0000c398       ??_C@_1FM@PKHPHILM@?$AAH?$AAU?$AAB?$AA?5?$AAS?$AAt?$AAa?$AAt?$AAu?$AAs?$AA?5?$AAC?$AAh?$AAa?$AAn?$AAg?$AAe?$AA?5?$AA?$CI?$AAB?$AA?$CJ?$AA?5?$AAw?$AAi?$AAt?$AAh?$AA?5?$AAF?$AAo?$AAr?$AAc?$AAe@ 1000d398     usbh_ehcdmdd_common_topaz_v1:chw.obj
 0001:0000c3f8       ??_C@_1FA@BDNPPCPE@?$AAH?$AAS?$AAE?$AAr?$AAr?$AAo?$AAr?$AA?5?$AAb?$AAu?$AAt?$AA?5?$AAl?$AAe?$AAt?$AA?5?$AAc?$AAo?$AAn?$AAt?$AAi?$AAn?$AAu?$AAe?$AA?5?$AAU?$AAS?$AAB?$AAS?$AAT?$AAS?$AA?$CI@ 1000d3f8     usbh_ehcdmdd_common_topaz_v1:chw.obj
 0001:0000c448       ??_C@_1HO@JAOFLGIG@?$AA?$CB?$AA?$CB?$AA?$CB?$AAi?$AAn?$AAt?$AAe?$AAr?$AAr?$AAu?$AAp?$AAt?$AA?$CB?$AA?$CB?$AA?$CB?$AA?$CB?$AA?5?$AAo?$AAn?$AA?5?$AAf?$AAr?$AAa?$AAm?$AAe?$AA?5?$AAi?$AAn?$AAd?$AAe?$AAx?$AA?5@ 1000d448     usbh_ehcdmdd_common_topaz_v1:chw.obj
 0001:0000c4c8       ??_C@_1DO@PGOJPICB@?$AAm?$AA_?$AAf?$AAU?$AAs?$AAb?$AAI?$AAn?$AAt?$AAe?$AAr?$AAr?$AAu?$AAp?$AAt?$AAT?$AAh?$AAr?$AAe?$AAa?$AAd?$AAC?$AAl?$AAo?$AAs?$AAi?$AAn?$AAg?$AA?$AN?$AA?6?$AA?$AA@ 1000d4c8     usbh_ehcdmdd_common_topaz_v1:chw.obj
 0001:0000c508       ??_C@_1DA@HJBBKMCK@?$AAH?$AAU?$AAB?$AA?5?$AAS?$AAT?$AAA?$AAT?$AAU?$AAS?$AA?5?$AAC?$AAH?$AAA?$AAN?$AAG?$AAE?$AA?5?$AA?$CI?$AAC?$AA?$CJ?$AA?$AN?$AA?6?$AA?$AA@ 1000d508     usbh_ehcdmdd_common_topaz_v1:chw.obj
 0001:0000c538       ??_C@_1DE@EIIFONGG@?$AAD?$AAi?$AAs?$AAc?$AAo?$AAn?$AAn?$AAe?$AAc?$AAt?$AA?5?$AAw?$AAi?$AAt?$AAh?$AA?5?$AAn?$AAo?$AAt?$AAh?$AAi?$AAn?$AAg?$AA?$AN?$AA?6?$AA?$AA@ 1000d538     usbh_ehcdmdd_common_topaz_v1:chw.obj
 0001:0000c56c       ??_C@_1BK@LCKDFJGC@?$AAh?$AA?5?$AAo?$AAt?$AAg?$AAs?$AAc?$AA?5?$AA?$CF?$AAx?$AA?$AN?$AA?6?$AA?$AA@ 1000d56c     usbh_ehcdmdd_common_topaz_v1:chw.obj
 0001:0000c588       ??_C@_1FG@EKHFLMHA@?$AAm?$AAi?$AAn?$AAi?$AA?9?$AAA?$AA?5?$AAu?$AAn?$AAp?$AAl?$AAu?$AAg?$AAg?$AAe?$AAd?$AA?4?$AA?4?$AA?4?$AA?5?$AAg?$AAo?$AAi?$AAn?$AAg?$AA?5?$AAb?$AAa?$AAc?$AAk?$AA?5?$AAi@ 1000d588     usbh_ehcdmdd_common_topaz_v1:chw.obj
 0001:0000c5e0       ??_C@_1CC@BBFDADPB@?$AAH?$AAo?$AAs?$AAt?$AA?5?$AA?9?$AA?5?$AAS?$AAU?$AAS?$AAP?$AAE?$AAN?$AAD?$AA?$AN?$AA?6?$AA?$AA@ 1000d5e0     usbh_ehcdmdd_common_topaz_v1:chw.obj
 0001:0000c608       ??_C@_1EK@EOIJHJGA@?$AAU?$AAS?$AAB?$AA?5?$AAH?$AAo?$AAs?$AAt?$AA?5?$AAi?$AAn?$AA?5?$AAI?$AAd?$AAl?$AAe?$AA?5?$AAS?$AAt?$AAa?$AAt?$AAe?$AA?5?$AAa?$AAn?$AAd?$AA?5?$AAS?$AAu?$AAs?$AAp?$AAe@ 1000d608     usbh_ehcdmdd_common_topaz_v1:chw.obj
 0001:0000c658       ??_C@_1EE@MDIPFHOI@?$AA?$CL?$AAC?$AAH?$AAW?$AA?3?$AA?3?$AAE?$AAn?$AAt?$AAe?$AAr?$AAe?$AAd?$AA?5?$AAU?$AAS?$AAB?$AAI?$AAn?$AAt?$AAe?$AAr?$AAr?$AAu?$AAp?$AAt?$AAT?$AAh?$AAr?$AAe?$AAa?$AAd@ 1000d658     usbh_ehcdmdd_common_topaz_v1:chw.obj
 0001:0000c69c       ??_C@_1DA@GCMJDHBK@?$AAH?$AAU?$AAB?$AA?5?$AAS?$AAt?$AAa?$AAt?$AAu?$AAs?$AA?5?$AAC?$AAh?$AAa?$AAn?$AAg?$AAe?$AA?5?$AA?$CI?$AAA?$AA?$CJ?$AA?$AN?$AA?6?$AA?$AA@ 1000d69c     usbh_ehcdmdd_common_topaz_v1:chw.obj
 0001:0000c6d0       ??_C@_1GM@LHAFDILO@?$AAE?$AAR?$AAR?$AAO?$AAR?$AA?3?$AA?5?$AAU?$AAf?$AAn?$AAP?$AAd?$AAd?$AA_?$AAI?$AAn?$AAi?$AAt?$AA?3?$AA?5?$AAI?$AAn?$AAt?$AAe?$AAr?$AAr?$AAu?$AAp?$AAt?$AA?5?$AAi?$AAn@ 1000d6d0     usbh_ehcdmdd_common_topaz_v1:chw.obj
 0001:0000c740       ??_C@_1EK@OFGOAKAI@?$AAH?$AAo?$AAs?$AAt?$AA?3?$AA?5?$AAH?$AAo?$AAs?$AAt?$AA?5?$AAD?$AAr?$AAi?$AAv?$AAe?$AAr?$AA?5?$AAi?$AAn?$AA?5?$AAc?$AAh?$AAa?$AAr?$AAg?$AAe?$AA?5?$AAn?$AAo?$AAw?$AA?$CB@ 1000d740     usbh_ehcdmdd_common_topaz_v1:chw.obj
 0001:0000c790       ??_C@_1FA@GPDFECOO@?$AAH?$AAo?$AAs?$AAt?$AA?3?$AA?5?$AAW?$AAa?$AAi?$AAt?$AAi?$AAn?$AAg?$AA?5?$AAf?$AAo?$AAr?$AA?5?$AAs?$AAi?$AAg?$AAn?$AAa?$AAl?$AA?5?$AAf?$AAr?$AAo?$AAm?$AA?5?$AAX?$AAC@ 1000d790     usbh_ehcdmdd_common_topaz_v1:chw.obj
 0001:0000c7e0       ??_C@_1EO@NDPDOJGH@?$AAU?$AAF?$AAN?$AA?3?$AA?5?$AAC?$AAr?$AAe?$AAa?$AAt?$AAe?$AA?5?$AAE?$AAv?$AAe?$AAn?$AAt?$AA?5?$AAF?$AAa?$AAi?$AAl?$AAe?$AAd?$AA?5?$AAf?$AAo?$AAr?$AA?5?$AAd?$AAe?$AAt@ 1000d7e0     usbh_ehcdmdd_common_topaz_v1:chw.obj
 0001:0000c830       ??_C@_1EE@OLDBENPI@?$AAU?$AAF?$AAN?$AA?3?$AA?5?$AAC?$AAr?$AAe?$AAa?$AAt?$AAe?$AAd?$AA?5?$AAa?$AA?5?$AAn?$AAe?$AAw?$AA?5?$AAD?$AAe?$AAt?$AAa?$AAc?$AAh?$AA?5?$AAE?$AAv?$AAe?$AAn?$AAt?$AA?$AN@ 1000d830     usbh_ehcdmdd_common_topaz_v1:chw.obj
 0001:0000c878       ??_C@_1EO@CPBNBNCB@?$AAU?$AAF?$AAN?$AA?3?$AA?5?$AAO?$AAp?$AAe?$AAn?$AAe?$AAd?$AA?5?$AAa?$AAn?$AA?5?$AAe?$AAx?$AAi?$AAs?$AAt?$AAi?$AAn?$AAg?$AA?5?$AAD?$AAe?$AAt?$AAa?$AAc?$AAh?$AA?5?$AAE@ 1000d878     usbh_ehcdmdd_common_topaz_v1:chw.obj
 0001:0000c8c8       ??_C@_1EK@KBAJIEHD@?$AAU?$AAF?$AAN?$AA?3?$AA?5?$AAC?$AAr?$AAe?$AAa?$AAt?$AAe?$AA?5?$AAE?$AAv?$AAe?$AAn?$AAt?$AA?5?$AAF?$AAa?$AAi?$AAl?$AAe?$AAd?$AA?5?$AAf?$AAo?$AAr?$AA?5?$AAx?$AAc?$AAv@ 1000d8c8     usbh_ehcdmdd_common_topaz_v1:chw.obj
 0001:0000c918       ??_C@_1EA@CDEDEFDH@?$AAU?$AAF?$AAN?$AA?3?$AA?5?$AAC?$AAr?$AAe?$AAa?$AAt?$AAe?$AAd?$AA?5?$AAa?$AA?5?$AAn?$AAe?$AAw?$AA?5?$AAX?$AAC?$AAV?$AAR?$AA?5?$AAE?$AAv?$AAe?$AAn?$AAt?$AA?$AN?$AA?6?$AA?$AA@ 1000d918     usbh_ehcdmdd_common_topaz_v1:chw.obj
 0001:0000c958       ??_C@_1EK@IADMCEKM@?$AAU?$AAF?$AAN?$AA?3?$AA?5?$AAO?$AAp?$AAe?$AAn?$AAe?$AAd?$AA?5?$AAa?$AAn?$AA?5?$AAe?$AAx?$AAi?$AAs?$AAt?$AAi?$AAn?$AAg?$AA?5?$AAX?$AAC?$AAV?$AAR?$AA?5?$AAE?$AAv?$AAe@ 1000d958     usbh_ehcdmdd_common_topaz_v1:chw.obj
 0001:0000c9a4       ??_C@_1DE@FIHFMDFA@?$AAU?$AAS?$AAB?$AAH?$AAo?$AAs?$AAt?$AA?3?$AA?5?$AAC?$AAr?$AAe?$AAa?$AAt?$AAe?$AAE?$AAv?$AAe?$AAn?$AAt?$AA?3?$AA?$CF?$AAs?$AA?$AN?$AA?6?$AA?$AA@ 1000d9a4     usbh_ehcdmdd_common_topaz_v1:chw.obj
 0001:0000c9d8       ??_C@_1BA@JAHEEJIA@?$AAU?$AAS?$AAB?$AAX?$AAC?$AAV?$AAR?$AA?$AA@ 1000d9d8     usbh_ehcdmdd_common_topaz_v1:chw.obj
 0001:0000c9e8       ??_C@_1EK@DLKEEKEI@?$AAU?$AAF?$AAN?$AA?3?$AA?5?$AAC?$AAr?$AAe?$AAa?$AAt?$AAe?$AA?5?$AAE?$AAv?$AAe?$AAn?$AAt?$AA?5?$AAF?$AAa?$AAi?$AAl?$AAe?$AAd?$AA?5?$AAf?$AAo?$AAr?$AA?5?$AAf?$AAu?$AAn@ 1000d9e8     usbh_ehcdmdd_common_topaz_v1:chw.obj
 0001:0000ca38       ??_C@_1EA@NFBAADLP@?$AAU?$AAF?$AAN?$AA?3?$AA?5?$AAC?$AAr?$AAe?$AAa?$AAt?$AAe?$AAd?$AA?5?$AAa?$AA?5?$AAn?$AAe?$AAw?$AA?5?$AAF?$AAu?$AAn?$AAc?$AA?5?$AAE?$AAv?$AAe?$AAn?$AAt?$AA?$AN?$AA?6?$AA?$AA@ 1000da38     usbh_ehcdmdd_common_topaz_v1:chw.obj
 0001:0000ca78       ??_C@_1FC@JKFHCGKK@?$AAU?$AAS?$AAB?$AAH?$AAo?$AAs?$AAt?$AA?3?$AA?5?$AAO?$AAp?$AAe?$AAn?$AAe?$AAd?$AA?5?$AAa?$AAn?$AA?5?$AAe?$AAx?$AAi?$AAs?$AAt?$AAi?$AAn?$AAg?$AA?5?$AAF?$AAu?$AAn?$AAc@ 1000da78     usbh_ehcdmdd_common_topaz_v1:chw.obj
 0001:0000cacc       ??_C@_1CM@EMEKFINL@?$AAC?$AAH?$AAW?$AA?3?$AA?5?$AAC?$AAr?$AAe?$AAa?$AAt?$AAe?$AAE?$AAv?$AAe?$AAn?$AAt?$AA?3?$AA?$CF?$AAs?$AA?$AN?$AA?6?$AA?$AA@ 1000dacc     usbh_ehcdmdd_common_topaz_v1:chw.obj
 0001:0000caf8       ??_C@_1BA@MLDLNLBG@?$AAU?$AAS?$AAB?$AAH?$AAo?$AAs?$AAt?$AA?$AA@ 1000daf8     usbh_ehcdmdd_common_topaz_v1:chw.obj
 0001:0000cb08       ??_C@_1GM@ELGEFHAB@?$AAU?$AAS?$AAB?$AA?5?$AAI?$AAn?$AAt?$AAe?$AAr?$AAr?$AAu?$AAp?$AAt?$AA?5?$AAT?$AAh?$AAr?$AAe?$AAa?$AAd?$AA?5?$AAr?$AAu?$AAn?$AAn?$AAi?$AAn?$AAg?$AA?5?$AAa?$AAg?$AAa@ 1000db08     usbh_ehcdmdd_common_topaz_v1:chw.obj
 0001:0000cb78       ??_C@_1LE@LBECPNE@?$AA?$CB?$AAU?$AAH?$AAC?$AAI?$AA?5?$AA?9?$AA?5?$AAC?$AAH?$AAW?$AA?3?$AA?3?$AAU?$AAp?$AAd?$AAa?$AAt?$AAe?$AAF?$AAr?$AAa?$AAm?$AAe?$AAC?$AAo?$AAu?$AAn?$AAt?$AAe?$AAr?$AA?5@ 1000db78     usbh_ehcdmdd_common_topaz_v1:chw.obj
 0001:0000cc30       ??_C@_1HC@IPBALCKF@?$AAR?$AAo?$AAo?$AAt?$AA?5?$AAh?$AAu?$AAb?$AA?0?$AA?5?$AAa?$AAf?$AAt?$AAe?$AAr?$AA?5?$AAr?$AAe?$AAs?$AAe?$AAt?$AA?5?$AA?$CG?$AA?5?$AAe?$AAn?$AAa?$AAb?$AAl?$AAe?$AA?0?$AA?5@ 1000dc30     usbh_ehcdmdd_common_topaz_v1:chw.obj
 0001:0000cca4       ??_C@_1CO@NCFLIPAA@?$AA?9?$AAE?$AAn?$AAt?$AAe?$AAr?$AAL?$AAo?$AAw?$AAP?$AAo?$AAw?$AAe?$AAr?$AAM?$AAo?$AAd?$AAe?$AA?$CI?$AA?$CJ?$AA?$AN?$AA?6?$AA?$AA@ 1000dca4     usbh_ehcdmdd_common_topaz_v1:chw.obj
 0001:0000ccd4       ??_C@_1CE@HMNFKKGB@?$AAU?$AAS?$AAB?$AA?5?$AAC?$AAl?$AAo?$AAc?$AAk?$AA?5?$AAs?$AAt?$AAa?$AAr?$AAt?$AA?$AN?$AA?6?$AA?$AA@ 1000dcd4     usbh_ehcdmdd_common_topaz_v1:chw.obj
 0001:0000ccf8       ??_C@_1DG@GDMEJBMH@?$AAP?$AAo?$AAw?$AAe?$AAr?$AAM?$AAg?$AAm?$AAt?$AA?5?$AAw?$AAi?$AAt?$AAh?$AA?5?$AAn?$AAo?$AA?5?$AAa?$AAc?$AAt?$AAi?$AAo?$AAn?$AA?$AN?$AA?6?$AA?$AA@ 1000dcf8     usbh_ehcdmdd_common_topaz_v1:chw.obj
 0001:0000cd30       ??_C@_1CO@OBIJJHOL@?$AA?9?$AAP?$AAo?$AAw?$AAe?$AAr?$AAM?$AAg?$AAm?$AAt?$AAC?$AAa?$AAl?$AAl?$AAB?$AAa?$AAc?$AAk?$AA?$CI?$AA?$CJ?$AA?$AN?$AA?6?$AA?$AA@ 1000dd30     usbh_ehcdmdd_common_topaz_v1:chw.obj
 0001:0000cd60       ??_C@_1CE@IDOAGBCF@?$AAR?$AAe?$AAs?$AAu?$AAm?$AAe?$AA?5?$AAt?$AAh?$AAe?$AA?5?$AAp?$AAo?$AAr?$AAt?$AA?$AN?$AA?6?$AA?$AA@ 1000dd60     usbh_ehcdmdd_common_topaz_v1:chw.obj
 0001:0000cd84       ??_C@_1DC@PANPENJE@?$AA?9?$AAS?$AAu?$AAs?$AAp?$AAe?$AAn?$AAd?$AAH?$AAo?$AAs?$AAt?$AAC?$AAo?$AAn?$AAt?$AAr?$AAo?$AAl?$AAl?$AAe?$AAr?$AA?$AN?$AA?6?$AA?$AA@ 1000dd84     usbh_ehcdmdd_common_topaz_v1:chw.obj
 0001:0000cdb8       ??_C@_1DC@FOJLBFDA@?$AA?$CL?$AAS?$AAu?$AAs?$AAp?$AAe?$AAn?$AAd?$AAH?$AAo?$AAs?$AAt?$AAC?$AAo?$AAn?$AAt?$AAr?$AAo?$AAl?$AAl?$AAe?$AAr?$AA?$AN?$AA?6?$AA?$AA@ 1000ddb8     usbh_ehcdmdd_common_topaz_v1:chw.obj
 0001:0000cdf0       ??_C@_1FA@CINLDKJL@?$AA?7?$AA?7?$AAC?$AAH?$AAW?$AA?5?$AA?9?$AA?5?$AAF?$AAA?$AAI?$AAL?$AAE?$AAD?$AA?5?$AAW?$AAH?$AAI?$AAL?$AAE?$AA?5?$AAD?$AAU?$AAM?$AAP?$AAI?$AAN?$AAG?$AA?5?$AAU?$AAS?$AAB@ 1000ddf0     usbh_ehcdmdd_common_topaz_v1:chw.obj
 0001:0000ce40       ??_C@_1CC@FCJFIKJP@?$AA?7?$AA?7?$AAR?$AAu?$AAn?$AA?1?$AAS?$AAt?$AAo?$AAp?$AA?5?$AA?$DN?$AA?5?$AA?$CF?$AAs?$AA?6?$AA?$AA@ 1000de40     usbh_ehcdmdd_common_topaz_v1:chw.obj
 0001:0000ce64       ??_C@_19PENBCILL@?$AAS?$AAt?$AAo?$AAp?$AA?$AA@ 1000de64     usbh_ehcdmdd_common_topaz_v1:chw.obj
 0001:0000ce70       ??_C@_17NMIMIGP@?$AAR?$AAu?$AAn?$AA?$AA@ 1000de70     usbh_ehcdmdd_common_topaz_v1:chw.obj
 0001:0000ce78       ??_C@_1DM@BNPFABFC@?$AA?7?$AA?7?$AAH?$AAo?$AAs?$AAt?$AA?5?$AAC?$AAo?$AAn?$AAt?$AAr?$AAo?$AAl?$AAl?$AAe?$AAr?$AA?5?$AAR?$AAe?$AAs?$AAe?$AAt?$AA?5?$AA?$DN?$AA?5?$AA?$CF?$AAs?$AA?6?$AA?$AA@ 1000de78     usbh_ehcdmdd_common_topaz_v1:chw.obj
 0001:0000ceb4       ??_C@_1BA@MICNGLHI@?$AAN?$AAo?$AAt?$AA?5?$AAS?$AAe?$AAt?$AA?$AA@ 1000deb4     usbh_ehcdmdd_common_topaz_v1:chw.obj
 0001:0000cec4       ??_C@_17PNBAHNJB@?$AAS?$AAe?$AAt?$AA?$AA@ 1000dec4     usbh_ehcdmdd_common_topaz_v1:chw.obj
 0001:0000ced0       ??_C@_1GI@CJDDJLJ@?$AA?7?$AAC?$AAH?$AAW?$AA?5?$AA?9?$AA?5?$AAU?$AAS?$AAB?$AA?5?$AAC?$AAO?$AAM?$AAM?$AAA?$AAN?$AAD?$AA?5?$AAR?$AAE?$AAG?$AAI?$AAS?$AAT?$AAE?$AAR?$AA?5?$AA?$CI?$AAU?$AAS?$AAB@ 1000ded0     usbh_ehcdmdd_common_topaz_v1:chw.obj
 0001:0000cf38       ??_C@_1FA@HOJIMDFK@?$AA?7?$AA?7?$AAC?$AAH?$AAW?$AA?5?$AA?9?$AA?5?$AAF?$AAA?$AAI?$AAL?$AAE?$AAD?$AA?5?$AAW?$AAH?$AAI?$AAL?$AAE?$AA?5?$AAD?$AAU?$AAM?$AAP?$AAI?$AAN?$AAG?$AA?5?$AAU?$AAS?$AAB@ 1000df38     usbh_ehcdmdd_common_topaz_v1:chw.obj
 0001:0000cf88       ??_C@_1CM@HJBFIEJM@?$AA?7?$AA?7?$AAU?$AAS?$AAB?$AA?5?$AAI?$AAn?$AAt?$AAe?$AAr?$AAr?$AAu?$AAp?$AAt?$AA?5?$AA?$DN?$AA?5?$AA?$CF?$AAs?$AA?6?$AA?$AA@ 1000df88     usbh_ehcdmdd_common_topaz_v1:chw.obj
 0001:0000cfb4       ??_C@_1DI@FEJALCMH@?$AA?7?$AA?7?$AAU?$AAS?$AAB?$AA?5?$AAE?$AAr?$AAr?$AAo?$AAr?$AA?5?$AAI?$AAn?$AAt?$AAe?$AAr?$AAr?$AAu?$AAp?$AAt?$AA?5?$AA?$DN?$AA?5?$AA?$CF?$AAs?$AA?6?$AA?$AA@ 1000dfb4     usbh_ehcdmdd_common_topaz_v1:chw.obj
 0001:0000cfec       ??_C@_1DE@EKNDKMKA@?$AA?7?$AA?7?$AAH?$AAo?$AAs?$AAt?$AA?5?$AAS?$AAy?$AAs?$AAt?$AAe?$AAm?$AA?5?$AAE?$AAr?$AAr?$AAo?$AAr?$AA?5?$AA?$DN?$AA?5?$AA?$CF?$AAs?$AA?6?$AA?$AA@ 1000dfec     usbh_ehcdmdd_common_topaz_v1:chw.obj
 0001:0000d020       ??_C@_1CC@GDBEJMLN@?$AA?7?$AA?7?$AAH?$AAC?$AAH?$AAa?$AAl?$AAt?$AAe?$AAd?$AA?5?$AA?$DN?$AA?5?$AA?$CF?$AAs?$AA?6?$AA?$AA@ 1000e020     usbh_ehcdmdd_common_topaz_v1:chw.obj
 0001:0000d044       ??_C@_1BG@BOOFOFNO@?$AAN?$AAo?$AAt?$AA?5?$AAH?$AAa?$AAl?$AAt?$AAe?$AAd?$AA?$AA@ 1000e044     usbh_ehcdmdd_common_topaz_v1:chw.obj
 0001:0000d05c       ??_C@_1O@OAOPMKLB@?$AAH?$AAa?$AAl?$AAt?$AAe?$AAd?$AA?$AA@ 1000e05c     usbh_ehcdmdd_common_topaz_v1:chw.obj
 0001:0000d070       ??_C@_1GG@MOAIJENA@?$AA?7?$AAC?$AAH?$AAW?$AA?5?$AA?9?$AA?5?$AAU?$AAS?$AAB?$AA?5?$AAS?$AAT?$AAA?$AAT?$AAU?$AAS?$AA?5?$AAR?$AAE?$AAG?$AAI?$AAS?$AAT?$AAE?$AAR?$AA?5?$AA?$CI?$AAU?$AAS?$AAB?$AAS@ 1000e070     usbh_ehcdmdd_common_topaz_v1:chw.obj
 0001:0000d0d8       ??_C@_1FC@FIEEKJDM@?$AA?7?$AA?7?$AAC?$AAH?$AAW?$AA?5?$AA?9?$AA?5?$AAF?$AAA?$AAI?$AAL?$AAE?$AAD?$AA?5?$AAW?$AAH?$AAI?$AAL?$AAE?$AA?5?$AAD?$AAU?$AAM?$AAP?$AAI?$AAN?$AAG?$AA?5?$AAU?$AAS?$AAB@ 1000e0d8     usbh_ehcdmdd_common_topaz_v1:chw.obj
 0001:0000d130       ??_C@_1GO@FCNOGNDE@?$AA?7?$AAC?$AAH?$AAW?$AA?5?$AA?9?$AA?5?$AAU?$AAS?$AAB?$AA?5?$AAI?$AAN?$AAT?$AAE?$AAR?$AAR?$AAU?$AAP?$AAT?$AA?5?$AAR?$AAE?$AAG?$AAI?$AAS?$AAT?$AAE?$AAR?$AA?5?$AA?$CI?$AAU@ 1000e130     usbh_ehcdmdd_common_topaz_v1:chw.obj
 0001:0000d1a0       ??_C@_1EO@HHCCBPHE@?$AA?7?$AA?7?$AAC?$AAH?$AAW?$AA?5?$AA?9?$AA?5?$AAF?$AAA?$AAI?$AAL?$AAE?$AAD?$AA?5?$AAW?$AAH?$AAI?$AAL?$AAE?$AA?5?$AAD?$AAU?$AAM?$AAP?$AAI?$AAN?$AAG?$AA?5?$AAF?$AAR?$AAN@ 1000e1a0     usbh_ehcdmdd_common_topaz_v1:chw.obj
 0001:0000d1f0       ??_C@_1EA@KMAMFMHL@?$AA?7?$AA?7?$AAF?$AAr?$AAa?$AAm?$AAe?$AA?5?$AAi?$AAn?$AAd?$AAe?$AAx?$AA?5?$AA?$CI?$AAb?$AAi?$AAt?$AAs?$AA?5?$AA1?$AA1?$AA?3?$AA3?$AA?$CJ?$AA?5?$AA?$DN?$AA?5?$AA?$CF?$AAd?$AA?6?$AA?$AA@ 1000e1f0     usbh_ehcdmdd_common_topaz_v1:chw.obj
 0001:0000d230       ??_C@_1EK@EDJKFKKL@?$AA?7?$AA?7?$AAM?$AAi?$AAc?$AAr?$AAo?$AAF?$AAr?$AAa?$AAm?$AAe?$AA?5?$AAn?$AAu?$AAm?$AAb?$AAe?$AAr?$AA?5?$AA?$CI?$AAb?$AAi?$AAt?$AAs?$AA?5?$AA2?$AA?3?$AA0?$AA?$CJ?$AA?5?$AA?$DN@ 1000e230     usbh_ehcdmdd_common_topaz_v1:chw.obj
 0001:0000d280       ??_C@_1GI@GBDLEJOC@?$AA?7?$AAC?$AAH?$AAW?$AA?5?$AA?9?$AA?5?$AAF?$AAR?$AAA?$AAM?$AAE?$AA?5?$AAN?$AAU?$AAM?$AAB?$AAE?$AAR?$AA?5?$AAR?$AAE?$AAG?$AAI?$AAS?$AAT?$AAE?$AAR?$AA?5?$AA?$CI?$AAF?$AAR@ 1000e280     usbh_ehcdmdd_common_topaz_v1:chw.obj
 0001:0000d2e8       ??_C@_1FG@PNNMPAJC@?$AA?7?$AA?7?$AAC?$AAH?$AAW?$AA?5?$AA?9?$AA?5?$AAF?$AAA?$AAI?$AAL?$AAE?$AAD?$AA?5?$AAW?$AAH?$AAI?$AAL?$AAE?$AA?5?$AAD?$AAU?$AAM?$AAP?$AAI?$AAN?$AAG?$AA?5?$AAF?$AAL?$AAB@ 1000e2e8     usbh_ehcdmdd_common_topaz_v1:chw.obj
 0001:0000d340       ??_C@_1GI@IENAJBGM@?$AA?7?$AA?7?$AAF?$AAL?$AAB?$AAA?$AAS?$AAE?$AAA?$AAD?$AAD?$AA?5?$AAa?$AAd?$AAd?$AAr?$AAe?$AAs?$AAs?$AA?5?$AAb?$AAa?$AAs?$AAe?$AA?5?$AA?$CI?$AAb?$AAi?$AAt?$AAs?$AA?5?$AA1@ 1000e340     usbh_ehcdmdd_common_topaz_v1:chw.obj
 0001:0000d3a8       ??_C@_1IG@DAOFPJDD@?$AA?7?$AAC?$AAH?$AAW?$AA?5?$AA?9?$AA?5?$AAF?$AAR?$AAA?$AAM?$AAE?$AA?5?$AAL?$AAI?$AAS?$AAT?$AA?5?$AAB?$AAA?$AAS?$AAE?$AA?5?$AAA?$AAD?$AAD?$AAR?$AAE?$AAS?$AAS?$AA?5?$AAR@ 1000e3a8     usbh_ehcdmdd_common_topaz_v1:chw.obj
 0001:0000d430       ??_C@_1FA@KDJOBDNF@?$AA?7?$AA?7?$AAC?$AAH?$AAW?$AA?5?$AA?9?$AA?5?$AAF?$AAA?$AAI?$AAL?$AAE?$AAD?$AA?5?$AAW?$AAH?$AAI?$AAL?$AAE?$AA?5?$AAD?$AAU?$AAM?$AAP?$AAI?$AAN?$AAG?$AA?5?$AAS?$AAO?$AAF@ 1000e430     usbh_ehcdmdd_common_topaz_v1:chw.obj
 0001:0000d480       ??_C@_1DC@IMLMPEKL@?$AA?7?$AA?7?$AAC?$AAH?$AAW?$AA?5?$AAC?$AAT?$AAL?$AAD?$AAS?$AAS?$AAE?$AAG?$AAM?$AAE?$AAN?$AAT?$AA?5?$AA?$DN?$AA?5?$AA?$CF?$AAx?$AA?6?$AA?$AA@ 1000e480     usbh_ehcdmdd_common_topaz_v1:chw.obj
 0001:0000d4b4       ??_C@_1CO@JNDLEHIM@?$AA?7?$AA?7?$AAC?$AAH?$AAW?$AA?5?$AAC?$AAO?$AAN?$AAF?$AAI?$AAG?$AAF?$AAL?$AAA?$AAG?$AA?5?$AA?$DN?$AA?5?$AA?$CF?$AAx?$AA?6?$AA?$AA@ 1000e4b4     usbh_ehcdmdd_common_topaz_v1:chw.obj
 0001:0000d4e8       ??_C@_1EI@ICGKKOFG@?$AA?7?$AAC?$AAH?$AAW?$AA?5?$AA?9?$AA?5?$AAA?$AAS?$AAY?$AAN?$AAC?$AAL?$AAI?$AAS?$AAT?$AAA?$AAD?$AAD?$AAR?$AA?5?$AA?$DN?$AA?5?$AA0?$AAx?$AA?$CF?$AAX?$AA?4?$AA?5?$AAD?$AAu?$AAm@ 1000e4e8     usbh_ehcdmdd_common_topaz_v1:chw.obj
 0001:0000d530       ??_C@_1FE@MJBCKJEH@?$AA?7?$AA?7?$AAC?$AAH?$AAW?$AA?5?$AA?9?$AA?5?$AAF?$AAA?$AAI?$AAL?$AAE?$AAD?$AA?5?$AAW?$AAH?$AAI?$AAL?$AAE?$AA?5?$AAD?$AAU?$AAM?$AAP?$AAI?$AAN?$AAG?$AA?5?$AAP?$AAO?$AAR@ 1000e530     usbh_ehcdmdd_common_topaz_v1:chw.obj
 0001:0000d588       ??_C@_1EA@COLCHOIE@?$AA?7?$AA?7?$AAH?$AAu?$AAb?$AA?5?$AAS?$AAt?$AAa?$AAt?$AAe?$AA?5?$AAt?$AAh?$AAi?$AAs?$AA?5?$AAp?$AAo?$AAr?$AAt?$AA?5?$AAD?$AAi?$AAs?$AAa?$AAb?$AAl?$AAe?$AAd?$AA?6?$AA?$AA@ 1000e588     usbh_ehcdmdd_common_topaz_v1:chw.obj
 0001:0000d5c8       ??_C@_1CO@NJFFGMHB@?$AA?7?$AA?7?$AAC?$AAo?$AAn?$AAn?$AAe?$AAc?$AAt?$AA?5?$AAS?$AAt?$AAa?$AAt?$AAu?$AAs?$AA?5?$AA?$DN?$AA?5?$AA?$CF?$AAs?$AA?6?$AA?$AA@ 1000e5c8     usbh_ehcdmdd_common_topaz_v1:chw.obj
 0001:0000d5f8       ??_C@_1CE@BKHLEMML@?$AAN?$AAo?$AA?5?$AAD?$AAe?$AAv?$AAi?$AAc?$AAe?$AA?5?$AAP?$AAr?$AAe?$AAs?$AAe?$AAn?$AAt?$AA?$AA@ 1000e5f8     usbh_ehcdmdd_common_topaz_v1:chw.obj
 0001:0000d61c       ??_C@_1BO@BNKELDOA@?$AAD?$AAe?$AAv?$AAi?$AAc?$AAe?$AA?5?$AAP?$AAr?$AAe?$AAs?$AAe?$AAn?$AAt?$AA?$AA@ 1000e61c     usbh_ehcdmdd_common_topaz_v1:chw.obj
 0001:0000d63c       ??_C@_1DM@IALKIFOG@?$AA?7?$AA?7?$AAC?$AAo?$AAn?$AAn?$AAe?$AAc?$AAt?$AA?5?$AAS?$AAt?$AAa?$AAt?$AAu?$AAs?$AA?5?$AAC?$AAh?$AAa?$AAn?$AAg?$AAe?$AA?5?$AA?$DN?$AA?5?$AA?$CF?$AAs?$AA?6?$AA?$AA@ 1000e63c     usbh_ehcdmdd_common_topaz_v1:chw.obj
 0001:0000d678       ??_C@_1EI@MHFOFDE@?$AA?7?$AA?7?$AAP?$AAo?$AAr?$AAt?$AA?5?$AAE?$AAn?$AAa?$AAb?$AAl?$AAe?$AA?1?$AAD?$AAi?$AAs?$AAa?$AAb?$AAl?$AAe?$AA?5?$AAC?$AAh?$AAa?$AAn?$AAg?$AAe?$AA?5?$AA?5?$AA?$DN?$AA?5@ 1000e678     usbh_ehcdmdd_common_topaz_v1:chw.obj
 0001:0000d6c0       ??_C@_1CI@HLOFBIAL@?$AA?7?$AA?7?$AAL?$AAi?$AAn?$AAe?$AA?5?$AAS?$AAt?$AAa?$AAt?$AAu?$AAs?$AA?5?$AA?$DN?$AA?5?$AA?$CF?$AAd?$AA?6?$AA?$AA@ 1000e6c0     usbh_ehcdmdd_common_topaz_v1:chw.obj
 0001:0000d6e8       ??_C@_1CM@ECMIMKLE@?$AA?7?$AA?7?$AAR?$AAe?$AAs?$AAu?$AAm?$AAe?$AA?5?$AAD?$AAe?$AAt?$AAe?$AAc?$AAt?$AA?5?$AA?$DN?$AA?5?$AA?$CF?$AAs?$AA?6?$AA?$AA@ 1000e6e8     usbh_ehcdmdd_common_topaz_v1:chw.obj
 0001:0000d714       ??_C@_1CG@JNFFMMPC@?$AA?7?$AA?7?$AAP?$AAo?$AAr?$AAt?$AA?5?$AAR?$AAe?$AAs?$AAe?$AAt?$AA?5?$AA?$DN?$AA?5?$AA?$CF?$AAs?$AA?6?$AA?$AA@ 1000e714     usbh_ehcdmdd_common_topaz_v1:chw.obj
 0001:0000d73c       ??_C@_1BE@HCJIFAIL@?$AAN?$AAo?$AAt?$AA?5?$AAR?$AAe?$AAs?$AAe?$AAt?$AA?$AA@ 1000e73c     usbh_ehcdmdd_common_topaz_v1:chw.obj
 0001:0000d750       ??_C@_1M@PNBPANGG@?$AAR?$AAe?$AAs?$AAe?$AAt?$AA?$AA@ 1000e750     usbh_ehcdmdd_common_topaz_v1:chw.obj
 0001:0000d75c       ??_C@_1CE@IINGCJBA@?$AA?7?$AA?7?$AAH?$AAu?$AAb?$AA?5?$AAS?$AAt?$AAa?$AAt?$AAe?$AA?5?$AA?$DN?$AA?5?$AA?$CF?$AAs?$AA?6?$AA?$AA@ 1000e75c     usbh_ehcdmdd_common_topaz_v1:chw.obj
 0001:0000d780       ??_C@_1O@PFBIKACK@?$AAE?$AAn?$AAa?$AAb?$AAl?$AAe?$AA?$AA@ 1000e780     usbh_ehcdmdd_common_topaz_v1:chw.obj
 0001:0000d790       ??_C@_1BA@CHDFGDCJ@?$AAS?$AAu?$AAs?$AAp?$AAe?$AAn?$AAd?$AA?$AA@ 1000e790     usbh_ehcdmdd_common_topaz_v1:chw.obj
 0001:0000d7a0       ??_C@_1IE@HABAAOJJ@?$AA?7?$AAC?$AAH?$AAW?$AA?5?$AA?9?$AA?5?$AAP?$AAO?$AAR?$AAT?$AA?5?$AAS?$AAT?$AAA?$AAT?$AAU?$AAS?$AA?5?$AAA?$AAN?$AAD?$AA?5?$AAC?$AAO?$AAN?$AAT?$AAR?$AAO?$AAL?$AA?5?$AAR@ 1000e7a0     usbh_ehcdmdd_common_topaz_v1:chw.obj
 0001:0000d824       ??_C@_1DG@GHFBFGDF@?$AAC?$AAH?$AAW?$AA?5?$AA?9?$AA?5?$AAD?$AAU?$AAM?$AAP?$AA?5?$AAR?$AAE?$AAG?$AAI?$AAS?$AAT?$AAE?$AAR?$AAS?$AA?5?$AAD?$AAO?$AAN?$AAE?$AA?6?$AA?$AA@ 1000e824     usbh_ehcdmdd_common_topaz_v1:chw.obj
 0001:0000d85c       ??_C@_1DI@GCACGEGK@?$AAC?$AAH?$AAW?$AA?5?$AA?9?$AA?5?$AAD?$AAU?$AAM?$AAP?$AA?5?$AAR?$AAE?$AAG?$AAI?$AAS?$AAT?$AAE?$AAR?$AAS?$AA?5?$AAB?$AAE?$AAG?$AAI?$AAN?$AA?6?$AA?$AA@ 1000e85c     usbh_ehcdmdd_common_topaz_v1:chw.obj
 0001:0000d894       ??_7CTransfer@@6B@         1000e894     usbh_ehcdmdd_common_topaz_v1:trans.obj
 0001:0000d8a0       ??_C@_1LK@NOKJIPGM@?$AAC?$AAT?$AAr?$AAa?$AAn?$AAs?$AAf?$AAe?$AAr?$AA?3?$AA?3?$AA?$HO?$AAC?$AAT?$AAr?$AAa?$AAn?$AAs?$AAf?$AAe?$AAr?$AA?$CI?$AA?$CJ?$AA?5?$AA?$CI?$AAt?$AAh?$AAi?$AAs?$AA?$DN?$AA0?$AAx@ 1000e8a0     usbh_ehcdmdd_common_topaz_v1:trans.obj
 0001:0000d960       ??_C@_1LM@CLNPCLAL@?$AAC?$AAQ?$AAT?$AAr?$AAa?$AAn?$AAs?$AAf?$AAe?$AAr?$AA?3?$AA?3?$AAI?$AAn?$AAi?$AAt?$AA?5?$AA?$CI?$AAt?$AAh?$AAi?$AAs?$AA?$DN?$AA0?$AAx?$AA?$CF?$AAx?$AA?0?$AAi?$AAd?$AA?$DN?$AA0@ 1000e960     usbh_ehcdmdd_common_topaz_v1:trans.obj
 0001:0000da20       ??_C@_1GI@DEJENGNL@?$AAC?$AAP?$AAi?$AAp?$AAe?$AA?$CI?$AA?$CF?$AAs?$AA?$CJ?$AA?3?$AA?3?$AAI?$AAs?$AAs?$AAu?$AAe?$AAT?$AAr?$AAa?$AAn?$AAs?$AAf?$AAe?$AAr?$AA?5?$AA?9?$AA?5?$AAn?$AAo?$AA?5?$AAm?$AAe@ 1000ea20     usbh_ehcdmdd_common_topaz_v1:trans.obj
 0001:0000da88       ??_C@_1CK@EEDMLIDO@?$AAI?$AAs?$AAs?$AAu?$AAe?$AAT?$AAr?$AAa?$AAn?$AAs?$AAf?$AAe?$AAr?$AA?5?$AAB?$AAu?$AAf?$AAf?$AAe?$AAr?$AA?$AA@ 1000ea88     usbh_ehcdmdd_common_topaz_v1:trans.obj
 0001:0000dab8       ??_C@_1FC@JFJBHHOO@?$AAC?$AAT?$AAr?$AAa?$AAn?$AAs?$AAf?$AAe?$AAr?$AA?3?$AA?5?$AAB?$AAa?$AAd?$AA?5?$AAb?$AAu?$AAf?$AAf?$AAe?$AAr?$AA?5?$AAt?$AAo?$AA?5?$AAm?$AAe?$AAm?$AAs?$AAe?$AAt?$AA?5@ 1000eab8     usbh_ehcdmdd_common_topaz_v1:trans.obj
 0001:0000db10       ??_C@_1LM@JGBFFJBF@?$AAC?$AA?3?$AA?2?$AAW?$AAI?$AAN?$AAC?$AAE?$AAR?$AAO?$AAO?$AAT?$AAS?$AA?2?$AAT?$AAo?$AAp?$AAa?$AAz?$AA?2?$AAW?$AAI?$AAN?$AAC?$AAE?$AA6?$AA0?$AA0?$AA?2?$AAP?$AAL?$AAA@ 1000eb10     usbh_ehcdmdd_common_topaz_v1:trans.obj
 0001:0000dbd0       ??_C@_1GO@EEFDOHBH@?$AAC?$AAP?$AAi?$AAp?$AAe?$AA?$CI?$AA?$CF?$AAs?$AA?$CJ?$AA?3?$AA?3?$AAI?$AAs?$AAs?$AAu?$AAe?$AAT?$AAr?$AAa?$AAn?$AAs?$AAf?$AAe?$AAr?$AA?5?$AA?9?$AA?5?$AAn?$AAo?$AA?5?$AAm?$AAe@ 1000ebd0     usbh_ehcdmdd_common_topaz_v1:trans.obj
 0001:0000dc40       ??_C@_1DG@OIBCBHKK@?$AAI?$AAs?$AAs?$AAu?$AAe?$AAT?$AAr?$AAa?$AAn?$AAs?$AAf?$AAe?$AAr?$AA?5?$AAS?$AAE?$AAT?$AAU?$AAP?$AA?5?$AAB?$AAu?$AAf?$AAf?$AAe?$AAr?$AA?$AA@ 1000ec40     usbh_ehcdmdd_common_topaz_v1:trans.obj
 0001:0000dc78       ??_C@_1EM@KFFIANIM@?$AAC?$AAT?$AAr?$AAa?$AAn?$AAs?$AAf?$AAe?$AAr?$AA?3?$AA?3?$AAI?$AAn?$AAi?$AAt?$AA?5?$AA?$CI?$AAt?$AAh?$AAi?$AAs?$AA?$DN?$AA0?$AAx?$AA?$CF?$AAx?$AA?0?$AAi?$AAd?$AA?$DN?$AA0?$AAx@ 1000ec78     usbh_ehcdmdd_common_topaz_v1:trans.obj
 0001:0000dcc8       ??_C@_1FM@HOOBCKCH@?$AAC?$AAQ?$AAT?$AAr?$AAa?$AAn?$AAs?$AAf?$AAe?$AAr?$AA?3?$AA?3?$AAA?$AAd?$AAd?$AAT?$AAr?$AAa?$AAn?$AAs?$AAf?$AAe?$AAr?$AA?5?$AA?$CI?$AAt?$AAh?$AAi?$AAs?$AA?$DN?$AA0?$AAx@ 1000ecc8     usbh_ehcdmdd_common_topaz_v1:trans.obj
 0001:0000dd28       ??_C@_1LA@PHHAKCJP@?$AAC?$AAQ?$AAu?$AAe?$AAu?$AAe?$AAd?$AAP?$AAi?$AAp?$AAe?$AA?$CI?$AA?$CF?$AAs?$AA?$CJ?$AA?3?$AA?3?$AAC?$AAh?$AAe?$AAc?$AAk?$AAF?$AAo?$AAr?$AAD?$AAo?$AAn?$AAe?$AAT?$AAr?$AAa@ 1000ed28     usbh_ehcdmdd_common_topaz_v1:trans.obj
 0001:0000ddd8       ??_C@_1FO@HOCBNIDJ@?$AAC?$AAQ?$AAT?$AAr?$AAa?$AAn?$AAs?$AAf?$AAe?$AAr?$AA?3?$AA?3?$AAD?$AAo?$AAn?$AAe?$AAT?$AAr?$AAa?$AAn?$AAs?$AAf?$AAe?$AAr?$AA?5?$AA?$CI?$AAt?$AAh?$AAi?$AAs?$AA?$DN?$AA0@ 1000edd8     usbh_ehcdmdd_common_topaz_v1:trans.obj
 0001:0000de38       ??_C@_1GA@LCLHDHLL@?$AAC?$AAQ?$AAT?$AAr?$AAa?$AAn?$AAs?$AAf?$AAe?$AAr?$AA?3?$AA?3?$AAA?$AAb?$AAo?$AAr?$AAt?$AAT?$AAr?$AAa?$AAn?$AAs?$AAf?$AAe?$AAr?$AA?5?$AA?$CI?$AAt?$AAh?$AAi?$AAs?$AA?$DN@ 1000ee38     usbh_ehcdmdd_common_topaz_v1:trans.obj
 0001:0000de98       ??_C@_1GI@FMPNEOID@?$AAC?$AAQ?$AAT?$AAr?$AAa?$AAn?$AAs?$AAf?$AAe?$AAr?$AA?3?$AA?3?$AAI?$AAs?$AAT?$AAr?$AAa?$AAn?$AAs?$AAf?$AAe?$AAr?$AAD?$AAo?$AAn?$AAe?$AA?5?$AA?$CI?$AAt?$AAh?$AAi?$AAs@ 1000ee98     usbh_ehcdmdd_common_topaz_v1:trans.obj
 0001:0000df00       ??_C@_1CK@OOCENHGM@?$AAC?$AAQ?$AAT?$AAr?$AAa?$AAn?$AAs?$AAf?$AAe?$AAr?$AA?3?$AA?5?$AAH?$AAa?$AAl?$AAt?$AAe?$AAd?$AA?$AN?$AA?6?$AA?$AA@ 1000ef00     usbh_ehcdmdd_common_topaz_v1:trans.obj
 0001:0000df30       ??_C@_1EG@FDPFCBKF@?$AAT?$AAD?$AA?5?$AAT?$AAo?$AAk?$AAe?$AAn?$AA?3?$AA?5?$AAD?$AAa?$AAt?$AAa?$AAB?$AAu?$AAf?$AAf?$AAe?$AAr?$AAE?$AAr?$AAr?$AAo?$AAr?$AA?5?$AAi?$AAn?$AA?5?$AAO?$AAU?$AAT@ 1000ef30     usbh_ehcdmdd_common_topaz_v1:trans.obj
 0001:0000df78       ??_C@_1EE@LLFNFPJJ@?$AAT?$AAD?$AA?5?$AAT?$AAo?$AAk?$AAe?$AAn?$AA?3?$AA?5?$AAD?$AAa?$AAt?$AAa?$AAB?$AAu?$AAf?$AAf?$AAe?$AAr?$AAE?$AAr?$AAr?$AAo?$AAr?$AA?5?$AAi?$AAn?$AA?5?$AAI?$AAN?$AA?$AN@ 1000ef78     usbh_ehcdmdd_common_topaz_v1:trans.obj
 0001:0000dfc0       ??_C@_1GC@LFCCAJDE@?$AAC?$AAQ?$AAT?$AAr?$AAa?$AAn?$AAs?$AAf?$AAe?$AAr?$AA?3?$AA?3?$AAI?$AAs?$AAT?$AAr?$AAa?$AAn?$AAs?$AAf?$AAe?$AAr?$AAD?$AAo?$AAn?$AAe?$AA?5?$AA?$CI?$AAt?$AAh?$AAi?$AAs@ 1000efc0     usbh_ehcdmdd_common_topaz_v1:trans.obj
 0001:0000e024       ??_7CIsochTransfer@@6B@    1000f024     usbh_ehcdmdd_common_topaz_v1:trans.obj
 0001:0000e040       ??_C@_1LE@NPCNNEEO@?$AAc?$AA?3?$AA?2?$AAw?$AAi?$AAn?$AAc?$AAe?$AAr?$AAo?$AAo?$AAt?$AAs?$AA?2?$AAt?$AAo?$AAp?$AAa?$AAz?$AA?2?$AAw?$AAi?$AAn?$AAc?$AAe?$AA6?$AA0?$AA0?$AA?2?$AAp?$AAl?$AAa@ 1000f040     usbh_ehcdmdd_common_topaz_v1:trans.obj
 0001:0000e0f4       ??_7CITransfer@@6B@        1000f0f4     usbh_ehcdmdd_common_topaz_v1:trans.obj
 0001:0000e110       ??_C@_1FM@OAOHMNCD@?$AAC?$AAI?$AAT?$AAr?$AAa?$AAn?$AAs?$AAf?$AAe?$AAr?$AA?3?$AA?3?$AAA?$AAd?$AAd?$AAT?$AAr?$AAa?$AAn?$AAs?$AAf?$AAe?$AAr?$AA?5?$AA?$CI?$AAt?$AAh?$AAi?$AAs?$AA?$DN?$AA0?$AAx@ 1000f110     usbh_ehcdmdd_common_topaz_v1:trans.obj
 0001:0000e170       ??_C@_1FO@JHKNGPD@?$AAC?$AAI?$AAT?$AAr?$AAa?$AAn?$AAs?$AAf?$AAe?$AAr?$AA?3?$AA?3?$AAS?$AAc?$AAh?$AAe?$AAd?$AAu?$AAl?$AAe?$AAT?$AAD?$AA?5?$AA?$CI?$AAt?$AAh?$AAi?$AAs?$AA?$DN?$AA0?$AAx?$AA?$CF@ 1000f170     usbh_ehcdmdd_common_topaz_v1:trans.obj
 0001:0000e1d0       ??_C@_1IA@GPBFBECG@?$AAC?$AAI?$AAT?$AAr?$AAa?$AAn?$AAs?$AAf?$AAe?$AAr?$AA?3?$AA?3?$AAS?$AAc?$AAh?$AAe?$AAd?$AAu?$AAl?$AAe?$AAT?$AAD?$AA?5?$AA?$CI?$AAt?$AAh?$AAi?$AAs?$AA?$DN?$AA0?$AAx?$AA?$CF@ 1000f1d0     usbh_ehcdmdd_common_topaz_v1:trans.obj
 0001:0000e250       ??_C@_1JA@MMFDMIBD@?$AAC?$AAI?$AAT?$AAr?$AAa?$AAn?$AAs?$AAf?$AAe?$AAr?$AA?3?$AA?3?$AA?3?$AAI?$AAs?$AAT?$AAr?$AAa?$AAn?$AAs?$AAf?$AAe?$AAr?$AAD?$AAo?$AAn?$AAe?$AA?5?$AA?$CI?$AAt?$AAh?$AAi@ 1000f250     usbh_ehcdmdd_common_topaz_v1:trans.obj
 0001:0000e2e0       ??_C@_1GC@HMMEFEGP@?$AAC?$AAI?$AAT?$AAr?$AAa?$AAn?$AAs?$AAf?$AAe?$AAr?$AA?3?$AA?3?$AAA?$AAb?$AAo?$AAr?$AAt?$AAT?$AAr?$AAa?$AAn?$AAs?$AAf?$AAe?$AAr?$AA?5?$AA?$CI?$AAt?$AAh?$AAi?$AAs?$AA?$DN@ 1000f2e0     usbh_ehcdmdd_common_topaz_v1:trans.obj
 0001:0000e348       ??_C@_1KG@GHEKBGJB@?$AAC?$AAI?$AAT?$AAr?$AAa?$AAn?$AAs?$AAf?$AAe?$AAr?$AA?3?$AA?3?$AAD?$AAo?$AAn?$AAe?$AAT?$AAr?$AAa?$AAn?$AAs?$AAf?$AAe?$AAr?$AA?5?$AA?$CI?$AAt?$AAh?$AAi?$AAs?$AA?$DN?$AA0@ 1000f348     usbh_ehcdmdd_common_topaz_v1:trans.obj
 0001:0000e3f0       ??_7CSITransfer@@6B@       1000f3f0     usbh_ehcdmdd_common_topaz_v1:trans.obj
 0001:0000e410       ??_C@_1IK@NLLPLEIF@?$AAC?$AAS?$AAI?$AAT?$AAr?$AAa?$AAn?$AAs?$AAf?$AAe?$AAr?$AA?3?$AA?3?$AAA?$AAd?$AAd?$AAT?$AAr?$AAa?$AAn?$AAs?$AAf?$AAe?$AAr?$AA?5?$AA?$CI?$AAt?$AAh?$AAi?$AAs?$AA?$DN?$AA0@ 1000f410     usbh_ehcdmdd_common_topaz_v1:trans.obj
 0001:0000e4a0       ??_C@_1LE@CHDJGKIJ@?$AAC?$AAS?$AAI?$AAT?$AAr?$AAa?$AAn?$AAs?$AAf?$AAe?$AAr?$AA?3?$AA?3?$AAS?$AAc?$AAh?$AAe?$AAd?$AAu?$AAl?$AAe?$AAT?$AAD?$AA?5?$AA?$CI?$AAt?$AAh?$AAi?$AAs?$AA?$DN?$AA0?$AAx@ 1000f4a0     usbh_ehcdmdd_common_topaz_v1:trans.obj
 0001:0000e558       ??_C@_1IG@HAOLAFMA@?$AAC?$AAI?$AAT?$AAr?$AAa?$AAn?$AAs?$AAf?$AAe?$AAr?$AA?3?$AA?3?$AAD?$AAo?$AAn?$AAe?$AAT?$AAr?$AAa?$AAn?$AAs?$AAf?$AAe?$AAr?$AA?5?$AA?$CI?$AAt?$AAh?$AAi?$AAs?$AA?$DN?$AA0@ 1000f558     usbh_ehcdmdd_common_topaz_v1:trans.obj
 0001:0000e5e0       ??_C@_1CC@KMLAOLOE@?$AAC?$AAN?$AAe?$AAx?$AAt?$AAL?$AAi?$AAn?$AAk?$AAP?$AAo?$AAi?$AAn?$AAt?$AAe?$AAr?$AA?$AA@ 1000f5e0     usbh_ehcdmdd_common_topaz_v1:ctd.obj
 0001:0000e608       ??_C@_1LI@JPOPDPIO@?$AAC?$AA?3?$AA?2?$AAW?$AAI?$AAN?$AAC?$AAE?$AAR?$AAO?$AAO?$AAT?$AAS?$AA?2?$AAT?$AAo?$AAp?$AAa?$AAz?$AA?2?$AAW?$AAI?$AAN?$AAC?$AAE?$AA6?$AA0?$AA0?$AA?2?$AAP?$AAL?$AAA@ 1000f608     usbh_ehcdmdd_common_topaz_v1:ctd.obj
 0001:0000e6c0       ??_C@_1LA@NELPONEA@?$AAc?$AA?3?$AA?2?$AAw?$AAi?$AAn?$AAc?$AAe?$AAr?$AAo?$AAo?$AAt?$AAs?$AA?2?$AAt?$AAo?$AAp?$AAa?$AAz?$AA?2?$AAw?$AAi?$AAn?$AAc?$AAe?$AA6?$AA0?$AA0?$AA?2?$AAp?$AAl?$AAa@ 1000f6c0     usbh_ehcdmdd_common_topaz_v1:ctd.obj
 0001:0000e770       ??_C@_1EO@OFFJOBOE@?$AAE?$AAH?$AAC?$AAD?$AA?3?$AA?5?$AAi?$AAo?$AAP?$AAo?$AAr?$AAt?$AAB?$AAa?$AAs?$AAe?$AA?5?$AA0?$AAx?$AA?$CF?$AAX?$AA?0?$AA?5?$AAp?$AAo?$AAr?$AAt?$AAB?$AAa?$AAs?$AAe?$AA?5@ 1000f770     usbh_ehcdpdd_common_topaz_v1:system.obj
 0001:0000e7c0       ??_C@_1FE@IJIAHJGH@?$AAE?$AAH?$AAC?$AAD?$AA?3?$AA?5?$AAi?$AAo?$AAP?$AAh?$AAy?$AAs?$AAi?$AAc?$AAa?$AAl?$AAB?$AAa?$AAs?$AAe?$AA?5?$AA0?$AAx?$AA?$CF?$AAX?$AA?0?$AA?5?$AAI?$AAo?$AAS?$AAp?$AAa@ 1000f7c0     usbh_ehcdpdd_common_topaz_v1:system.obj
 0001:0000e818       ??_C@_1EK@IDLONLLI@?$AAE?$AAH?$AAC?$AAD?$AA?3?$AA?5?$AAF?$AAa?$AAi?$AAl?$AAe?$AAd?$AA?5?$AAT?$AAr?$AAa?$AAn?$AAs?$AAB?$AAu?$AAs?$AAA?$AAd?$AAd?$AAr?$AAT?$AAo?$AAV?$AAi?$AAr?$AAt?$AAu@ 1000f818     usbh_ehcdpdd_common_topaz_v1:system.obj
 0001:0000e864       ??_C@_1CC@IGBPDHCE@?$AAI?$AAn?$AAi?$AAt?$AAi?$AAa?$AAl?$AAi?$AAz?$AAe?$AAE?$AAH?$AAC?$AAI?$AA?$AN?$AA?6?$AA?$AA@ 1000f864     usbh_ehcdpdd_common_topaz_v1:system.obj
 0001:0000e888       ??_C@_1BM@KKKMKIHE@?$AAH?$AAc?$AAd?$AAC?$AAa?$AAp?$AAa?$AAb?$AAi?$AAl?$AAi?$AAt?$AAy?$AA?$AA@ 1000f888     usbh_ehcdpdd_common_topaz_v1:system.obj
 0001:0000e8a4       ??_C@_1DE@LILAJAFN@?$AAU?$AAS?$AAB?$AAH?$AAo?$AAs?$AAt?$AA?5?$AAO?$AAT?$AAG?$AAS?$AAu?$AAp?$AAp?$AAo?$AAr?$AAt?$AA?5?$AA?$DN?$AA?5?$AA?$CF?$AAd?$AA?$AN?$AA?6?$AA?$AA@ 1000f8a4     usbh_ehcdpdd_common_topaz_v1:system.obj
 0001:0000e8d8       ??_C@_1BAK@HPDDFLLI@?$AAE?$AAH?$AAC?$AAD?$AA?3?$AA?5?$AAR?$AAe?$AAa?$AAd?$AA?5?$AAc?$AAo?$AAn?$AAf?$AAi?$AAg?$AA?5?$AAf?$AAr?$AAo?$AAm?$AA?5?$AAr?$AAe?$AAg?$AAi?$AAs?$AAt?$AAr?$AAy?$AA?3@ 1000f8d8     usbh_ehcdpdd_common_topaz_v1:system.obj
 0001:0000e9e4       ??_C@_15LIBIHNCL@?$AAN?$AAO?$AA?$AA@ 1000f9e4     usbh_ehcdpdd_common_topaz_v1:system.obj
 0001:0000e9ec       ??_C@_17FGJJPDOI@?$AAY?$AAE?$AAS?$AA?$AA@ 1000f9ec     usbh_ehcdpdd_common_topaz_v1:system.obj
 0001:0000e9f4       ??_C@_1CI@NIAEKGLK@?$AAO?$AAT?$AAG?$AAG?$AAr?$AAo?$AAu?$AAp?$AAN?$AAa?$AAm?$AAe?$AA?5?$AA?$DN?$AA?5?$AA?$CF?$AAs?$AA?$AN?$AA?6?$AA?$AA@ 1000f9f4     usbh_ehcdpdd_common_topaz_v1:system.obj
 0001:0000ea1c       ??_C@_1BC@GDFGLIEL@?$AAO?$AAT?$AAG?$AAG?$AAr?$AAo?$AAu?$AAp?$AA?$AA@ 1000fa1c     usbh_ehcdpdd_common_topaz_v1:system.obj
 0001:0000ea30       ??_C@_1BG@HHFAGDDC@?$AAO?$AAT?$AAG?$AAS?$AAu?$AAp?$AAp?$AAo?$AAr?$AAt?$AA?$AA@ 1000fa30     usbh_ehcdpdd_common_topaz_v1:system.obj
 0001:0000ea48       ??_C@_1IM@JNEHECOI@?$AAI?$AAn?$AAi?$AAt?$AAi?$AAa?$AAl?$AAi?$AAz?$AAe?$AAE?$AAH?$AAC?$AAI?$AA?3?$AAD?$AAD?$AAK?$AAR?$AAe?$AAg?$AA_?$AAG?$AAe?$AAt?$AAW?$AAi?$AAn?$AAd?$AAo?$AAw?$AAI@ 1000fa48     usbh_ehcdpdd_common_topaz_v1:system.obj
 0001:0000ead8       ??_C@_1HG@IFCIGIJA@?$AAI?$AAn?$AAi?$AAt?$AAi?$AAa?$AAl?$AAi?$AAz?$AAe?$AAE?$AAH?$AAC?$AAI?$AA?3?$AAG?$AAe?$AAt?$AAR?$AAe?$AAg?$AAi?$AAs?$AAt?$AAr?$AAy?$AAC?$AAo?$AAn?$AAf?$AAi?$AAg@ 1000fad8     usbh_ehcdpdd_common_topaz_v1:system.obj
 0001:0000eb50       ??_C@_1CC@NPEFILDH@?$AAP?$AAh?$AAy?$AAs?$AAi?$AAc?$AAa?$AAl?$AAP?$AAa?$AAg?$AAe?$AAS?$AAi?$AAz?$AAe?$AA?$AA@ 1000fb50     usbh_ehcdpdd_common_topaz_v1:system.obj
 0001:0000eb78       ??_C@_1GK@FOJFGKHH@?$AA?$CB?$AAE?$AAH?$AAC?$AAD?$AA?3?$AAG?$AAe?$AAt?$AAR?$AAe?$AAg?$AAi?$AAs?$AAt?$AAr?$AAy?$AAC?$AAo?$AAn?$AAf?$AAi?$AAg?$AA?5?$AAR?$AAe?$AAg?$AAO?$AAp?$AAe?$AAn?$AAK@ 1000fb78     usbh_ehcdpdd_common_topaz_v1:system.obj
 0001:0000ec0c       FslUfnIsUSBKitlEnable      1000fc0c f   i_hwinit.obj
 0001:0000eca0       SetPHYPowerMgmt            1000fca0 f   i_hwinit.obj
 0001:0000ecb4       gfnGetOTGGroup             1000fcb4 f   i_hwinit.obj
 0001:0000ecd0       gfnIsOTGSupport            1000fcd0 f   i_hwinit.obj
 0001:0000ecf0       InitializeTransceiver      1000fcf0 f   i_hwinit.obj
 0001:0000f8fc       BSPUsbhCheckConfigPower    100108fc f   i_hwinit.obj
 0001:0000f94c       BSPUsbSetWakeUp            1001094c f   i_hwinit.obj
 0001:0000fbc0       BSPUsbCheckWakeUp          10010bc0 f   i_hwinit.obj
 0001:0000fcd4       BSPUsbHostLowPowerModeEnable 10010cd4 f   i_hwinit.obj
 0001:0000fcec       BSPUSBHostVbusControl      10010cec f   i_hwinit.obj
 0001:0000fda0       BSPNeedCloseVBus           10010da0 f   i_hwinit.obj
 0001:0000fdb8       IsLowPowerSameAsSuspend    10010db8 f   i_hwinit.obj
 0001:0000fdfc       GetUSBPortType             10010dfc f   i_hwinit.obj
 0001:0000fe1c       BSPGetUSBControllerType    10010e1c f   i_hwinit.obj
 0001:0000fe34       USBClockInit               10010e34 f   i_usbclock.obj
 0001:0000fe60       USBClockGatingLock         10010e60 f   i_usbclock.obj
 0001:0000febc       USBClockGatingUnlock       10010ebc f   i_usbclock.obj
 0001:0000fed8       BSPUSBClockCreateFileMapping 10010ed8 f   i_usbclock.obj
 0001:0001010c       BSPUSBClockDeleteFileMapping 1001110c f   i_usbclock.obj
 0001:00010170       BSPUSBClockSwitch          10011170 f   i_usbclock.obj
 0001:000104a4       PowerDownSchemeExist       100114a4 f   i_usbutils.obj
 0001:00010548       BSPUsbXvrEnableVBUSIntr    10011548 f   i_usbutils.obj
 0001:000105c8       BSPUsbXvrEnableIDIntr      100115c8 f   i_usbutils.obj
 0001:00010648       BSPUsbEnableLowPowerIntr   10011648 f   i_usbutils.obj
 0001:00010698       BSPUsbSetBusConfig         10011698 f   i_usbutils.obj
 0001:000106dc       BSPUSBInterruptControl     100116dc f   i_usbutils.obj
 0001:00010748       BSPPhyShowDevDiscon        10011748 f   i_usbutils.obj
 0001:00010760       BSPUsbPhyStartUp           10011760 f   i_usbutils.obj
 0001:00010764       BSPUsbSetCurrentLimitation 10011764 f   i_usbutils.obj
 0001:00010778       BSPUsbPhyRegDump           10011778 f   i_usbutils.obj
 0001:0001077c       BSPUSBSwitchModulePower    1001177c f   i_usbutils.obj
 0001:00010790       BSPHostDisconDetect        10011790 f   i_usbutils.obj
 0001:000107a4       DllMain                    100117a4 f   usbh_usb2com_common_topaz_v1:hcddrv.obj
 0001:00010868       HcdGetFrameNumber          10011868 f   usbh_usb2com_common_topaz_v1:hcddrv.obj
 0001:000108bc       HcdGetFrameLength          100118bc f   usbh_usb2com_common_topaz_v1:hcddrv.obj
 0001:00010910       HcdSetFrameLength          10011910 f   usbh_usb2com_common_topaz_v1:hcddrv.obj
 0001:00010968       HcdStopAdjustingFrame      10011968 f   usbh_usb2com_common_topaz_v1:hcddrv.obj
 0001:000109b8       HcdOpenPipe                100119b8 f   usbh_usb2com_common_topaz_v1:hcddrv.obj
 0001:00010a00       HcdClosePipe               10011a00 f   usbh_usb2com_common_topaz_v1:hcddrv.obj
 0001:00010a44       HcdResetPipe               10011a44 f   usbh_usb2com_common_topaz_v1:hcddrv.obj
 0001:00010a88       HcdIsPipeHalted            10011a88 f   usbh_usb2com_common_topaz_v1:hcddrv.obj
 0001:00010ad0       HcdIssueTransfer           10011ad0 f   usbh_usb2com_common_topaz_v1:hcddrv.obj
 0001:00010b90       HcdAbortTransfer           10011b90 f   usbh_usb2com_common_topaz_v1:hcddrv.obj
 0001:00010be8       HcdDisableDevice           10011be8 f   usbh_usb2com_common_topaz_v1:hcddrv.obj
 0001:00010c40       HcdSuspendResume           10011c40 f   usbh_usb2com_common_topaz_v1:hcddrv.obj
 0001:00010c98       HcdMdd_CreateMemoryObject  10011c98 f   usbh_usb2com_common_topaz_v1:hcddrv.obj
 0001:00010dd4       HcdMdd_CreateHcdObject_Customized 10011dd4 f   usbh_usb2com_common_topaz_v1:hcddrv.obj
 0001:00010ebc       HcdMdd_DestroyHcdObject    10011ebc f   usbh_usb2com_common_topaz_v1:hcddrv.obj
 0001:00010f3c       HcdMdd_DestroyMemoryObject 10011f3c f   usbh_usb2com_common_topaz_v1:hcddrv.obj
 0001:00010fac       HcdMdd_PowerUp             10011fac f   usbh_usb2com_common_topaz_v1:hcddrv.obj
 0001:00011030       HcdMdd_PowerDown           10012030 f   usbh_usb2com_common_topaz_v1:hcddrv.obj
 0001:00011080       HcdMdd_SetCapability       10012080 f   usbh_usb2com_common_topaz_v1:hcddrv.obj
 0001:000110d4       HcdMdd_SetSubHubTestMode   100120d4 f   usbh_usb2com_common_topaz_v1:hcddrv.obj
 0001:0001118c       HCD_Init                   1001218c f   usbh_usb2com_common_topaz_v1:hcddrv.obj
 0001:0001143c       HCD_PowerUp                1001243c f   usbh_usb2com_common_topaz_v1:hcddrv.obj
 0001:00011458       HCD_PowerDown              10012458 f   usbh_usb2com_common_topaz_v1:hcddrv.obj
 0001:00011474       HCD_Deinit                 10012474 f   usbh_usb2com_common_topaz_v1:hcddrv.obj
 0001:000114dc       HCD_Open                   100124dc f   usbh_usb2com_common_topaz_v1:hcddrv.obj
 0001:00011518       HCD_Close                  10012518 f   usbh_usb2com_common_topaz_v1:hcddrv.obj
 0001:0001154c       HCD_Read                   1001254c f   usbh_usb2com_common_topaz_v1:hcddrv.obj
 0001:00011588       HCD_Write                  10012588 f   usbh_usb2com_common_topaz_v1:hcddrv.obj
 0001:000115c4       HCD_Seek                   100125c4 f   usbh_usb2com_common_topaz_v1:hcddrv.obj
 0001:00011600       HCD_IOControl              10012600 f   usbh_usb2com_common_topaz_v1:hcddrv.obj
 0001:00011658       ?InittedOK@CPhysMem@@QAAHXZ 10012658 f i usbh_usb2com_common_topaz_v1:hcddrv.obj
 0001:00011688       ??_GCPhysMem@@QAAPAXI@Z    10012688 f i usbh_usb2com_common_topaz_v1:hcddrv.obj
 0001:000116cc       ?GetRootHub@CHcd@@QAAPAVCRootHub@@XZ 100126cc f i usbh_usb2com_common_topaz_v1:hcddrv.obj
 0001:000116fc       ??0CHcd@@QAA@XZ            100126fc f   usbh_usb2com_common_topaz_v1:hcd.obj
 0001:00011760       ??1CHcd@@UAA@XZ            10012760 f   usbh_usb2com_common_topaz_v1:hcd.obj
 0001:00011870       ?SetRootHub@CHcd@@QAAPAVCRootHub@@PAV2@@Z 10012870 f   usbh_usb2com_common_topaz_v1:hcd.obj
 0001:000118d0       ?OpenPipe@CHcd@@QAAHIPBU_USB_ENDPOINT_DESCRIPTOR@@PAI@Z 100128d0 f   usbh_usb2com_common_topaz_v1:hcd.obj
 0001:00011a34       ?ClosePipe@CHcd@@QAAHII@Z  10012a34 f   usbh_usb2com_common_topaz_v1:hcd.obj
 0001:00011b60       ?IssueTransfer@CHcd@@QAAHIIP6AKPAX@Z0KPBXKKPBKK0K2PAK4PAH44@Z 10012b60 f   usbh_usb2com_common_topaz_v1:hcd.obj
 0001:00011d3c       ?AbortTransfer@CHcd@@QAAHIIP6AKPAX@Z0PBX@Z 10012d3c f   usbh_usb2com_common_topaz_v1:hcd.obj
 0001:00011ea0       ?IsPipeHalted@CHcd@@QAAHIIPAH@Z 10012ea0 f   usbh_usb2com_common_topaz_v1:hcd.obj
 0001:00012008       ?ResetPipe@CHcd@@QAAHII@Z  10013008 f   usbh_usb2com_common_topaz_v1:hcd.obj
 0001:00012134       ?DisableDevice@CHcd@@UAAHIH@Z 10013134 f   usbh_usb2com_common_topaz_v1:hcd.obj
 0001:0001225c       ?SuspendResume@CHcd@@UAAHIH@Z 1001325c f   usbh_usb2com_common_topaz_v1:hcd.obj
 0001:00012388       ??0LockObject@@QAA@XZ      10013388 f i usbh_usb2com_common_topaz_v1:hcd.obj
 0001:000123b8       ?WaitForPortStatusChange@CHcd@@UAAHPAX@Z 100133b8 f i usbh_usb2com_common_topaz_v1:hcd.obj
 0001:000123e0       ?SuspendHC@CHcd@@UAAHXZ    100133e0 f i usbh_usb2com_common_topaz_v1:hcd.obj
 0001:00012408       ?ResumeNotification@CHcd@@MAAHXZ 10013408 f i usbh_usb2com_common_topaz_v1:hcd.obj
 0001:000124a8       ?Lock@LockObject@@QAAXXZ   100134a8 f i usbh_usb2com_common_topaz_v1:hcd.obj
 0001:000124c4       ?Unlock@LockObject@@QAAXXZ 100134c4 f i usbh_usb2com_common_topaz_v1:hcd.obj
 0001:000124e0       ??_ECHcd@@UAAPAXI@Z        100134e0 f i usbh_usb2com_common_topaz_v1:hcd.obj
 0001:000124e0       ??_GCHcd@@UAAPAXI@Z        100134e0 f i usbh_usb2com_common_topaz_v1:hcd.obj
 0001:00012524       ??1LockObject@@QAA@XZ      10013524 f i usbh_usb2com_common_topaz_v1:hcd.obj
 0001:00012540       ??0CPhysMem@@QAA@KKPAE0@Z  10013540 f   usbh_usb2com_common_topaz_v1:cphysmem.obj
 0001:00012b88       ?ReInit@CPhysMem@@QAAXXZ   10013b88 f   usbh_usb2com_common_topaz_v1:cphysmem.obj
 0001:00013094       ?ValidateHeaps@CPhysMem@@AAAHH@Z 10014094 f   usbh_usb2com_common_topaz_v1:cphysmem.obj
 0001:00013a54       ?CreateNewNode@CPhysMem@@AAAPAUtMEMLIST@@KKK@Z 10014a54 f   usbh_usb2com_common_topaz_v1:cphysmem.obj
 0001:00013c64       ?DeleteNode@CPhysMem@@AAAHPAUtMEMLIST@@@Z 10014c64 f   usbh_usb2com_common_topaz_v1:cphysmem.obj
 0001:00013cfc       ?FindFreeBlock@CPhysMem@@AAAPAUtMEMLIST@@KH@Z 10014cfc f   usbh_usb2com_common_topaz_v1:cphysmem.obj
 0001:00013e64       ?AddNodeToFreeList@CPhysMem@@AAAHPAUtMEMLIST@@H@Z 10014e64 f   usbh_usb2com_common_topaz_v1:cphysmem.obj
 0001:000141c4       ??1CPhysMem@@QAA@XZ        100151c4 f   usbh_usb2com_common_topaz_v1:cphysmem.obj
 0001:00014268       ?FreeList@CPhysMem@@AAAHPAPAUtMEMLIST@@@Z 10015268 f   usbh_usb2com_common_topaz_v1:cphysmem.obj
 0001:0001434c       ?AllocateSpecialMemory@CPhysMem@@QAAHKQAPAE@Z 1001534c f   usbh_usb2com_common_topaz_v1:cphysmem.obj
 0001:00014518       ?FreeSpecialMemory@CPhysMem@@QAAXQAE@Z 10015518 f   usbh_usb2com_common_topaz_v1:cphysmem.obj
 0001:000145d8       ?AllocateMemory@CPhysMem@@QAAHPBGKQAPAEKPAH@Z 100155d8 f   usbh_usb2com_common_topaz_v1:cphysmem.obj
 0001:00014db0       ?FreeMemory@CPhysMem@@QAAXQAEKK@Z 10015db0 f   usbh_usb2com_common_topaz_v1:cphysmem.obj
 0001:000152b0       ?ReleaseBlockedCalls@CPhysMem@@QAAHXZ 100162b0 f   usbh_usb2com_common_topaz_v1:cphysmem.obj
 0001:000152fc       ?InitializeListHead@@YAXPAUtMEMLIST@@@Z 100162fc f i usbh_usb2com_common_topaz_v1:cphysmem.obj
 0001:00015330       ?FirstNode@@YAPAUtMEMLIST@@PAU1@@Z 10016330 f i usbh_usb2com_common_topaz_v1:cphysmem.obj
 0001:00015360       ?InsertNodeBefore@@YAXPAUtMEMLIST@@0@Z 10016360 f i usbh_usb2com_common_topaz_v1:cphysmem.obj
 0001:000153c4       ?PaToVa@CPhysMem@@QAAPAEK@Z 100163c4 f i usbh_usb2com_common_topaz_v1:cphysmem.obj
 0001:000154b4       ?RemoveNode@@YAXPAUtMEMLIST@@@Z 100164b4 f i usbh_usb2com_common_topaz_v1:cphysmem.obj
 0001:00015528       ?VaToPa@CPhysMem@@QAAKPAE@Z 10016528 f i usbh_usb2com_common_topaz_v1:cphysmem.obj
 0001:00015610       PulseEvent                 10016610 f i usbh_usb2com_common_topaz_v1:cphysmem.obj
 0001:00015648       ??0CDeviceGlobal@@QAA@XZ   10016648 f   usbh_usb2com_common_topaz_v1:cdevice.obj
 0001:00015750       ??1CDeviceGlobal@@UAA@XZ   10016750 f   usbh_usb2com_common_topaz_v1:cdevice.obj
 0001:000157a0       ?Initialize@CDeviceGlobal@@QAAHPAX@Z 100167a0 f   usbh_usb2com_common_topaz_v1:cdevice.obj
 0001:00015bc0       ?DeInitialize@CDeviceGlobal@@UAAXXZ 10016bc0 f   usbh_usb2com_common_topaz_v1:cdevice.obj
 0001:00015d94       ?ReserveAddress@CDeviceGlobal@@QAAHAAE@Z 10016d94 f   usbh_usb2com_common_topaz_v1:cdevice.obj
 0001:00015fa8       ?FreeAddress@CDeviceGlobal@@QAAXE@Z 10016fa8 f   usbh_usb2com_common_topaz_v1:cdevice.obj
 0001:00016160       ?TransferDoneCallbackSetEvent@CDevice@@KAKPAX@Z 10017160 f   usbh_usb2com_common_topaz_v1:cdevice.obj
 0001:000161d8       ??0CDevice@@QAA@EABU_USB_DEVICE_INFO@@HHEQAVCDeviceGlobal@@QAVCHub@@E@Z 100171d8 f   usbh_usb2com_common_topaz_v1:cdevice.obj
 0001:00016400       ??1CDevice@@UAA@XZ         10017400 f   usbh_usb2com_common_topaz_v1:cdevice.obj
 0001:00016778       ?GetUSB2TT@CDevice@@UAAPAVCHub@@PAE0@Z 10017778 f   usbh_usb2com_common_topaz_v1:cdevice.obj
 0001:00016868       ?CreateUsbConfigurationStructure@CDevice@@QBAHAAU_NON_CONST_USB_CONFIGURATION@@QAEI@Z 10017868 f   usbh_usb2com_common_topaz_v1:cdevice.obj
 0001:00017464       ?DeleteUsbConfigurationStructure@CDevice@@QBAXAAU_NON_CONST_USB_CONFIGURATION@@@Z 10018464 f   usbh_usb2com_common_topaz_v1:cdevice.obj
 0001:00017778       ?AllocatePipeArray@CDevice@@IAAHXZ 10018778 f   usbh_usb2com_common_topaz_v1:cdevice.obj
 0001:00017c94       ?DumpDeviceDescriptor@CDevice@@QBAXQAU_USB_DEVICE_DESCRIPTOR@@@Z 10018c94 f   usbh_usb2com_common_topaz_v1:cdevice.obj
 0001:00018124       ?DumpConfigDescriptor@CDevice@@QBAXQAU_USB_CONFIGURATION_DESCRIPTOR@@@Z 10019124 f   usbh_usb2com_common_topaz_v1:cdevice.obj
 0001:0001850c       ?DumpInterfaceDescriptor@CDevice@@QBAXQAU_USB_INTERFACE_DESCRIPTOR@@@Z 1001950c f   usbh_usb2com_common_topaz_v1:cdevice.obj
 0001:00018808       ?DumpEndpointDescriptor@CDevice@@QBAXQAU_USB_ENDPOINT_DESCRIPTOR@@@Z 10019808 f   usbh_usb2com_common_topaz_v1:cdevice.obj
 0001:00018ba0       ?DumpExtendedBytes@CDevice@@QBAXQAEK@Z 10019ba0 f   usbh_usb2com_common_topaz_v1:cdevice.obj
 0001:00018d6c       ??0CHub@@QAA@EABU_USB_DEVICE_INFO@@HHEABU_USB_HUB_DESCRIPTOR@@QAVCHcd@@QAV0@E@Z 10019d6c f   usbh_usb2com_common_topaz_v1:cdevice.obj
 0001:00019110       ??1CHub@@UAA@XZ            1001a110 f   usbh_usb2com_common_topaz_v1:cdevice.obj
 0001:00019444       ?HubStatusChangeThreadStub@CHub@@KAKPAX@Z 1001a444 f   usbh_usb2com_common_topaz_v1:cdevice.obj
 0001:00019478       ?HubStatusChangeThread@CHub@@AAAKXZ 1001a478 f   usbh_usb2com_common_topaz_v1:cdevice.obj
 0001:0001a5b0       ?SubHubTestModeEnable@CHub@@UAAHGG@Z 1001b5b0 f   usbh_usb2com_common_topaz_v1:cdevice.obj
 0001:0001a5fc       ?DisableDevice@CDevice@@UAA?AW4HCD_REQUEST_STATUS@@IH@Z 1001b5fc f   usbh_usb2com_common_topaz_v1:cdevice.obj
 0001:0001a700       ?SuspendResume@CDevice@@UAA?AW4HCD_REQUEST_STATUS@@IH@Z 1001b700 f   usbh_usb2com_common_topaz_v1:cdevice.obj
 0001:0001a8c4       ?DumpHubDescriptor@CHub@@SAXQAU_USB_HUB_DESCRIPTOR@@@Z 1001b8c4 f   usbh_usb2com_common_topaz_v1:cdevice.obj
 0001:0001ae88       ?MessageBoxSpecial@CHub@@QAAHPAUHWND__@@PBGI@Z 1001be88 f   usbh_usb2com_common_topaz_v1:cdevice.obj
 0001:0001b088       ?AttachDevice@CHub@@IAAXEHH@Z 1001c088 f   usbh_usb2com_common_topaz_v1:cdevice.obj
 0001:0001dc0c       ?GetDescriptor@CHub@@IAAHQAVCPipeAbs@@EEEGPAX@Z 1001ec0c f   usbh_usb2com_common_topaz_v1:cdevice.obj
 0001:0001e1ac       ?DetachDownstreamDeviceThreadStub@CHub@@KAKPAX@Z 1001f1ac f   usbh_usb2com_common_topaz_v1:cdevice.obj
 0001:0001e1e0       ?DetachDownstreamDeviceThread@CHub@@IAAKXZ 1001f1e0 f   usbh_usb2com_common_topaz_v1:cdevice.obj
 0001:0001e35c       ?DetachDevice@CHub@@IAAXE@Z 1001f35c f   usbh_usb2com_common_topaz_v1:cdevice.obj
 0001:0001e9e8       ?AllocateDeviceArray@CHub@@IAAHXZ 1001f9e8 f   usbh_usb2com_common_topaz_v1:cdevice.obj
 0001:0001ee7c       ?HandleDetach@CHub@@UAAXXZ 1001fe7c f   usbh_usb2com_common_topaz_v1:cdevice.obj
 0001:0001f598       ?OpenPipe@CHub@@UAA?AW4HCD_REQUEST_STATUS@@IQBU_USB_ENDPOINT_DESCRIPTOR@@QAI@Z 10020598 f   usbh_usb2com_common_topaz_v1:cdevice.obj
 0001:0001f854       ?ClosePipe@CHub@@UAA?AW4HCD_REQUEST_STATUS@@II@Z 10020854 f   usbh_usb2com_common_topaz_v1:cdevice.obj
 0001:0001fb14       ?IssueTransfer@CHub@@UAA?AW4HCD_REQUEST_STATUS@@IIQ6AKPAX@ZQAXKQBXKKQBKK2K3QAK5QAH55@Z 10020b14 f   usbh_usb2com_common_topaz_v1:cdevice.obj
 0001:0001fe58       ?AbortTransfer@CHub@@UAA?AW4HCD_REQUEST_STATUS@@IIQ6AKPAX@ZQAXQBX@Z 10020e58 f   usbh_usb2com_common_topaz_v1:cdevice.obj
 0001:00020134       ?IsPipeHalted@CHub@@UAA?AW4HCD_REQUEST_STATUS@@IIQAH@Z 10021134 f   usbh_usb2com_common_topaz_v1:cdevice.obj
 0001:00020400       ?ResetPipe@CHub@@UAA?AW4HCD_REQUEST_STATUS@@II@Z 10021400 f   usbh_usb2com_common_topaz_v1:cdevice.obj
 0001:00020708       ?DisableDevice@CHub@@UAA?AW4HCD_REQUEST_STATUS@@IH@Z 10021708 f   usbh_usb2com_common_topaz_v1:cdevice.obj
 0001:000208a8       ?SuspendResume@CHub@@UAA?AW4HCD_REQUEST_STATUS@@IH@Z 100218a8 f   usbh_usb2com_common_topaz_v1:cdevice.obj
 0001:00020b78       ?DisableOffStreamDevice@CHub@@UAAHIH@Z 10021b78 f   usbh_usb2com_common_topaz_v1:cdevice.obj
 0001:00020e48       ?SuspendResumeOffStreamDevice@CHub@@UAAHIH@Z 10021e48 f   usbh_usb2com_common_topaz_v1:cdevice.obj
 0001:000210f0       ??0CRootHub@@QAA@ABU_USB_DEVICE_INFO@@HHABU_USB_HUB_DESCRIPTOR@@QAVCHcd@@@Z 100220f0 f   usbh_usb2com_common_topaz_v1:cdevice.obj
 0001:000211f4       ??1CRootHub@@UAA@XZ        100221f4 f   usbh_usb2com_common_topaz_v1:cdevice.obj
 0001:000212ac       ?EnterOperationalState@CRootHub@@UAAHQAVCPipeAbs@@@Z 100222ac f   usbh_usb2com_common_topaz_v1:cdevice.obj
 0001:000215d4       ?PowerAllHubPorts@CRootHub@@EAAHXZ 100225d4 f   usbh_usb2com_common_topaz_v1:cdevice.obj
 0001:00021680       ?WaitForPortStatusChange@CRootHub@@EAAHAAEAAU_USB_HUB_AND_PORT_STATUS@@PAK@Z 10022680 f   usbh_usb2com_common_topaz_v1:cdevice.obj
 0001:00021bf8       ?GetStatus@CRootHub@@EAAHEAAU_USB_HUB_AND_PORT_STATUS@@PAK@Z 10022bf8 f   usbh_usb2com_common_topaz_v1:cdevice.obj
 0001:00021d50       ?ResetAndEnablePort@CRootHub@@EAAHE@Z 10022d50 f   usbh_usb2com_common_topaz_v1:cdevice.obj
 0001:00021eac       ?DisablePort@CRootHub@@EAAXE@Z 10022eac f   usbh_usb2com_common_topaz_v1:cdevice.obj
 0001:00021fec       ?SetOrClearFeature@CRootHub@@EAAHGEG@Z 10022fec f   usbh_usb2com_common_topaz_v1:cdevice.obj
 0001:00022324       ?SetOrClearRemoteWakup@CRootHub@@EAAHH@Z 10023324 f   usbh_usb2com_common_topaz_v1:cdevice.obj
 0001:0002234c       ?SubHubTestModeEnable@CRootHub@@UAAHGG@Z 1002334c f   usbh_usb2com_common_topaz_v1:cdevice.obj
 0001:00022504       ??0CExternalHub@@QAA@EABU_USB_DEVICE_INFO@@HHEABU_USB_HUB_DESCRIPTOR@@QAVCHcd@@QAVCHub@@E@Z 10023504 f   usbh_usb2com_common_topaz_v1:cdevice.obj
 0001:00022608       ??1CExternalHub@@UAA@XZ    10023608 f   usbh_usb2com_common_topaz_v1:cdevice.obj
 0001:000226c0       ?EnterOperationalState@CExternalHub@@UAAHQAVCPipeAbs@@@Z 100236c0 f   usbh_usb2com_common_topaz_v1:cdevice.obj
 0001:00022cd4       ?SubHubTestModeEnable@CExternalHub@@UAAHGG@Z 10023cd4 f   usbh_usb2com_common_topaz_v1:cdevice.obj
 0001:00023130       ?PowerAllHubPorts@CExternalHub@@EAAHXZ 10024130 f   usbh_usb2com_common_topaz_v1:cdevice.obj
 0001:000233e8       ?GetStatusChangeBitmap@CExternalHub@@AAAHAAK@Z 100243e8 f   usbh_usb2com_common_topaz_v1:cdevice.obj
 0001:000238b8       ?WaitForPortStatusChange@CExternalHub@@EAAHAAEAAU_USB_HUB_AND_PORT_STATUS@@PAK@Z 100248b8 f   usbh_usb2com_common_topaz_v1:cdevice.obj
 0001:00023bf4       ?GetStatus@CExternalHub@@EAAHEAAU_USB_HUB_AND_PORT_STATUS@@PAK@Z 10024bf4 f   usbh_usb2com_common_topaz_v1:cdevice.obj
 0001:00023ff4       ?ResetAndEnablePort@CExternalHub@@EAAHE@Z 10024ff4 f   usbh_usb2com_common_topaz_v1:cdevice.obj
 0001:00024318       ?DisablePort@CExternalHub@@EAAXE@Z 10025318 f   usbh_usb2com_common_topaz_v1:cdevice.obj
 0001:0002440c       ?SetOrClearFeature@CExternalHub@@EAAHGEG@Z 1002540c f   usbh_usb2com_common_topaz_v1:cdevice.obj
 0001:000249e4       ?SetOrClearRemoteWakup@CExternalHub@@EAAHH@Z 100259e4 f   usbh_usb2com_common_topaz_v1:cdevice.obj
 0001:00024cf8       ??0CFunction@@QAA@EABU_USB_DEVICE_INFO@@HHEQAVCHcd@@QAVCHub@@E@Z 10025cf8 f   usbh_usb2com_common_topaz_v1:cdevice.obj
 0001:00024e44       ??1CFunction@@UAA@XZ       10025e44 f   usbh_usb2com_common_topaz_v1:cdevice.obj
 0001:00024fac       ?EnterOperationalState@CFunction@@UAAHQAVCPipeAbs@@@Z 10025fac f   usbh_usb2com_common_topaz_v1:cdevice.obj
 0001:0002543c       ?OpenPipe@CFunction@@UAA?AW4HCD_REQUEST_STATUS@@IQBU_USB_ENDPOINT_DESCRIPTOR@@QAI@Z 1002643c f   usbh_usb2com_common_topaz_v1:cdevice.obj
 0001:00025ddc       ?ClosePipe@CFunction@@UAA?AW4HCD_REQUEST_STATUS@@II@Z 10026ddc f   usbh_usb2com_common_topaz_v1:cdevice.obj
 0001:000260b0       ?IssueTransfer@CFunction@@UAA?AW4HCD_REQUEST_STATUS@@IIQ6AKPAX@ZQAXKQBXKKQBKK2K3QAK5QAH55@Z 100270b0 f   usbh_usb2com_common_topaz_v1:cdevice.obj
 0001:0002633c       ?AbortTransfer@CFunction@@UAA?AW4HCD_REQUEST_STATUS@@IIQ6AKPAX@ZQAXQBX@Z 1002733c f   usbh_usb2com_common_topaz_v1:cdevice.obj
 0001:00026508       ?IsPipeHalted@CFunction@@UAA?AW4HCD_REQUEST_STATUS@@IIQAH@Z 10027508 f   usbh_usb2com_common_topaz_v1:cdevice.obj
 0001:00026720       ?ResetPipe@CFunction@@UAA?AW4HCD_REQUEST_STATUS@@II@Z 10027720 f   usbh_usb2com_common_topaz_v1:cdevice.obj
 0001:000269a0       ?HandleDetach@CFunction@@EAAXXZ 100279a0 f   usbh_usb2com_common_topaz_v1:cdevice.obj
 0001:00026ed8       ?SetOrClearFeature@CFunction@@AAAHEGEG@Z 10027ed8 f   usbh_usb2com_common_topaz_v1:cdevice.obj
 0001:00027468       ??_GCDeviceGlobal@@UAAPAXI@Z 10028468 f i usbh_usb2com_common_topaz_v1:cdevice.obj
 0001:00027468       ??_ECDeviceGlobal@@UAAPAXI@Z 10028468 f i usbh_usb2com_common_topaz_v1:cdevice.obj
 0001:000274ac       ?UnlockCountdown@Countdown@@QAAXXZ 100284ac f i usbh_usb2com_common_topaz_v1:cdevice.obj
 0001:000274e0       SetEvent                   100284e0 f i usbh_usb2com_common_topaz_v1:cdevice.obj
 0001:00027518       ?ResumeNotification@CDevice@@UAAHXZ 10028518 f i usbh_usb2com_common_topaz_v1:cdevice.obj
 0001:00027540       ??_GCDevice@@UAAPAXI@Z     10028540 f i usbh_usb2com_common_topaz_v1:cdevice.obj
 0001:00027540       ??_ECDevice@@UAAPAXI@Z     10028540 f i usbh_usb2com_common_topaz_v1:cdevice.obj
 0001:00027584       ?FreeAddress@CDevice@@QAAXE@Z 10028584 f i usbh_usb2com_common_topaz_v1:cdevice.obj
 0001:000275ac       ?ResumeNotification@CHub@@UAAHXZ 100285ac f i usbh_usb2com_common_topaz_v1:cdevice.obj
 0001:00027668       ??_ECHub@@UAAPAXI@Z        10028668 f i usbh_usb2com_common_topaz_v1:cdevice.obj
 0001:00027668       ??_GCHub@@UAAPAXI@Z        10028668 f i usbh_usb2com_common_topaz_v1:cdevice.obj
 0001:000276ac       ResetEvent                 100286ac f i usbh_usb2com_common_topaz_v1:cdevice.obj
 0001:000276e4       ?WaitForAPIReadyWrapper@@YAKKK@Z 100286e4 f i usbh_usb2com_common_topaz_v1:cdevice.obj
 0001:000277cc       ?CeCallUserProcWrapper@@YAHPBG0PAXK1KPAK@Z 100287cc f i usbh_usb2com_common_topaz_v1:cdevice.obj
 0001:000278d4       ?Addr0LockEntry@CDeviceGlobal@@QAA?AW4e_CritSec_Status@@K@Z 100288d4 f i usbh_usb2com_common_topaz_v1:cdevice.obj
 0001:00027910       ?Addr0LockLeave@CDeviceGlobal@@QAAXXZ 10028910 f i usbh_usb2com_common_topaz_v1:cdevice.obj
 0001:00027930       ?GetpUSBDSelectConfigurationProc@CDeviceGlobal@@QAAP6AHPBU_USB_DEVICE@@PAE@ZXZ 10028930 f i usbh_usb2com_common_topaz_v1:cdevice.obj
 0001:00027960       ?ReserveAddress@CDevice@@QAAHAAE@Z 10028960 f i usbh_usb2com_common_topaz_v1:cdevice.obj
 0001:000279a0       ?ObjCountdownDec@CDeviceGlobal@@QAAXXZ 100289a0 f i usbh_usb2com_common_topaz_v1:cdevice.obj
 0001:000279c0       GetCurrentThread           100289c0 f i usbh_usb2com_common_topaz_v1:cdevice.obj
 0001:000279d8       ?ObjCountdownInc@CDeviceGlobal@@QAAHXZ 100289d8 f i usbh_usb2com_common_topaz_v1:cdevice.obj
 0001:00027a10       ?Addr0LockPrepareDelete@CDeviceGlobal@@QAAXXZ 10028a10 f i usbh_usb2com_common_topaz_v1:cdevice.obj
 0001:00027a30       ?GetDeviceAddress@CDevice@@QAAEXZ 10028a30 f i usbh_usb2com_common_topaz_v1:cdevice.obj
 0001:00027a60       ?GetDeviceType@CRootHub@@EBAPBGXZ 10028a60 f i usbh_usb2com_common_topaz_v1:cdevice.obj
 0001:00027a90       ?GetDeviceTypeInt@CRootHub@@EBA?BKXZ 10028a90 f i usbh_usb2com_common_topaz_v1:cdevice.obj
 0001:00027ab8       ??_GCRootHub@@UAAPAXI@Z    10028ab8 f i usbh_usb2com_common_topaz_v1:cdevice.obj
 0001:00027ab8       ??_ECRootHub@@UAAPAXI@Z    10028ab8 f i usbh_usb2com_common_topaz_v1:cdevice.obj
 0001:00027afc       ?GetDeviceType@CExternalHub@@EBAPBGXZ 10028afc f i usbh_usb2com_common_topaz_v1:cdevice.obj
 0001:00027b2c       ?GetDeviceTypeInt@CExternalHub@@EBA?BKXZ 10028b2c f i usbh_usb2com_common_topaz_v1:cdevice.obj
 0001:00027b54       ??_GCExternalHub@@UAAPAXI@Z 10028b54 f i usbh_usb2com_common_topaz_v1:cdevice.obj
 0001:00027b54       ??_ECExternalHub@@UAAPAXI@Z 10028b54 f i usbh_usb2com_common_topaz_v1:cdevice.obj
 0001:00027b98       ?GetDeviceType@CFunction@@EBAPBGXZ 10028b98 f i usbh_usb2com_common_topaz_v1:cdevice.obj
 0001:00027bc8       ?GetDeviceTypeInt@CFunction@@EBA?BKXZ 10028bc8 f i usbh_usb2com_common_topaz_v1:cdevice.obj
 0001:00027bf0       ??_ECFunction@@UAAPAXI@Z   10028bf0 f i usbh_usb2com_common_topaz_v1:cdevice.obj
 0001:00027bf0       ??_GCFunction@@UAAPAXI@Z   10028bf0 f i usbh_usb2com_common_topaz_v1:cdevice.obj
 0001:00027c34       ?GetpUSBDAttachProc@CDeviceGlobal@@QAAP6AHPAXIIPBU_USB_DEVICE@@PAPAX@ZXZ 10028c34 f i usbh_usb2com_common_topaz_v1:cdevice.obj
 0001:00027c64       ?GetpHcdContext@CDeviceGlobal@@QAAPAXXZ 10028c64 f i usbh_usb2com_common_topaz_v1:cdevice.obj
 0001:00027c94       ?GetpUSBDDetachProc@CDeviceGlobal@@QAAP6AHPAX@ZXZ 10028c94 f i usbh_usb2com_common_topaz_v1:cdevice.obj
 0001:00027cc4       ?EnterCritSec_Ex@CritSec_Ex@@QAA?AW4e_CritSec_Status@@K@Z 10028cc4 f   usbh_usb2com_common_topaz_v1:sync.obj
 0001:00027f08       ?LeaveCritSec_Ex@CritSec_Ex@@QAAXXZ 10028f08 f   usbh_usb2com_common_topaz_v1:sync.obj
 0001:0002801c       ??0CritSec_Ex@@QAA@XZ      1002901c f   usbh_usb2com_common_topaz_v1:sync.obj
 0001:000280a8       ?Initialize@CritSec_Ex@@QAAXXZ 100290a8 f   usbh_usb2com_common_topaz_v1:sync.obj
 0001:00028110       ?PrepareDeleteCritSec_Ex@CritSec_Ex@@QAAXXZ 10029110 f   usbh_usb2com_common_topaz_v1:sync.obj
 0001:00028194       ??1CritSec_Ex@@QAA@XZ      10029194 f   usbh_usb2com_common_topaz_v1:sync.obj
 0001:000282b8       ??0Countdown@@QAA@K@Z      100292b8 f   usbh_usb2com_common_topaz_v1:sync.obj
 0001:00028350       ?IncrCountdown@Countdown@@QAAHXZ 10029350 f   usbh_usb2com_common_topaz_v1:sync.obj
 0001:000283f0       ?DecrCountdown@Countdown@@QAAXXZ 100293f0 f   usbh_usb2com_common_topaz_v1:sync.obj
 0001:000284ac       ?LockCountdown@Countdown@@AAAXXZ 100294ac f   usbh_usb2com_common_topaz_v1:sync.obj
 0001:000284e0       ?WaitForCountdown@Countdown@@QAAXH@Z 100294e0 f   usbh_usb2com_common_topaz_v1:sync.obj
 0001:00028574       ??1Countdown@@QAA@XZ       10029574 f   usbh_usb2com_common_topaz_v1:sync.obj
 0001:000285ac       GetCurrentThreadId         100295ac f i usbh_usb2com_common_topaz_v1:sync.obj
 0001:000285d8       ??0CEhcd@@QAA@PAXPAVCPhysMem@@PBGRAEKK@Z 100295d8 f   usbh_ehcdmdd_common_topaz_v1:cehcd.obj
 0001:000286f8       ??1CEhcd@@UAA@XZ           100296f8 f   usbh_ehcdmdd_common_topaz_v1:cehcd.obj
 0001:00028874       ?DeviceDeInitialize@CEhcd@@UAAXXZ 10029874 f   usbh_ehcdmdd_common_topaz_v1:cehcd.obj
 0001:000289c4       ?DeviceInitialize@CEhcd@@UAAHXZ 100299c4 f   usbh_ehcdmdd_common_topaz_v1:cehcd.obj
 0001:00028d7c       ?CreateHCDObject@@YAPAVCHcd@@PAXPAVCPhysMem@@KPBGRAEK@Z 10029d7c f   usbh_ehcdmdd_common_topaz_v1:cehcd.obj
 0001:00028e0c       ?SignalCheckForDoneTransfers@CHW@@UAAXXZ 10029e0c f i usbh_ehcdmdd_common_topaz_v1:cehcd.obj
 0001:00028e2c       ?GetForceReAttach@CHW@@UAAKXZ 10029e2c f i usbh_ehcdmdd_common_topaz_v1:cehcd.obj
 0001:00028e5c       ?SetForceReAttach@CHW@@UAAXK@Z 10029e5c f i usbh_ehcdmdd_common_topaz_v1:cehcd.obj
 0001:00028e80       ?GetCapability@CHW@@UAAKXZ 10029e80 f i usbh_ehcdmdd_common_topaz_v1:cehcd.obj
 0001:00028eb0       ?SignalHubStatusChange@CHW@@UAAXXZ 10029eb0 f i usbh_ehcdmdd_common_topaz_v1:cehcd.obj
 0001:00028ee8       ?AddedTt@CEhcd@@UAAHEE@Z   10029ee8 f i usbh_ehcdmdd_common_topaz_v1:cehcd.obj
 0001:00028f28       ?DeleteTt@CEhcd@@UAAHEE@Z  10029f28 f i usbh_ehcdmdd_common_topaz_v1:cehcd.obj
 0001:00028f68       ??_ECEhcd@@UAAPAXI@Z       10029f68 f i usbh_ehcdmdd_common_topaz_v1:cehcd.obj
 0001:00028f68       ??_GCEhcd@@UAAPAXI@Z       10029f68 f i usbh_ehcdmdd_common_topaz_v1:cehcd.obj
 0001:00028fac       ?GetNumberOfPort@CHW@@QAAKXZ 10029fac f i usbh_ehcdmdd_common_topaz_v1:cehcd.obj
 0001:00028fdc       ??0CPipe@@QAA@QBU_USB_ENDPOINT_DESCRIPTOR@@HHEEEQAVCEhcd@@@Z 10029fdc f   usbh_ehcdmdd_common_topaz_v1:cpipe.obj
 0001:000291b0       ??1CPipe@@UAA@XZ           1002a1b0 f   usbh_ehcdmdd_common_topaz_v1:cpipe.obj
 0001:00029274       ?GetCPhysMem@CPipe@@UAAPAVCPhysMem@@XZ 1002a274 f   usbh_ehcdmdd_common_topaz_v1:cpipe.obj
 0001:000292b0       ?IsPipeHalted@CPipe@@UAA?AW4HCD_REQUEST_STATUS@@QAH@Z 1002a2b0 f   usbh_ehcdmdd_common_topaz_v1:cpipe.obj
 0001:00029428       ?ClearHaltedFlag@CPipe@@UAAXXZ 1002a428 f   usbh_ehcdmdd_common_topaz_v1:cpipe.obj
 0001:000295a0       ??0CQueuedPipe@@QAA@QBU_USB_ENDPOINT_DESCRIPTOR@@HHEEEQAVCEhcd@@@Z 1002a5a0 f   usbh_ehcdmdd_common_topaz_v1:cpipe.obj
 0001:000296c4       ??1CQueuedPipe@@UAA@XZ     1002a6c4 f   usbh_ehcdmdd_common_topaz_v1:cpipe.obj
 0001:00029868       ?AbortTransfer@CQueuedPipe@@UAA?AW4HCD_REQUEST_STATUS@@Q6AKPAX@ZQAXPBX@Z 1002a868 f   usbh_ehcdmdd_common_topaz_v1:cpipe.obj
 0001:00029c3c       ?ClearHaltedFlag@CQueuedPipe@@UAAXXZ 1002ac3c f   usbh_ehcdmdd_common_topaz_v1:cpipe.obj
 0001:00029dc4       ?AbortQueue@CQueuedPipe@@IAAXXZ 1002adc4 f   usbh_ehcdmdd_common_topaz_v1:cpipe.obj
 0001:0002a110       ?IssueTransfer@CQueuedPipe@@UAA?AW4HCD_REQUEST_STATUS@@EQ6AKPAX@ZQAXKQBXKKQBKK2K3QAK5QAH55@Z 1002b110 f   usbh_ehcdmdd_common_topaz_v1:cpipe.obj
 0001:0002a514       ?StopTransfers@CQueuedPipe@@UAAXXZ 1002b514 f   usbh_ehcdmdd_common_topaz_v1:cpipe.obj
 0001:0002a580       ?ScheduleTransfer@CQueuedPipe@@UAA?AW4HCD_REQUEST_STATUS@@XZ 1002b580 f   usbh_ehcdmdd_common_topaz_v1:cpipe.obj
 0001:0002a824       ?CheckForDoneTransfers@CQueuedPipe@@UAAHXZ 1002b824 f   usbh_ehcdmdd_common_topaz_v1:cpipe.obj
 0001:0002aa1c       ??0CBulkPipe@@QAA@QBU_USB_ENDPOINT_DESCRIPTOR@@HHEEEQAVCEhcd@@@Z 1002ba1c f   usbh_ehcdmdd_common_topaz_v1:cpipe.obj
 0001:0002abc4       ??1CBulkPipe@@UAA@XZ       1002bbc4 f   usbh_ehcdmdd_common_topaz_v1:cpipe.obj
 0001:0002ac84       ?RemoveQHeadFromQueue@CBulkPipe@@MAAHXZ 1002bc84 f   usbh_ehcdmdd_common_topaz_v1:cpipe.obj
 0001:0002ad3c       ?InsertQHeadToQueue@CBulkPipe@@MAAHXZ 1002bd3c f   usbh_ehcdmdd_common_topaz_v1:cpipe.obj
 0001:0002adf4       ?OpenPipe@CBulkPipe@@UAA?AW4HCD_REQUEST_STATUS@@XZ 1002bdf4 f   usbh_ehcdmdd_common_topaz_v1:cpipe.obj
 0001:0002b230       ?ClosePipe@CBulkPipe@@UAA?AW4HCD_REQUEST_STATUS@@XZ 1002c230 f   usbh_ehcdmdd_common_topaz_v1:cpipe.obj
 0001:0002b394       ?AreTransferParametersValid@CBulkPipe@@EBAHPBUSTRANSFER@@@Z 1002c394 f   usbh_ehcdmdd_common_topaz_v1:cpipe.obj
 0001:0002b62c       ??0CControlPipe@@QAA@QBU_USB_ENDPOINT_DESCRIPTOR@@HHEEEQAVCEhcd@@@Z 1002c62c f   usbh_ehcdmdd_common_topaz_v1:cpipe.obj
 0001:0002b794       ??1CControlPipe@@UAA@XZ    1002c794 f   usbh_ehcdmdd_common_topaz_v1:cpipe.obj
 0001:0002b854       ?OpenPipe@CControlPipe@@UAA?AW4HCD_REQUEST_STATUS@@XZ 1002c854 f   usbh_ehcdmdd_common_topaz_v1:cpipe.obj
 0001:0002bc2c       ?ClosePipe@CControlPipe@@UAA?AW4HCD_REQUEST_STATUS@@XZ 1002cc2c f   usbh_ehcdmdd_common_topaz_v1:cpipe.obj
 0001:0002bd90       ?RemoveQHeadFromQueue@CControlPipe@@MAAHXZ 1002cd90 f   usbh_ehcdmdd_common_topaz_v1:cpipe.obj
 0001:0002be48       ?InsertQHeadToQueue@CControlPipe@@MAAHXZ 1002ce48 f   usbh_ehcdmdd_common_topaz_v1:cpipe.obj
 0001:0002bf00       ?IssueTransfer@CControlPipe@@UAA?AW4HCD_REQUEST_STATUS@@EQ6AKPAX@ZQAXKQBXKKQBKK2K3QAK5QAH55@Z 1002cf00 f   usbh_ehcdmdd_common_topaz_v1:cpipe.obj
 0001:0002c110       ?ChangeMaxPacketSize@CControlPipe@@UAAXG@Z 1002d110 f   usbh_ehcdmdd_common_topaz_v1:cpipe.obj
 0001:0002c39c       ?AreTransferParametersValid@CControlPipe@@EBAHPBUSTRANSFER@@@Z 1002d39c f   usbh_ehcdmdd_common_topaz_v1:cpipe.obj
 0001:0002c6e8       ??0CInterruptPipe@@QAA@QBU_USB_ENDPOINT_DESCRIPTOR@@HHEEEQAVCEhcd@@@Z 1002d6e8 f   usbh_ehcdmdd_common_topaz_v1:cpipe.obj
 0001:0002cc20       ??1CInterruptPipe@@UAA@XZ  1002dc20 f   usbh_ehcdmdd_common_topaz_v1:cpipe.obj
 0001:0002cd28       ?OpenPipe@CInterruptPipe@@UAA?AW4HCD_REQUEST_STATUS@@XZ 1002dd28 f   usbh_ehcdmdd_common_topaz_v1:cpipe.obj
 0001:0002d080       ?ClosePipe@CInterruptPipe@@UAA?AW4HCD_REQUEST_STATUS@@XZ 1002e080 f   usbh_ehcdmdd_common_topaz_v1:cpipe.obj
 0001:0002d1e4       ?AreTransferParametersValid@CInterruptPipe@@EBAHPBUSTRANSFER@@@Z 1002e1e4 f   usbh_ehcdmdd_common_topaz_v1:cpipe.obj
 0001:0002d444       ??0CIsochronousPipe@@QAA@QBU_USB_ENDPOINT_DESCRIPTOR@@HHEEEQAVCEhcd@@@Z 1002e444 f   usbh_ehcdmdd_common_topaz_v1:cpipe.obj
 0001:0002dd78       ??1CIsochronousPipe@@UAA@XZ 1002ed78 f   usbh_ehcdmdd_common_topaz_v1:cpipe.obj
 0001:0002e150       ?AllocateCITD@CIsochronousPipe@@QAAPAVCITD@@PAVCITransfer@@@Z 1002f150 f   usbh_ehcdmdd_common_topaz_v1:cpipe.obj
 0001:0002e334       ?AllocateCSITD@CIsochronousPipe@@QAAPAVCSITD@@PAVCSITransfer@@PAV2@@Z 1002f334 f   usbh_ehcdmdd_common_topaz_v1:cpipe.obj
 0001:0002e51c       ?FreeCITD@CIsochronousPipe@@QAAXPAVCITD@@@Z 1002f51c f   usbh_ehcdmdd_common_topaz_v1:cpipe.obj
 0001:0002e6c8       ?FreeCSITD@CIsochronousPipe@@QAAXPAVCSITD@@@Z 1002f6c8 f   usbh_ehcdmdd_common_topaz_v1:cpipe.obj
 0001:0002e878       ?OpenPipe@CIsochronousPipe@@UAA?AW4HCD_REQUEST_STATUS@@XZ 1002f878 f   usbh_ehcdmdd_common_topaz_v1:cpipe.obj
 0001:0002eacc       ?ClosePipe@CIsochronousPipe@@UAA?AW4HCD_REQUEST_STATUS@@XZ 1002facc f   usbh_ehcdmdd_common_topaz_v1:cpipe.obj
 0001:0002ec44       ?AbortTransfer@CIsochronousPipe@@UAA?AW4HCD_REQUEST_STATUS@@Q6AKPAX@ZQAXPBX@Z 1002fc44 f   usbh_ehcdmdd_common_topaz_v1:cpipe.obj
 0001:0002ee78       ?IssueTransfer@CIsochronousPipe@@UAA?AW4HCD_REQUEST_STATUS@@EQ6AKPAX@ZQAXKQBXKKQBKK2K3QAK5QAH55@Z 1002fe78 f   usbh_ehcdmdd_common_topaz_v1:cpipe.obj
 0001:0002f48c       ?ScheduleTransfer@CIsochronousPipe@@UAA?AW4HCD_REQUEST_STATUS@@XZ 1003048c f   usbh_ehcdmdd_common_topaz_v1:cpipe.obj
 0001:0002f598       ?CheckForDoneTransfers@CIsochronousPipe@@UAAHXZ 10030598 f   usbh_ehcdmdd_common_topaz_v1:cpipe.obj
 0001:0002f7f0       ?AreTransferParametersValid@CIsochronousPipe@@EBAHPBUSTRANSFER@@@Z 100307f0 f   usbh_ehcdmdd_common_topaz_v1:cpipe.obj
 0001:0002fc20       ?CreateBulkPipe@@YAPAVCPipeAbs@@QBU_USB_ENDPOINT_DESCRIPTOR@@HHEEEQAVCHcd@@@Z 10030c20 f   usbh_ehcdmdd_common_topaz_v1:cpipe.obj
 0001:0002fcb4       ?CreateControlPipe@@YAPAVCPipeAbs@@QBU_USB_ENDPOINT_DESCRIPTOR@@HHEEEQAVCHcd@@@Z 10030cb4 f   usbh_ehcdmdd_common_topaz_v1:cpipe.obj
 0001:0002fd48       ?CreateInterruptPipe@@YAPAVCPipeAbs@@QBU_USB_ENDPOINT_DESCRIPTOR@@HHEEEQAVCHcd@@@Z 10030d48 f   usbh_ehcdmdd_common_topaz_v1:cpipe.obj
 0001:0002fddc       ?CreateIsochronousPipe@@YAPAVCPipeAbs@@QBU_USB_ENDPOINT_DESCRIPTOR@@HHEEEQAVCHcd@@@Z 10030ddc f   usbh_ehcdmdd_common_topaz_v1:cpipe.obj
 0001:0002fe70       ??0CPipeAbs@@QAA@E@Z       10030e70 f i usbh_ehcdmdd_common_topaz_v1:cpipe.obj
 0001:0002feb8       ?ChangeMaxPacketSize@CPipeAbs@@UAAXG@Z 10030eb8 f i usbh_ehcdmdd_common_topaz_v1:cpipe.obj
 0001:0002ff10       ??_ECPipeAbs@@UAAPAXI@Z    10030f10 f i usbh_ehcdmdd_common_topaz_v1:cpipe.obj
 0001:0002ff10       ??_GCPipeAbs@@UAAPAXI@Z    10030f10 f i usbh_ehcdmdd_common_topaz_v1:cpipe.obj
 0001:0002ff54       ??1CPipeAbs@@UAA@XZ        10030f54 f i usbh_ehcdmdd_common_topaz_v1:cpipe.obj
 0001:0002ff78       ??_GCPipe@@UAAPAXI@Z       10030f78 f i usbh_ehcdmdd_common_topaz_v1:cpipe.obj
 0001:0002ff78       ??_ECPipe@@UAAPAXI@Z       10030f78 f i usbh_ehcdmdd_common_topaz_v1:cpipe.obj
 0001:0002ffbc       ?GetPhysMem@CHW@@QAAPAVCPhysMem@@XZ 10030fbc f i usbh_ehcdmdd_common_topaz_v1:cpipe.obj
 0001:0002ffec       ??_GCQueuedPipe@@UAAPAXI@Z 10030fec f i usbh_ehcdmdd_common_topaz_v1:cpipe.obj
 0001:0002ffec       ??_ECQueuedPipe@@UAAPAXI@Z 10030fec f i usbh_ehcdmdd_common_topaz_v1:cpipe.obj
 0001:00030030       ?InvalidNextTD@CQH@@QAAXXZ 10031030 f i usbh_ehcdmdd_common_topaz_v1:cpipe.obj
 0001:000300e8       ?CheckStructure@CQH@@QAAHXZ 100310e8 f i usbh_ehcdmdd_common_topaz_v1:cpipe.obj
 0001:00030194       ?GetNextTransfer@CTransfer@@QAAPAV1@XZ 10031194 f i usbh_ehcdmdd_common_topaz_v1:cpipe.obj
 0001:000301c4       ?SetNextTransfer@CTransfer@@QAAXPAV1@@Z 100311c4 f i usbh_ehcdmdd_common_topaz_v1:cpipe.obj
 0001:000301e8       ?GetSTransfer@CTransfer@@QAA?AUSTRANSFER@@XZ 100311e8 f i usbh_ehcdmdd_common_topaz_v1:cpipe.obj
 0001:00030224       ?GetQHead@CQueuedPipe@@QAAPAVCQH@@XZ 10031224 f i usbh_ehcdmdd_common_topaz_v1:cpipe.obj
 0001:00030254       ?ResetOverlayDataToggle@CQH@@QAAXXZ 10031254 f i usbh_ehcdmdd_common_topaz_v1:cpipe.obj
 0001:00030288       ?DoNotCallBack@CTransfer@@QAAXXZ 10031288 f i usbh_ehcdmdd_common_topaz_v1:cpipe.obj
 0001:000302dc       ??0CQTransfer@@QAA@QAVCPipe@@QAVCPhysMem@@PAUSTRANSFER@@@Z 100312dc f i usbh_ehcdmdd_common_topaz_v1:cpipe.obj
 0001:0003033c       ??_GCQTransfer@@UAAPAXI@Z  1003133c f i usbh_ehcdmdd_common_topaz_v1:cpipe.obj
 0001:0003033c       ??_ECQTransfer@@UAAPAXI@Z  1003133c f i usbh_ehcdmdd_common_topaz_v1:cpipe.obj
 0001:00030380       ?GetTransfer@CQTD@@QAAPAVCQTransfer@@XZ 10031380 f i usbh_ehcdmdd_common_topaz_v1:cpipe.obj
 0001:000303b8       ?CheckStructure@CQTD@@QAAXXZ 100313b8 f i usbh_ehcdmdd_common_topaz_v1:cpipe.obj
 0001:00030428       ?IsActive@CQH@@QAAHXZ      10031428 f i usbh_ehcdmdd_common_topaz_v1:cpipe.obj
 0001:000304b0       ?GetCQTDList@CQTransfer@@QAAPAVCQTD@@XZ 100314b0 f i usbh_ehcdmdd_common_topaz_v1:cpipe.obj
 0001:000304e0       ?GetPipeType@CBulkPipe@@UBAPBGXZ 100314e0 f i usbh_ehcdmdd_common_topaz_v1:cpipe.obj
 0001:0003050c       ??_ECBulkPipe@@UAAPAXI@Z   1003150c f i usbh_ehcdmdd_common_topaz_v1:cpipe.obj
 0001:0003050c       ??_GCBulkPipe@@UAAPAXI@Z   1003150c f i usbh_ehcdmdd_common_topaz_v1:cpipe.obj
 0001:00030550       ?AsyncQueueQH@CHW@@QAAPAVCQH@@PAV2@@Z 10031550 f i usbh_ehcdmdd_common_topaz_v1:cpipe.obj
 0001:0003058c       ?SetDTC@CQH@@QAAXH@Z       1003158c f i usbh_ehcdmdd_common_topaz_v1:cpipe.obj
 0001:00030600       ?AddToBusyPipeList@CHW@@QAAHQAVCPipe@@H@Z 10031600 f i usbh_ehcdmdd_common_topaz_v1:cpipe.obj
 0001:00030640       ??_GCQH@@QAAPAXI@Z         10031640 f i usbh_ehcdmdd_common_topaz_v1:cpipe.obj
 0001:00030684       ??1CQH@@QAA@XZ             10031684 f i usbh_ehcdmdd_common_topaz_v1:cpipe.obj
 0001:00030698       ?GetPhysAddr@CQH@@QAAKXZ   10031698 f i usbh_ehcdmdd_common_topaz_v1:cpipe.obj
 0001:000306d0       ?RemoveFromBusyPipeList@CHW@@QAAXQAVCPipe@@@Z 100316d0 f i usbh_ehcdmdd_common_topaz_v1:cpipe.obj
 0001:000306f4       ?GetPipeType@CControlPipe@@UBAPBGXZ 100316f4 f i usbh_ehcdmdd_common_topaz_v1:cpipe.obj
 0001:00030720       ??_GCControlPipe@@UAAPAXI@Z 10031720 f i usbh_ehcdmdd_common_topaz_v1:cpipe.obj
 0001:00030720       ??_ECControlPipe@@UAAPAXI@Z 10031720 f i usbh_ehcdmdd_common_topaz_v1:cpipe.obj
 0001:00030764       ?SetControlEnpt@CQH@@QAAXH@Z 10031764 f i usbh_ehcdmdd_common_topaz_v1:cpipe.obj
 0001:000307d8       ?SetDeviceAddress@CQH@@QAAXK@Z 100317d8 f i usbh_ehcdmdd_common_topaz_v1:cpipe.obj
 0001:00030820       ?SetMaxPacketLength@CQH@@QAAXK@Z 10031820 f i usbh_ehcdmdd_common_topaz_v1:cpipe.obj
 0001:00030884       ?GetPipeType@CInterruptPipe@@UBAPBGXZ 10031884 f i usbh_ehcdmdd_common_topaz_v1:cpipe.obj
 0001:000308b4       ?RemoveQHeadFromQueue@CInterruptPipe@@MAAHXZ 100318b4 f i usbh_ehcdmdd_common_topaz_v1:cpipe.obj
 0001:000308dc       ?InsertQHeadToQueue@CInterruptPipe@@MAAHXZ 100318dc f i usbh_ehcdmdd_common_topaz_v1:cpipe.obj
 0001:00030904       ??_GCInterruptPipe@@UAAPAXI@Z 10031904 f i usbh_ehcdmdd_common_topaz_v1:cpipe.obj
 0001:00030904       ??_ECInterruptPipe@@UAAPAXI@Z 10031904 f i usbh_ehcdmdd_common_topaz_v1:cpipe.obj
 0001:00030948       ?SetReLoad@CQH@@QAAXK@Z    10031948 f i usbh_ehcdmdd_common_topaz_v1:cpipe.obj
 0001:00030994       ?SetINT@CQH@@QAAXH@Z       10031994 f i usbh_ehcdmdd_common_topaz_v1:cpipe.obj
 0001:00030a08       ?PeriodQeueuQHead@CHW@@QAAPAVCQH@@PAV2@EEH@Z 10031a08 f i usbh_ehcdmdd_common_topaz_v1:cpipe.obj
 0001:00030a54       ?PeriodDeQueueuQHead@CHW@@QAAHPAVCQH@@@Z 10031a54 f i usbh_ehcdmdd_common_topaz_v1:cpipe.obj
 0001:00030a90       ?GetPipeType@CIsochronousPipe@@UBAPBGXZ 10031a90 f i usbh_ehcdmdd_common_topaz_v1:cpipe.obj
 0001:00030ac0       ?StopTransfers@CIsochronousPipe@@UAAXXZ 10031ac0 f i usbh_ehcdmdd_common_topaz_v1:cpipe.obj
 0001:00030ad4       ??_GCIsochronousPipe@@UAAPAXI@Z 10031ad4 f i usbh_ehcdmdd_common_topaz_v1:cpipe.obj
 0001:00030ad4       ??_ECIsochronousPipe@@UAAPAXI@Z 10031ad4 f i usbh_ehcdmdd_common_topaz_v1:cpipe.obj
 0001:00030b18       ??_GCITD@@QAAPAXI@Z        10031b18 f i usbh_ehcdmdd_common_topaz_v1:cpipe.obj
 0001:00030b5c       ??1CITD@@QAA@XZ            10031b5c f i usbh_ehcdmdd_common_topaz_v1:cpipe.obj
 0001:00030b78       ?CheckStructure@CITD@@QAAHXZ 10031b78 f i usbh_ehcdmdd_common_topaz_v1:cpipe.obj
 0001:00030c20       ??_GCSITD@@QAAPAXI@Z       10031c20 f i usbh_ehcdmdd_common_topaz_v1:cpipe.obj
 0001:00030c64       ??1CSITD@@QAA@XZ           10031c64 f i usbh_ehcdmdd_common_topaz_v1:cpipe.obj
 0001:00030c80       ?CheckStructure@CSITD@@QAAHXZ 10031c80 f i usbh_ehcdmdd_common_topaz_v1:cpipe.obj
 0001:00030d28       ?GetStartFrame@CIsochTransfer@@QAAKXZ 10031d28 f i usbh_ehcdmdd_common_topaz_v1:cpipe.obj
 0001:00030d58       ?SetStartFrame@CIsochTransfer@@QAAHK@Z 10031d58 f i usbh_ehcdmdd_common_topaz_v1:cpipe.obj
 0001:00030dd8       ??0TransactionTrasnlate@@QAA@EEPAV0@@Z 10031dd8 f   usbh_ehcdmdd_common_topaz_v1:usb2lib.obj
 0001:00030ea4       ??1TransactionTrasnlate@@QAA@XZ 10031ea4 f   usbh_ehcdmdd_common_topaz_v1:usb2lib.obj
 0001:00030f58       ?AddedEp@TransactionTrasnlate@@QAAHPAU_EndpointBuget@@@Z 10031f58 f   usbh_ehcdmdd_common_topaz_v1:usb2lib.obj
 0001:000315a0       ?DeletedEp@TransactionTrasnlate@@QAAHPAU_EndpointBuget@@@Z 100325a0 f   usbh_ehcdmdd_common_topaz_v1:usb2lib.obj
 0001:000316f4       ?FindBestTimeSlot@TransactionTrasnlate@@AAAHGGPAU_ENDPOINTBUGETLIST@@PAK@Z 100326f4 f   usbh_ehcdmdd_common_topaz_v1:usb2lib.obj
 0001:000317dc       ?InsertEp@TransactionTrasnlate@@AAAHKPAU_EndpointBuget@@@Z 100327dc f   usbh_ehcdmdd_common_topaz_v1:usb2lib.obj
 0001:00031a48       ?RemoveEp@TransactionTrasnlate@@AAAHKPAU_EndpointBuget@@@Z 10032a48 f   usbh_ehcdmdd_common_topaz_v1:usb2lib.obj
 0001:00031c64       ??0USB2lib@@QAA@XZ         10032c64 f   usbh_ehcdmdd_common_topaz_v1:usb2lib.obj
 0001:00031d6c       ??1USB2lib@@QAA@XZ         10032d6c f   usbh_ehcdmdd_common_topaz_v1:usb2lib.obj
 0001:00031e1c       ?AddedTt@USB2lib@@QAAHEE@Z 10032e1c f   usbh_ehcdmdd_common_topaz_v1:usb2lib.obj
 0001:00031f08       ?DeleteTt@USB2lib@@QAAHEE@Z 10032f08 f   usbh_ehcdmdd_common_topaz_v1:usb2lib.obj
 0001:000320ac       ?GetTT@USB2lib@@QAAPAVTransactionTrasnlate@@EE@Z 100330ac f   usbh_ehcdmdd_common_topaz_v1:usb2lib.obj
 0001:00032160       ?Add_bitstuff@USB2lib@@ABAII@Z 10033160 f   usbh_ehcdmdd_common_topaz_v1:usb2lib.obj
 0001:00032194       ?Compute_nonsplit_overhead@USB2lib@@AAAHPAU_EndpointBuget@@@Z 10033194 f   usbh_ehcdmdd_common_topaz_v1:usb2lib.obj
 0001:000322e8       ?AllocUsb2BusTime@USB2lib@@QAAHEEPAU_EndpointBuget@@@Z 100332e8 f   usbh_ehcdmdd_common_topaz_v1:usb2lib.obj
 0001:00032af0       ?FreeUsb2BusTime@USB2lib@@QAAXEEPAU_EndpointBuget@@@Z 10033af0 f   usbh_ehcdmdd_common_topaz_v1:usb2lib.obj
 0001:00032d38       ?GetSMASK@USB2lib@@QAAEPAU_EndpointBuget@@@Z 10033d38 f   usbh_ehcdmdd_common_topaz_v1:usb2lib.obj
 0001:00032e38       ?GetCMASK@USB2lib@@QAAEPAU_EndpointBuget@@@Z 10033e38 f   usbh_ehcdmdd_common_topaz_v1:usb2lib.obj
 0001:00033000       ?ConvertBtoHFrame@USB2lib@@AAAXEEPAE0@Z 10034000 f   usbh_ehcdmdd_common_topaz_v1:usb2lib.obj
 0001:0003309c       ?GetNextTT@TransactionTrasnlate@@QAAPAV1@XZ 1003409c f i usbh_ehcdmdd_common_topaz_v1:usb2lib.obj
 0001:000330cc       ??_GTransactionTrasnlate@@QAAPAXI@Z 100340cc f i usbh_ehcdmdd_common_topaz_v1:usb2lib.obj
 0001:00033110       ?GetHubAddress@TransactionTrasnlate@@QAAEXZ 10034110 f i usbh_ehcdmdd_common_topaz_v1:usb2lib.obj
 0001:0003313c       ?GetHubPort@TransactionTrasnlate@@QAAEXZ 1003413c f i usbh_ehcdmdd_common_topaz_v1:usb2lib.obj
 0001:0003316c       ?SetNextTT@TransactionTrasnlate@@QAAPAV1@PAV1@@Z 1003416c f i usbh_ehcdmdd_common_topaz_v1:usb2lib.obj
 0001:000331b4       ??0CDummyPipe@@QAA@QAVCPhysMem@@@Z 100341b4 f   usbh_ehcdmdd_common_topaz_v1:chw.obj
 0001:000332a4       ??0CPeriodicMgr@@QAA@QAVCPhysMem@@K@Z 100342a4 f   usbh_ehcdmdd_common_topaz_v1:chw.obj
 0001:000334b0       ??1CPeriodicMgr@@QAA@XZ    100344b0 f   usbh_ehcdmdd_common_topaz_v1:chw.obj
 0001:00033548       ?Init@CPeriodicMgr@@QAAHXZ 10034548 f   usbh_ehcdmdd_common_topaz_v1:chw.obj
 0001:000339d0       ?DeInit@CPeriodicMgr@@QAAXXZ 100349d0 f   usbh_ehcdmdd_common_topaz_v1:chw.obj
 0001:00033b30       ?QueueITD@CPeriodicMgr@@QAAHPAVCITD@@K@Z 10034b30 f   usbh_ehcdmdd_common_topaz_v1:chw.obj
 0001:00033cd8       ?QueueSITD@CPeriodicMgr@@QAAHPAVCSITD@@K@Z 10034cd8 f   usbh_ehcdmdd_common_topaz_v1:chw.obj
 0001:00033e80       ?DeQueueTD@CPeriodicMgr@@QAAHKK@Z 10034e80 f   usbh_ehcdmdd_common_topaz_v1:chw.obj
 0001:00034090       ?QueueQHead@CPeriodicMgr@@QAAPAVCQH@@PAV2@EEH@Z 10035090 f   usbh_ehcdmdd_common_topaz_v1:chw.obj
 0001:000343c0       ?DequeueQHead@CPeriodicMgr@@QAAHPAVCQH@@@Z 100353c0 f   usbh_ehcdmdd_common_topaz_v1:chw.obj
 0001:00034610       ??0CAsyncMgr@@QAA@QAVCPhysMem@@@Z 10035610 f   usbh_ehcdmdd_common_topaz_v1:chw.obj
 0001:000346b8       ??1CAsyncMgr@@QAA@XZ       100356b8 f   usbh_ehcdmdd_common_topaz_v1:chw.obj
 0001:000346dc       ?Init@CAsyncMgr@@QAAHXZ    100356dc f   usbh_ehcdmdd_common_topaz_v1:chw.obj
 0001:000347d4       ?DeInit@CAsyncMgr@@QAAXXZ  100357d4 f   usbh_ehcdmdd_common_topaz_v1:chw.obj
 0001:0003487c       ?QueueQH@CAsyncMgr@@QAAPAVCQH@@PAV2@@Z 1003587c f   usbh_ehcdmdd_common_topaz_v1:chw.obj
 0001:00034928       ?DequeueQHead@CAsyncMgr@@QAAHPAVCQH@@@Z 10035928 f   usbh_ehcdmdd_common_topaz_v1:chw.obj
 0001:00034aa4       ?Init@CBusyPipeList@@QAAHXZ 10035aa4 f   usbh_ehcdmdd_common_topaz_v1:chw.obj
 0001:00034c24       ?DeInit@CBusyPipeList@@QAAXXZ 10035c24 f   usbh_ehcdmdd_common_topaz_v1:chw.obj
 0001:00034d44       ?SignalCheckForDoneTransfers@CBusyPipeList@@QAAXXZ 10035d44 f   usbh_ehcdmdd_common_topaz_v1:chw.obj
 0001:00034dd4       ?CheckForDoneTransfersThreadStub@CBusyPipeList@@CAKPAX@Z 10035dd4 f   usbh_ehcdmdd_common_topaz_v1:chw.obj
 0001:00034e08       ?CheckForDoneTransfersThread@CBusyPipeList@@AAAKXZ 10035e08 f   usbh_ehcdmdd_common_topaz_v1:chw.obj
 0001:0003513c       ?AddToBusyPipeList@CBusyPipeList@@QAAHQAVCPipe@@H@Z 1003613c f   usbh_ehcdmdd_common_topaz_v1:chw.obj
 0001:0003539c       ?RemoveFromBusyPipeList@CBusyPipeList@@QAAXQAVCPipe@@@Z 1003639c f   usbh_ehcdmdd_common_topaz_v1:chw.obj
 0001:00035660       ??0CHW@@QAA@SAEKKQAVCPhysMem@@PAXPBG@Z 10036660 f   usbh_ehcdmdd_common_topaz_v1:chw.obj
 0001:000359d0       ??1CHW@@UAA@XZ             100369d0 f   usbh_ehcdmdd_common_topaz_v1:chw.obj
 0001:00035ab8       ?DisableAsyncSchedule@CHW@@QAAHXZ 10036ab8 f   usbh_ehcdmdd_common_topaz_v1:chw.obj
 0001:00035b9c       ?EnableAsyncSchedule@CHW@@QAAHXZ 10036b9c f   usbh_ehcdmdd_common_topaz_v1:chw.obj
 0001:00035c8c       ?PowerOnAllPorts@CHW@@QAAHXZ 10036c8c f   usbh_ehcdmdd_common_topaz_v1:chw.obj
 0001:00035d80       ?WriteAsyncListAddr@CHW@@QAAXK@Z 10036d80 f   usbh_ehcdmdd_common_topaz_v1:chw.obj
 0001:00035da4       ?ConfigureHS@CHW@@QAAHXZ   10036da4 f   usbh_ehcdmdd_common_topaz_v1:chw.obj
 0001:00036320       ?Initialize@CHW@@UAAHXZ    10037320 f   usbh_ehcdmdd_common_topaz_v1:chw.obj
 0001:00036860       ?DeInitialize@CHW@@UAAXXZ  10037860 f   usbh_ehcdmdd_common_topaz_v1:chw.obj
 0001:00036a88       ?EnterOperationalState@CHW@@QAAXXZ 10037a88 f   usbh_ehcdmdd_common_topaz_v1:chw.obj
 0001:00036c7c       ?RunStopUSBController@CHW@@QAAXH@Z 10037c7c f   usbh_ehcdmdd_common_topaz_v1:chw.obj
 0001:00036d8c       ?StartHostController@CHW@@QAAXXZ 10037d8c f   usbh_ehcdmdd_common_topaz_v1:chw.obj
 0001:00036fb4       ?StopHostController@CHW@@QAAXXZ 10037fb4 f   usbh_ehcdmdd_common_topaz_v1:chw.obj
 0001:00037088       ?AsyncBell@CHW@@QAAHXZ     10038088 f   usbh_ehcdmdd_common_topaz_v1:chw.obj
 0001:0003713c       ?AsyncDequeueQH@CHW@@QAAHPAVCQH@@@Z 1003813c f   usbh_ehcdmdd_common_topaz_v1:chw.obj
 0001:00037194       ?PeriodQueueITD@CHW@@QAAHPAVCITD@@K@Z 10038194 f   usbh_ehcdmdd_common_topaz_v1:chw.obj
 0001:0003721c       ?PeriodQueueSITD@CHW@@QAAHPAVCSITD@@K@Z 1003821c f   usbh_ehcdmdd_common_topaz_v1:chw.obj
 0001:000372a4       ?PeriodDeQueueTD@CHW@@QAAHKK@Z 100382a4 f   usbh_ehcdmdd_common_topaz_v1:chw.obj
 0001:00037348       ?CeResumeThreadStub@CHW@@CAKPAX@Z 10038348 f   usbh_ehcdmdd_common_topaz_v1:chw.obj
 0001:0003737c       ?CeResumeThread@CHW@@AAAKXZ 1003837c f   usbh_ehcdmdd_common_topaz_v1:chw.obj
 0001:00037534       ?UsbInterruptThreadStub@CHW@@CAKPAX@Z 10038534 f   usbh_ehcdmdd_common_topaz_v1:chw.obj
 0001:00037574       ?UsbInterruptThread@CHW@@AAAKXZ 10038574 f   usbh_ehcdmdd_common_topaz_v1:chw.obj
 0001:00038e24       ?UpdateFrameCounter@CHW@@AAAXXZ 10039e24 f   usbh_ehcdmdd_common_topaz_v1:chw.obj
 0001:00038f68       ?GetFrameNumber@CHW@@UAAHPAK@Z 10039f68 f   usbh_ehcdmdd_common_topaz_v1:chw.obj
 0001:00038fec       ?GetFrameLength@CHW@@UAAHPAG@Z 10039fec f   usbh_ehcdmdd_common_topaz_v1:chw.obj
 0001:00039024       ?SetFrameLength@CHW@@UAAHPAXG@Z 1003a024 f   usbh_ehcdmdd_common_topaz_v1:chw.obj
 0001:0003904c       ?StopAdjustingFrame@CHW@@UAAHXZ 1003a04c f   usbh_ehcdmdd_common_topaz_v1:chw.obj
 0001:00039074       ?DidPortStatusChange@CHW@@UAAHE@Z 1003a074 f   usbh_ehcdmdd_common_topaz_v1:chw.obj
 0001:000392e0       ?GetPortStatus@CHW@@UAAHEAAU_USB_HUB_AND_PORT_STATUS@@PAK@Z 1003a2e0 f   usbh_ehcdmdd_common_topaz_v1:chw.obj
 0001:00039938       ?RootHubFeature@CHW@@UAAHEEG@Z 1003a938 f   usbh_ehcdmdd_common_topaz_v1:chw.obj
 0001:00039b68       ?ResetAndEnablePort@CHW@@UAAHE@Z 1003ab68 f   usbh_ehcdmdd_common_topaz_v1:chw.obj
 0001:00039eb8       ?DisablePort@CHW@@UAAXE@Z  1003aeb8 f   usbh_ehcdmdd_common_topaz_v1:chw.obj
 0001:00039f5c       ?WaitForPortStatusChange@CHW@@UAAHPAX@Z 1003af5c f   usbh_ehcdmdd_common_topaz_v1:chw.obj
 0001:00039ff4       ?EnterLowPowerMode@CHW@@QAAXXZ 1003aff4 f   usbh_ehcdmdd_common_topaz_v1:chw.obj
 0001:0003a32c       ?PowerMgmtCallback@CHW@@UAAXH@Z 1003b32c f   usbh_ehcdmdd_common_topaz_v1:chw.obj
 0001:0003a840       ?SuspendHostController@CHW@@AAAXXZ 1003b840 f   usbh_ehcdmdd_common_topaz_v1:chw.obj
 0001:0003aa08       ?ResumeHostController@CHW@@AAAXXZ 1003ba08 f   usbh_ehcdmdd_common_topaz_v1:chw.obj
 0001:0003ac24       ?SetCapability@CHW@@UAAKK@Z 1003bc24 f   usbh_ehcdmdd_common_topaz_v1:chw.obj
 0001:0003ac74       ?GetPortSpeed@CHW@@QAAGG@Z 1003bc74 f   usbh_ehcdmdd_common_topaz_v1:chw.obj
 0001:0003acbc       ?IsOTGHostDevice@CHW@@UAAHXZ 1003bcbc f   usbh_ehcdmdd_common_topaz_v1:chw.obj
 0001:0003ad44       ?StopUSBClock@CHW@@QAAHXZ  1003bd44 f   usbh_ehcdmdd_common_topaz_v1:chw.obj
 0001:0003ad88       ?StartUSBClock@CHW@@QAAHXZ 1003bd88 f   usbh_ehcdmdd_common_topaz_v1:chw.obj
 0001:0003adcc       ?WakeUpSysIntr@CHW@@UAAXXZ 1003bdcc f   usbh_ehcdmdd_common_topaz_v1:chw.obj
 0001:0003adf8       ?DumpUSBCMD@CHW@@AAAXXZ    1003bdf8 f   usbh_ehcdmdd_common_topaz_v1:chw.obj
 0001:0003af60       ?DumpUSBSTS@CHW@@AAAXXZ    1003bf60 f   usbh_ehcdmdd_common_topaz_v1:chw.obj
 0001:0003b170       ?DumpUSBINTR@CHW@@AAAXXZ   1003c170 f   usbh_ehcdmdd_common_topaz_v1:chw.obj
 0001:0003b220       ?DumpFRNUM@CHW@@AAAXXZ     1003c220 f   usbh_ehcdmdd_common_topaz_v1:chw.obj
 0001:0003b344       ?DumpFLBASEADD@CHW@@AAAXXZ 1003c344 f   usbh_ehcdmdd_common_topaz_v1:chw.obj
 0001:0003b448       ?DumpSOFMOD@CHW@@AAAXXZ    1003c448 f   usbh_ehcdmdd_common_topaz_v1:chw.obj
 0001:0003b584       ?DumpPORTSC@CHW@@AAAXG@Z   1003c584 f   usbh_ehcdmdd_common_topaz_v1:chw.obj
 0001:0003b974       ?DumpAllRegisters@CHW@@AAAXXZ 1003c974 f   usbh_ehcdmdd_common_topaz_v1:chw.obj
 0001:0003ba6c       ?IssueTransfer@CDummyPipe@@UAA?AW4HCD_REQUEST_STATUS@@EQ6AKPAX@ZQAXKQBXKKQBKK2K3QAK5QAH55@Z 1003ca6c f i usbh_ehcdmdd_common_topaz_v1:chw.obj
 0001:0003ba94       ?OpenPipe@CDummyPipe@@UAA?AW4HCD_REQUEST_STATUS@@XZ 1003ca94 f i usbh_ehcdmdd_common_topaz_v1:chw.obj
 0001:0003babc       ?ClosePipe@CDummyPipe@@UAA?AW4HCD_REQUEST_STATUS@@XZ 1003cabc f i usbh_ehcdmdd_common_topaz_v1:chw.obj
 0001:0003bae4       ?IsPipeHalted@CDummyPipe@@UAA?AW4HCD_REQUEST_STATUS@@QAH@Z 1003cae4 f i usbh_ehcdmdd_common_topaz_v1:chw.obj
 0001:0003bb48       ?ClearHaltedFlag@CDummyPipe@@UAAXXZ 1003cb48 f i usbh_ehcdmdd_common_topaz_v1:chw.obj
 0001:0003bb5c       ?StopTransfers@CDummyPipe@@UAAXXZ 1003cb5c f i usbh_ehcdmdd_common_topaz_v1:chw.obj
 0001:0003bb70       ?AbortTransfer@CDummyPipe@@UAA?AW4HCD_REQUEST_STATUS@@Q6AKPAX@ZQAXPBX@Z 1003cb70 f i usbh_ehcdmdd_common_topaz_v1:chw.obj
 0001:0003bb98       ?GetCPhysMem@CDummyPipe@@UAAPAVCPhysMem@@XZ 1003cb98 f i usbh_ehcdmdd_common_topaz_v1:chw.obj
 0001:0003bbc8       ?ScheduleTransfer@CDummyPipe@@EAA?AW4HCD_REQUEST_STATUS@@XZ 1003cbc8 f i usbh_ehcdmdd_common_topaz_v1:chw.obj
 0001:0003bbf0       ?GetPipeType@CDummyPipe@@MBAPBGXZ 1003cbf0 f i usbh_ehcdmdd_common_topaz_v1:chw.obj
 0001:0003bc20       ?AreTransferParametersValid@CDummyPipe@@MBAHPBUSTRANSFER@@@Z 1003cc20 f i usbh_ehcdmdd_common_topaz_v1:chw.obj
 0001:0003bc48       ?CheckForDoneTransfers@CDummyPipe@@MAAHXZ 1003cc48 f i usbh_ehcdmdd_common_topaz_v1:chw.obj
 0001:0003bc70       ??_ECDummyPipe@@UAAPAXI@Z  1003cc70 f i usbh_ehcdmdd_common_topaz_v1:chw.obj
 0001:0003bc70       ??_GCDummyPipe@@UAAPAXI@Z  1003cc70 f i usbh_ehcdmdd_common_topaz_v1:chw.obj
 0001:0003bcb4       ??1CDummyPipe@@UAA@XZ      1003ccb4 f i usbh_ehcdmdd_common_topaz_v1:chw.obj
 0001:0003bce0       ??0CNextLinkPointer@@QAA@XZ 1003cce0 f i usbh_ehcdmdd_common_topaz_v1:chw.obj
 0001:0003bd14       ?GetDWORD@CNextLinkPointer@@QAAKXZ 1003cd14 f i usbh_ehcdmdd_common_topaz_v1:chw.obj
 0001:0003bd40       ?SetNextPointer@CNextLinkPointer@@QAAHKW4NEXTLINKTYPE@@H@Z 1003cd40 f i usbh_ehcdmdd_common_topaz_v1:chw.obj
 0001:0003bdac       ?SetLinkValid@CNextLinkPointer@@QAAHH@Z 1003cdac f i usbh_ehcdmdd_common_topaz_v1:chw.obj
 0001:0003be44       ?SetLinkType@CNextLinkPointer@@QAA?AW4NEXTLINKTYPE@@W42@@Z 1003ce44 f i usbh_ehcdmdd_common_topaz_v1:chw.obj
 0001:0003bea8       ?SetPointer@CNextLinkPointer@@QAAKK@Z 1003cea8 f i usbh_ehcdmdd_common_topaz_v1:chw.obj
 0001:0003bf4c       ?QueueQHead@CQH@@QAAHPAV1@@Z 1003cf4c f i usbh_ehcdmdd_common_topaz_v1:chw.obj
 0001:0003bfd8       ?SetDWORD@CNextLinkPointer@@QAAKK@Z 1003cfd8 f i usbh_ehcdmdd_common_topaz_v1:chw.obj
 0001:0003c018       ?GetLinkValid@CNextLinkPointer@@QAAHXZ 1003d018 f i usbh_ehcdmdd_common_topaz_v1:chw.obj
 0001:0003c064       ?GetPhysAddr@CITD@@QAAKXZ  1003d064 f i usbh_ehcdmdd_common_topaz_v1:chw.obj
 0001:0003c094       ?GetPhysAddr@CSITD@@QAAKXZ 1003d094 f i usbh_ehcdmdd_common_topaz_v1:chw.obj
 0001:0003c0cc       ?GetLinkType@CNextLinkPointer@@QAA?AW4NEXTLINKTYPE@@XZ 1003d0cc f i usbh_ehcdmdd_common_topaz_v1:chw.obj
 0001:0003c100       ?GetPointer@CNextLinkPointer@@QAAKXZ 1003d100 f i usbh_ehcdmdd_common_topaz_v1:chw.obj
 0001:0003c134       ?GetNextLinkPointer@CNextLinkPointer@@QAAPAV1@PAVCPhysMem@@@Z 1003d134 f i usbh_ehcdmdd_common_topaz_v1:chw.obj
 0001:0003c1f0       ?SetSMask@CQH@@QAAXE@Z     1003d1f0 f i usbh_ehcdmdd_common_topaz_v1:chw.obj
 0001:0003c238       ?GetNextQueueQHead@CQH@@QAAPAV1@QAVCPhysMem@@@Z 1003d238 f i usbh_ehcdmdd_common_topaz_v1:chw.obj
 0001:0003c2d8       ?SetReclamationFlag@CQH@@QAAXH@Z 1003d2d8 f i usbh_ehcdmdd_common_topaz_v1:chw.obj
 0001:0003c34c       ??0CRegistryEdit@@QAA@PAUHKEY__@@PBG@Z 1003d34c f i usbh_ehcdmdd_common_topaz_v1:chw.obj
 0001:0003c3c4       ??0CBusyPipeList@@QAA@K@Z  1003d3c4 f i usbh_ehcdmdd_common_topaz_v1:chw.obj
 0001:0003c408       ?Read_CapLength@CHW@@AAAEXZ 1003d408 f i usbh_ehcdmdd_common_topaz_v1:chw.obj
 0001:0003c43c       ?Read_HCSParams@CHW@@AAA?ATHCSPARAMS@1@XZ 1003d43c f i usbh_ehcdmdd_common_topaz_v1:chw.obj
 0001:0003c48c       ??_ECHW@@UAAPAXI@Z         1003d48c f i usbh_ehcdmdd_common_topaz_v1:chw.obj
 0001:0003c48c       ??_GCHW@@UAAPAXI@Z         1003d48c f i usbh_ehcdmdd_common_topaz_v1:chw.obj
 0001:0003c4d0       ??1CRegistryEdit@@QAA@XZ   1003d4d0 f i usbh_ehcdmdd_common_topaz_v1:chw.obj
 0001:0003c500       ??1CBusyPipeList@@QAA@XZ   1003d500 f i usbh_ehcdmdd_common_topaz_v1:chw.obj
 0001:0003c524       ?Read_USBCMD@CHW@@AAA?ATUSBCMD@1@XZ 1003d524 f i usbh_ehcdmdd_common_topaz_v1:chw.obj
 0001:0003c5c0       ?Write_USBCMD@CHW@@AAAXTUSBCMD@1@@Z 1003d5c0 f i usbh_ehcdmdd_common_topaz_v1:chw.obj
 0001:0003c690       ?Read_USBSTS@CHW@@AAA?ATUSBSTS@1@XZ 1003d690 f i usbh_ehcdmdd_common_topaz_v1:chw.obj
 0001:0003c784       ?Read_HHCCP_CAP@CHW@@AAA?ATHCCP_CAP@1@XZ 1003d784 f i usbh_ehcdmdd_common_topaz_v1:chw.obj
 0001:0003c7d4       ?Read_PORTSC@CHW@@AAA?ATPORTSC@1@I@Z 1003d7d4 f i usbh_ehcdmdd_common_topaz_v1:chw.obj
 0001:0003c8dc       ?Write_PORTSC@CHW@@AAAXITPORTSC@1@@Z 1003d8dc f i usbh_ehcdmdd_common_topaz_v1:chw.obj
 0001:0003c9c8       ?Write_EHCIRegister@CHW@@AAAXKK@Z 1003d9c8 f i usbh_ehcdmdd_common_topaz_v1:chw.obj
 0001:0003ca4c       ?GetFrameListPhysAddr@CPeriodicMgr@@QAAKXZ 1003da4c f i usbh_ehcdmdd_common_topaz_v1:chw.obj
 0001:0003ca7c       ?GetPhysAddr@CAsyncMgr@@QAAKXZ 1003da7c f i usbh_ehcdmdd_common_topaz_v1:chw.obj
 0001:0003cae0       ?Write_USBINTR@CHW@@AAAXTUSBINTR@1@@Z 1003dae0 f i usbh_ehcdmdd_common_topaz_v1:chw.obj
 0001:0003cb64       ?Write_FRINDEX@CHW@@AAAXTFRINDEX@1@@Z 1003db64 f i usbh_ehcdmdd_common_topaz_v1:chw.obj
 0001:0003cbe4       ?Read_EHCIRegister@CHW@@AAAKK@Z 1003dbe4 f i usbh_ehcdmdd_common_topaz_v1:chw.obj
 0001:0003cc70       ?Read_TXFILLTUNING@CHW@@AAA?ATTXFILLTUNING@1@XZ 1003dc70 f i usbh_ehcdmdd_common_topaz_v1:chw.obj
 0001:0003ccc0       ?Write_TXFILLTUNING@CHW@@AAAXTTXFILLTUNING@1@@Z 1003dcc0 f i usbh_ehcdmdd_common_topaz_v1:chw.obj
 0001:0003ccec       ?GetRegValue@CRegistryEdit@@QAAHPBGPAEK@Z 1003dcec f i usbh_ehcdmdd_common_topaz_v1:chw.obj
 0001:0003cd70       ?IsKeyOpened@CRegistryEdit@@QAAHXZ 1003dd70 f i usbh_ehcdmdd_common_topaz_v1:chw.obj
 0001:0003cdbc       ?Clear_USBSTS@CHW@@AAAXXZ  1003ddbc f i usbh_ehcdmdd_common_topaz_v1:chw.obj
 0001:0003ce10       ?Write_USBSTS@CHW@@AAAXTUSBSTS@1@@Z 1003de10 f i usbh_ehcdmdd_common_topaz_v1:chw.obj
 0001:0003ce94       ?Read_FRINDEX@CHW@@AAA?ATFRINDEX@1@XZ 1003de94 f i usbh_ehcdmdd_common_topaz_v1:chw.obj
 0001:0003cf34       ?Read_OTGSC@CHW@@AAA?ATOTGSC@1@XZ 1003df34 f i usbh_ehcdmdd_common_topaz_v1:chw.obj
 0001:0003cfd4       ?Read_USBINTR@CHW@@AAA?ATUSBINTR@1@XZ 1003dfd4 f i usbh_ehcdmdd_common_topaz_v1:chw.obj
 0001:0003d074       ??0CTransfer@@QAA@QAVCPipe@@QAVCPhysMem@@PAUSTRANSFER@@@Z 1003e074 f   usbh_ehcdmdd_common_topaz_v1:trans.obj
 0001:0003d15c       ??1CTransfer@@UAA@XZ       1003e15c f   usbh_ehcdmdd_common_topaz_v1:trans.obj
 0001:0003d270       ?Init@CTransfer@@UAAHXZ    1003e270 f   usbh_ehcdmdd_common_topaz_v1:trans.obj
 0001:0003d868       ??1CQTransfer@@UAA@XZ      1003e868 f   usbh_ehcdmdd_common_topaz_v1:trans.obj
 0001:0003d918       ?AddTransfer@CQTransfer@@UAAHXZ 1003e918 f   usbh_ehcdmdd_common_topaz_v1:trans.obj
 0001:0003e470       ?DoneTransfer@CQTransfer@@QAAHXZ 1003f470 f   usbh_ehcdmdd_common_topaz_v1:trans.obj
 0001:0003e8d4       ?AbortTransfer@CQTransfer@@QAAHXZ 1003f8d4 f   usbh_ehcdmdd_common_topaz_v1:trans.obj
 0001:0003e994       ?IsTransferDone@CQTransfer@@QAAHXZ 1003f994 f   usbh_ehcdmdd_common_topaz_v1:trans.obj
 0001:0003ec7c       ??0CIsochTransfer@@QAA@QAVCIsochronousPipe@@QAVCEhcd@@PAUSTRANSFER@@@Z 1003fc7c f   usbh_ehcdmdd_common_topaz_v1:trans.obj
 0001:0003ed70       ??0CITransfer@@QAA@QAVCIsochronousPipe@@QAVCEhcd@@PAUSTRANSFER@@@Z 1003fd70 f   usbh_ehcdmdd_common_topaz_v1:trans.obj
 0001:0003ee6c       ??1CITransfer@@UAA@XZ      1003fe6c f   usbh_ehcdmdd_common_topaz_v1:trans.obj
 0001:0003f0e8       ?ArmTD@CITransfer@@QAAHXZ  100400e8 f   usbh_ehcdmdd_common_topaz_v1:trans.obj
 0001:0003f5b4       ?AddTransfer@CITransfer@@UAAHXZ 100405b4 f   usbh_ehcdmdd_common_topaz_v1:trans.obj
 0001:0003f844       ?ScheduleTD@CITransfer@@UAAHKK@Z 10040844 f   usbh_ehcdmdd_common_topaz_v1:trans.obj
 0001:0003fc2c       ?IsTransferDone@CITransfer@@UAAHKK@Z 10040c2c f   usbh_ehcdmdd_common_topaz_v1:trans.obj
 0001:000402f0       ?AbortTransfer@CITransfer@@UAAHXZ 100412f0 f   usbh_ehcdmdd_common_topaz_v1:trans.obj
 0001:00040650       ?DoneTransfer@CITransfer@@UAAHKK@Z 10041650 f   usbh_ehcdmdd_common_topaz_v1:trans.obj
 0001:000408f8       ??0CSITransfer@@QAA@QAVCIsochronousPipe@@QAVCEhcd@@PAUSTRANSFER@@@Z 100418f8 f   usbh_ehcdmdd_common_topaz_v1:trans.obj
 0001:00040958       ??1CSITransfer@@UAA@XZ     10041958 f   usbh_ehcdmdd_common_topaz_v1:trans.obj
 0001:00040b98       ?ArmTD@CSITransfer@@QAAHXZ 10041b98 f   usbh_ehcdmdd_common_topaz_v1:trans.obj
 0001:00040ec8       ?AddTransfer@CSITransfer@@UAAHXZ 10041ec8 f   usbh_ehcdmdd_common_topaz_v1:trans.obj
 0001:00041134       ?ScheduleTD@CSITransfer@@UAAHKK@Z 10042134 f   usbh_ehcdmdd_common_topaz_v1:trans.obj
 0001:0004152c       ?IsTransferDone@CSITransfer@@UAAHKK@Z 1004252c f   usbh_ehcdmdd_common_topaz_v1:trans.obj
 0001:00041c40       ?AbortTransfer@CSITransfer@@UAAHXZ 10042c40 f   usbh_ehcdmdd_common_topaz_v1:trans.obj
 0001:00041f44       ?DoneTransfer@CSITransfer@@UAAHKK@Z 10042f44 f   usbh_ehcdmdd_common_topaz_v1:trans.obj
 0001:00042200       ??_ECTransfer@@UAAPAXI@Z   10043200 f i usbh_ehcdmdd_common_topaz_v1:trans.obj
 0001:00042200       ??_GCTransfer@@UAAPAXI@Z   10043200 f i usbh_ehcdmdd_common_topaz_v1:trans.obj
 0001:00042244       ?GetNextTD@CQTD@@QAAPAV1@XZ 10043244 f i usbh_ehcdmdd_common_topaz_v1:trans.obj
 0001:0004227c       ??_GCQTD@@QAAPAXI@Z        1004327c f i usbh_ehcdmdd_common_topaz_v1:trans.obj
 0001:000422c0       ??1CQTD@@QAA@XZ            100432c0 f i usbh_ehcdmdd_common_topaz_v1:trans.obj
 0001:000422dc       ?GetPhysAddr@CQTD@@QAAKXZ  100432dc f i usbh_ehcdmdd_common_topaz_v1:trans.obj
 0001:00042314       ?SetAltNextQTDPointer@CQTD@@QAAXK@Z 10043314 f i usbh_ehcdmdd_common_topaz_v1:trans.obj
 0001:0004238c       ?GetEndptDescriptor@CPipe@@QAA?AU_USB_ENDPOINT_DESCRIPTOR@@XZ 1004338c f i usbh_ehcdmdd_common_topaz_v1:trans.obj
 0001:000423c8       ?DeActiveTD@CQTD@@QAAXXZ   100433c8 f i usbh_ehcdmdd_common_topaz_v1:trans.obj
 0001:00042410       ??_ECIsochTransfer@@UAAPAXI@Z 10043410 f i usbh_ehcdmdd_common_topaz_v1:trans.obj
 0001:00042410       ??_GCIsochTransfer@@UAAPAXI@Z 10043410 f i usbh_ehcdmdd_common_topaz_v1:trans.obj
 0001:00042454       ??1CIsochTransfer@@UAA@XZ  10043454 f i usbh_ehcdmdd_common_topaz_v1:trans.obj
 0001:00042578       ?GetMaxTransferPerItd@CIsochTransfer@@QAAKXZ 10043578 f i usbh_ehcdmdd_common_topaz_v1:trans.obj
 0001:000425b8       ?GetPipe@CIsochTransfer@@QAAQAVCIsochronousPipe@@XZ 100435b8 f i usbh_ehcdmdd_common_topaz_v1:trans.obj
 0001:000425e8       ?GetMaxTransferPerItd@CIsochronousPipe@@QAAKXZ 100435e8 f i usbh_ehcdmdd_common_topaz_v1:trans.obj
 0001:00042618       ??_GCITransfer@@UAAPAXI@Z  10043618 f i usbh_ehcdmdd_common_topaz_v1:trans.obj
 0001:00042618       ??_ECITransfer@@UAAPAXI@Z  10043618 f i usbh_ehcdmdd_common_topaz_v1:trans.obj
 0001:0004265c       ?GetFrameSize@CPeriodicMgr@@QAAKXZ 1004365c f i usbh_ehcdmdd_common_topaz_v1:trans.obj
 0001:0004268c       ?GetPeriodicMgr@CHW@@QAAAAVCPeriodicMgr@@XZ 1004368c f i usbh_ehcdmdd_common_topaz_v1:trans.obj
 0001:000426b8       ??_ECSITransfer@@UAAPAXI@Z 100436b8 f i usbh_ehcdmdd_common_topaz_v1:trans.obj
 0001:000426b8       ??_GCSITransfer@@UAAPAXI@Z 100436b8 f i usbh_ehcdmdd_common_topaz_v1:trans.obj
 0001:000426fc       ?SetIOC@CSITD@@QAAXH@Z     100436fc f i usbh_ehcdmdd_common_topaz_v1:trans.obj
 0001:00042770       ??2CNextLinkPointer@@SAPAXIQAVCPhysMem@@@Z 10043770 f   usbh_ehcdmdd_common_topaz_v1:ctd.obj
 0001:00042878       ??3CNextLinkPointer@@SAXPAX@Z 10043878 f   usbh_ehcdmdd_common_topaz_v1:ctd.obj
 0001:000428d0       ??0CITD@@QAA@PAVCITransfer@@@Z 100438d0 f   usbh_ehcdmdd_common_topaz_v1:ctd.obj
 0001:00042a8c       ?ReInit@CITD@@QAAXPAVCITransfer@@@Z 10043a8c f   usbh_ehcdmdd_common_topaz_v1:ctd.obj
 0001:00042bdc       ?SetIOC@CITD@@QAAXH@Z      10043bdc f   usbh_ehcdmdd_common_topaz_v1:ctd.obj
 0001:00042d30       ?IssueTransfer@CITD@@QAAKKPAK0HH@Z 10043d30 f   usbh_ehcdmdd_common_topaz_v1:ctd.obj
 0001:00043428       ??0CSITD@@QAA@PAVCSITransfer@@PAV0@@Z 10044428 f   usbh_ehcdmdd_common_topaz_v1:ctd.obj
 0001:00043704       ?ReInit@CSITD@@QAAXPAVCSITransfer@@PAV1@@Z 10044704 f   usbh_ehcdmdd_common_topaz_v1:ctd.obj
 0001:000439bc       ?IssueTransfer@CSITD@@QAAKKKKHH@Z 100449bc f   usbh_ehcdmdd_common_topaz_v1:ctd.obj
 0001:00043ec8       ??0CQTD@@QAA@PAVCQTransfer@@PAVCQH@@@Z 10044ec8 f   usbh_ehcdmdd_common_topaz_v1:ctd.obj
 0001:000440cc       ?IssueTransfer@CQTD@@QAAKKHKPAUPhysBufferArray@@H@Z 100450cc f   usbh_ehcdmdd_common_topaz_v1:ctd.obj
 0001:00044560       ?QueueNextTD@CQTD@@QAAPAV1@PAV1@@Z 10045560 f   usbh_ehcdmdd_common_topaz_v1:ctd.obj
 0001:000445d0       ??0CQH@@QAA@PAVCPipe@@@Z   100455d0 f   usbh_ehcdmdd_common_topaz_v1:ctd.obj
 0001:00044b04       ?QueueTD@CQH@@QAAHPAVCQTD@@@Z 10045b04 f   usbh_ehcdmdd_common_topaz_v1:ctd.obj
 0001:00044c4c       ?GetDeviceAddress@CPipe@@QAAEXZ 10045c4c f i usbh_ehcdmdd_common_topaz_v1:ctd.obj
 0001:00044c7c       ?GetSMask@CPipe@@QAAEXZ    10045c7c f i usbh_ehcdmdd_common_topaz_v1:ctd.obj
 0001:00044cac       ?GetCMask@CPipe@@QAAEXZ    10045cac f i usbh_ehcdmdd_common_topaz_v1:ctd.obj
 0001:00044cdc       ?IsHighSpeed@CPipe@@QAAHXZ 10045cdc f i usbh_ehcdmdd_common_topaz_v1:ctd.obj
 0001:00044d0c       ?IsLowSpeed@CPipe@@QAAHXZ  10045d0c f i usbh_ehcdmdd_common_topaz_v1:ctd.obj
 0001:00044d3c       HcdPdd_DllMain             10045d3c f   usbh_ehcdpdd_common_topaz_v1:system.obj
 0001:00044d7c       ConfigureEHCICard          10045d7c f   usbh_ehcdpdd_common_topaz_v1:system.obj
 0001:00044ed8       HcdPdd_Init                10045ed8 f   usbh_ehcdpdd_common_topaz_v1:system.obj
 0001:000458ac       HcdPdd_CheckConfigPower    100468ac f   usbh_ehcdpdd_common_topaz_v1:system.obj
 0001:000458e8       HcdPdd_PowerUp             100468e8 f   usbh_ehcdpdd_common_topaz_v1:system.obj
 0001:0004591c       HcdPdd_PowerDown           1004691c f   usbh_ehcdpdd_common_topaz_v1:system.obj
 0001:00045950       HcdPdd_Deinit              10046950 f   usbh_ehcdpdd_common_topaz_v1:system.obj
 0001:00045a7c       HcdPdd_Open                10046a7c f   usbh_ehcdpdd_common_topaz_v1:system.obj
 0001:00045abc       HcdPdd_Close               10046abc f   usbh_ehcdpdd_common_topaz_v1:system.obj
 0001:00045aec       HcdPdd_Read                10046aec f   usbh_ehcdpdd_common_topaz_v1:system.obj
 0001:00045b2c       HcdPdd_Write               10046b2c f   usbh_ehcdpdd_common_topaz_v1:system.obj
 0001:00045b6c       HcdPdd_Seek                10046b6c f   usbh_ehcdpdd_common_topaz_v1:system.obj
 0001:00045bac       HcdPdd_IOControl           10046bac f   usbh_ehcdpdd_common_topaz_v1:system.obj
 0001:00045c80       HcdPdd_InitiatePowerUp     10046c80 f   usbh_ehcdpdd_common_topaz_v1:system.obj
 0001:00045c94       KernelIoControl            10046c94 f   coredll:COREDLL.dll
 0001:00045ca4       NKDbgPrintfW               10046ca4 f   coredll:COREDLL.dll
 0001:00045cb4       StringCchCopyW             10046cb4 f   coredll:COREDLL.dll
 0001:00045cc4       Sleep                      10046cc4 f   coredll:COREDLL.dll
 0001:00045cd4       InterlockedCompareExchange 10046cd4 f   coredll:COREDLL.dll
 0001:00045ce4       GetLastError               10046ce4 f   coredll:COREDLL.dll
 0001:00045cf4       MapViewOfFile              10046cf4 f   coredll:COREDLL.dll
 0001:00045d04       CreateFileMappingW         10046d04 f   coredll:COREDLL.dll
 0001:00045d14       CloseHandle                10046d14 f   coredll:COREDLL.dll
 0001:00045d24       UnmapViewOfFile            10046d24 f   coredll:COREDLL.dll
 0001:00045d34       DeleteCriticalSection      10046d34 f   coredll:COREDLL.dll
 0001:00045d44       InitializeCriticalSection  10046d44 f   coredll:COREDLL.dll
 0001:00045d54       DisableThreadLibraryCalls  10046d54 f   coredll:COREDLL.dll
 0001:00045d64       RegisterDbgZones           10046d64 f   coredll:COREDLL.dll
 0001:00045d74       LeaveCriticalSection       10046d74 f   coredll:COREDLL.dll
 0001:00045d84       EnterCriticalSection       10046d84 f   coredll:COREDLL.dll
 0001:00045d94       RegCloseKey                10046d94 f   coredll:COREDLL.dll
 0001:00045da4       RegQueryValueExW           10046da4 f   coredll:COREDLL.dll
 0001:00045db4       RegOpenKeyExW              10046db4 f   coredll:COREDLL.dll
 0001:00045dc4       OpenDeviceKey              10046dc4 f   coredll:COREDLL.dll
 0001:00045dd4       CreateEventW               10046dd4 f   coredll:COREDLL.dll
 0001:00045de4       AllocPhysMem               10046de4 f   coredll:COREDLL.dll
 0001:00045df4       LocalAlloc                 10046df4 f   coredll:COREDLL.dll
 0001:00045e04       FreePhysMem                10046e04 f   coredll:COREDLL.dll
 0001:00045e14       LocalFree                  10046e14 f   coredll:COREDLL.dll
 0001:00045e24       WaitForSingleObject        10046e24 f   coredll:COREDLL.dll
 0001:00045e34       GetTickCount               10046e34 f   coredll:COREDLL.dll
 0001:00045e44       EventModify                10046e44 f   coredll:COREDLL.dll
 0001:00045e54       GetProcAddressW            10046e54 f   coredll:COREDLL.dll
 0001:00045e64       LoadDriver                 10046e64 f   coredll:COREDLL.dll
 0001:00045e74       FreeLibrary                10046e74 f   coredll:COREDLL.dll
 0001:00045e84       StringCchCatW              10046e84 f   coredll:COREDLL.dll
 0001:00045e94       SetLastError               10046e94 f   coredll:COREDLL.dll
 0001:00045ea4       LoadLibraryW               10046ea4 f   coredll:COREDLL.dll
 0001:00045eb4       CeGetThreadPriority        10046eb4 f   coredll:COREDLL.dll
 0001:00045ec4       CeSetThreadPriority        10046ec4 f   coredll:COREDLL.dll
 0001:00045ed4       CreateThread               10046ed4 f   coredll:COREDLL.dll
 0001:00045ee4       __GetUserKData             10046ee4 f   coredll:COREDLL.dll
 0001:00045ef4       RaiseException             10046ef4 f   coredll:COREDLL.dll
 0001:00045f04       TerminateThread            10046f04 f   coredll:COREDLL.dll
 0001:00045f14       InterruptInitialize        10046f14 f   coredll:COREDLL.dll
 0001:00045f24       InterruptDisable           10046f24 f   coredll:COREDLL.dll
 0001:00045f34       ExitThread                 10046f34 f   coredll:COREDLL.dll
 0001:00045f44       InterruptDone              10046f44 f   coredll:COREDLL.dll
 0001:00045f54       WaitForMultipleObjects     10046f54 f   coredll:COREDLL.dll
 0001:00045f64       SetInterruptEvent          10046f64 f   coredll:COREDLL.dll
 0001:00045f74       FreeIntChainHandler        10046f74 f   coredll:COREDLL.dll
 0001:00045f84       StringCchCopyNW            10046f84 f   coredll:COREDLL.dll
 0001:00045f94       DDKReg_GetIsrInfo          10046f94 f   coredll:COREDLL.dll
 0001:00045fa4       DDKReg_GetWindowInfo       10046fa4 f   coredll:COREDLL.dll
 0001:00045fb4       StallExecution             10046fb4 f   ceddk:CEDDK.dll
 0001:00045fc4       BusTransBusAddrToVirtual   10046fc4 f   ceddk:CEDDK.dll
 0001:00045fd4       CloseBusAccessHandle       10046fd4 f   ceddk:CEDDK.dll
 0001:00045fe4       CreateBusAccessHandle      10046fe4 f   ceddk:CEDDK.dll
 0001:00045ff4       HalFreeCommonBuffer        10046ff4 f   ceddk:CEDDK.dll
 0001:00046004       HalAllocateCommonBuffer    10047004 f   ceddk:CEDDK.dll
 0001:00046014       DDKIomuxSelectInput        10047014 f   cspddk:CSPDDK.dll
 0001:00046024       DDKGpioWriteDataPin        10047024 f   cspddk:CSPDDK.dll
 0001:00046034       DDKGpioSetConfig           10047034 f   cspddk:CSPDDK.dll
 0001:00046044       DDKIomuxSetPadConfig       10047044 f   cspddk:CSPDDK.dll
 0001:00046054       DDKIomuxSetPinMux          10047054 f   cspddk:CSPDDK.dll
 0001:00046064       DDKClockSetGatingMode      10047064 f   cspddk:CSPDDK.dll
 0001:00046074       DDKClockGetGatingMode      10047074 f   cspddk:CSPDDK.dll
 0001:00046084       DDKClockConfigBaud         10047084 f   cspddk:CSPDDK.dll
 0001:00046094       _DllMainCRTStartup         10047094 f   corelib0:pegdmain.obj
 0001:0004623c       __security_init_cookie     1004723c f   corelib0:seccinit.obj
 0001:00046304       __GSHandlerCheck           10047304 f   corelib0:gshandler.obj
 0001:0004634c       __GSHandlerCheckCommon     1004734c f   corelib0:gshandler.obj
 0001:000463f4       __security_check_cookie    100473f4 f   corelib0:armsecgs.obj
 0001:00046408       __gsfailure                10047408 f   corelib0:armsecgs.obj
 0001:0004644c       exit                       1004744c f   corelib0:cexit.obj
 0001:000465cc       _exit                      100475cc f   corelib0:cexit.obj
 0001:000465f0       _cexit                     100475f0 f   corelib0:cexit.obj
 0001:0004660c       _c_exit                    1004760c f   corelib0:cexit.obj
 0001:00046628       GetCurrentProcess          10047628 f i corelib0:cexit.obj
 0001:00046640       _initterm                  10047640 f   corelib0:crt0dat.obj
 0001:00046694       _cinit                     10047694 f   corelib0:crt0dat.obj
 0001:000466d0       _onexit                    100476d0 f   corelib0:onexit.obj
 0001:000469d4       atexit                     100479d4 f   corelib0:onexit.obj
 0001:00046a28       ??2@YAPAXI@Z               10047a28 f   corelib1:COREDLL.dll
 0001:00046a38       ??3@YAXPAX@Z               10047a38 f   corelib1:COREDLL.dll
 0001:00046a48       _purecall                  10047a48 f   corelib1:COREDLL.dll
 0001:00046a58       memset                     10047a58 f   corelib1:COREDLL.dll
 0001:00046a68       __rt_udiv                  10047a68 f   corelib1:COREDLL.dll
 0001:00046a78       wcslen                     10047a78 f   corelib1:COREDLL.dll
 0001:00046a88       memcpy                     10047a88 f   corelib1:COREDLL.dll
 0001:00046a98       memcmp                     10047a98 f   corelib1:COREDLL.dll
 0001:00046aa8       __C_specific_handler       10047aa8 f   corelib1:COREDLL.dll
 0001:00046ab8       __rt_sdiv                  10047ab8 f   corelib1:COREDLL.dll
 0001:00046ac8       free                       10047ac8 f   corelib1:COREDLL.dll
 0001:00046ad8       malloc                     10047ad8 f   corelib1:COREDLL.dll
 0001:00046ae8       _XcptFilter                10047ae8 f   corelib1:COREDLL.dll
 0001:00046af8       __security_gen_cookie2     10047af8 f   corelib1:COREDLL.dll
 0001:00046b08       __report_gsfailure         10047b08 f   corelib1:COREDLL.dll
 0001:00046b18       realloc                    10047b18 f   corelib1:COREDLL.dll
 0001:00046b28       _msize                     10047b28 f   corelib1:COREDLL.dll
 0001:00046b38       InterlockedExchange        10047b38 f   coredll:COREDLL.dll
 0001:00046b48       TerminateProcess           10047b48 f   coredll:COREDLL.dll
 0001:00046d8c       __IMPORT_DESCRIPTOR_COREDLL 10047d8c     coredll:COREDLL.dll
 0001:00046da0       __IMPORT_DESCRIPTOR_CEDDK  10047da0     ceddk:CEDDK.dll
 0001:00046db4       __IMPORT_DESCRIPTOR_CSPDDK 10047db4     cspddk:CSPDDK.dll
 0001:00046dc8       __NULL_IMPORT_DESCRIPTOR   10047dc8     coredll:COREDLL.dll
 0002:00000000       __imp_HalFreeCommonBuffer  10049000     ceddk:CEDDK.dll
 0002:00000004       __imp_CreateBusAccessHandle 10049004     ceddk:CEDDK.dll
 0002:00000008       __imp_CloseBusAccessHandle 10049008     ceddk:CEDDK.dll
 0002:0000000c       __imp_BusTransBusAddrToVirtual 1004900c     ceddk:CEDDK.dll
 0002:00000010       __imp_StallExecution       10049010     ceddk:CEDDK.dll
 0002:00000014       __imp_HalAllocateCommonBuffer 10049014     ceddk:CEDDK.dll
 0002:00000018       \177CEDDK_NULL_THUNK_DATA  10049018     ceddk:CEDDK.dll
 0002:0000001c       __imp_CreateFileMappingW   1004901c     coredll:COREDLL.dll
 0002:00000020       __imp_CloseHandle          10049020     coredll:COREDLL.dll
 0002:00000024       __imp_UnmapViewOfFile      10049024     coredll:COREDLL.dll
 0002:00000028       __imp_DeleteCriticalSection 10049028     coredll:COREDLL.dll
 0002:0000002c       __imp_InitializeCriticalSection 1004902c     coredll:COREDLL.dll
 0002:00000030       __imp_DisableThreadLibraryCalls 10049030     coredll:COREDLL.dll
 0002:00000034       __imp_RegisterDbgZones     10049034     coredll:COREDLL.dll
 0002:00000038       __imp_LeaveCriticalSection 10049038     coredll:COREDLL.dll
 0002:0000003c       __imp_EnterCriticalSection 1004903c     coredll:COREDLL.dll
 0002:00000040       __imp_RegCloseKey          10049040     coredll:COREDLL.dll
 0002:00000044       __imp_RegQueryValueExW     10049044     coredll:COREDLL.dll
 0002:00000048       __imp_RegOpenKeyExW        10049048     coredll:COREDLL.dll
 0002:0000004c       __imp_OpenDeviceKey        1004904c     coredll:COREDLL.dll
 0002:00000050       __imp_CreateEventW         10049050     coredll:COREDLL.dll
 0002:00000054       __imp_AllocPhysMem         10049054     coredll:COREDLL.dll
 0002:00000058       __imp_LocalAlloc           10049058     coredll:COREDLL.dll
 0002:0000005c       __imp_FreePhysMem          1004905c     coredll:COREDLL.dll
 0002:00000060       __imp_LocalFree            10049060     coredll:COREDLL.dll
 0002:00000064       __imp_WaitForSingleObject  10049064     coredll:COREDLL.dll
 0002:00000068       __imp_GetTickCount         10049068     coredll:COREDLL.dll
 0002:0000006c       __imp_EventModify          1004906c     coredll:COREDLL.dll
 0002:00000070       __imp_MapViewOfFile        10049070     coredll:COREDLL.dll
 0002:00000074       __imp_LoadDriver           10049074     coredll:COREDLL.dll
 0002:00000078       __imp_FreeLibrary          10049078     coredll:COREDLL.dll
 0002:0000007c       __imp_StringCchCatW        1004907c     coredll:COREDLL.dll
 0002:00000080       __imp_SetLastError         10049080     coredll:COREDLL.dll
 0002:00000084       __imp_LoadLibraryW         10049084     coredll:COREDLL.dll
 0002:00000088       __imp_CeGetThreadPriority  10049088     coredll:COREDLL.dll
 0002:0000008c       __imp_CeSetThreadPriority  1004908c     coredll:COREDLL.dll
 0002:00000090       __imp_CreateThread         10049090     coredll:COREDLL.dll
 0002:00000094       __imp___GetUserKData       10049094     coredll:COREDLL.dll
 0002:00000098       __imp_RaiseException       10049098     coredll:COREDLL.dll
 0002:0000009c       __imp_TerminateThread      1004909c     coredll:COREDLL.dll
 0002:000000a0       __imp_InterruptInitialize  100490a0     coredll:COREDLL.dll
 0002:000000a4       __imp_InterruptDisable     100490a4     coredll:COREDLL.dll
 0002:000000a8       __imp_ExitThread           100490a8     coredll:COREDLL.dll
 0002:000000ac       __imp_InterruptDone        100490ac     coredll:COREDLL.dll
 0002:000000b0       __imp_WaitForMultipleObjects 100490b0     coredll:COREDLL.dll
 0002:000000b4       __imp_SetInterruptEvent    100490b4     coredll:COREDLL.dll
 0002:000000b8       __imp_FreeIntChainHandler  100490b8     coredll:COREDLL.dll
 0002:000000bc       __imp_StringCchCopyNW      100490bc     coredll:COREDLL.dll
 0002:000000c0       __imp_DDKReg_GetIsrInfo    100490c0     coredll:COREDLL.dll
 0002:000000c4       __imp_DDKReg_GetWindowInfo 100490c4     coredll:COREDLL.dll
 0002:000000c8       __imp_GetLastError         100490c8     coredll:COREDLL.dll
 0002:000000cc       __imp_InterlockedCompareExchange 100490cc     coredll:COREDLL.dll
 0002:000000d0       __imp_Sleep                100490d0     coredll:COREDLL.dll
 0002:000000d4       __imp_StringCchCopyW       100490d4     coredll:COREDLL.dll
 0002:000000d8       __imp_NKDbgPrintfW         100490d8     coredll:COREDLL.dll
 0002:000000dc       __imp_GetProcAddressW      100490dc     coredll:COREDLL.dll
 0002:000000e0       __imp_KernelIoControl      100490e0     coredll:COREDLL.dll
 0002:000000e4       __imp_InterlockedExchange  100490e4     coredll:COREDLL.dll
 0002:000000e8       __imp__msize               100490e8     corelib1:COREDLL.dll
 0002:000000ec       __imp_realloc              100490ec     corelib1:COREDLL.dll
 0002:000000f0       __imp___report_gsfailure   100490f0     corelib1:COREDLL.dll
 0002:000000f4       __imp___security_gen_cookie2 100490f4     corelib1:COREDLL.dll
 0002:000000f8       __imp__XcptFilter          100490f8     corelib1:COREDLL.dll
 0002:000000fc       __imp_malloc               100490fc     corelib1:COREDLL.dll
 0002:00000100       __imp_free                 10049100     corelib1:COREDLL.dll
 0002:00000104       __imp___rt_sdiv            10049104     corelib1:COREDLL.dll
 0002:00000108       __imp_??2@YAPAXI@Z         10049108     corelib1:COREDLL.dll
 0002:0000010c       __imp_??3@YAXPAX@Z         1004910c     corelib1:COREDLL.dll
 0002:00000110       __imp__purecall            10049110     corelib1:COREDLL.dll
 0002:00000114       __imp_memset               10049114     corelib1:COREDLL.dll
 0002:00000118       __imp___rt_udiv            10049118     corelib1:COREDLL.dll
 0002:0000011c       __imp_wcslen               1004911c     corelib1:COREDLL.dll
 0002:00000120       __imp_memcpy               10049120     corelib1:COREDLL.dll
 0002:00000124       __imp_memcmp               10049124     corelib1:COREDLL.dll
 0002:00000128       __imp___C_specific_handler 10049128     corelib1:COREDLL.dll
 0002:0000012c       __imp_TerminateProcess     1004912c     coredll:COREDLL.dll
 0002:00000130       \177COREDLL_NULL_THUNK_DATA 10049130     coredll:COREDLL.dll
 0002:00000134       __imp_DDKClockConfigBaud   10049134     cspddk:CSPDDK.dll
 0002:00000138       __imp_DDKClockGetGatingMode 10049138     cspddk:CSPDDK.dll
 0002:0000013c       __imp_DDKClockSetGatingMode 1004913c     cspddk:CSPDDK.dll
 0002:00000140       __imp_DDKIomuxSetPinMux    10049140     cspddk:CSPDDK.dll
 0002:00000144       __imp_DDKIomuxSetPadConfig 10049144     cspddk:CSPDDK.dll
 0002:00000148       __imp_DDKGpioSetConfig     10049148     cspddk:CSPDDK.dll
 0002:0000014c       __imp_DDKGpioWriteDataPin  1004914c     cspddk:CSPDDK.dll
 0002:00000150       __imp_DDKIomuxSelectInput  10049150     cspddk:CSPDDK.dll
 0002:00000154       \177CSPDDK_NULL_THUNK_DATA 10049154     cspddk:CSPDDK.dll
 0002:000001b8       dpCurSettings              100491b8     usbh_usb2com_common_topaz_v1:hcddrv.obj
 0002:000005fc       ?gc_HcdFuncs@@3U_HCD_FUNCS@@A 100495fc     usbh_usb2com_common_topaz_v1:hcddrv.obj
 0002:000006f0       ?cszDeviceType@?1??GetDeviceType@CRootHub@@EBAPBGXZ@4PBGB 100496f0     usbh_usb2com_common_topaz_v1:cdevice.obj
 0002:000006f8       ?cszDeviceType@?1??GetDeviceType@CExternalHub@@EBAPBGXZ@4PBGB 100496f8     usbh_usb2com_common_topaz_v1:cdevice.obj
 0002:000006fc       ?cszDeviceType@?1??GetDeviceType@CFunction@@EBAPBGXZ@4PBGB 100496fc     usbh_usb2com_common_topaz_v1:cdevice.obj
 0002:000007b0       ?cszPipeType@?1??GetPipeType@CInterruptPipe@@UBAPBGXZ@4PBGB 100497b0     usbh_ehcdmdd_common_topaz_v1:cpipe.obj
 0002:000007b4       ?cszPipeType@?1??GetPipeType@CIsochronousPipe@@UBAPBGXZ@4PBGB 100497b4     usbh_ehcdmdd_common_topaz_v1:cpipe.obj
 0002:000007b8       ?CMASKS@USB2lib@@0PAEA     100497b8     usbh_ehcdmdd_common_topaz_v1:usb2lib.obj
 0002:00000818       ?periodTable@CPeriodicMgr@@0PAU_PERIOD_TABLE@@A 10049818     usbh_ehcdmdd_common_topaz_v1:chw.obj
 0002:000008d8       ?cszPipeType@?1??GetPipeType@CDummyPipe@@MBAPBGXZ@4PBGB 100498d8     usbh_ehcdmdd_common_topaz_v1:chw.obj
 0002:00000938       __security_cookie          10049938     corelib0:seccinit.obj
 0002:0000093c       __security_cookie_complement 1004993c     corelib0:seccinit.obj
 0002:00000940       m_hUSBClockGatingHandle    10049940     i_usbclock.obj
 0002:00000944       pUSBClkGating              10049944     i_usbclock.obj
 0002:00000948       g_IstThreadPriority        10049948     usbh_usb2com_common_topaz_v1:hcddrv.obj
 0002:0000094c       ?g_CSection@@3UCRITICAL_SECTION@@A 1004994c     usbh_usb2com_common_topaz_v1:hcddrv.obj
 0002:00000960       g_dwContext                10049960     usbh_usb2com_common_topaz_v1:hcddrv.obj
 0002:00000964       ?ghDetach@@3PAXA           10049964     usbh_usb2com_common_topaz_v1:cdevice.obj
 0002:00000968       ?m_dwGlobalTransferID@CTransfer@@1KA 10049968     usbh_ehcdmdd_common_topaz_v1:trans.obj
 0002:0000096c       _exitflag                  1004996c     corelib0:cexit.obj
 0002:0000096e       gSel                       1004996e     <common>
 0002:00000970       gQueueHead                 10049970     <common>
 0002:00000980       gszOTGGroup                10049980     <common>
 0002:000009bc       gRegs                      100499bc     <common>
 0002:000009c0       gdwOTGSupport              100499c0     <common>
 0002:000009c4       __onexitend                100499c4     <common>
 0002:000009c8       __onexitbegin              100499c8     <common>
 0002:000009cc       g_pcsExit                  100499cc     <common>
 0002:000009d0       _pRawDllMain               100499d0     <common>

 entry point at        0001:00046094

 Static symbols

 0001:0000f0b0       InitializeMux              100100b0 f   i_hwinit.obj
 0001:0000f108       InitializeOTGMux           10010108 f   i_hwinit.obj
 0001:0000f10c       InitializeHost2Mux         1001010c f   i_hwinit.obj
 0001:0000f1c8       SelectUSBCore              100101c8 f   i_hwinit.obj
 0001:0000f210       ConfigH2                   10010210 f   i_hwinit.obj
 0001:0000f52c       ConfigOTG                  1001052c f   i_hwinit.obj
 0001:000102f4       USBClockSet                100112f4 f   i_usbclock.obj
 0001:000113b4       ?GetInterruptThreadPriority@@YAKPAG@Z 100123b4 f   usbh_usb2com_common_topaz_v1:hcddrv.obj
 0001:00045018       InitializeEHCI             10046018 f   usbh_ehcdpdd_common_topaz_v1:system.obj
 0001:00045790       GetRegistryPhysicalMemSize 10046790 f   usbh_ehcdpdd_common_topaz_v1:system.obj
 0001:000460e8       _DllMainCRTStartupHelper   100470e8 f   corelib0:pegdmain.obj
 0001:00046470       doexit                     10047470 f   corelib0:cexit.obj
 0001:0004672c       lockexit                   1004772c f   corelib0:onexit.obj
 0001:000467c8       unlockexit                 100477c8 f   corelib0:onexit.obj
 0001:000467f4       _onexit_nolock             100477f4 f   corelib0:onexit.obj
